Archive member included to satisfy reference by file (symbol)

..\..\..\Libraries\libs\libplatform.a(audio.o)
                              Output\obj\Libraries\bsp\bsp_sys.o (adpll_init)
..\..\..\Libraries\libs\libplatform.a(cm.o)
                              Output\obj\Libraries\bsp\bsp_param.o (cm_sync)
..\..\..\Libraries\libs\libplatform.a(os_flash.o)
                              Output\obj\Examples\Internal_Flash\Source\Internal_Flash.o (os_spiflash_read)
..\..\..\Libraries\libs\libplatform.a(xcfg.o)
                              Output\obj\Libraries\bsp\bsp_sys.o (xcfg_init)
..\..\..\Libraries\libs\libplatform.a(device.o)
                              Output\obj\Libraries\bsp\bsp_sys.o (dev_init)
..\..\..\Libraries\libs\libplatform.a(main.o)
                              Output\obj\Libraries\bsp\bsp_bt.o (delay_5ms)
..\..\..\Libraries\libs\libplatform.a(interrupt.o)
                              Output\obj\Libraries\bsp\bsp_fot.o (tick_get)
..\..\..\Libraries\libs\libplatform.a(startup.o)
                              ..\..\..\Libraries\libs\libplatform.a(interrupt.o) (user_timer_isr_en)
..\..\..\Libraries\libs\libplatform.a(sys_hook.o)
                              ..\..\..\Libraries\libs\libplatform.a(startup.o) (sys_hook_init)
..\..\..\Libraries\libs\libplatform.a(reset.o)
                              (_start)
..\..\..\Libraries\libs\libplatform.a(spiflash.o)
                              ..\..\..\Libraries\libs\libplatform.a(os_flash.o) (spiflash_program)
..\..\..\Libraries\libs\libplatform.a(debug.o)
                              ..\..\..\Libraries\libs\libplatform.a(main.o) (debug_set)
..\..\..\Libraries\libs\libplatform.a(fot_update.o)
                              ..\..\..\Libraries\libs\libplatform.a(xcfg.o) (get_spiloader_offset)
..\..\..\Libraries\libs\libplatform.a(lock.o)
                              ..\..\..\Libraries\libs\libplatform.a(main.o) (lock_init)
..\..\..\Libraries\libs\libplatform.a(patch.o)
                              ..\..\..\Libraries\libs\libplatform.a(main.o) (patch_init)
..\..\..\Libraries\libs\libplatform.a(power.o)
                              Output\obj\Libraries\bsp\bsp_sys.o (pmu_init)
..\..\..\Libraries\libs\libplatform.a(rc.o)
                              ..\..\..\Libraries\libs\libplatform.a(main.o) (rc_compile)
..\..\..\Libraries\libs\libplatform.a(s_sys.o)
                              ..\..\..\Libraries\libs\libplatform.a(main.o) (s_bcnt)
..\..\..\Libraries\libs\libplatform.a(sys.o)
                              ..\..\..\Libraries\libs\libplatform.a(main.o) (sys_get_rc2m_clkhz)
..\..\..\Libraries\libs\libplatform.a(sys_clk.o)
                              Output\obj\Libraries\BT\ble\ble.o (get_cur_sysclk)
..\..\..\Libraries\libs\libplatform.a(voltage_trim.o)
                              ..\..\..\Libraries\libs\libplatform.a(main.o) (voltage_trim_value_init)
..\..\..\Libraries\libs\libplatform.a(weak_symbol.o)
                              ..\..\..\Libraries\libs\libplatform.a(main.o) (update_complete)
..\..\..\Libraries\libs\libplatform.a(huart.o)
                              ..\..\..\Libraries\libs\libplatform.a(interrupt.o) (huart_isr)
..\..\..\Libraries\libs\libplatform.a(usb.o)
                              ..\..\..\Libraries\libs\libplatform.a(startup.o) (thread_usb_entry)
..\..\..\Libraries\libs\libplatform.a(bt.o)
                              ..\..\..\Libraries\libs\libplatform.a(reset.o) (bthw_txrx_isr)
..\..\..\Libraries\libs\libbtstack.a(nanos.o)
                              ..\..\..\Libraries\libs\libplatform.a(startup.o) (nanos_var_init)
..\..\..\Libraries\libs\libbtstack.a(patch.o)
                              ..\..\..\Libraries\libs\libplatform.a(patch.o) (bb_patch_init)
..\..\..\Libraries\libs\libbtstack.a(platform.o)
                              ..\..\..\Libraries\libs\libplatform.a(interrupt.o) (timer_sync_init)
..\..\..\Libraries\libs\libbtstack.a(bt_sco.o)
                              ..\..\..\Libraries\libs\libplatform.a(interrupt.o) (bt_codec_isr)
..\..\..\Libraries\libs\libbtstack.a(bt_acl.o)
                              ..\..\..\Libraries\libs\libbtstack.a(patch.o) (bt_acl_env)
..\..\..\Libraries\libs\libbtstack.a(ble_con.o)
                              ..\..\..\Libraries\libs\libbtstack.a(patch.o) (ble_con_evt_prio_check)
..\..\..\Libraries\libs\libbtstack.a(bb_utils.o)
                              ..\..\..\Libraries\libs\libbtstack.a(ble_con.o) (bb_sca2ppm)
..\..\..\Libraries\libs\libbtstack.a(bb_int.o)
                              ..\..\..\Libraries\libs\libplatform.a(bt.o) (bb_hal_isr)
..\..\..\Libraries\libs\libbtstack.a(bb.o)
                              ..\..\..\Libraries\libs\libbtstack.a(nanos.o) (bb_get_heap_info)
..\..\..\Libraries\libs\libbtstack.a(platform.o)
                              ..\..\..\Libraries\libs\libbtstack.a(bb.o) (dummy_void)
..\..\..\Libraries\libs\libbtstack.a(extern_tws.o)
                              ..\..\..\Libraries\libs\libbtstack.a(bb_int.o) (cfg_bt_tws_limit_pair_time)
..\..\..\Libraries\libs\libbtstack.a(extern_bt.o)
                              ..\..\..\Libraries\libs\libbtstack.a(bb_int.o) (cfg_bt_sniff_clk_sel)
..\..\..\Libraries\libs\libbtstack.a(extern.o)
                              ..\..\..\Libraries\libs\libplatform.a(reset.o) (ext_aubuf_isr)
..\..\..\Libraries\libs\libbtstack.a(spp.o)
                              Output\obj\Libraries\bsp\bsp_fot.o (bt_spp_tx)
..\..\..\Libraries\libs\libbtstack.a(sdp_util.o)
                              ..\..\..\Libraries\libs\libbtstack.a(spp.o) (mfi_search_uuid128)
..\..\..\Libraries\libs\libbtstack.a(sdp_tbl.o)
                              Output\obj\Libraries\BT\spp\profile.o (sdp_spp_service_record)
..\..\..\Libraries\libs\libbtstack.a(sdp_server.o)
                              Output\obj\Libraries\BT\spp\profile.o (sdp_add_service)
..\..\..\Libraries\libs\libbtstack.a(sdp_client.o)
                              ..\..\..\Libraries\libs\libbtstack.a(sdp_server.o) (sdp_client_init)
..\..\..\Libraries\libs\libbtstack.a(rfcomm.o)
                              ..\..\..\Libraries\libs\libbtstack.a(spp.o) (rfcomm_can_send_packet_now)
..\..\..\Libraries\libs\libbtstack.a(btstack_link_key_db.o)
                              Output\obj\Libraries\BT\spp\bt.o (link_info_page_size)
..\..\..\Libraries\libs\libbtstack.a(btstack_util.o)
                              ..\..\..\Libraries\libs\libbtstack.a(rfcomm.o) (bd_addr_cmp)
..\..\..\Libraries\libs\libbtstack.a(btstack_txpkt.o)
                              Output\obj\Libraries\BT\ble\ab_link\app.o (txpkt_init)
..\..\..\Libraries\libs\libbtstack.a(btstack_run_loop.o)
                              ..\..\..\Libraries\libs\libbtstack.a(rfcomm.o) (btstack_run_loop_set_timer_handler)
..\..\..\Libraries\libs\libbtstack.a(btstack_memory.o)
                              ..\..\..\Libraries\libs\libbtstack.a(rfcomm.o) (btstack_memory_rfcomm_multiplexer_get)
..\..\..\Libraries\libs\libbtstack.a(btstack_linked_list.o)
                              ..\..\..\Libraries\libs\libbtstack.a(rfcomm.o) (btstack_linked_list_empty)
..\..\..\Libraries\libs\libbtstack.a(btstack_link_ctrl.o)
                              ..\..\..\Libraries\libs\libbtstack.a(spp.o) (provide_link_ctrl_context_for_bd_addr)
..\..\..\Libraries\libs\libbtstack.a(sm.o)
                              Output\obj\Libraries\bsp\bsp_bt.o (gap_random_address_set_mode)
..\..\..\Libraries\libs\libbtstack.a(le_device_db_memory.o)
                              ..\..\..\Libraries\libs\libbtstack.a(sm.o) (le_device_db_set_local_bd_addr)
..\..\..\Libraries\libs\libbtstack.a(gatt_server.o)
                              Output\obj\Libraries\BT\ble\ab_link\app.o (ble_init_att_for_handle)
..\..\..\Libraries\libs\libbtstack.a(gatt_profile.o)
                              Output\obj\Libraries\BT\ble\ab_link\app.o (ble_gatts_service_add)
..\..\..\Libraries\libs\libbtstack.a(att_server.o)
                              Output\obj\Libraries\bsp\bsp_bt.o (att_server_init)
..\..\..\Libraries\libs\libbtstack.a(att_dispatch.o)
                              ..\..\..\Libraries\libs\libbtstack.a(att_server.o) (att_dispatch_register_server)
..\..\..\Libraries\libs\libbtstack.a(att_db.o)
                              ..\..\..\Libraries\libs\libbtstack.a(gatt_server.o) (att_uuid_for_handle)
..\..\..\Libraries\libs\libbtstack.a(ad_parser.o)
                              ..\..\..\Libraries\libs\libbtstack.a(gatt_server.o) (ad_param)
..\..\..\Libraries\libs\libbtstack.a(btstack_main.o)
                              Output\obj\Libraries\bsp\bsp_bt.o (le_sm_init)
..\..\..\Libraries\libs\libbtstack.a(btstack_hal.o)
                              ..\..\..\Libraries\libs\libbtstack.a(btstack_run_loop.o) (hal_tick_init)
..\..\..\Libraries\libs\libbtstack.a(btstack_api.o)
                              ..\..\..\Libraries\libs\libplatform.a(startup.o) (btstack_var_init)
..\..\..\Libraries\libs\libbtstack.a(bt_api.o)
                              Output\obj\Libraries\bsp\bsp_bt.o (bt_setup)
..\..\..\Libraries\libs\libbtstack.a(ble_api.o)
                              ..\..\..\Libraries\libs\libbtstack.a(gatt_server.o) (ble_get_status)
..\..\..\Libraries\libs\libbtstack.a(bb_sche.o)
                              ..\..\..\Libraries\libs\libbtstack.a(ble_con.o) (bb_sche_frag_ble_dur_set)
..\..\..\Libraries\libs\libbtstack.a(patch_asm.o)
                              ..\..\..\Libraries\libs\libbtstack.a(patch.o) (bb_v1_patch0)
..\..\..\Libraries\libs\libbtstack.a(bb_dbg.o)
                              ..\..\..\Libraries\libs\libbtstack.a(bb.o) (bb_dbg_init)
..\..\..\Libraries\libs\libbtstack.a(bb_clk.o)
                              ..\..\..\Libraries\libs\libbtstack.a(bb.o) (bb_clk_init)
..\..\..\Libraries\libs\libbtstack.a(aes.o)
                              ..\..\..\Libraries\libs\libbtstack.a(bb.o) (aes_init)
..\..\..\Libraries\libs\libbtstack.a(vs_proc.o)
                              ..\..\..\Libraries\libs\libbtstack.a(btstack_api.o) (bt_fcc_test_ctrl)
..\..\..\Libraries\libs\libbtstack.a(vs_fcc.o)
                              ..\..\..\Libraries\libs\libbtstack.a(vs_proc.o) (vs_fcc_test_cmd_do)
..\..\..\Libraries\libs\libbtstack.a(vs.o)
                              ..\..\..\Libraries\libs\libbtstack.a(bb.o) (vs_init)
..\..\..\Libraries\libs\libbtstack.a(rf_smart.o)
                              ..\..\..\Libraries\libs\libbtstack.a(vs_fcc.o) (rfphy_pll_afc)
..\..\..\Libraries\libs\libbtstack.a(rf.o)
                              ..\..\..\Libraries\libs\libbtstack.a(bt_acl.o) (rf_txpwr_get_dbm)
..\..\..\Libraries\libs\libbtstack.a(bt_hook.o)
                              ..\..\..\Libraries\libs\libbtstack.a(bb.o) (bt_isr_hook)
..\..\..\Libraries\libs\libbtstack.a(ble_hook.o)
                              ..\..\..\Libraries\libs\libbtstack.a(bb.o) (ble_isr_hook)
..\..\..\Libraries\libs\libbtstack.a(hct_tl.o)
                              ..\..\..\Libraries\libs\libbtstack.a(bb_int.o) (hct_queue_is_empty)
..\..\..\Libraries\libs\libbtstack.a(hct_msg.o)
                              ..\..\..\Libraries\libs\libbtstack.a(hct_tl.o) (hci_look_for_cmd_desc)
..\..\..\Libraries\libs\libbtstack.a(hct_fc.o)
                              ..\..\..\Libraries\libs\libbtstack.a(hct_tl.o) (hci_fc_acl_packet_sent)
..\..\..\Libraries\libs\libbtstack.a(hct.o)
                              ..\..\..\Libraries\libs\libbtstack.a(vs_proc.o) (hci_send_2_host)
..\..\..\Libraries\libs\libbtstack.a(tws_sco.o)
                              ..\..\..\Libraries\libs\libbtstack.a(bt_hook.o) (bt_sco_get_index)
..\..\..\Libraries\libs\libbtstack.a(tws_acl.o)
                              ..\..\..\Libraries\libs\libbtstack.a(patch_asm.o) (tws_switch_acl_is_pause)
..\..\..\Libraries\libs\libbtstack.a(lm.o)
                              ..\..\..\Libraries\libs\libbtstack.a(btstack_main.o) (lm_set_scan_int)
..\..\..\Libraries\libs\libbtstack.a(bt_hal.o)
                              ..\..\..\Libraries\libs\libbtstack.a(bt_hook.o) (bt_channel_assess)
..\..\..\Libraries\libs\libbtstack.a(bt21.o)
                              ..\..\..\Libraries\libs\libbtstack.a(bb.o) (bt_buf_acl_rx_free)
..\..\..\Libraries\libs\libbtstack.a(bc.o)
                              ..\..\..\Libraries\libs\libbtstack.a(bt21.o) (bc_init)
..\..\..\Libraries\libs\libbtstack.a(ble_hal.o)
                              ..\..\..\Libraries\libs\libbtstack.a(ble_con.o) (ble_channel_assess)
..\..\..\Libraries\libs\libbtstack.a(ble_adv.o)
                              ..\..\..\Libraries\libs\libbtstack.a(ble_hal.o) (ble_adv_init)
..\..\..\Libraries\libs\libbtstack.a(ble.o)
                              ..\..\..\Libraries\libs\libbtstack.a(bb.o) (ble_var_init)
..\..\..\Libraries\libs\libbtstack.a(extern_ble.o)
                              ..\..\..\Libraries\libs\libbtstack.a(gatt_server.o) (ble_client_cfg_callback)
..\..\..\Libraries\libs\libbtstack.a(l2cap_test.o)
                              ..\..\..\Libraries\libs\libbtstack.a(btstack_main.o) (l2cap_vd_acl_init)
..\..\..\Libraries\libs\libbtstack.a(l2cap.o)
                              ..\..\..\Libraries\libs\libbtstack.a(btstack_main.o) (l2cap_init)
..\..\..\Libraries\libs\libbtstack.a(hci_sco.o)
                              ..\..\..\Libraries\libs\libbtstack.a(btstack_api.o) (sco_init_var)
..\..\..\Libraries\libs\libbtstack.a(hci_dump.o)
                              ..\..\..\Libraries\libs\libbtstack.a(btstack_api.o) (hci_dump_open)
..\..\..\Libraries\libs\libbtstack.a(hci_cmd.o)
                              ..\..\..\Libraries\libs\libbtstack.a(sm.o) (hci_le_long_term_key_negative_reply)
..\..\..\Libraries\libs\libbtstack.a(hci.o)
                              ..\..\..\Libraries\libs\libbtstack.a(l2cap.o) (gap_get_connection_parameter_range)
..\..\..\Libraries\libs\libbtstack.a(hid_usage.o)
                              ..\..\..\Libraries\libs\libbtstack.a(bt_api.o) (hid_report_set)
..\..\..\Libraries\libs\libbtstack.a(hid_device.o)
                              ..\..\..\Libraries\libs\libbtstack.a(bt_api.o) (bt_hid_is_connected)
..\..\..\Libraries\libs\libbtstack.a(hfp_hf.o)
                              ..\..\..\Libraries\libs\libbtstack.a(btstack_api.o) (hfp_hf_get_siri_status)
..\..\..\Libraries\libs\libbtstack.a(hfp.o)
                              ..\..\..\Libraries\libs\libbtstack.a(btstack_main.o) (hfp_var_init)
..\..\..\Libraries\libs\libbtstack.a(avdtp.o)
                              ..\..\..\Libraries\libs\libbtstack.a(bt_hook.o) (a2dp_get_play_index)
..\..\..\Libraries\libs\libbtstack.a(a2dp.o)
                              ..\..\..\Libraries\libs\libbtstack.a(btstack_api.o) (a2dp_is_playing)
..\..\..\Libraries\libs\libbtstack.a(btstack_memory_pool.o)
                              ..\..\..\Libraries\libs\libbtstack.a(btstack_memory.o) (btstack_memory_pool_get)
..\..\..\Libraries\libs\libbtstack.a(btstack_adv0.o)
                              ..\..\..\Libraries\libs\libbtstack.a(btstack_api.o) (btstack_adv0_ctrl)
..\..\..\Libraries\libs\libbtstack.a(hci_transport_hcic.o)
                              ..\..\..\Libraries\libs\libbtstack.a(hci.o) (hcic_rx_flush)
..\..\..\Libraries\libs\libbtstack.a(btstack_chipset_inner.o)
                              ..\..\..\Libraries\libs\libbtstack.a(btstack_api.o) (btstack_chipset_inner_instance)
..\..\..\Libraries\libs\libbtstack.a(lm_hook.o)
                              ..\..\..\Libraries\libs\libbtstack.a(lm.o) (lm_init_hook)
..\..\..\Libraries\libs\libbtstack.a(lm_sp.o)
                              ..\..\..\Libraries\libs\libbtstack.a(lm.o) (lm_oob_f1)
..\..\..\Libraries\libs\libbtstack.a(lm_proc.o)
                              ..\..\..\Libraries\libs\libbtstack.a(lm.o) (lm_msg_env)
..\..\..\Libraries\libs\libbtstack.a(lm_key.o)
                              ..\..\..\Libraries\libs\libbtstack.a(lm.o) (lm_e22)
..\..\..\Libraries\libs\libbtstack.a(lc.o)
                              ..\..\..\Libraries\libs\libbtstack.a(bt21.o) (lc_init)
..\..\..\Libraries\libs\libbtstack.a(mgr.o)
                              ..\..\..\Libraries\libs\libbtstack.a(ble.o) (mgr_init)
..\..\..\Libraries\libs\libbtstack.a(ll.o)
                              ..\..\..\Libraries\libs\libbtstack.a(ble.o) (ll_init)
..\..\..\Libraries\libs\libbtstack.a(ble_test.o)
                              ..\..\..\Libraries\libs\libbtstack.a(ble_hal.o) (ble_test_init)
..\..\..\Libraries\libs\libbtstack.a(ble_scan.o)
                              ..\..\..\Libraries\libs\libbtstack.a(ble.o) (ble_get_scan_var)
..\..\..\Libraries\libs\libbtstack.a(ble_per_adv.o)
                              ..\..\..\Libraries\libs\libbtstack.a(ble.o) (ble_get_per_adv_var)
..\..\..\Libraries\libs\libbtstack.a(ble_init.o)
                              ..\..\..\Libraries\libs\libbtstack.a(ble_hal.o) (ble_init_init)
..\..\..\Libraries\libs\libbtstack.a(ble_buf.o)
                              ..\..\..\Libraries\libs\libbtstack.a(ble.o) (ble_buf_init)
..\..\..\Libraries\libs\libbtstack.a(ble_adv0.o)
                              ..\..\..\Libraries\libs\libbtstack.a(ble.o) (ble_adv0_init)
..\..\..\Libraries\libs\libbtstack.a(extern_hfhs.o)
                              ..\..\..\Libraries\libs\libbtstack.a(hfp.o) (hfp_notice_network_time)
..\..\..\Libraries\libs\libbtstack.a(l2cap_signaling.o)
                              ..\..\..\Libraries\libs\libbtstack.a(l2cap.o) (l2cap_next_sig_id)
..\..\..\Libraries\libs\libbtstack.a(lc_hook.o)
                              ..\..\..\Libraries\libs\libbtstack.a(lm_proc.o) (lc_auto_sniff_step_set)
..\..\..\Libraries\libs\libbtstack.a(lm_sco.o)
                              ..\..\..\Libraries\libs\libbtstack.a(lc.o) (lm_init_sync)
..\..\..\Libraries\libs\libbtstack.a(lc_util.o)
                              ..\..\..\Libraries\libs\libbtstack.a(lc.o) (lc_compute_pkt_types)
..\..\..\Libraries\libs\libbtstack.a(lc_sniff.o)
                              ..\..\..\Libraries\libs\libbtstack.a(lc.o) (lc_sniff_init)
..\..\..\Libraries\libs\libbtstack.a(lc_sco.o)
                              ..\..\..\Libraries\libs\libbtstack.a(lc.o) (lc_sco_init)
..\..\..\Libraries\libs\libbtstack.a(lc_proc.o)
                              ..\..\..\Libraries\libs\libbtstack.a(lc.o) (lc_msg_env)
..\..\..\Libraries\libs\libbtstack.a(lc_lmppdu.o)
                              ..\..\..\Libraries\libs\libbtstack.a(lc_proc.o) (lmp_estab_allowed)
..\..\..\Libraries\libs\libbtstack.a(mgr_proc.o)
                              ..\..\..\Libraries\libs\libbtstack.a(mgr.o) (mgr_msg_env)
..\..\..\Libraries\libs\libbtstack.a(mgr_init.o)
                              ..\..\..\Libraries\libs\libbtstack.a(mgr_proc.o) (ble_init_end_ind_func)
..\..\..\Libraries\libs\libbtstack.a(mgr_hci.o)
                              ..\..\..\Libraries\libs\libbtstack.a(mgr_proc.o) (hci_command_mgr_func)
..\..\..\Libraries\libs\libbtstack.a(ll_scan.o)
                              ..\..\..\Libraries\libs\libbtstack.a(mgr_hci.o) (hci_le_set_scan_param_cmd_func)
..\..\..\Libraries\libs\libbtstack.a(ll_adv.o)
                              ..\..\..\Libraries\libs\libbtstack.a(mgr_hci.o) (hci_le_rd_adv_ch_tx_pw_cmd_func)
..\..\..\Libraries\libs\libbtstack.a(ll_proc.o)
                              ..\..\..\Libraries\libs\libbtstack.a(ll.o) (ll_msg_env)
..\..\..\Libraries\libs\libbtstack.a(ll_ping.o)
                              ..\..\..\Libraries\libs\libbtstack.a(ll_proc.o) (hci_rd_auth_payl_to_cmd_func)
..\..\..\Libraries\libs\libbtstack.a(ll_phy_upd.o)
                              ..\..\..\Libraries\libs\libbtstack.a(ll_proc.o) (hci_le_rd_phy_cmd_func)
..\..\..\Libraries\libs\libbtstack.a(ll_past.o)
                              ..\..\..\Libraries\libs\libbtstack.a(ll_proc.o) (hci_le_per_adv_set_info_transf_cmd_func)
..\..\..\Libraries\libs\libbtstack.a(ll_length.o)
                              ..\..\..\Libraries\libs\libbtstack.a(ll_proc.o) (hci_le_set_data_len_cmd_func)
..\..\..\Libraries\libs\libbtstack.a(ll_feature.o)
                              ..\..\..\Libraries\libs\libbtstack.a(ll_proc.o) (hci_le_rd_rem_feats_cmd_func)
..\..\..\Libraries\libs\libbtstack.a(ll_encrypt.o)
                              ..\..\..\Libraries\libs\libbtstack.a(ll_proc.o) (hci_le_en_enc_cmd_func)
..\..\..\Libraries\libs\libbtstack.a(ll_disconnect.o)
                              ..\..\..\Libraries\libs\libbtstack.a(ll_proc.o) (ble_disc_ind_func)
..\..\..\Libraries\libs\libbtstack.a(ll_con_upd.o)
                              ..\..\..\Libraries\libs\libbtstack.a(ll_proc.o) (hci_le_con_upd_cmd_func)
..\..\..\Libraries\libs\libbtstack.a(ll_cntl.o)
                              ..\..\..\Libraries\libs\libbtstack.a(ll.o) (ll_cntl_tx_check)
..\..\..\Libraries\libs\libbtstack.a(ll_clk_acc.o)
                              ..\..\..\Libraries\libs\libbtstack.a(ll_cntl.o) (ll_clk_acc_req_func)
..\..\..\Libraries\libs\libbtstack.a(ll_chmap_upd.o)
                              ..\..\..\Libraries\libs\libbtstack.a(ll_cntl.o) (ll_channel_map_ind_func)
..\..\..\Libraries\libs\libbtstack.a(aes_rpa.o)
                              ..\..\..\Libraries\libs\libbtstack.a(ll_adv.o) (aes_rpa_gen)
..\..\..\Libraries\libs\libbtstack.a(scan_hook.o)
                              ..\..\..\Libraries\libs\libbtstack.a(ll_scan.o) (ble_scan_end_ind_hook)
..\..\..\Libraries\libs\libbtstack.a(adv_hook.o)
                              ..\..\..\Libraries\libs\libbtstack.a(ll_adv.o) (ble_adv_end_ind_hook)
..\..\..\Libraries\libs\libbtstack.a(ll_version.o)
                              ..\..\..\Libraries\libs\libbtstack.a(ll_proc.o) (ll_op_ver_exch_ind_func)
..\..\..\Libraries\libs\libbtstack.a(ll_pwr.o)
                              ..\..\..\Libraries\libs\libbtstack.a(ll_proc.o) (hci_rd_tx_pwr_lvl_cmd_func)
..\..\..\Libraries\libs\libdrivers.a(usb_device_hid.o)
                              Output\obj\Libraries\bsp\bsp_sys.o (ude_tmr_isr)
..\..\..\Libraries\libs\libdrivers.a(usb_device_printer.o)
                              ..\..\..\Libraries\libs\libplatform.a(usb.o) (ude_bulk_tx_process)
..\..\..\Libraries\libs\libdrivers.a(usb_device_run_loop.o)
                              ..\..\..\Libraries\libs\libdrivers.a(usb_device_hid.o) (ude_cfgval_get)
..\..\..\Libraries\libs\libdrivers.a(usb_host_manage.o)
                              ..\..\..\Libraries\libs\libplatform.a(device.o) (usb_host_init)
..\..\..\Libraries\libs\libdrivers.a(usb_host_storage.o)
                              ..\..\..\Libraries\libs\libdrivers.a(usb_host_manage.o) (uhs_start)
..\..\..\Libraries\libs\libdrivers.a(usb_comm.o)
                              ..\..\..\Libraries\libs\libdrivers.a(usb_host_storage.o) (usb_interrupt_disable)
..\..\..\Libraries\libs\libdrivers.a(usb_detect.o)
                              ..\..\..\Libraries\libs\libdrivers.a(usb_host_manage.o) (usbchk_switch_otg_device)
..\..\..\Libraries\libs\libdrivers.a(usb_device_desc.o)
                              ..\..\..\Libraries\libs\libdrivers.a(usb_device_run_loop.o) (usb_get_hid_config_descriptor)
..\..\..\Libraries\libs\libdrivers.a(usb_device_enum.o)
                              ..\..\..\Libraries\libs\libdrivers.a(usb_device_run_loop.o) (ude_run_loop_execute)
..\..\..\Libraries\libs\libdrivers.a(usb_device_ep.o)
                              ..\..\..\Libraries\libs\libdrivers.a(usb_device_hid.o) (usb_set_cur_ep)
..\..\..\Libraries\libs\libdrivers.a(usb_host_enum.o)
                              ..\..\..\Libraries\libs\libdrivers.a(usb_host_manage.o) (uhe_start)
..\..\..\Libraries\libs\libdrivers.a(weak_symbol.o)
                              ..\..\..\Libraries\libs\libdrivers.a(usb_host_enum.o) (iphone_power_set)
..\..\..\Libraries\libs\libdrivers.a(usb_device_audio.o)
                              ..\..\..\Libraries\libs\libdrivers.a(usb_device_enum.o) (uda_get_spk_mute)

Allocating common symbols
Common symbol       size              file

fot_var             0x22              Output\obj\Libraries\bsp\bsp_fot.o
f_bt                0x7               Output\obj\Libraries\bsp\bsp_bt.o
mySavePara          0x40              Output\obj\Examples\Internal_Flash\Source\Internal_Flash.o
ticks_50ms          0x4               Output\obj\Libraries\bsp\bsp_sys.o
g_ucMcuId           0x20              Output\obj\Examples\Internal_Flash\Source\Internal_Flash.o
xcfg_cb             0xae              Output\obj\Libraries\bsp\bsp_sys.o

Discarded input sections

 .text          0x0000000000000000        0x0 Output\obj\Libraries\bsp\bsp_bt.o
 .data          0x0000000000000000        0x0 Output\obj\Libraries\bsp\bsp_bt.o
 .bss           0x0000000000000000        0x0 Output\obj\Libraries\bsp\bsp_bt.o
 .text.ble_get_scan_data
                0x0000000000000000        0x4 Output\obj\Libraries\bsp\bsp_bt.o
 .text.ble_get_adv_data
                0x0000000000000000        0x4 Output\obj\Libraries\bsp\bsp_bt.o
 .text.bsp_spp_disinit
                0x0000000000000000       0xda Output\obj\Libraries\bsp\bsp_bt.o
 .text.bsp_bt_close
                0x0000000000000000        0x2 Output\obj\Libraries\bsp\bsp_bt.o
 .text.tws_user_key_process
                0x0000000000000000        0x2 Output\obj\Libraries\bsp\bsp_bt.o
 .text.tws_warning_process
                0x0000000000000000        0x2 Output\obj\Libraries\bsp\bsp_bt.o
 .text.bsp_bt_vol_change
                0x0000000000000000        0x2 Output\obj\Libraries\bsp\bsp_bt.o
 .text.bsp_bt_get_hfp_vol
                0x0000000000000000        0x4 Output\obj\Libraries\bsp\bsp_bt.o
 .text.bsp_bt_call_volume_msg
                0x0000000000000000        0x2 Output\obj\Libraries\bsp\bsp_bt.o
 .text          0x0000000000000000        0x0 Output\obj\Libraries\bsp\bsp_cm.o
 .data          0x0000000000000000        0x0 Output\obj\Libraries\bsp\bsp_cm.o
 .bss           0x0000000000000000        0x0 Output\obj\Libraries\bsp\bsp_cm.o
 .text          0x0000000000000000        0x0 Output\obj\Libraries\bsp\bsp_fot.o
 .data          0x0000000000000000        0x0 Output\obj\Libraries\bsp\bsp_fot.o
 .bss           0x0000000000000000        0x0 Output\obj\Libraries\bsp\bsp_fot.o
 .text          0x0000000000000000        0x0 Output\obj\Libraries\bsp\bsp_param.o
 .data          0x0000000000000000        0x0 Output\obj\Libraries\bsp\bsp_param.o
 .bss           0x0000000000000000        0x0 Output\obj\Libraries\bsp\bsp_param.o
 .text          0x0000000000000000        0x0 Output\obj\Libraries\bsp\bsp_sys.o
 .data          0x0000000000000000        0x0 Output\obj\Libraries\bsp\bsp_sys.o
 .bss           0x0000000000000000        0x0 Output\obj\Libraries\bsp\bsp_sys.o
 .text.bsp_get_bat_level
                0x0000000000000000        0x6 Output\obj\Libraries\bsp\bsp_sys.o
 .rodata        0x0000000000000000       0x20 Output\obj\Libraries\bsp\bsp_sys.o
 .text          0x0000000000000000        0x0 Output\obj\Libraries\BT\ble\ab_link\app.o
 .data          0x0000000000000000        0x0 Output\obj\Libraries\BT\ble\ab_link\app.o
 .bss           0x0000000000000000        0x0 Output\obj\Libraries\BT\ble\ab_link\app.o
 .text.ble_send_packet1
                0x0000000000000000       0x28 Output\obj\Libraries\BT\ble\ab_link\app.o
 .text.ble_send_packet2
                0x0000000000000000       0x28 Output\obj\Libraries\BT\ble\ab_link\app.o
 .text.ble_read_value
                0x0000000000000000       0x24 Output\obj\Libraries\BT\ble\ab_link\app.o
 .text.bsp_ble_process
                0x0000000000000000        0x2 Output\obj\Libraries\BT\ble\ab_link\app.o
 .text          0x0000000000000000        0x0 Output\obj\Libraries\BT\ble\adv0.o
 .data          0x0000000000000000        0x0 Output\obj\Libraries\BT\ble\adv0.o
 .bss           0x0000000000000000        0x0 Output\obj\Libraries\BT\ble\adv0.o
 .text          0x0000000000000000        0x0 Output\obj\Libraries\BT\ble\ble.o
 .data          0x0000000000000000        0x0 Output\obj\Libraries\BT\ble\ble.o
 .bss           0x0000000000000000        0x0 Output\obj\Libraries\BT\ble\ble.o
 .text.ble_enter_transmit
                0x0000000000000000       0x3a Output\obj\Libraries\BT\ble\ble.o
 .text.ble_exit_transmit
                0x0000000000000000       0x32 Output\obj\Libraries\BT\ble\ble.o
 .text.ble_get_bat_level
                0x0000000000000000        0x8 Output\obj\Libraries\BT\ble\ble.o
 .sbss          0x0000000000000000        0x1 Output\obj\Libraries\BT\ble\ble.o
 .text          0x0000000000000000        0x0 Output\obj\Libraries\BT\spp\bt.o
 .data          0x0000000000000000        0x0 Output\obj\Libraries\BT\spp\bt.o
 .bss           0x0000000000000000        0x0 Output\obj\Libraries\BT\spp\bt.o
 .text.bt_clr_master_addr
                0x0000000000000000        0x2 Output\obj\Libraries\BT\spp\bt.o
 .text.bt_save_master_addr
                0x0000000000000000        0x2 Output\obj\Libraries\BT\spp\bt.o
 .text.bt_get_master_addr
                0x0000000000000000        0x4 Output\obj\Libraries\BT\spp\bt.o
 .text.bt_clr_all_link_info
                0x0000000000000000        0x8 Output\obj\Libraries\BT\spp\bt.o
 .text.bt_tws_clr_link_info
                0x0000000000000000        0x2 Output\obj\Libraries\BT\spp\bt.o
 .text.bt_get_rand_seed
                0x0000000000000000        0xa Output\obj\Libraries\BT\spp\bt.o
 .rodata        0x0000000000000000        0xa Output\obj\Libraries\BT\spp\bt.o
 .text          0x0000000000000000        0x0 Output\obj\Libraries\BT\spp\hid.o
 .data          0x0000000000000000        0x0 Output\obj\Libraries\BT\spp\hid.o
 .bss           0x0000000000000000        0x0 Output\obj\Libraries\BT\spp\hid.o
 .text.bsp_bt_hid_photo
                0x0000000000000000        0x4 Output\obj\Libraries\BT\spp\hid.o
 .text.bsp_bt_hid_vol_change
                0x0000000000000000        0x4 Output\obj\Libraries\BT\spp\hid.o
 .text.bsp_bt_hid_screen_left
                0x0000000000000000       0x32 Output\obj\Libraries\BT\spp\hid.o
 .text.bsp_bt_hid_screen_right
                0x0000000000000000       0x32 Output\obj\Libraries\BT\spp\hid.o
 .comment       0x0000000000000000       0x12 Output\obj\Libraries\BT\spp\hid.o
 .text          0x0000000000000000        0x0 Output\obj\Libraries\BT\spp\profile.o
 .bss           0x0000000000000000        0x0 Output\obj\Libraries\BT\spp\profile.o
 .text          0x0000000000000000        0x0 Output\obj\Libraries\BT\spp\spp.o
 .data          0x0000000000000000        0x0 Output\obj\Libraries\BT\spp\spp.o
 .bss           0x0000000000000000        0x0 Output\obj\Libraries\BT\spp\spp.o
 .text.bsp_spp_process
                0x0000000000000000        0x2 Output\obj\Libraries\BT\spp\spp.o
 .text          0x0000000000000000        0x0 Output\obj\Libraries\Device\Source\gw3323_clk.o
 .data          0x0000000000000000        0x0 Output\obj\Libraries\Device\Source\gw3323_clk.o
 .bss           0x0000000000000000        0x0 Output\obj\Libraries\Device\Source\gw3323_clk.o
 .text.clock_gate0_cmd
                0x0000000000000000       0x16 Output\obj\Libraries\Device\Source\gw3323_clk.o
 .text.clock_gate1_cmd
                0x0000000000000000       0x16 Output\obj\Libraries\Device\Source\gw3323_clk.o
 .text.clock_gate2_cmd
                0x0000000000000000       0x16 Output\obj\Libraries\Device\Source\gw3323_clk.o
 .comment       0x0000000000000000       0x12 Output\obj\Libraries\Device\Source\gw3323_clk.o
 .text          0x0000000000000000        0x0 Output\obj\Libraries\Device\Source\gw3323_gpio.o
 .data          0x0000000000000000        0x0 Output\obj\Libraries\Device\Source\gw3323_gpio.o
 .bss           0x0000000000000000        0x0 Output\obj\Libraries\Device\Source\gw3323_gpio.o
 .text.gpio_init
                0x0000000000000000       0xf6 Output\obj\Libraries\Device\Source\gw3323_gpio.o
 .text.gpio_func_mapping
                0x0000000000000000       0x5a Output\obj\Libraries\Device\Source\gw3323_gpio.o
 .text.gpio_pic_config_reset
                0x0000000000000000        0xa Output\obj\Libraries\Device\Source\gw3323_gpio.o
 .text.gpio_pic_config
                0x0000000000000000       0x88 Output\obj\Libraries\Device\Source\gw3323_gpio.o
 .com_text.isr  0x0000000000000000       0x28 Output\obj\Libraries\Device\Source\gw3323_gpio.o
 .text          0x0000000000000000        0x0 Output\obj\Libraries\Device\Source\gw3323_spi.o
 .data          0x0000000000000000        0x0 Output\obj\Libraries\Device\Source\gw3323_spi.o
 .bss           0x0000000000000000        0x0 Output\obj\Libraries\Device\Source\gw3323_spi.o
 .text.spi_init
                0x0000000000000000       0x28 Output\obj\Libraries\Device\Source\gw3323_spi.o
 .text.spi_cmd  0x0000000000000000       0x10 Output\obj\Libraries\Device\Source\gw3323_spi.o
 .text.spi_dir_sel
                0x0000000000000000       0x16 Output\obj\Libraries\Device\Source\gw3323_spi.o
 .text.spi_it_cmd
                0x0000000000000000       0x12 Output\obj\Libraries\Device\Source\gw3323_spi.o
 .text.spi_lfsr_cmd
                0x0000000000000000       0x12 Output\obj\Libraries\Device\Source\gw3323_spi.o
 .text.spi_multi_bit_bus_cmd
                0x0000000000000000       0x12 Output\obj\Libraries\Device\Source\gw3323_spi.o
 .text.spi_hold_rx_cmd
                0x0000000000000000       0x12 Output\obj\Libraries\Device\Source\gw3323_spi.o
 .text.spi_hold_tx_cmd
                0x0000000000000000       0x12 Output\obj\Libraries\Device\Source\gw3323_spi.o
 .text.spi_soft_hold_cmd
                0x0000000000000000       0x12 Output\obj\Libraries\Device\Source\gw3323_spi.o
 .text.spi_get_flag
                0x0000000000000000        0xa Output\obj\Libraries\Device\Source\gw3323_spi.o
 .text.spi_clear_flag
                0x0000000000000000        0x8 Output\obj\Libraries\Device\Source\gw3323_spi.o
 .text.spi_set_dma_cnt
                0x0000000000000000        0x4 Output\obj\Libraries\Device\Source\gw3323_spi.o
 .text.spi_set_dma_addr
                0x0000000000000000        0x4 Output\obj\Libraries\Device\Source\gw3323_spi.o
 .text.spi_receive_data
                0x0000000000000000        0x8 Output\obj\Libraries\Device\Source\gw3323_spi.o
 .text.spi_send_data
                0x0000000000000000        0x4 Output\obj\Libraries\Device\Source\gw3323_spi.o
 .comment       0x0000000000000000       0x12 Output\obj\Libraries\Device\Source\gw3323_spi.o
 .text          0x0000000000000000        0x0 Output\obj\Libraries\libs\strong_symbol.o
 .data          0x0000000000000000        0x0 Output\obj\Libraries\libs\strong_symbol.o
 .bss           0x0000000000000000        0x0 Output\obj\Libraries\libs\strong_symbol.o
 .text.aac_dec_init
                0x0000000000000000        0x2 Output\obj\Libraries\libs\strong_symbol.o
 .text.aac_decode_init
                0x0000000000000000        0x2 Output\obj\Libraries\libs\strong_symbol.o
 .text.aac_dec_frame
                0x0000000000000000        0x4 Output\obj\Libraries\libs\strong_symbol.o
 .text.aac_nor_dec_frame
                0x0000000000000000        0x4 Output\obj\Libraries\libs\strong_symbol.o
 .text.aac_tws_dec_frame
                0x0000000000000000        0x4 Output\obj\Libraries\libs\strong_symbol.o
 .text.aac_cache_free_do
                0x0000000000000000        0x2 Output\obj\Libraries\libs\strong_symbol.o
 .text.aac_cache_read_do
                0x0000000000000000        0x4 Output\obj\Libraries\libs\strong_symbol.o
 .text.tws_pack_aac
                0x0000000000000000        0x4 Output\obj\Libraries\libs\strong_symbol.o
 .com_text.aac.obuf
                0x0000000000000000        0x2 Output\obj\Libraries\libs\strong_symbol.o
 .aacdec.text   0x0000000000000000        0x2 Output\obj\Libraries\libs\strong_symbol.o
 .text.btstack_tws_init
                0x0000000000000000        0x2 Output\obj\Libraries\libs\strong_symbol.o
 .text.a2dp_play_init
                0x0000000000000000        0x2 Output\obj\Libraries\libs\strong_symbol.o
 .bcom_text.sbc.play
                0x0000000000000000       0x28 Output\obj\Libraries\libs\strong_symbol.o
 .bcom_text.sbc_cache
                0x0000000000000000        0xc Output\obj\Libraries\libs\strong_symbol.o
 .sbcdec.code   0x0000000000000000        0x6 Output\obj\Libraries\libs\strong_symbol.o
 .com_text.bb.tws
                0x0000000000000000        0x2 Output\obj\Libraries\libs\strong_symbol.o
 .bcom_text.bb.btisr
                0x0000000000000000       0x12 Output\obj\Libraries\libs\strong_symbol.o
 .text.bt_tws_set_spr
                0x0000000000000000        0x4 Output\obj\Libraries\libs\strong_symbol.o
 .com_text.sbc.play
                0x0000000000000000        0x2 Output\obj\Libraries\libs\strong_symbol.o
 .bcom_text.sbc.send
                0x0000000000000000        0x2 Output\obj\Libraries\libs\strong_symbol.o
 .bcom_text.lc.tws
                0x0000000000000000        0x4 Output\obj\Libraries\libs\strong_symbol.o
 .bcom_text.a2dp.lost
                0x0000000000000000        0x4 Output\obj\Libraries\libs\strong_symbol.o
 .bcom_text.sbc
                0x0000000000000000        0x2 Output\obj\Libraries\libs\strong_symbol.o
 .bcom_text.bb.tws_switch
                0x0000000000000000        0x4 Output\obj\Libraries\libs\strong_symbol.o
 .bcom_text.bb.bttx
                0x0000000000000000        0x6 Output\obj\Libraries\libs\strong_symbol.o
 .text.tws_set_snoop_ticks
                0x0000000000000000        0x4 Output\obj\Libraries\libs\strong_symbol.o
 .text.ble_test_start
                0x0000000000000000        0x4 Output\obj\Libraries\libs\strong_symbol.o
 .text.ble_test_stop
                0x0000000000000000        0x4 Output\obj\Libraries\libs\strong_symbol.o
 .text.huart_init
                0x0000000000000000        0x2 Output\obj\Libraries\libs\strong_symbol.o
 .com_text.bt_rec
                0x0000000000000000        0x2 Output\obj\Libraries\libs\strong_symbol.o
 .text.bt_sco_fill_remote_buf
                0x0000000000000000        0x2 Output\obj\Libraries\libs\strong_symbol.o
 .text.btstack_pbap
                0x0000000000000000        0x2 Output\obj\Libraries\libs\strong_symbol.o
 .text.bsp_charge_ctrl_process
                0x0000000000000000        0x2 Output\obj\Libraries\libs\strong_symbol.o
 .text.usb_dev_isr
                0x0000000000000000        0x2 Output\obj\Libraries\libs\strong_symbol.o
 .text.ude_isoc_tx_process
                0x0000000000000000        0x2 Output\obj\Libraries\libs\strong_symbol.o
 .text.ude_isoc_rx_process
                0x0000000000000000        0x2 Output\obj\Libraries\libs\strong_symbol.o
 .text.lock_code_usbdev
                0x0000000000000000        0x2 Output\obj\Libraries\libs\strong_symbol.o
 .text.unlock_code_usbdev
                0x0000000000000000        0x2 Output\obj\Libraries\libs\strong_symbol.o
 .text.dac_get_max_anl_vol
                0x0000000000000000        0x4 Output\obj\Libraries\libs\strong_symbol.o
 .com_text.dac  0x0000000000000000        0x2 Output\obj\Libraries\libs\strong_symbol.o
 .text.bsp.dac  0x0000000000000000        0x2 Output\obj\Libraries\libs\strong_symbol.o
 .text          0x0000000000000000        0x0 Output\obj\Examples\Internal_Flash\Source\Internal_Flash.o
 .data          0x0000000000000000        0x0 Output\obj\Examples\Internal_Flash\Source\Internal_Flash.o
 .bss           0x0000000000000000        0x0 Output\obj\Examples\Internal_Flash\Source\Internal_Flash.o
 .text.read_bluetooth_name
                0x0000000000000000       0x80 Output\obj\Examples\Internal_Flash\Source\Internal_Flash.o
 .text          0x0000000000000000        0x0 Output\obj\Examples\Internal_Flash\Project\config.o
 .data          0x0000000000000000        0x0 Output\obj\Examples\Internal_Flash\Project\config.o
 .bss           0x0000000000000000        0x0 Output\obj\Examples\Internal_Flash\Project\config.o
 .text          0x0000000000000000        0x0 Output\obj\Examples\Internal_Flash\Project\main.o
 .data          0x0000000000000000        0x0 Output\obj\Examples\Internal_Flash\Project\main.o
 .bss           0x0000000000000000        0x0 Output\obj\Examples\Internal_Flash\Project\main.o
 .text          0x0000000000000000        0x0 ..\..\..\Libraries\libs\libplatform.a(audio.o)
 .data          0x0000000000000000        0x0 ..\..\..\Libraries\libs\libplatform.a(audio.o)
 .bss           0x0000000000000000        0x0 ..\..\..\Libraries\libs\libplatform.a(audio.o)
 .com_text.dac  0x0000000000000000       0x66 ..\..\..\Libraries\libs\libplatform.a(audio.o)
 .text.spires   0x0000000000000000       0x40 ..\..\..\Libraries\libs\libplatform.a(audio.o)
 .text          0x0000000000000000        0x0 ..\..\..\Libraries\libs\libplatform.a(cm.o)
 .data          0x0000000000000000        0x0 ..\..\..\Libraries\libs\libplatform.a(cm.o)
 .text.cm_move_allpages
                0x0000000000000000      0x140 ..\..\..\Libraries\libs\libplatform.a(cm.o)
 .text.cm_get_startaddr
                0x0000000000000000        0xa ..\..\..\Libraries\libs\libplatform.a(cm.o)
 .text.cm_get_area
                0x0000000000000000       0x14 ..\..\..\Libraries\libs\libplatform.a(cm.o)
 .text.cm_release_all
                0x0000000000000000       0x90 ..\..\..\Libraries\libs\libplatform.a(cm.o)
 .text.cm_read8
                0x0000000000000000       0x28 ..\..\..\Libraries\libs\libplatform.a(cm.o)
 .text.cm_read16
                0x0000000000000000       0x28 ..\..\..\Libraries\libs\libplatform.a(cm.o)
 .text.cm_read32
                0x0000000000000000       0x24 ..\..\..\Libraries\libs\libplatform.a(cm.o)
 .text.cm_write8
                0x0000000000000000       0x28 ..\..\..\Libraries\libs\libplatform.a(cm.o)
 .text.cm_write16
                0x0000000000000000       0x28 ..\..\..\Libraries\libs\libplatform.a(cm.o)
 .text.cm_write32
                0x0000000000000000       0x24 ..\..\..\Libraries\libs\libplatform.a(cm.o)
 .text.cm_clear
                0x0000000000000000       0x60 ..\..\..\Libraries\libs\libplatform.a(cm.o)
 .text          0x0000000000000000        0x0 ..\..\..\Libraries\libs\libplatform.a(os_flash.o)
 .data          0x0000000000000000        0x0 ..\..\..\Libraries\libs\libplatform.a(os_flash.o)
 .bss           0x0000000000000000        0x0 ..\..\..\Libraries\libs\libplatform.a(os_flash.o)
 .text          0x0000000000000000        0x0 ..\..\..\Libraries\libs\libplatform.a(xcfg.o)
 .data          0x0000000000000000        0x0 ..\..\..\Libraries\libs\libplatform.a(xcfg.o)
 .bss           0x0000000000000000        0x0 ..\..\..\Libraries\libs\libplatform.a(xcfg.o)
 .text          0x0000000000000000        0x0 ..\..\..\Libraries\libs\libplatform.a(device.o)
 .data          0x0000000000000000        0x0 ..\..\..\Libraries\libs\libplatform.a(device.o)
 .bss           0x0000000000000000        0x0 ..\..\..\Libraries\libs\libplatform.a(device.o)
 .text.sd_disable
                0x0000000000000000       0x18 ..\..\..\Libraries\libs\libplatform.a(device.o)
 .text.sd_disable_user
                0x0000000000000000       0x46 ..\..\..\Libraries\libs\libplatform.a(device.o)
 .text.sd_enable_user
                0x0000000000000000       0x2c ..\..\..\Libraries\libs\libplatform.a(device.o)
 .com_text.device
                0x0000000000000000       0x10 ..\..\..\Libraries\libs\libplatform.a(device.o)
 .com_text.device.udisk
                0x0000000000000000        0xe ..\..\..\Libraries\libs\libplatform.a(device.o)
 .com_text.device.filter
                0x0000000000000000       0xe0 ..\..\..\Libraries\libs\libplatform.a(device.o)
 .text.device   0x0000000000000000       0x40 ..\..\..\Libraries\libs\libplatform.a(device.o)
 .text.dev_is_invalid
                0x0000000000000000        0xe ..\..\..\Libraries\libs\libplatform.a(device.o)
 .com_text.sd.api
                0x0000000000000000       0x3c ..\..\..\Libraries\libs\libplatform.a(device.o)
 .text.fs_lock  0x0000000000000000       0x14 ..\..\..\Libraries\libs\libplatform.a(device.o)
 .text.fs_unlock
                0x0000000000000000       0x12 ..\..\..\Libraries\libs\libplatform.a(device.o)
 .sbss          0x0000000000000000        0x4 ..\..\..\Libraries\libs\libplatform.a(device.o)
 .text          0x0000000000000000        0x0 ..\..\..\Libraries\libs\libplatform.a(main.o)
 .data          0x0000000000000000        0x0 ..\..\..\Libraries\libs\libplatform.a(main.o)
 .com_text.exception.do
                0x0000000000000000       0x5a ..\..\..\Libraries\libs\libplatform.a(main.o)
 .com_text.ledseg
                0x0000000000000000       0x40 ..\..\..\Libraries\libs\libplatform.a(main.o)
 .text.uart0_mapping_sel
                0x0000000000000000       0x18 ..\..\..\Libraries\libs\libplatform.a(main.o)
 .text.compiler
                0x0000000000000000       0x20 ..\..\..\Libraries\libs\libplatform.a(main.o)
 .com_text.ledseg.table
                0x0000000000000000        0xc ..\..\..\Libraries\libs\libplatform.a(main.o)
 .text          0x0000000000000000        0x0 ..\..\..\Libraries\libs\libplatform.a(interrupt.o)
 .data          0x0000000000000000        0x0 ..\..\..\Libraries\libs\libplatform.a(interrupt.o)
 .bss           0x0000000000000000        0x0 ..\..\..\Libraries\libs\libplatform.a(interrupt.o)
 .text.sys_irq_init
                0x0000000000000000       0x54 ..\..\..\Libraries\libs\libplatform.a(interrupt.o)
 .text.timer1_irq_init
                0x0000000000000000       0x38 ..\..\..\Libraries\libs\libplatform.a(interrupt.o)
 .com_text.tws.isr
                0x0000000000000000       0x22 ..\..\..\Libraries\libs\libplatform.a(interrupt.o)
 .text.huart_irq_init
                0x0000000000000000       0x3a ..\..\..\Libraries\libs\libplatform.a(interrupt.o)
 .rodata.str1.4
                0x0000000000000000       0x19 ..\..\..\Libraries\libs\libplatform.a(interrupt.o)
 .text.watch_point_set
                0x0000000000000000       0x48 ..\..\..\Libraries\libs\libplatform.a(interrupt.o)
 .text.wdt_init
                0x0000000000000000       0x3a ..\..\..\Libraries\libs\libplatform.a(interrupt.o)
 .text          0x0000000000000000        0x0 ..\..\..\Libraries\libs\libplatform.a(startup.o)
 .data          0x0000000000000000        0x0 ..\..\..\Libraries\libs\libplatform.a(startup.o)
 .com_text.sndp.api
                0x0000000000000000       0x26 ..\..\..\Libraries\libs\libplatform.a(startup.o)
 .text          0x0000000000000000        0x0 ..\..\..\Libraries\libs\libplatform.a(sys_hook.o)
 .data          0x0000000000000000        0x0 ..\..\..\Libraries\libs\libplatform.a(sys_hook.o)
 .bss           0x0000000000000000        0x0 ..\..\..\Libraries\libs\libplatform.a(sys_hook.o)
 .text          0x0000000000000000        0x0 ..\..\..\Libraries\libs\libplatform.a(reset.o)
 .data          0x0000000000000000        0x0 ..\..\..\Libraries\libs\libplatform.a(reset.o)
 .bss           0x0000000000000000        0x0 ..\..\..\Libraries\libs\libplatform.a(reset.o)
 .text          0x0000000000000000        0x0 ..\..\..\Libraries\libs\libplatform.a(spiflash.o)
 .data          0x0000000000000000        0x0 ..\..\..\Libraries\libs\libplatform.a(spiflash.o)
 .bss           0x0000000000000000        0x0 ..\..\..\Libraries\libs\libplatform.a(spiflash.o)
 .text          0x0000000000000000        0x0 ..\..\..\Libraries\libs\libplatform.a(debug.o)
 .data          0x0000000000000000        0x0 ..\..\..\Libraries\libs\libplatform.a(debug.o)
 .bss           0x0000000000000000        0x0 ..\..\..\Libraries\libs\libplatform.a(debug.o)
 .text.debug_dump_info_nanos_schedule
                0x0000000000000000        0x2 ..\..\..\Libraries\libs\libplatform.a(debug.o)
 .text.debug_dump_info_nanos_timer
                0x0000000000000000        0x2 ..\..\..\Libraries\libs\libplatform.a(debug.o)
 .text          0x0000000000000000        0x0 ..\..\..\Libraries\libs\libplatform.a(fot_update.o)
 .data          0x0000000000000000        0x0 ..\..\..\Libraries\libs\libplatform.a(fot_update.o)
 .text.param_fot_head_info_write
                0x0000000000000000        0x2 ..\..\..\Libraries\libs\libplatform.a(fot_update.o)
 .text.param_fot_head_info_read
                0x0000000000000000        0x2 ..\..\..\Libraries\libs\libplatform.a(fot_update.o)
 .text.param_fot_addr_write
                0x0000000000000000        0x2 ..\..\..\Libraries\libs\libplatform.a(fot_update.o)
 .text.param_fot_addr_read
                0x0000000000000000        0x2 ..\..\..\Libraries\libs\libplatform.a(fot_update.o)
 .text.is_fot_update_en
                0x0000000000000000        0x4 ..\..\..\Libraries\libs\libplatform.a(fot_update.o)
 .text.fot_head_crc_get
                0x0000000000000000       0x9c ..\..\..\Libraries\libs\libplatform.a(fot_update.o)
 .text.fot_get_info
                0x0000000000000000       0x50 ..\..\..\Libraries\libs\libplatform.a(fot_update.o)
 .text          0x0000000000000000        0x0 ..\..\..\Libraries\libs\libplatform.a(lock.o)
 .data          0x0000000000000000        0x0 ..\..\..\Libraries\libs\libplatform.a(lock.o)
 .text.unlock_whcode
                0x0000000000000000       0x3c ..\..\..\Libraries\libs\libplatform.a(lock.o)
 .text.lock_whcode
                0x0000000000000000       0x58 ..\..\..\Libraries\libs\libplatform.a(lock.o)
 .text.unlock_dcode
                0x0000000000000000       0x54 ..\..\..\Libraries\libs\libplatform.a(lock.o)
 .text.lock_dcode
                0x0000000000000000       0x58 ..\..\..\Libraries\libs\libplatform.a(lock.o)
 .text.lock_code_bt_sleep
                0x0000000000000000       0x54 ..\..\..\Libraries\libs\libplatform.a(lock.o)
 .text.unlock_code_bt_sleep
                0x0000000000000000       0x38 ..\..\..\Libraries\libs\libplatform.a(lock.o)
 .text.lock_code_pwrsave
                0x0000000000000000       0x3c ..\..\..\Libraries\libs\libplatform.a(lock.o)
 .text.unlock_code_pwrsave
                0x0000000000000000       0x38 ..\..\..\Libraries\libs\libplatform.a(lock.o)
 .text.lock_code_charge
                0x0000000000000000       0x3c ..\..\..\Libraries\libs\libplatform.a(lock.o)
 .text.unlock_code_charge
                0x0000000000000000        0x8 ..\..\..\Libraries\libs\libplatform.a(lock.o)
 .text.unlock_code_bt_voice
                0x0000000000000000       0x38 ..\..\..\Libraries\libs\libplatform.a(lock.o)
 .text.lock_code_usbdev
                0x0000000000000000       0x54 ..\..\..\Libraries\libs\libplatform.a(lock.o)
 .text.unlock_code_usbdev
                0x0000000000000000       0x38 ..\..\..\Libraries\libs\libplatform.a(lock.o)
 .text.load_code_btdec
                0x0000000000000000       0x54 ..\..\..\Libraries\libs\libplatform.a(lock.o)
 .text.unlock_code_btdec
                0x0000000000000000       0x38 ..\..\..\Libraries\libs\libplatform.a(lock.o)
 .text.load_code_bt_voice
                0x0000000000000000       0x5c ..\..\..\Libraries\libs\libplatform.a(lock.o)
 .text.lock_ram_mp3enc
                0x0000000000000000       0x4c ..\..\..\Libraries\libs\libplatform.a(lock.o)
 .text.unlock_ram_mp3enc
                0x0000000000000000       0x38 ..\..\..\Libraries\libs\libplatform.a(lock.o)
 .text.lock_code_sniff
                0x0000000000000000       0x4c ..\..\..\Libraries\libs\libplatform.a(lock.o)
 .text.unlock_code_sniff
                0x0000000000000000       0x38 ..\..\..\Libraries\libs\libplatform.a(lock.o)
 .text.unlock_code_huart
                0x0000000000000000        0x8 ..\..\..\Libraries\libs\libplatform.a(lock.o)
 .text.lock_code_huart
                0x0000000000000000       0x54 ..\..\..\Libraries\libs\libplatform.a(lock.o)
 .text.lock_code_bb_test
                0x0000000000000000       0x54 ..\..\..\Libraries\libs\libplatform.a(lock.o)
 .text.unlock_code_bb_test
                0x0000000000000000       0x38 ..\..\..\Libraries\libs\libplatform.a(lock.o)
 .text.unlock_code_fota
                0x0000000000000000       0x38 ..\..\..\Libraries\libs\libplatform.a(lock.o)
 .text          0x0000000000000000        0x0 ..\..\..\Libraries\libs\libplatform.a(patch.o)
 .data          0x0000000000000000        0x0 ..\..\..\Libraries\libs\libplatform.a(patch.o)
 .bss           0x0000000000000000        0x0 ..\..\..\Libraries\libs\libplatform.a(patch.o)
 .text          0x0000000000000000        0x0 ..\..\..\Libraries\libs\libplatform.a(power.o)
 .data          0x0000000000000000        0x0 ..\..\..\Libraries\libs\libplatform.a(power.o)
 .bss           0x0000000000000000        0x0 ..\..\..\Libraries\libs\libplatform.a(power.o)
 .com_text.voltage.trim
                0x0000000000000000        0xa ..\..\..\Libraries\libs\libplatform.a(power.o)
 .text          0x0000000000000000        0x0 ..\..\..\Libraries\libs\libplatform.a(rc.o)
 .data          0x0000000000000000        0x0 ..\..\..\Libraries\libs\libplatform.a(rc.o)
 .bss           0x0000000000000000        0x0 ..\..\..\Libraries\libs\libplatform.a(rc.o)
 .text.compiler
                0x0000000000000000        0x2 ..\..\..\Libraries\libs\libplatform.a(rc.o)
 .text          0x0000000000000000        0x0 ..\..\..\Libraries\libs\libplatform.a(s_sys.o)
 .data          0x0000000000000000        0x0 ..\..\..\Libraries\libs\libplatform.a(s_sys.o)
 .bss           0x0000000000000000        0x0 ..\..\..\Libraries\libs\libplatform.a(s_sys.o)
 .text          0x0000000000000000        0x0 ..\..\..\Libraries\libs\libplatform.a(sys.o)
 .data          0x0000000000000000        0x0 ..\..\..\Libraries\libs\libplatform.a(sys.o)
 .bss           0x0000000000000000        0x0 ..\..\..\Libraries\libs\libplatform.a(sys.o)
 .text.dbg_clk_out
                0x0000000000000000       0x44 ..\..\..\Libraries\libs\libplatform.a(sys.o)
 .text.sys_clk_output
                0x0000000000000000      0x136 ..\..\..\Libraries\libs\libplatform.a(sys.o)
 .text.__divdi3
                0x0000000000000000       0x5c ..\..\..\Libraries\libs\libplatform.a(sys.o)
 .text.__umoddi3
                0x0000000000000000       0x30 ..\..\..\Libraries\libs\libplatform.a(sys.o)
 .text.get_random
                0x0000000000000000       0x26 ..\..\..\Libraries\libs\libplatform.a(sys.o)
 .text.random_init
                0x0000000000000000        0xa ..\..\..\Libraries\libs\libplatform.a(sys.o)
 .text.convert_uni2gbk
                0x0000000000000000       0x8a ..\..\..\Libraries\libs\libplatform.a(sys.o)
 .text.lrc      0x0000000000000000       0x58 ..\..\..\Libraries\libs\libplatform.a(sys.o)
 .text.utf8_convert_to_unicode
                0x0000000000000000       0x72 ..\..\..\Libraries\libs\libplatform.a(sys.o)
 .com_text.sys  0x0000000000000000       0x1e ..\..\..\Libraries\libs\libplatform.a(sys.o)
 .text.sw_reset_source_get
                0x0000000000000000       0x2a ..\..\..\Libraries\libs\libplatform.a(sys.o)
 .sleep_text.sleep
                0x0000000000000000      0x128 ..\..\..\Libraries\libs\libplatform.a(sys.o)
 .text.sys.power
                0x0000000000000000       0x96 ..\..\..\Libraries\libs\libplatform.a(sys.o)
 .text          0x0000000000000000        0x0 ..\..\..\Libraries\libs\libplatform.a(sys_clk.o)
 .data          0x0000000000000000        0x0 ..\..\..\Libraries\libs\libplatform.a(sys_clk.o)
 .bss           0x0000000000000000        0x0 ..\..\..\Libraries\libs\libplatform.a(sys_clk.o)
 .com_text.sys  0x0000000000000000        0x4 ..\..\..\Libraries\libs\libplatform.a(sys_clk.o)
 .text.sys_clk.aec
                0x0000000000000000      0x200 ..\..\..\Libraries\libs\libplatform.a(sys_clk.o)
 .text.set_uart0_baud
                0x0000000000000000       0x38 ..\..\..\Libraries\libs\libplatform.a(sys_clk.o)
 .text.set_uart1_baud
                0x0000000000000000       0x38 ..\..\..\Libraries\libs\libplatform.a(sys_clk.o)
 .text.set_uart1_baud_rc2m_clk
                0x0000000000000000       0x24 ..\..\..\Libraries\libs\libplatform.a(sys_clk.o)
 .text.sys_clk_get
                0x0000000000000000        0xa ..\..\..\Libraries\libs\libplatform.a(sys_clk.o)
 .text.sys_clk_req
                0x0000000000000000       0x5e ..\..\..\Libraries\libs\libplatform.a(sys_clk.o)
 .text.sys_clk_free
                0x0000000000000000       0x5c ..\..\..\Libraries\libs\libplatform.a(sys_clk.o)
 .text.sys_clk_free_all
                0x0000000000000000       0x50 ..\..\..\Libraries\libs\libplatform.a(sys_clk.o)
 .text          0x0000000000000000        0x0 ..\..\..\Libraries\libs\libplatform.a(voltage_trim.o)
 .data          0x0000000000000000        0x0 ..\..\..\Libraries\libs\libplatform.a(voltage_trim.o)
 .text          0x0000000000000000        0x0 ..\..\..\Libraries\libs\libplatform.a(weak_symbol.o)
 .data          0x0000000000000000        0x0 ..\..\..\Libraries\libs\libplatform.a(weak_symbol.o)
 .bss           0x0000000000000000        0x0 ..\..\..\Libraries\libs\libplatform.a(weak_symbol.o)
 .text.music_eq_get_bass_tbl
                0x0000000000000000        0x4 ..\..\..\Libraries\libs\libplatform.a(weak_symbol.o)
 .text.music_eq_get_treble_tbl
                0x0000000000000000        0x4 ..\..\..\Libraries\libs\libplatform.a(weak_symbol.o)
 .text.mic_eq_get_bass_tbl
                0x0000000000000000        0x4 ..\..\..\Libraries\libs\libplatform.a(weak_symbol.o)
 .text.mic_eq_get_treble_tbl
                0x0000000000000000        0x4 ..\..\..\Libraries\libs\libplatform.a(weak_symbol.o)
 .text.music_eq_get_tbl
                0x0000000000000000        0x4 ..\..\..\Libraries\libs\libplatform.a(weak_symbol.o)
 .text.bass_treble_get_coef_tbl
                0x0000000000000000        0x4 ..\..\..\Libraries\libs\libplatform.a(weak_symbol.o)
 .text.stream   0x0000000000000000        0x8 ..\..\..\Libraries\libs\libplatform.a(weak_symbol.o)
 .com_text.rec  0x0000000000000000        0x2 ..\..\..\Libraries\libs\libplatform.a(weak_symbol.o)
 .text.update   0x0000000000000000        0x4 ..\..\..\Libraries\libs\libplatform.a(weak_symbol.o)
 .text.qtest    0x0000000000000000       0x1a ..\..\..\Libraries\libs\libplatform.a(weak_symbol.o)
 .text.dacr_is_output
                0x0000000000000000        0x4 ..\..\..\Libraries\libs\libplatform.a(weak_symbol.o)
 .text.sd_is_online
                0x0000000000000000        0x4 ..\..\..\Libraries\libs\libplatform.a(weak_symbol.o)
 .sbss          0x0000000000000000        0x1 ..\..\..\Libraries\libs\libplatform.a(weak_symbol.o)
 .text          0x0000000000000000        0x0 ..\..\..\Libraries\libs\libplatform.a(huart.o)
 .data          0x0000000000000000        0x0 ..\..\..\Libraries\libs\libplatform.a(huart.o)
 .bss           0x0000000000000000        0x0 ..\..\..\Libraries\libs\libplatform.a(huart.o)
 .com_huart.text
                0x0000000000000000      0x1b2 ..\..\..\Libraries\libs\libplatform.a(huart.o)
 .text.huart_tx_done
                0x0000000000000000        0x2 ..\..\..\Libraries\libs\libplatform.a(huart.o)
 .text.lock_code_huart
                0x0000000000000000        0x2 ..\..\..\Libraries\libs\libplatform.a(huart.o)
 .text.huart_irq_init
                0x0000000000000000        0x2 ..\..\..\Libraries\libs\libplatform.a(huart.o)
 .text.huart.huart_init_do
                0x0000000000000000      0x194 ..\..\..\Libraries\libs\libplatform.a(huart.o)
 .text.huart.huart_exit
                0x0000000000000000       0x12 ..\..\..\Libraries\libs\libplatform.a(huart.o)
 .text.huart.huart_setbaudrate
                0x0000000000000000       0x36 ..\..\..\Libraries\libs\libplatform.a(huart.o)
 .com_text.huart.huart_getchar
                0x0000000000000000       0x2e ..\..\..\Libraries\libs\libplatform.a(huart.o)
 .com_huart.rodata
                0x0000000000000000       0x58 ..\..\..\Libraries\libs\libplatform.a(huart.o)
 .sbss          0x0000000000000000        0xc ..\..\..\Libraries\libs\libplatform.a(huart.o)
 .comment       0x0000000000000000       0x13 ..\..\..\Libraries\libs\libplatform.a(huart.o)
 .riscv.attributes
                0x0000000000000000       0x32 ..\..\..\Libraries\libs\libplatform.a(huart.o)
 .text          0x0000000000000000        0x0 ..\..\..\Libraries\libs\libplatform.a(usb.o)
 .data          0x0000000000000000        0x0 ..\..\..\Libraries\libs\libplatform.a(usb.o)
 .bss           0x0000000000000000        0x0 ..\..\..\Libraries\libs\libplatform.a(usb.o)
 .text          0x0000000000000000        0x0 ..\..\..\Libraries\libs\libplatform.a(bt.o)
 .data          0x0000000000000000        0x0 ..\..\..\Libraries\libs\libplatform.a(bt.o)
 .bss           0x0000000000000000        0x0 ..\..\..\Libraries\libs\libplatform.a(bt.o)
 .com_text.isr.txrx
                0x0000000000000000        0x2 ..\..\..\Libraries\libs\libplatform.a(bt.o)
 .text.update   0x0000000000000000        0x4 ..\..\..\Libraries\libs\libplatform.a(bt.o)
 .bt_voice.plc  0x0000000000000000       0x48 ..\..\..\Libraries\libs\libplatform.a(bt.o)
 .rodata.str1.4
                0x0000000000000000        0xd ..\..\..\Libraries\libs\libplatform.a(bt.o)
 .com_text.btstack.uart
                0x0000000000000000       0x26 ..\..\..\Libraries\libs\libplatform.a(bt.o)
 .data          0x0000000000000000        0x0 ..\..\..\Libraries\libs\libbtstack.a(nanos.o)
 .bss           0x0000000000000000        0x0 ..\..\..\Libraries\libs\libbtstack.a(nanos.o)
 .com_text.md.nanos
                0x0000000000000000       0x3c ..\..\..\Libraries\libs\libbtstack.a(nanos.o)
 .data          0x0000000000000000        0x0 ..\..\..\Libraries\libs\libbtstack.a(patch.o)
 .bss           0x0000000000000000        0x0 ..\..\..\Libraries\libs\libbtstack.a(patch.o)
 .data          0x0000000000000000        0x0 ..\..\..\Libraries\libs\libbtstack.a(platform.o)
 .bss           0x0000000000000000        0x0 ..\..\..\Libraries\libs\libbtstack.a(platform.o)
 .com_text.bb.isr.timer
                0x0000000000000000        0x2 ..\..\..\Libraries\libs\libbtstack.a(platform.o)
 .data          0x0000000000000000        0x0 ..\..\..\Libraries\libs\libbtstack.a(bt_sco.o)
 .bss           0x0000000000000000        0x0 ..\..\..\Libraries\libs\libbtstack.a(bt_sco.o)
 .bt_voice.bb.cvsd
                0x0000000000000000        0x2 ..\..\..\Libraries\libs\libbtstack.a(bt_sco.o)
 .bt_voice.plc  0x0000000000000000        0x2 ..\..\..\Libraries\libs\libbtstack.a(bt_sco.o)
 .data          0x0000000000000000        0x0 ..\..\..\Libraries\libs\libbtstack.a(bt_acl.o)
 .bss           0x0000000000000000        0x0 ..\..\..\Libraries\libs\libbtstack.a(bt_acl.o)
 .data          0x0000000000000000        0x0 ..\..\..\Libraries\libs\libbtstack.a(ble_con.o)
 .bss           0x0000000000000000        0x0 ..\..\..\Libraries\libs\libbtstack.a(ble_con.o)
 .data          0x0000000000000000        0x0 ..\..\..\Libraries\libs\libbtstack.a(bb_utils.o)
 .bss           0x0000000000000000        0x0 ..\..\..\Libraries\libs\libbtstack.a(bb_utils.o)
 .srodata       0x0000000000000000        0x5 ..\..\..\Libraries\libs\libbtstack.a(bb_utils.o)
 .data          0x0000000000000000        0x0 ..\..\..\Libraries\libs\libbtstack.a(bb_int.o)
 .bss           0x0000000000000000        0x0 ..\..\..\Libraries\libs\libbtstack.a(bb_int.o)
 .com_text.bb.isr.timer
                0x0000000000000000       0x48 ..\..\..\Libraries\libs\libbtstack.a(bb_int.o)
 .text.bb.timer.init
                0x0000000000000000       0x76 ..\..\..\Libraries\libs\libbtstack.a(bb_int.o)
 .text.bb.timer.kill
                0x0000000000000000       0x22 ..\..\..\Libraries\libs\libbtstack.a(bb_int.o)
 .com_text.bb.timer.get
                0x0000000000000000       0x24 ..\..\..\Libraries\libs\libbtstack.a(bb_int.o)
 .sleep_text.bb
                0x0000000000000000      0x232 ..\..\..\Libraries\libs\libbtstack.a(bb_int.o)
 .com_text.bb.sleep
                0x0000000000000000       0x4c ..\..\..\Libraries\libs\libbtstack.a(bb_int.o)
 .data          0x0000000000000000        0x0 ..\..\..\Libraries\libs\libbtstack.a(bb.o)
 .text.update   0x0000000000000000       0x1a ..\..\..\Libraries\libs\libbtstack.a(bb.o)
 .data          0x0000000000000000        0x0 ..\..\..\Libraries\libs\libbtstack.a(platform.o)
 .bss           0x0000000000000000        0x0 ..\..\..\Libraries\libs\libbtstack.a(platform.o)
 .com_text.cpu.sfr
                0x0000000000000000       0x3c ..\..\..\Libraries\libs\libbtstack.a(platform.o)
 .com_text.sco  0x0000000000000000        0x8 ..\..\..\Libraries\libs\libbtstack.a(platform.o)
 .data          0x0000000000000000        0x0 ..\..\..\Libraries\libs\libbtstack.a(extern_tws.o)
 .bss           0x0000000000000000        0x0 ..\..\..\Libraries\libs\libbtstack.a(extern_tws.o)
 .sdata         0x0000000000000000        0x7 ..\..\..\Libraries\libs\libbtstack.a(extern_tws.o)
 .data          0x0000000000000000        0x0 ..\..\..\Libraries\libs\libbtstack.a(extern_bt.o)
 .bss           0x0000000000000000        0x0 ..\..\..\Libraries\libs\libbtstack.a(extern_bt.o)
 .com_text.bt_rec
                0x0000000000000000        0x2 ..\..\..\Libraries\libs\libbtstack.a(extern_bt.o)
 .com_text.aec  0x0000000000000000        0x4 ..\..\..\Libraries\libs\libbtstack.a(extern_bt.o)
 .bt_voice.sco  0x0000000000000000        0x2 ..\..\..\Libraries\libs\libbtstack.a(extern_bt.o)
 .bt_voice.bb.cvsd
                0x0000000000000000        0x2 ..\..\..\Libraries\libs\libbtstack.a(extern_bt.o)
 .text          0x0000000000000000       0x28 ..\..\..\Libraries\libs\libbtstack.a(extern.o)
 .data          0x0000000000000000        0x0 ..\..\..\Libraries\libs\libbtstack.a(extern.o)
 .bss           0x0000000000000000        0x0 ..\..\..\Libraries\libs\libbtstack.a(extern.o)
 .text.huart    0x0000000000000000        0x2 ..\..\..\Libraries\libs\libbtstack.a(extern.o)
 .com_text.huart
                0x0000000000000000        0xe ..\..\..\Libraries\libs\libbtstack.a(extern.o)
 .com_text.ticks
                0x0000000000000000        0x4 ..\..\..\Libraries\libs\libbtstack.a(extern.o)
 .sbss          0x0000000000000000        0x1 ..\..\..\Libraries\libs\libbtstack.a(extern.o)
 .data          0x0000000000000000        0x0 ..\..\..\Libraries\libs\libbtstack.a(spp.o)
 .bss           0x0000000000000000        0x0 ..\..\..\Libraries\libs\libbtstack.a(spp.o)
 .sbss          0x0000000000000000        0x1 ..\..\..\Libraries\libs\libbtstack.a(spp.o)
 .text          0x0000000000000000        0x0 ..\..\..\Libraries\libs\libbtstack.a(sdp_util.o)
 .data          0x0000000000000000        0x0 ..\..\..\Libraries\libs\libbtstack.a(sdp_util.o)
 .bss           0x0000000000000000        0x0 ..\..\..\Libraries\libs\libbtstack.a(sdp_util.o)
 .text          0x0000000000000000        0x0 ..\..\..\Libraries\libs\libbtstack.a(sdp_tbl.o)
 .data          0x0000000000000000        0x0 ..\..\..\Libraries\libs\libbtstack.a(sdp_tbl.o)
 .bss           0x0000000000000000        0x0 ..\..\..\Libraries\libs\libbtstack.a(sdp_tbl.o)
 .rodata.sdp.tbl.avctp_controller
                0x0000000000000000       0x44 ..\..\..\Libraries\libs\libbtstack.a(sdp_tbl.o)
 .rodata.sdp.tbl.avctp_target2
                0x0000000000000000       0x41 ..\..\..\Libraries\libs\libbtstack.a(sdp_tbl.o)
 .rodata.sdp.tbl.avdtp
                0x0000000000000000       0x41 ..\..\..\Libraries\libs\libbtstack.a(sdp_tbl.o)
 .rodata.sdp.tbl.hfp
                0x0000000000000000       0x50 ..\..\..\Libraries\libs\libbtstack.a(sdp_tbl.o)
 .rodata.sdp.tbl.hid_consumer
                0x0000000000000000       0xd2 ..\..\..\Libraries\libs\libbtstack.a(sdp_tbl.o)
 .rodata.sdp.tbl.hid_did
                0x0000000000000000       0x40 ..\..\..\Libraries\libs\libbtstack.a(sdp_tbl.o)
 .rodata.sdp.tbl.hid_keyboard
                0x0000000000000000      0x115 ..\..\..\Libraries\libs\libbtstack.a(sdp_tbl.o)
 .rodata.sdp.tbl.hid_tscreen
                0x0000000000000000      0x110 ..\..\..\Libraries\libs\libbtstack.a(sdp_tbl.o)
 .rodata.sdp.tbl.hid_tscreen_ext
                0x0000000000000000      0x119 ..\..\..\Libraries\libs\libbtstack.a(sdp_tbl.o)
 .rodata.sdp.tbl.spp_dueros
                0x0000000000000000       0x51 ..\..\..\Libraries\libs\libbtstack.a(sdp_tbl.o)
 .data          0x0000000000000000        0x0 ..\..\..\Libraries\libs\libbtstack.a(sdp_server.o)
 .bss           0x0000000000000000        0x0 ..\..\..\Libraries\libs\libbtstack.a(sdp_server.o)
 .text.stack.sdp.server_rmv
                0x0000000000000000       0x2c ..\..\..\Libraries\libs\libbtstack.a(sdp_server.o)
 .data          0x0000000000000000        0x0 ..\..\..\Libraries\libs\libbtstack.a(sdp_client.o)
 .bss           0x0000000000000000        0x0 ..\..\..\Libraries\libs\libbtstack.a(sdp_client.o)
 .data          0x0000000000000000        0x0 ..\..\..\Libraries\libs\libbtstack.a(rfcomm.o)
 .bss           0x0000000000000000        0x0 ..\..\..\Libraries\libs\libbtstack.a(rfcomm.o)
 .text          0x0000000000000000        0x0 ..\..\..\Libraries\libs\libbtstack.a(btstack_link_key_db.o)
 .sbss          0x0000000000000000        0x1 ..\..\..\Libraries\libs\libbtstack.a(btstack_link_key_db.o)
 .data          0x0000000000000000        0x0 ..\..\..\Libraries\libs\libbtstack.a(btstack_util.o)
 .bss           0x0000000000000000        0x0 ..\..\..\Libraries\libs\libbtstack.a(btstack_util.o)
 .data          0x0000000000000000        0x0 ..\..\..\Libraries\libs\libbtstack.a(btstack_txpkt.o)
 .bss           0x0000000000000000        0x0 ..\..\..\Libraries\libs\libbtstack.a(btstack_txpkt.o)
 .text          0x0000000000000000        0x0 ..\..\..\Libraries\libs\libbtstack.a(btstack_run_loop.o)
 .bss           0x0000000000000000        0x0 ..\..\..\Libraries\libs\libbtstack.a(btstack_run_loop.o)
 .text          0x0000000000000000       0x22 ..\..\..\Libraries\libs\libbtstack.a(btstack_memory.o)
 .data          0x0000000000000000        0x0 ..\..\..\Libraries\libs\libbtstack.a(btstack_memory.o)
 .text          0x0000000000000000       0x54 ..\..\..\Libraries\libs\libbtstack.a(btstack_linked_list.o)
 .data          0x0000000000000000        0x0 ..\..\..\Libraries\libs\libbtstack.a(btstack_linked_list.o)
 .bss           0x0000000000000000        0x0 ..\..\..\Libraries\libs\libbtstack.a(btstack_linked_list.o)
 .com_text.fifo.search
                0x0000000000000000       0x28 ..\..\..\Libraries\libs\libbtstack.a(btstack_linked_list.o)
 .com_text.fifo.add
                0x0000000000000000       0x5e ..\..\..\Libraries\libs\libbtstack.a(btstack_linked_list.o)
 .btdec.a2dp.list
                0x0000000000000000      0x1be ..\..\..\Libraries\libs\libbtstack.a(btstack_linked_list.o)
 .data          0x0000000000000000        0x0 ..\..\..\Libraries\libs\libbtstack.a(btstack_link_ctrl.o)
 .bss           0x0000000000000000        0x0 ..\..\..\Libraries\libs\libbtstack.a(btstack_link_ctrl.o)
 .sbss          0x0000000000000000        0x1 ..\..\..\Libraries\libs\libbtstack.a(btstack_link_ctrl.o)
 .data          0x0000000000000000        0x0 ..\..\..\Libraries\libs\libbtstack.a(sm.o)
 .data          0x0000000000000000        0x0 ..\..\..\Libraries\libs\libbtstack.a(le_device_db_memory.o)
 .bss           0x0000000000000000        0x0 ..\..\..\Libraries\libs\libbtstack.a(le_device_db_memory.o)
 .data          0x0000000000000000        0x0 ..\..\..\Libraries\libs\libbtstack.a(gatt_server.o)
 .bss           0x0000000000000000        0x0 ..\..\..\Libraries\libs\libbtstack.a(gatt_server.o)
 .com_text.ble_frame1
                0x0000000000000000       0x2a ..\..\..\Libraries\libs\libbtstack.a(gatt_server.o)
 .text.ble.notify_handle
                0x0000000000000000       0x54 ..\..\..\Libraries\libs\libbtstack.a(gatt_server.o)
 .sbss          0x0000000000000000        0x1 ..\..\..\Libraries\libs\libbtstack.a(gatt_server.o)
 .data          0x0000000000000000        0x0 ..\..\..\Libraries\libs\libbtstack.a(gatt_profile.o)
 .bss           0x0000000000000000        0x0 ..\..\..\Libraries\libs\libbtstack.a(gatt_profile.o)
 .data          0x0000000000000000        0x0 ..\..\..\Libraries\libs\libbtstack.a(att_server.o)
 .bss           0x0000000000000000        0x0 ..\..\..\Libraries\libs\libbtstack.a(att_server.o)
 .data          0x0000000000000000        0x0 ..\..\..\Libraries\libs\libbtstack.a(att_dispatch.o)
 .bss           0x0000000000000000        0x0 ..\..\..\Libraries\libs\libbtstack.a(att_dispatch.o)
 .data          0x0000000000000000        0x0 ..\..\..\Libraries\libs\libbtstack.a(att_db.o)
 .bss           0x0000000000000000        0x0 ..\..\..\Libraries\libs\libbtstack.a(att_db.o)
 .text          0x0000000000000000      0x1ea ..\..\..\Libraries\libs\libbtstack.a(ad_parser.o)
 .data          0x0000000000000000        0x0 ..\..\..\Libraries\libs\libbtstack.a(ad_parser.o)
 .bss           0x0000000000000000        0x0 ..\..\..\Libraries\libs\libbtstack.a(ad_parser.o)
 .data          0x0000000000000000        0x0 ..\..\..\Libraries\libs\libbtstack.a(btstack_main.o)
 .bss           0x0000000000000000        0x0 ..\..\..\Libraries\libs\libbtstack.a(btstack_main.o)
 .data          0x0000000000000000        0x0 ..\..\..\Libraries\libs\libbtstack.a(btstack_hal.o)
 .bss           0x0000000000000000        0x0 ..\..\..\Libraries\libs\libbtstack.a(btstack_hal.o)
 .com_text.stack.uart_isr
                0x0000000000000000       0x7e ..\..\..\Libraries\libs\libbtstack.a(btstack_hal.o)
 .text.stack.hal
                0x0000000000000000       0xa2 ..\..\..\Libraries\libs\libbtstack.a(btstack_hal.o)
 .com_text.stack.util
                0x0000000000000000       0x12 ..\..\..\Libraries\libs\libbtstack.a(btstack_hal.o)
 .sbss          0x0000000000000000        0x9 ..\..\..\Libraries\libs\libbtstack.a(btstack_hal.o)
 .data          0x0000000000000000        0x0 ..\..\..\Libraries\libs\libbtstack.a(btstack_api.o)
 .com_text.bb.sleep
                0x0000000000000000       0x34 ..\..\..\Libraries\libs\libbtstack.a(btstack_api.o)
 .sleep_text.sleep
                0x0000000000000000        0x8 ..\..\..\Libraries\libs\libbtstack.a(btstack_api.o)
 .com_text.sco  0x0000000000000000       0x44 ..\..\..\Libraries\libs\libbtstack.a(btstack_api.o)
 .sbss          0x0000000000000000        0x7 ..\..\..\Libraries\libs\libbtstack.a(btstack_api.o)
 .data          0x0000000000000000        0x0 ..\..\..\Libraries\libs\libbtstack.a(bt_api.o)
 .bss           0x0000000000000000        0x0 ..\..\..\Libraries\libs\libbtstack.a(bt_api.o)
 .text.stack.sleep
                0x0000000000000000       0xc0 ..\..\..\Libraries\libs\libbtstack.a(bt_api.o)
 .text.stack.api.hid_con
                0x0000000000000000       0x3a ..\..\..\Libraries\libs\libbtstack.a(bt_api.o)
 .text.stack.api.hid_disc
                0x0000000000000000       0x34 ..\..\..\Libraries\libs\libbtstack.a(bt_api.o)
 .text.stack.api.hid_send
                0x0000000000000000       0xa6 ..\..\..\Libraries\libs\libbtstack.a(bt_api.o)
 .com_text.timer
                0x0000000000000000       0x1a ..\..\..\Libraries\libs\libbtstack.a(bt_api.o)
 .sbss          0x0000000000000000        0x1 ..\..\..\Libraries\libs\libbtstack.a(bt_api.o)
 .data          0x0000000000000000        0x0 ..\..\..\Libraries\libs\libbtstack.a(ble_api.o)
 .bss           0x0000000000000000        0x0 ..\..\..\Libraries\libs\libbtstack.a(ble_api.o)
 .sbss          0x0000000000000000        0x1 ..\..\..\Libraries\libs\libbtstack.a(ble_api.o)
 .data          0x0000000000000000        0x0 ..\..\..\Libraries\libs\libbtstack.a(bb_sche.o)
 .text          0x0000000000000000        0x0 ..\..\..\Libraries\libs\libbtstack.a(patch_asm.o)
 .data          0x0000000000000000        0x0 ..\..\..\Libraries\libs\libbtstack.a(patch_asm.o)
 .bss           0x0000000000000000        0x0 ..\..\..\Libraries\libs\libbtstack.a(patch_asm.o)
 .data          0x0000000000000000        0x0 ..\..\..\Libraries\libs\libbtstack.a(bb_dbg.o)
 .bss           0x0000000000000000        0x0 ..\..\..\Libraries\libs\libbtstack.a(bb_dbg.o)
 .com_text.bb.putc
                0x0000000000000000       0x60 ..\..\..\Libraries\libs\libbtstack.a(bb_dbg.o)
 .data          0x0000000000000000        0x0 ..\..\..\Libraries\libs\libbtstack.a(bb_clk.o)
 .bss           0x0000000000000000        0x0 ..\..\..\Libraries\libs\libbtstack.a(bb_clk.o)
 .text          0x0000000000000000        0x0 ..\..\..\Libraries\libs\libbtstack.a(aes.o)
 .data          0x0000000000000000        0x0 ..\..\..\Libraries\libs\libbtstack.a(aes.o)
 .data          0x0000000000000000        0x0 ..\..\..\Libraries\libs\libbtstack.a(vs_proc.o)
 .bss           0x0000000000000000        0x0 ..\..\..\Libraries\libs\libbtstack.a(vs_proc.o)
 .data          0x0000000000000000        0x0 ..\..\..\Libraries\libs\libbtstack.a(vs_fcc.o)
 .bss           0x0000000000000000        0x0 ..\..\..\Libraries\libs\libbtstack.a(vs_fcc.o)
 .text.bb.vs.fcc_ble.do
                0x0000000000000000       0x7a ..\..\..\Libraries\libs\libbtstack.a(vs_fcc.o)
 .data          0x0000000000000000        0x0 ..\..\..\Libraries\libs\libbtstack.a(vs.o)
 .bss           0x0000000000000000        0x0 ..\..\..\Libraries\libs\libbtstack.a(vs.o)
 .data          0x0000000000000000        0x0 ..\..\..\Libraries\libs\libbtstack.a(rf_smart.o)
 .bss           0x0000000000000000        0x0 ..\..\..\Libraries\libs\libbtstack.a(rf_smart.o)
 .text.update   0x0000000000000000       0x44 ..\..\..\Libraries\libs\libbtstack.a(rf_smart.o)
 .data          0x0000000000000000        0x0 ..\..\..\Libraries\libs\libbtstack.a(rf.o)
 .bss           0x0000000000000000        0x0 ..\..\..\Libraries\libs\libbtstack.a(rf.o)
 .sleep_text.bb
                0x0000000000000000       0x30 ..\..\..\Libraries\libs\libbtstack.a(rf.o)
 .data          0x0000000000000000        0x0 ..\..\..\Libraries\libs\libbtstack.a(bt_hook.o)
 .bss           0x0000000000000000        0x0 ..\..\..\Libraries\libs\libbtstack.a(bt_hook.o)
 .com_text.bt21.test.fcc
                0x0000000000000000       0xa0 ..\..\..\Libraries\libs\libbtstack.a(bt_hook.o)
 .data          0x0000000000000000        0x0 ..\..\..\Libraries\libs\libbtstack.a(ble_hook.o)
 .bss           0x0000000000000000        0x0 ..\..\..\Libraries\libs\libbtstack.a(ble_hook.o)
 .data          0x0000000000000000        0x0 ..\..\..\Libraries\libs\libbtstack.a(hct_tl.o)
 .com_text.bb.sleep
                0x0000000000000000       0x34 ..\..\..\Libraries\libs\libbtstack.a(hct_tl.o)
 .data          0x0000000000000000        0x0 ..\..\..\Libraries\libs\libbtstack.a(hct_msg.o)
 .bss           0x0000000000000000        0x0 ..\..\..\Libraries\libs\libbtstack.a(hct_msg.o)
 .data          0x0000000000000000        0x0 ..\..\..\Libraries\libs\libbtstack.a(hct_fc.o)
 .bss           0x0000000000000000        0x0 ..\..\..\Libraries\libs\libbtstack.a(hct_fc.o)
 .data          0x0000000000000000        0x0 ..\..\..\Libraries\libs\libbtstack.a(hct.o)
 .bss           0x0000000000000000        0x0 ..\..\..\Libraries\libs\libbtstack.a(hct.o)
 .text          0x0000000000000000        0x0 ..\..\..\Libraries\libs\libbtstack.a(tws_sco.o)
 .data          0x0000000000000000        0x0 ..\..\..\Libraries\libs\libbtstack.a(tws_sco.o)
 .bss           0x0000000000000000        0x0 ..\..\..\Libraries\libs\libbtstack.a(tws_sco.o)
 .text          0x0000000000000000        0x0 ..\..\..\Libraries\libs\libbtstack.a(tws_acl.o)
 .data          0x0000000000000000        0x0 ..\..\..\Libraries\libs\libbtstack.a(tws_acl.o)
 .bss           0x0000000000000000        0x0 ..\..\..\Libraries\libs\libbtstack.a(tws_acl.o)
 .data          0x0000000000000000        0x0 ..\..\..\Libraries\libs\libbtstack.a(lm.o)
 .bss           0x0000000000000000        0x0 ..\..\..\Libraries\libs\libbtstack.a(lm.o)
 .data          0x0000000000000000        0x0 ..\..\..\Libraries\libs\libbtstack.a(bt_hal.o)
 .bss           0x0000000000000000        0x0 ..\..\..\Libraries\libs\libbtstack.a(bt_hal.o)
 .com_rodata.bb.tbl
                0x0000000000000000       0x2a ..\..\..\Libraries\libs\libbtstack.a(bt_hal.o)
 .data          0x0000000000000000        0x0 ..\..\..\Libraries\libs\libbtstack.a(bt21.o)
 .bss           0x0000000000000000        0x0 ..\..\..\Libraries\libs\libbtstack.a(bt21.o)
 .com_text.bb.sleep
                0x0000000000000000       0x4e ..\..\..\Libraries\libs\libbtstack.a(bt21.o)
 .data          0x0000000000000000        0x0 ..\..\..\Libraries\libs\libbtstack.a(bc.o)
 .data          0x0000000000000000        0x0 ..\..\..\Libraries\libs\libbtstack.a(ble_hal.o)
 .bss           0x0000000000000000        0x0 ..\..\..\Libraries\libs\libbtstack.a(ble_hal.o)
 .data          0x0000000000000000        0x0 ..\..\..\Libraries\libs\libbtstack.a(ble_adv.o)
 .bss           0x0000000000000000        0x0 ..\..\..\Libraries\libs\libbtstack.a(ble_adv.o)
 .data          0x0000000000000000        0x0 ..\..\..\Libraries\libs\libbtstack.a(ble.o)
 .bss           0x0000000000000000        0x0 ..\..\..\Libraries\libs\libbtstack.a(ble.o)
 .data          0x0000000000000000        0x0 ..\..\..\Libraries\libs\libbtstack.a(extern_ble.o)
 .bss           0x0000000000000000        0x0 ..\..\..\Libraries\libs\libbtstack.a(extern_ble.o)
 .sbss          0x0000000000000000        0x1 ..\..\..\Libraries\libs\libbtstack.a(extern_ble.o)
 .srodata       0x0000000000000000        0x2 ..\..\..\Libraries\libs\libbtstack.a(extern_ble.o)
 .data          0x0000000000000000        0x0 ..\..\..\Libraries\libs\libbtstack.a(l2cap_test.o)
 .data          0x0000000000000000        0x0 ..\..\..\Libraries\libs\libbtstack.a(l2cap.o)
 .bss           0x0000000000000000        0x0 ..\..\..\Libraries\libs\libbtstack.a(l2cap.o)
 .sbss          0x0000000000000000        0x1 ..\..\..\Libraries\libs\libbtstack.a(l2cap.o)
 .text          0x0000000000000000        0x4 ..\..\..\Libraries\libs\libbtstack.a(hci_sco.o)
 .data          0x0000000000000000        0x0 ..\..\..\Libraries\libs\libbtstack.a(hci_sco.o)
 .bss           0x0000000000000000        0x0 ..\..\..\Libraries\libs\libbtstack.a(hci_sco.o)
 .sbss          0x0000000000000000        0x1 ..\..\..\Libraries\libs\libbtstack.a(hci_sco.o)
 .text          0x0000000000000000       0x18 ..\..\..\Libraries\libs\libbtstack.a(hci_dump.o)
 .data          0x0000000000000000        0xc ..\..\..\Libraries\libs\libbtstack.a(hci_dump.o)
 .bss           0x0000000000000000        0x0 ..\..\..\Libraries\libs\libbtstack.a(hci_dump.o)
 .rodata.str1.4
                0x0000000000000000       0x12 ..\..\..\Libraries\libs\libbtstack.a(hci_dump.o)
 .text.stack.util
                0x0000000000000000       0x82 ..\..\..\Libraries\libs\libbtstack.a(hci_dump.o)
 .text          0x0000000000000000        0x0 ..\..\..\Libraries\libs\libbtstack.a(hci_cmd.o)
 .data          0x0000000000000000        0x0 ..\..\..\Libraries\libs\libbtstack.a(hci_cmd.o)
 .bss           0x0000000000000000        0x0 ..\..\..\Libraries\libs\libbtstack.a(hci_cmd.o)
 .data          0x0000000000000000        0x0 ..\..\..\Libraries\libs\libbtstack.a(hci.o)
 .bss           0x0000000000000000        0x0 ..\..\..\Libraries\libs\libbtstack.a(hci.o)
 .com_text.timer
                0x0000000000000000        0xe ..\..\..\Libraries\libs\libbtstack.a(hci.o)
 .com_text.sco  0x0000000000000000        0xe ..\..\..\Libraries\libs\libbtstack.a(hci.o)
 .rodata.stack.hci_init
                0x0000000000000000       0x11 ..\..\..\Libraries\libs\libbtstack.a(hci.o)
 .data          0x0000000000000000        0x0 ..\..\..\Libraries\libs\libbtstack.a(hid_usage.o)
 .bss           0x0000000000000000        0x0 ..\..\..\Libraries\libs\libbtstack.a(hid_usage.o)
 .text.stack.api.hid_touch
                0x0000000000000000        0xa ..\..\..\Libraries\libs\libbtstack.a(hid_usage.o)
 .srodata       0x0000000000000000        0xe ..\..\..\Libraries\libs\libbtstack.a(hid_usage.o)
 .data          0x0000000000000000        0x0 ..\..\..\Libraries\libs\libbtstack.a(hid_device.o)
 .bss           0x0000000000000000        0x0 ..\..\..\Libraries\libs\libbtstack.a(hid_device.o)
 .sbss          0x0000000000000000        0x1 ..\..\..\Libraries\libs\libbtstack.a(hid_device.o)
 .data          0x0000000000000000        0x0 ..\..\..\Libraries\libs\libbtstack.a(hfp_hf.o)
 .bss           0x0000000000000000        0x0 ..\..\..\Libraries\libs\libbtstack.a(hfp_hf.o)
 .data          0x0000000000000000        0x0 ..\..\..\Libraries\libs\libbtstack.a(hfp.o)
 .bss           0x0000000000000000        0x0 ..\..\..\Libraries\libs\libbtstack.a(hfp.o)
 .sbss          0x0000000000000000        0x1 ..\..\..\Libraries\libs\libbtstack.a(hfp.o)
 .text          0x0000000000000000        0x0 ..\..\..\Libraries\libs\libbtstack.a(avdtp.o)
 .data          0x0000000000000000        0x0 ..\..\..\Libraries\libs\libbtstack.a(avdtp.o)
 .bss           0x0000000000000000        0x0 ..\..\..\Libraries\libs\libbtstack.a(avdtp.o)
 .com_text.acl.pend
                0x0000000000000000        0x4 ..\..\..\Libraries\libs\libbtstack.a(avdtp.o)
 .sbss          0x0000000000000000        0x1 ..\..\..\Libraries\libs\libbtstack.a(avdtp.o)
 .data          0x0000000000000000        0x0 ..\..\..\Libraries\libs\libbtstack.a(a2dp.o)
 .bss           0x0000000000000000        0x0 ..\..\..\Libraries\libs\libbtstack.a(a2dp.o)
 .sbss          0x0000000000000000        0x1 ..\..\..\Libraries\libs\libbtstack.a(a2dp.o)
 .text          0x0000000000000000        0x0 ..\..\..\Libraries\libs\libbtstack.a(btstack_memory_pool.o)
 .data          0x0000000000000000        0x0 ..\..\..\Libraries\libs\libbtstack.a(btstack_memory_pool.o)
 .bss           0x0000000000000000        0x0 ..\..\..\Libraries\libs\libbtstack.a(btstack_memory_pool.o)
 .data          0x0000000000000000        0x0 ..\..\..\Libraries\libs\libbtstack.a(btstack_adv0.o)
 .bss           0x0000000000000000        0x0 ..\..\..\Libraries\libs\libbtstack.a(btstack_adv0.o)
 .sbss          0x0000000000000000        0x1 ..\..\..\Libraries\libs\libbtstack.a(btstack_adv0.o)
 .data          0x0000000000000000        0x0 ..\..\..\Libraries\libs\libbtstack.a(hci_transport_hcic.o)
 .bss           0x0000000000000000        0x0 ..\..\..\Libraries\libs\libbtstack.a(hci_transport_hcic.o)
 .data          0x0000000000000000        0x0 ..\..\..\Libraries\libs\libbtstack.a(btstack_chipset_inner.o)
 .bss           0x0000000000000000        0x0 ..\..\..\Libraries\libs\libbtstack.a(btstack_chipset_inner.o)
 .data          0x0000000000000000        0x0 ..\..\..\Libraries\libs\libbtstack.a(lm_hook.o)
 .bss           0x0000000000000000        0x0 ..\..\..\Libraries\libs\libbtstack.a(lm_hook.o)
 .data          0x0000000000000000        0x0 ..\..\..\Libraries\libs\libbtstack.a(lm_sp.o)
 .text.lm.sha256
                0x0000000000000000      0x13a ..\..\..\Libraries\libs\libbtstack.a(lm_sp.o)
 .data          0x0000000000000000        0x0 ..\..\..\Libraries\libs\libbtstack.a(lm_proc.o)
 .bss           0x0000000000000000        0x0 ..\..\..\Libraries\libs\libbtstack.a(lm_proc.o)
 .text.bb.lm.inq.start
                0x0000000000000000      0x104 ..\..\..\Libraries\libs\libbtstack.a(lm_proc.o)
 .text.bb.lm.inq.stop
                0x0000000000000000       0x32 ..\..\..\Libraries\libs\libbtstack.a(lm_proc.o)
 .text.bb.lm.inq.res
                0x0000000000000000      0x222 ..\..\..\Libraries\libs\libbtstack.a(lm_proc.o)
 .data          0x0000000000000000        0x0 ..\..\..\Libraries\libs\libbtstack.a(lm_key.o)
 .bss           0x0000000000000000        0x0 ..\..\..\Libraries\libs\libbtstack.a(lm_key.o)
 .data          0x0000000000000000        0x0 ..\..\..\Libraries\libs\libbtstack.a(lc.o)
 .bss           0x0000000000000000        0x0 ..\..\..\Libraries\libs\libbtstack.a(lc.o)
 .com_text.lc   0x0000000000000000       0x9c ..\..\..\Libraries\libs\libbtstack.a(lc.o)
 .data          0x0000000000000000        0x0 ..\..\..\Libraries\libs\libbtstack.a(mgr.o)
 .bss           0x0000000000000000        0x0 ..\..\..\Libraries\libs\libbtstack.a(mgr.o)
 .text          0x0000000000000000        0x0 ..\..\..\Libraries\libs\libbtstack.a(ll.o)
 .data          0x0000000000000000        0x0 ..\..\..\Libraries\libs\libbtstack.a(ll.o)
 .bss           0x0000000000000000        0x0 ..\..\..\Libraries\libs\libbtstack.a(ll.o)
 .data          0x0000000000000000        0x0 ..\..\..\Libraries\libs\libbtstack.a(ble_test.o)
 .bss           0x0000000000000000        0x0 ..\..\..\Libraries\libs\libbtstack.a(ble_test.o)
 .com_text.ble.isr.test
                0x0000000000000000      0x17a ..\..\..\Libraries\libs\libbtstack.a(ble_test.o)
 .com_text.ble.isr.test.ind
                0x0000000000000000       0x5a ..\..\..\Libraries\libs\libbtstack.a(ble_test.o)
 .text.bb.ble.test.start
                0x0000000000000000      0x4b0 ..\..\..\Libraries\libs\libbtstack.a(ble_test.o)
 .text.bb.ble.test.stop
                0x0000000000000000      0x200 ..\..\..\Libraries\libs\libbtstack.a(ble_test.o)
 .srodata       0x0000000000000000        0x7 ..\..\..\Libraries\libs\libbtstack.a(ble_test.o)
 .data          0x0000000000000000        0x0 ..\..\..\Libraries\libs\libbtstack.a(ble_scan.o)
 .bss           0x0000000000000000        0x0 ..\..\..\Libraries\libs\libbtstack.a(ble_scan.o)
 .com_rodata.bb.tbl
                0x0000000000000000       0x10 ..\..\..\Libraries\libs\libbtstack.a(ble_scan.o)
 .data          0x0000000000000000        0x0 ..\..\..\Libraries\libs\libbtstack.a(ble_per_adv.o)
 .bss           0x0000000000000000        0x0 ..\..\..\Libraries\libs\libbtstack.a(ble_per_adv.o)
 .data          0x0000000000000000        0x0 ..\..\..\Libraries\libs\libbtstack.a(ble_init.o)
 .bss           0x0000000000000000        0x0 ..\..\..\Libraries\libs\libbtstack.a(ble_init.o)
 .data          0x0000000000000000        0x0 ..\..\..\Libraries\libs\libbtstack.a(ble_buf.o)
 .text          0x0000000000000000        0x0 ..\..\..\Libraries\libs\libbtstack.a(ble_adv0.o)
 .data          0x0000000000000000        0x0 ..\..\..\Libraries\libs\libbtstack.a(ble_adv0.o)
 .bss           0x0000000000000000        0x0 ..\..\..\Libraries\libs\libbtstack.a(ble_adv0.o)
 .data          0x0000000000000000        0x0 ..\..\..\Libraries\libs\libbtstack.a(extern_hfhs.o)
 .bss           0x0000000000000000        0x0 ..\..\..\Libraries\libs\libbtstack.a(extern_hfhs.o)
 .sbss          0x0000000000000000        0x1 ..\..\..\Libraries\libs\libbtstack.a(extern_hfhs.o)
 .srodata       0x0000000000000000        0x1 ..\..\..\Libraries\libs\libbtstack.a(extern_hfhs.o)
 .text          0x0000000000000000       0x38 ..\..\..\Libraries\libs\libbtstack.a(l2cap_signaling.o)
 .data          0x0000000000000000        0x0 ..\..\..\Libraries\libs\libbtstack.a(l2cap_signaling.o)
 .bss           0x0000000000000000        0x0 ..\..\..\Libraries\libs\libbtstack.a(l2cap_signaling.o)
 .data          0x0000000000000000        0x0 ..\..\..\Libraries\libs\libbtstack.a(lc_hook.o)
 .bss           0x0000000000000000        0x0 ..\..\..\Libraries\libs\libbtstack.a(lc_hook.o)
 .data          0x0000000000000000        0x0 ..\..\..\Libraries\libs\libbtstack.a(lm_sco.o)
 .bss           0x0000000000000000        0x0 ..\..\..\Libraries\libs\libbtstack.a(lm_sco.o)
 .data          0x0000000000000000        0x0 ..\..\..\Libraries\libs\libbtstack.a(lc_util.o)
 .bss           0x0000000000000000        0x0 ..\..\..\Libraries\libs\libbtstack.a(lc_util.o)
 .data          0x0000000000000000        0x0 ..\..\..\Libraries\libs\libbtstack.a(lc_sniff.o)
 .bss           0x0000000000000000        0x0 ..\..\..\Libraries\libs\libbtstack.a(lc_sniff.o)
 .data          0x0000000000000000        0x0 ..\..\..\Libraries\libs\libbtstack.a(lc_sco.o)
 .bss           0x0000000000000000        0x0 ..\..\..\Libraries\libs\libbtstack.a(lc_sco.o)
 .data          0x0000000000000000        0x0 ..\..\..\Libraries\libs\libbtstack.a(lc_proc.o)
 .bss           0x0000000000000000        0x0 ..\..\..\Libraries\libs\libbtstack.a(lc_proc.o)
 .data          0x0000000000000000        0x0 ..\..\..\Libraries\libs\libbtstack.a(lc_lmppdu.o)
 .bss           0x0000000000000000        0x0 ..\..\..\Libraries\libs\libbtstack.a(lc_lmppdu.o)
 .data          0x0000000000000000        0x0 ..\..\..\Libraries\libs\libbtstack.a(mgr_proc.o)
 .bss           0x0000000000000000        0x0 ..\..\..\Libraries\libs\libbtstack.a(mgr_proc.o)
 .data          0x0000000000000000        0x0 ..\..\..\Libraries\libs\libbtstack.a(mgr_init.o)
 .bss           0x0000000000000000        0x0 ..\..\..\Libraries\libs\libbtstack.a(mgr_init.o)
 .data          0x0000000000000000        0x0 ..\..\..\Libraries\libs\libbtstack.a(mgr_hci.o)
 .bss           0x0000000000000000        0x0 ..\..\..\Libraries\libs\libbtstack.a(mgr_hci.o)
 .data          0x0000000000000000        0x0 ..\..\..\Libraries\libs\libbtstack.a(ll_scan.o)
 .bss           0x0000000000000000        0x0 ..\..\..\Libraries\libs\libbtstack.a(ll_scan.o)
 .data          0x0000000000000000        0x0 ..\..\..\Libraries\libs\libbtstack.a(ll_adv.o)
 .bss           0x0000000000000000        0x0 ..\..\..\Libraries\libs\libbtstack.a(ll_adv.o)
 .data          0x0000000000000000        0x0 ..\..\..\Libraries\libs\libbtstack.a(ll_proc.o)
 .data          0x0000000000000000        0x0 ..\..\..\Libraries\libs\libbtstack.a(ll_ping.o)
 .bss           0x0000000000000000        0x0 ..\..\..\Libraries\libs\libbtstack.a(ll_ping.o)
 .data          0x0000000000000000        0x0 ..\..\..\Libraries\libs\libbtstack.a(ll_phy_upd.o)
 .bss           0x0000000000000000        0x0 ..\..\..\Libraries\libs\libbtstack.a(ll_phy_upd.o)
 .data          0x0000000000000000        0x0 ..\..\..\Libraries\libs\libbtstack.a(ll_past.o)
 .bss           0x0000000000000000        0x0 ..\..\..\Libraries\libs\libbtstack.a(ll_past.o)
 .data          0x0000000000000000        0x0 ..\..\..\Libraries\libs\libbtstack.a(ll_length.o)
 .bss           0x0000000000000000        0x0 ..\..\..\Libraries\libs\libbtstack.a(ll_length.o)
 .data          0x0000000000000000        0x0 ..\..\..\Libraries\libs\libbtstack.a(ll_feature.o)
 .bss           0x0000000000000000        0x0 ..\..\..\Libraries\libs\libbtstack.a(ll_feature.o)
 .data          0x0000000000000000        0x0 ..\..\..\Libraries\libs\libbtstack.a(ll_encrypt.o)
 .bss           0x0000000000000000        0x0 ..\..\..\Libraries\libs\libbtstack.a(ll_encrypt.o)
 .data          0x0000000000000000        0x0 ..\..\..\Libraries\libs\libbtstack.a(ll_disconnect.o)
 .bss           0x0000000000000000        0x0 ..\..\..\Libraries\libs\libbtstack.a(ll_disconnect.o)
 .data          0x0000000000000000        0x0 ..\..\..\Libraries\libs\libbtstack.a(ll_con_upd.o)
 .bss           0x0000000000000000        0x0 ..\..\..\Libraries\libs\libbtstack.a(ll_con_upd.o)
 .data          0x0000000000000000        0x0 ..\..\..\Libraries\libs\libbtstack.a(ll_cntl.o)
 .bss           0x0000000000000000        0x0 ..\..\..\Libraries\libs\libbtstack.a(ll_cntl.o)
 .data          0x0000000000000000        0x0 ..\..\..\Libraries\libs\libbtstack.a(ll_clk_acc.o)
 .bss           0x0000000000000000        0x0 ..\..\..\Libraries\libs\libbtstack.a(ll_clk_acc.o)
 .data          0x0000000000000000        0x0 ..\..\..\Libraries\libs\libbtstack.a(ll_chmap_upd.o)
 .bss           0x0000000000000000        0x0 ..\..\..\Libraries\libs\libbtstack.a(ll_chmap_upd.o)
 .data          0x0000000000000000        0x0 ..\..\..\Libraries\libs\libbtstack.a(aes_rpa.o)
 .bss           0x0000000000000000        0x0 ..\..\..\Libraries\libs\libbtstack.a(aes_rpa.o)
 .data          0x0000000000000000        0x0 ..\..\..\Libraries\libs\libbtstack.a(scan_hook.o)
 .bss           0x0000000000000000        0x0 ..\..\..\Libraries\libs\libbtstack.a(scan_hook.o)
 .data          0x0000000000000000        0x0 ..\..\..\Libraries\libs\libbtstack.a(adv_hook.o)
 .bss           0x0000000000000000        0x0 ..\..\..\Libraries\libs\libbtstack.a(adv_hook.o)
 .data          0x0000000000000000        0x0 ..\..\..\Libraries\libs\libbtstack.a(ll_version.o)
 .bss           0x0000000000000000        0x0 ..\..\..\Libraries\libs\libbtstack.a(ll_version.o)
 .data          0x0000000000000000        0x0 ..\..\..\Libraries\libs\libbtstack.a(ll_pwr.o)
 .bss           0x0000000000000000        0x0 ..\..\..\Libraries\libs\libbtstack.a(ll_pwr.o)
 .text          0x0000000000000000        0x0 ..\..\..\Libraries\libs\libdrivers.a(usb_device_hid.o)
 .data          0x0000000000000000        0x0 ..\..\..\Libraries\libs\libdrivers.a(usb_device_hid.o)
 .bss           0x0000000000000000        0x0 ..\..\..\Libraries\libs\libdrivers.a(usb_device_hid.o)
 .com_text.bulkep
                0x0000000000000000       0x80 ..\..\..\Libraries\libs\libdrivers.a(usb_device_hid.o)
 .text.usb_hid_ep_config
                0x0000000000000000        0xa ..\..\..\Libraries\libs\libdrivers.a(usb_device_hid.o)
 .text.usb_user_ep_config
                0x0000000000000000       0x2e ..\..\..\Libraries\libs\libdrivers.a(usb_device_hid.o)
 .text          0x0000000000000000        0x0 ..\..\..\Libraries\libs\libdrivers.a(usb_device_printer.o)
 .data          0x0000000000000000        0x0 ..\..\..\Libraries\libs\libdrivers.a(usb_device_printer.o)
 .bss           0x0000000000000000        0x0 ..\..\..\Libraries\libs\libdrivers.a(usb_device_printer.o)
 .com_text.bulkep
                0x0000000000000000       0xaa ..\..\..\Libraries\libs\libdrivers.a(usb_device_printer.o)
 .text.usb_printer_ep_config
                0x0000000000000000       0x12 ..\..\..\Libraries\libs\libdrivers.a(usb_device_printer.o)
 .text.udp_init
                0x0000000000000000       0xa2 ..\..\..\Libraries\libs\libdrivers.a(usb_device_printer.o)
 .sdata         0x0000000000000000        0x2 ..\..\..\Libraries\libs\libdrivers.a(usb_device_printer.o)
 .text          0x0000000000000000        0x0 ..\..\..\Libraries\libs\libdrivers.a(usb_device_run_loop.o)
 .data          0x0000000000000000        0x0 ..\..\..\Libraries\libs\libdrivers.a(usb_device_run_loop.o)
 .bss           0x0000000000000000        0x0 ..\..\..\Libraries\libs\libdrivers.a(usb_device_run_loop.o)
 .text.usb_device_exit
                0x0000000000000000       0x32 ..\..\..\Libraries\libs\libdrivers.a(usb_device_run_loop.o)
 .usbdev.com    0x0000000000000000       0xa8 ..\..\..\Libraries\libs\libdrivers.a(usb_device_run_loop.o)
 .text.usb_device_init
                0x0000000000000000       0xac ..\..\..\Libraries\libs\libdrivers.a(usb_device_run_loop.o)
 .text.usb_device_enter
                0x0000000000000000       0x74 ..\..\..\Libraries\libs\libdrivers.a(usb_device_run_loop.o)
 .com_text.usb.device
                0x0000000000000000       0x62 ..\..\..\Libraries\libs\libdrivers.a(usb_device_run_loop.o)
 .com_text.irq  0x0000000000000000       0x10 ..\..\..\Libraries\libs\libdrivers.a(usb_device_run_loop.o)
 .usb_buf.device.desc.buf
                0x0000000000000000      0x400 ..\..\..\Libraries\libs\libdrivers.a(usb_device_run_loop.o)
 .usb_buf.isoc  0x0000000000000000      0x140 ..\..\..\Libraries\libs\libdrivers.a(usb_device_run_loop.o)
 .usb_buf.printer
                0x0000000000000000       0x80 ..\..\..\Libraries\libs\libdrivers.a(usb_device_run_loop.o)
 .text          0x0000000000000000        0x0 ..\..\..\Libraries\libs\libdrivers.a(usb_host_manage.o)
 .data          0x0000000000000000        0x0 ..\..\..\Libraries\libs\libdrivers.a(usb_host_manage.o)
 .bss           0x0000000000000000        0x0 ..\..\..\Libraries\libs\libdrivers.a(usb_host_manage.o)
 .text.usb_host_var_init
                0x0000000000000000       0x3c ..\..\..\Libraries\libs\libdrivers.a(usb_host_manage.o)
 .text.uhs_is_iphone
                0x0000000000000000       0x12 ..\..\..\Libraries\libs\libdrivers.a(usb_host_manage.o)
 .text.usb.host.init
                0x0000000000000000       0x96 ..\..\..\Libraries\libs\libdrivers.a(usb_host_manage.o)
 .com_text.irq  0x0000000000000000       0x12 ..\..\..\Libraries\libs\libdrivers.a(usb_host_manage.o)
 .text.udisk_suspend
                0x0000000000000000       0x32 ..\..\..\Libraries\libs\libdrivers.a(usb_host_manage.o)
 .text.udisk_resume
                0x0000000000000000       0x4c ..\..\..\Libraries\libs\libdrivers.a(usb_host_manage.o)
 .com_text.usb.host
                0x0000000000000000       0x82 ..\..\..\Libraries\libs\libdrivers.a(usb_host_manage.o)
 .text.udisk_read
                0x0000000000000000       0x7c ..\..\..\Libraries\libs\libdrivers.a(usb_host_manage.o)
 .text.uhs_set_nluns
                0x0000000000000000        0xa ..\..\..\Libraries\libs\libdrivers.a(usb_host_manage.o)
 .text.udisk_write
                0x0000000000000000       0x54 ..\..\..\Libraries\libs\libdrivers.a(usb_host_manage.o)
 .buf.usb       0x0000000000000000       0x74 ..\..\..\Libraries\libs\libdrivers.a(usb_host_manage.o)
 .comment       0x0000000000000000       0x13 ..\..\..\Libraries\libs\libdrivers.a(usb_host_manage.o)
 .riscv.attributes
                0x0000000000000000       0x32 ..\..\..\Libraries\libs\libdrivers.a(usb_host_manage.o)
 .text          0x0000000000000000        0x0 ..\..\..\Libraries\libs\libdrivers.a(usb_host_storage.o)
 .data          0x0000000000000000        0x0 ..\..\..\Libraries\libs\libdrivers.a(usb_host_storage.o)
 .bss           0x0000000000000000        0x0 ..\..\..\Libraries\libs\libdrivers.a(usb_host_storage.o)
 .text.do_transfer
                0x0000000000000000       0xae ..\..\..\Libraries\libs\libdrivers.a(usb_host_storage.o)
 .text.do_receive
                0x0000000000000000       0xf6 ..\..\..\Libraries\libs\libdrivers.a(usb_host_storage.o)
 .text.do_request
                0x0000000000000000      0x20a ..\..\..\Libraries\libs\libdrivers.a(usb_host_storage.o)
 .text.do_scsi_request
                0x0000000000000000       0xf8 ..\..\..\Libraries\libs\libdrivers.a(usb_host_storage.o)
 .text.uhs_start
                0x0000000000000000      0x18c ..\..\..\Libraries\libs\libdrivers.a(usb_host_storage.o)
 .text.uhs_read
                0x0000000000000000       0x64 ..\..\..\Libraries\libs\libdrivers.a(usb_host_storage.o)
 .text.uhs_write
                0x0000000000000000       0x64 ..\..\..\Libraries\libs\libdrivers.a(usb_host_storage.o)
 .text.uhs_init
                0x0000000000000000       0x26 ..\..\..\Libraries\libs\libdrivers.a(usb_host_storage.o)
 .rodata        0x0000000000000000       0x57 ..\..\..\Libraries\libs\libdrivers.a(usb_host_storage.o)
 .comment       0x0000000000000000       0x13 ..\..\..\Libraries\libs\libdrivers.a(usb_host_storage.o)
 .riscv.attributes
                0x0000000000000000       0x32 ..\..\..\Libraries\libs\libdrivers.a(usb_host_storage.o)
 .text          0x0000000000000000        0x0 ..\..\..\Libraries\libs\libdrivers.a(usb_comm.o)
 .data          0x0000000000000000        0x0 ..\..\..\Libraries\libs\libdrivers.a(usb_comm.o)
 .bss           0x0000000000000000        0x0 ..\..\..\Libraries\libs\libdrivers.a(usb_comm.o)
 .text.usb_init
                0x0000000000000000       0x80 ..\..\..\Libraries\libs\libdrivers.a(usb_comm.o)
 .text.usb_host_enter
                0x0000000000000000       0x56 ..\..\..\Libraries\libs\libdrivers.a(usb_comm.o)
 .usbdev.com    0x0000000000000000       0x20 ..\..\..\Libraries\libs\libdrivers.a(usb_comm.o)
 .com_text.irq  0x0000000000000000       0x2a ..\..\..\Libraries\libs\libdrivers.a(usb_comm.o)
 .buf.usb.ctrl  0x0000000000000000       0x40 ..\..\..\Libraries\libs\libdrivers.a(usb_comm.o)
 .text          0x0000000000000000        0x0 ..\..\..\Libraries\libs\libdrivers.a(usb_detect.o)
 .data          0x0000000000000000        0x0 ..\..\..\Libraries\libs\libdrivers.a(usb_detect.o)
 .bss           0x0000000000000000        0x0 ..\..\..\Libraries\libs\libdrivers.a(usb_detect.o)
 .com_text.usb.dectect
                0x0000000000000000      0x108 ..\..\..\Libraries\libs\libdrivers.a(usb_detect.o)
 .buf.usbchk.cb
                0x0000000000000000        0x2 ..\..\..\Libraries\libs\libdrivers.a(usb_detect.o)
 .comment       0x0000000000000000       0x13 ..\..\..\Libraries\libs\libdrivers.a(usb_detect.o)
 .riscv.attributes
                0x0000000000000000       0x32 ..\..\..\Libraries\libs\libdrivers.a(usb_detect.o)
 .text          0x0000000000000000        0x0 ..\..\..\Libraries\libs\libdrivers.a(usb_device_desc.o)
 .data          0x0000000000000000        0x0 ..\..\..\Libraries\libs\libdrivers.a(usb_device_desc.o)
 .bss           0x0000000000000000        0x0 ..\..\..\Libraries\libs\libdrivers.a(usb_device_desc.o)
 .text.usb_get_device_descriptor
                0x0000000000000000        0x8 ..\..\..\Libraries\libs\libdrivers.a(usb_device_desc.o)
 .text.usb_get_config_descriptor
                0x0000000000000000        0x8 ..\..\..\Libraries\libs\libdrivers.a(usb_device_desc.o)
 .text.usb_get_lang_id_str_descriptor
                0x0000000000000000        0x8 ..\..\..\Libraries\libs\libdrivers.a(usb_device_desc.o)
 .text.usb_get_manufacturer_str_descriptor
                0x0000000000000000        0x8 ..\..\..\Libraries\libs\libdrivers.a(usb_device_desc.o)
 .text.usb_get_product_str_descriptor
                0x0000000000000000        0x8 ..\..\..\Libraries\libs\libdrivers.a(usb_device_desc.o)
 .text.usb_get_serial_str_descriptor
                0x0000000000000000        0x8 ..\..\..\Libraries\libs\libdrivers.a(usb_device_desc.o)
 .text.usb_get_hid_config_descriptor
                0x0000000000000000        0x8 ..\..\..\Libraries\libs\libdrivers.a(usb_device_desc.o)
 .text.usb_get_hid_report_descriptor
                0x0000000000000000        0x8 ..\..\..\Libraries\libs\libdrivers.a(usb_device_desc.o)
 .comment       0x0000000000000000       0x13 ..\..\..\Libraries\libs\libdrivers.a(usb_device_desc.o)
 .riscv.attributes
                0x0000000000000000       0x32 ..\..\..\Libraries\libs\libdrivers.a(usb_device_desc.o)
 .text          0x0000000000000000        0x0 ..\..\..\Libraries\libs\libdrivers.a(usb_device_enum.o)
 .data          0x0000000000000000        0x0 ..\..\..\Libraries\libs\libdrivers.a(usb_device_enum.o)
 .bss           0x0000000000000000        0xa ..\..\..\Libraries\libs\libdrivers.a(usb_device_enum.o)
 .usbdev.com    0x0000000000000000      0x9c2 ..\..\..\Libraries\libs\libdrivers.a(usb_device_enum.o)
 .text.usb_ep0_out_data_callback
                0x0000000000000000        0x4 ..\..\..\Libraries\libs\libdrivers.a(usb_device_enum.o)
 .text.usb_itf_in_req
                0x0000000000000000        0x4 ..\..\..\Libraries\libs\libdrivers.a(usb_device_enum.o)
 .comment       0x0000000000000000       0x13 ..\..\..\Libraries\libs\libdrivers.a(usb_device_enum.o)
 .riscv.attributes
                0x0000000000000000       0x32 ..\..\..\Libraries\libs\libdrivers.a(usb_device_enum.o)
 .text          0x0000000000000000        0x0 ..\..\..\Libraries\libs\libdrivers.a(usb_device_ep.o)
 .data          0x0000000000000000        0x0 ..\..\..\Libraries\libs\libdrivers.a(usb_device_ep.o)
 .text          0x0000000000000000        0x0 ..\..\..\Libraries\libs\libdrivers.a(usb_host_enum.o)
 .data          0x0000000000000000        0x0 ..\..\..\Libraries\libs\libdrivers.a(usb_host_enum.o)
 .bss           0x0000000000000000        0x0 ..\..\..\Libraries\libs\libdrivers.a(usb_host_enum.o)
 .text.wait_transfering
                0x0000000000000000       0x3c ..\..\..\Libraries\libs\libdrivers.a(usb_host_enum.o)
 .text.do_receive
                0x0000000000000000       0x90 ..\..\..\Libraries\libs\libdrivers.a(usb_host_enum.o)
 .text.do_skip_rxdata
                0x0000000000000000       0x4c ..\..\..\Libraries\libs\libdrivers.a(usb_host_enum.o)
 .text.do_request.isra.0
                0x0000000000000000      0x298 ..\..\..\Libraries\libs\libdrivers.a(usb_host_enum.o)
 .text.uhe_reset
                0x0000000000000000       0x34 ..\..\..\Libraries\libs\libdrivers.a(usb_host_enum.o)
 .rodata.str1.4
                0x0000000000000000        0xb ..\..\..\Libraries\libs\libdrivers.a(usb_host_enum.o)
 .text.uhe_start
                0x0000000000000000      0x22c ..\..\..\Libraries\libs\libdrivers.a(usb_host_enum.o)
 .text.uhe_clear_feature
                0x0000000000000000       0x44 ..\..\..\Libraries\libs\libdrivers.a(usb_host_enum.o)
 .text.uhe_init
                0x0000000000000000       0x24 ..\..\..\Libraries\libs\libdrivers.a(usb_host_enum.o)
 .rodata        0x0000000000000000       0x40 ..\..\..\Libraries\libs\libdrivers.a(usb_host_enum.o)
 .rodata.uhe    0x0000000000000000       0x40 ..\..\..\Libraries\libs\libdrivers.a(usb_host_enum.o)
 .comment       0x0000000000000000       0x13 ..\..\..\Libraries\libs\libdrivers.a(usb_host_enum.o)
 .riscv.attributes
                0x0000000000000000       0x32 ..\..\..\Libraries\libs\libdrivers.a(usb_host_enum.o)
 .text          0x0000000000000000        0x0 ..\..\..\Libraries\libs\libdrivers.a(weak_symbol.o)
 .data          0x0000000000000000        0x0 ..\..\..\Libraries\libs\libdrivers.a(weak_symbol.o)
 .bss           0x0000000000000000        0x0 ..\..\..\Libraries\libs\libdrivers.a(weak_symbol.o)
 .text.iphone_power_set
                0x0000000000000000       0x12 ..\..\..\Libraries\libs\libdrivers.a(weak_symbol.o)
 .comment       0x0000000000000000       0x13 ..\..\..\Libraries\libs\libdrivers.a(weak_symbol.o)
 .riscv.attributes
                0x0000000000000000       0x32 ..\..\..\Libraries\libs\libdrivers.a(weak_symbol.o)
 .text          0x0000000000000000        0x0 ..\..\..\Libraries\libs\libdrivers.a(usb_device_audio.o)
 .data          0x0000000000000000        0x0 ..\..\..\Libraries\libs\libdrivers.a(usb_device_audio.o)
 .bss           0x0000000000000000        0x0 ..\..\..\Libraries\libs\libdrivers.a(usb_device_audio.o)
 .usbdev.com    0x0000000000000000      0x36a ..\..\..\Libraries\libs\libdrivers.a(usb_device_audio.o)
 .ude.aubuf     0x0000000000000000      0x8d4 ..\..\..\Libraries\libs\libdrivers.a(usb_device_audio.o)
 .usbdev.com.table
                0x0000000000000000        0x3 ..\..\..\Libraries\libs\libdrivers.a(usb_device_audio.o)
 .comment       0x0000000000000000       0x13 ..\..\..\Libraries\libs\libdrivers.a(usb_device_audio.o)
 .riscv.attributes
                0x0000000000000000       0x32 ..\..\..\Libraries\libs\libdrivers.a(usb_device_audio.o)

Memory Configuration

Name             Origin             Length             Attributes
init             0x0000000010000000 0x0000000000000200
flash            0x0000000010000200 0x0000000000064000 xr
comm             0x0000000000017000 0x0000000000009000 xr
stack            0x0000000000010800 0x0000000000000400
heap             0x0000000000010c00 0x0000000000003000
data             0x0000000000013c00 0x0000000000003400
bram             0x0000000000020000 0x000000000000c000
cram             0x000000000002c000 0x0000000000014000
aram             0x0000000000050000 0x0000000000004000
dram             0x0000000000058000 0x0000000000004500
eram             0x0000000000054000 0x0000000000000a00
rram             0x0000000000055800 0x0000000000000260
*default*        0x0000000000000000 0xffffffffffffffff

Linker script and memory map

LOAD Output\obj\Libraries\bsp\bsp_bt.o
LOAD Output\obj\Libraries\bsp\bsp_cm.o
LOAD Output\obj\Libraries\bsp\bsp_fot.o
LOAD Output\obj\Libraries\bsp\bsp_param.o
LOAD Output\obj\Libraries\bsp\bsp_sys.o
LOAD Output\obj\Libraries\BT\ble\ab_link\app.o
LOAD Output\obj\Libraries\BT\ble\adv0.o
LOAD Output\obj\Libraries\BT\ble\ble.o
LOAD Output\obj\Libraries\BT\spp\bt.o
LOAD Output\obj\Libraries\BT\spp\hid.o
LOAD Output\obj\Libraries\BT\spp\profile.o
LOAD Output\obj\Libraries\BT\spp\spp.o
LOAD Output\obj\Libraries\Device\Source\gw3323_clk.o
LOAD Output\obj\Libraries\Device\Source\gw3323_gpio.o
LOAD Output\obj\Libraries\Device\Source\gw3323_spi.o
LOAD Output\obj\Libraries\libs\strong_symbol.o
LOAD Output\obj\Examples\Internal_Flash\Source\Internal_Flash.o
LOAD Output\obj\Examples\Internal_Flash\Project\config.o
LOAD Output\obj\Examples\Internal_Flash\Project\main.o
                0x0000000000064000                __max_flash_size = 0x64000
                0x0000000010000000                __base = 0x10000000
                0x0000000000010600                __cache_stack_vma = 0x10600
                0x0000000000000200                __cache_stack_size = 0x200
                0x0000000000010800                __stack_vma = 0x10800
                0x0000000000000400                __stack_ram_size = 0x400
                0x0000000000010c00                __heap_vma = 0x10c00
                0x0000000000003000                __heap_ram_size = 0x3000
                0x0000000000013c00                __data_vma = 0x13c00
                0x0000000000003400                __data_ram_size = 0x3400
                0x0000000000017000                __comm_vma = 0x17000
                0x0000000000009000                __comm_ram_size = 0x9000
                0x0000000000020000                __bram_vma = 0x20000
                0x000000000000c000                __bram_ram_size = 0xc000
                0x000000000002c000                __cram_vma = 0x2c000
                0x0000000000014000                __cram_ram_size = 0x14000
                0x0000000000050000                __aram_vma = 0x50000
                0x0000000000054000                __eram_vma = 0x54000
                0x0000000000058000                __dram_vma = 0x58000
                0x0000000000055800                __rram_vma = 0x55800

.init           0x0000000010000000       0x4e
 *(.reset)
 .reset         0x0000000010000000       0x4e ..\..\..\Libraries\libs\libplatform.a(reset.o)
                0x0000000010000000                _start

.comm           0x0000000000017000     0x6600 load address 0x0000000010000200
 *(.vector)
 .vector        0x0000000000017000      0x1a2 ..\..\..\Libraries\libs\libplatform.a(reset.o)
                0x00000000000170a0                _exception_isr
                0x00000000000170a2                nop_isr
 *(.plt)
 .plt           0x00000000000171a2       0x10 ..\..\..\Libraries\libs\libplatform.a(main.o)
 *(.com_text*)
 .com_text.fot  0x00000000000171b2       0x4e Output\obj\Libraries\bsp\bsp_fot.o
                0x00000000000171b2                fot_app_connect_auth
                0x00000000000171f4                bsp_fot_is_connect
 .com_text.const
                0x0000000000017200        0x7 Output\obj\Libraries\bsp\bsp_fot.o
 *fill*         0x0000000000017207        0x1 
 .com_text.timer
                0x0000000000017208       0x98 Output\obj\Libraries\bsp\bsp_sys.o
                0x0000000000017208                usr_tmr1ms_isr
                0x000000000001720a                usr_tmr5ms_thread
                0x0000000000017288                timer1_isr
 .com_text.sys  0x00000000000172a0        0x4 Output\obj\Libraries\bsp\bsp_sys.o
                0x00000000000172a0                spiflash_speed_up_en
 .com_text.gpio
                0x00000000000172a4       0x36 Output\obj\Libraries\Device\Source\gw3323_gpio.o
                0x00000000000172a4                gpio_set_bits
                0x00000000000172a8                gpio_reset_bits
                0x00000000000172ac                gpio_writebit
                0x00000000000172b6                gpio_write_data
                0x00000000000172c0                gpio_toggle_bits
                0x00000000000172c8                gpio_read_data
                0x00000000000172d0                gpio_read_bit
 .com_text.stack.uart_isr
                0x00000000000172da        0x4 Output\obj\Libraries\libs\strong_symbol.o
                0x00000000000172da                bt_uart_isr
 *fill*         0x00000000000172de        0x2 
 .com_text.data
                0x00000000000172e0     0x3000 Output\obj\Examples\Internal_Flash\Source\Internal_Flash.o
                0x00000000000172e0                erase_buff
                0x00000000000182e0                wbuff
                0x00000000000192e0                rbuff
 .com_text.spiflash
                0x000000000001a2e0      0x13e ..\..\..\Libraries\libs\libplatform.a(os_flash.o)
                0x000000000001a2e0                os_spiflash_read
                0x000000000001a31a                os_spiflash_program
                0x000000000001a3a0                os_spiflash_erase
 .com_text.sd.isr
                0x000000000001a41e       0x20 ..\..\..\Libraries\libs\libplatform.a(device.o)
                0x000000000001a41e                sdctl_isr
 .com_text.exception.hook
                0x000000000001a43e       0x3a ..\..\..\Libraries\libs\libplatform.a(main.o)
                0x000000000001a43e                sys_error_hook
 .com_text.exception
                0x000000000001a478       0x5e ..\..\..\Libraries\libs\libplatform.a(main.o)
                0x000000000001a478                exception_isr
 .com_text.delay
                0x000000000001a4d6       0x4e ..\..\..\Libraries\libs\libplatform.a(main.o)
                0x000000000001a4d6                delay_5ms
                0x000000000001a4f0                delay_ms
                0x000000000001a508                delay_us
 .com_text.irq  0x000000000001a524      0x17a ..\..\..\Libraries\libs\libplatform.a(interrupt.o)
                0x000000000001a524                bthw_isr
                0x000000000001a53e                aubuf_isr
                0x000000000001a5ba                timer0_isr
                0x000000000001a626                register_isr
                0x000000000001a660                tick_get
                0x000000000001a668                watch_point_isr
                0x000000000001a68c                tick_check_expire
 .com_text.timer
                0x000000000001a69e       0x10 ..\..\..\Libraries\libs\libplatform.a(startup.o)
 .com_text.irq  0x000000000001a6ae       0x5a ..\..\..\Libraries\libs\libplatform.a(reset.o)
                0x000000000001a6ae                cpu_irq_comm
                0x000000000001a700                btmdm_isr
 .com_text.util.isr
                0x000000000001a708        0x6 ..\..\..\Libraries\libs\libplatform.a(reset.o)
                0x000000000001a708                kick_soft_isr
 .com_text.spiflash
                0x000000000001a70e      0x154 ..\..\..\Libraries\libs\libplatform.a(spiflash.o)
                0x000000000001a7a0                spiflash_program
                0x000000000001a7ea                spiflash_erase
                0x000000000001a816                spiflash_get_id
 .com_text.debug
                0x000000000001a862      0x1aa ..\..\..\Libraries\libs\libplatform.a(debug.o)
                0x000000000001a934                debug_dump_err_cache_irq
 .com_text.sys  0x000000000001aa0c       0x68 ..\..\..\Libraries\libs\libplatform.a(s_sys.o)
                0x000000000001aa0c                s_ff1
                0x000000000001aa12                s_fl1
                0x000000000001aa18                s_log2
                0x000000000001aa20                s_clb
                0x000000000001aa26                s_bcnt
                0x000000000001aa2c                s_ror
                0x000000000001aa32                s_swapw
                0x000000000001aa38                s_bitrvti
                0x000000000001aa3e                s_clip16
                0x000000000001aa44                s_abs
                0x000000000001aa4a                mul_r
                0x000000000001aa56                dummy_func
                0x000000000001aa58                __ashrdi3
                0x000000000001aa66                __ashldi3
 .com_text.thread.driver
                0x000000000001aa74       0x56 ..\..\..\Libraries\libs\libplatform.a(usb.o)
                0x000000000001aa74                os_mq_usb_post
                0x000000000001aa9a                thread_user_kick
                0x000000000001aac8                thread_user_func_do
 *fill*         0x000000000001aaca        0x2 
 .com_text.thread.usb
                0x000000000001aacc       0xaa ..\..\..\Libraries\libs\libplatform.a(usb.o)
                0x000000000001aacc                thread_usb_entry
 .com_text.bthw
                0x000000000001ab76       0x22 ..\..\..\Libraries\libs\libplatform.a(bt.o)
                0x000000000001ab76                btstack_status_lock
                0x000000000001ab88                btstack_status_unlock
 .com_text.stack.thread
                0x000000000001ab98       0x32 ..\..\..\Libraries\libs\libplatform.a(bt.o)
                0x000000000001ab98                thread_btstack_pend
                0x000000000001abba                thread_btstack_post
 .com_text.stack.run_loop
                0x000000000001abca       0x48 ..\..\..\Libraries\libs\libplatform.a(bt.o)
                0x000000000001abca                thread_btstack_entry
 .com_text.bb.bthw
                0x000000000001ac12       0x3c ..\..\..\Libraries\libs\libplatform.a(bt.o)
                0x000000000001ac12                thread_bthw_entry
 .com_text.bb.nanos
                0x000000000001ac4e       0x16 ..\..\..\Libraries\libs\libbtstack.a(nanos.o)
                0x000000000001ac4e                nanos_event_set
 .com_text.bb.patch
                0x000000000001ac64       0x9a ..\..\..\Libraries\libs\libbtstack.a(patch.o)
                0x000000000001ac64                bb_v1_patch0_do
                0x000000000001ac72                bt_acl_cal_offset_fix
 .com_text.bb.ll.tx
                0x000000000001acfe        0x2 ..\..\..\Libraries\libs\libbtstack.a(platform.o)
                0x000000000001acfe                bb_ll_tx_cb
 .com_text.bb.ll.rx
                0x000000000001ad00        0x2 ..\..\..\Libraries\libs\libbtstack.a(platform.o)
                0x000000000001ad00                bb_ll_rx_cb
 .com_text.bb.lmp.rx
                0x000000000001ad02        0x2 ..\..\..\Libraries\libs\libbtstack.a(platform.o)
                0x000000000001ad02                bb_lmp_tx_cb
 .com_text.bb.lmp.tx
                0x000000000001ad04        0x2 ..\..\..\Libraries\libs\libbtstack.a(platform.o)
                0x000000000001ad04                bb_lmp_rx_cb
 .com_text.timer
                0x000000000001ad06        0x6 ..\..\..\Libraries\libs\libbtstack.a(platform.o)
                0x000000000001ad06                timer_get_tick
                0x000000000001ad0a                timer_sync
 .com_text.bb.sco
                0x000000000001ad0c       0x1e ..\..\..\Libraries\libs\libbtstack.a(bt_sco.o)
                0x000000000001ad0c                bt_sco_is_transp
                0x000000000001ad1c                bt_codec_isr
                0x000000000001ad1e                lc_sco_codec_pkt
 .com_text.bt21.isr
                0x000000000001ad2a      0x212 ..\..\..\Libraries\libs\libbtstack.a(bt_acl.o)
                0x000000000001adac                bt_acl_lmp_tx_isr
                0x000000000001ae14                bt_acl_data_tx_isr
                0x000000000001ae4a                bt_sco_audio_isr
                0x000000000001aefc                bt_acl_get_clkoff
 .com_text.ble.isr.con
                0x000000000001af3c       0x82 ..\..\..\Libraries\libs\libbtstack.a(ble_con.o)
                0x000000000001af3c                ble_con_rx_end
                0x000000000001af8e                ble_con_evt_prio_check
 .com_text.bb.utils
                0x000000000001afbe        0xa ..\..\..\Libraries\libs\libbtstack.a(bb_utils.o)
                0x000000000001afbe                bb_slot_to_duration
 .com_text.bb.isr
                0x000000000001afc8      0x19c ..\..\..\Libraries\libs\libbtstack.a(bb_int.o)
                0x000000000001affc                bb_lpcycles_2_hus
                0x000000000001b03e                bb_isr
                0x000000000001b152                bb_hal_isr
 .com_text.bb.btisr
                0x000000000001b164       0x2e ..\..\..\Libraries\libs\libbtstack.a(bb.o)
                0x000000000001b164                bb_acl_rx0_parse
                0x000000000001b168                bb_free_acl_buf
                0x000000000001b174                bb_alloc_acl_buf
 .com_text.bb.isr
                0x000000000001b192       0x32 ..\..\..\Libraries\libs\libbtstack.a(bb.o)
                0x000000000001b192                bb_notice_status
 .com_text.dummy
                0x000000000001b1c4        0x6 ..\..\..\Libraries\libs\libbtstack.a(platform.o)
                0x000000000001b1c4                dummy_void
                0x000000000001b1c6                dummy_false
 .com_text.aubuf.isr
                0x000000000001b1ca        0x2 ..\..\..\Libraries\libs\libbtstack.a(extern.o)
                0x000000000001b1ca                ext_aubuf_isr
 .com_text.pp.send_pkt
                0x000000000001b1cc       0x58 ..\..\..\Libraries\libs\libbtstack.a(spp.o)
                0x000000000001b1cc                spp_send_packet
 .com_text.spp.tx
                0x000000000001b224       0xd4 ..\..\..\Libraries\libs\libbtstack.a(spp.o)
                0x000000000001b224                spp_is_connect
                0x000000000001b238                spp_default_connected
                0x000000000001b24e                spp_custom1_connected
                0x000000000001b264                spp_custom2_connected
                0x000000000001b27a                bt_spp_tx
                0x000000000001b2a4                bt_spp_custom1_tx
                0x000000000001b2ce                bt_spp_custom2_tx
 .com_text.spp.send_kick
                0x000000000001b2f8        0xe ..\..\..\Libraries\libs\libbtstack.a(spp.o)
                0x000000000001b2f8                spp_send_kick
 .com_text.spp.send_req
                0x000000000001b306       0x12 ..\..\..\Libraries\libs\libbtstack.a(spp.o)
                0x000000000001b306                btstack_spp_send_req
 .com_text.spp.event_send
                0x000000000001b318       0x32 ..\..\..\Libraries\libs\libbtstack.a(spp.o)
                0x000000000001b318                spp_event_send
 .com_text.spp.rx_set_new_credit
                0x000000000001b34a       0x7e ..\..\..\Libraries\libs\libbtstack.a(spp.o)
                0x000000000001b34a                spp_set_rx_new_credit
                0x000000000001b358                spp_notify_rx_buffer_len
                0x000000000001b3ae                btstack_spp_rx_set_new_credit
 .com_text.txpkt.send
                0x000000000001b3c8      0x15e ..\..\..\Libraries\libs\libbtstack.a(btstack_txpkt.o)
                0x000000000001b3c8                txpkt_send
                0x000000000001b4a6                txpkt_event_send
 .com_text.stack.run_loop
                0x000000000001b526       0xe2 ..\..\..\Libraries\libs\libbtstack.a(btstack_run_loop.o)
                0x000000000001b526                btstack_cmp_abs_tick
                0x000000000001b52c                btstack_runtime_check
                0x000000000001b572                btstack_run_loop_execute_once
 .com_text.stack.thread
                0x000000000001b608        0xe ..\..\..\Libraries\libs\libbtstack.a(btstack_run_loop.o)
                0x000000000001b608                btstack_run_loop_embedded_trigger
 .com_text.stack.ticks
                0x000000000001b616       0x34 ..\..\..\Libraries\libs\libbtstack.a(btstack_run_loop.o)
 .com_text.stack.linked_list
                0x000000000001b64a       0x50 ..\..\..\Libraries\libs\libbtstack.a(btstack_linked_list.o)
                0x000000000001b64a                btstack_linked_list_empty
                0x000000000001b652                btstack_linked_list_iterator_init
                0x000000000001b65e                btstack_linked_list_iterator_has_next
                0x000000000001b67c                btstack_linked_list_iterator_next
 .com_text.ble.send_pkt
                0x000000000001b69a       0xd6 ..\..\..\Libraries\libs\libbtstack.a(gatt_server.o)
                0x000000000001b69a                ble_send_notify_packet
                0x000000000001b72c                att_event_server_send
 .com_text.stack.ble.mtu
                0x000000000001b770       0x10 ..\..\..\Libraries\libs\libbtstack.a(gatt_server.o)
                0x000000000001b770                ble_get_gatt_mtu
 .com_text.ble.send_kick
                0x000000000001b780        0xe ..\..\..\Libraries\libs\libbtstack.a(gatt_server.o)
                0x000000000001b780                ble_send_kick
 .com_text.stack.ticks
                0x000000000001b78e        0xa ..\..\..\Libraries\libs\libbtstack.a(btstack_hal.o)
                0x000000000001b790                sys_tick_handler
 .com_text.isr  0x000000000001b798       0x1a ..\..\..\Libraries\libs\libbtstack.a(btstack_hal.o)
                0x000000000001b798                bt_timer_isr
 .com_text.stack.api
                0x000000000001b7b2      0x13a ..\..\..\Libraries\libs\libbtstack.a(btstack_api.o)
                0x000000000001b7b2                bt_is_testmode
                0x000000000001b7c0                bt_is_l2cap_disconnected
                0x000000000001b7da                bt_is_disconnecting
                0x000000000001b7f4                btstack_status_update
                0x000000000001b802                btstack_set_play_status
                0x000000000001b82e                btstack_get_play_status
                0x000000000001b83e                bt_get_status
                0x000000000001b886                bt_get_disp_status
                0x000000000001b888                bt_is_calling
                0x000000000001b89e                bt_get_l2cap_status
                0x000000000001b8ca                bt_tws_get_status
 .com_text.stack.run_loop
                0x000000000001b8ec        0x2 ..\..\..\Libraries\libs\libbtstack.a(btstack_api.o)
                0x000000000001b8ec                btstack_msg
 .com_text.stack.ble.api0
                0x000000000001b8ee       0x10 ..\..\..\Libraries\libs\libbtstack.a(ble_api.o)
                0x000000000001b8ee                ble_get_status
 .com_text.stack.ble.api1
                0x000000000001b8fe       0x16 ..\..\..\Libraries\libs\libbtstack.a(ble_api.o)
                0x000000000001b8fe                ble_is_connect
 .com_text.bb.frag
                0x000000000001b914       0x3a ..\..\..\Libraries\libs\libbtstack.a(bb_sche.o)
 .com_text.bb.prog
                0x000000000001b94e      0x1f0 ..\..\..\Libraries\libs\libbtstack.a(bb_sche.o)
 .com_text.bb.patch
                0x000000000001bb3e       0x52 ..\..\..\Libraries\libs\libbtstack.a(patch_asm.o)
                0x000000000001bb3e                bb_v1_patch0
                0x000000000001bb4a                bb_v1_patch6
                0x000000000001bb52                bb_v1_patch7
                0x000000000001bb6c                bb_v1_patch8
 .com_text.bb.isr
                0x000000000001bb90       0x1a ..\..\..\Libraries\libs\libbtstack.a(aes.o)
                0x000000000001bb90                ble_ecpy_aes_res_cb
 .com_text.bb.isr
                0x000000000001bbaa       0x50 ..\..\..\Libraries\libs\libbtstack.a(rf.o)
                0x000000000001bbaa                rf_rssi_calc_dbm
                0x000000000001bbb4                rf_txpwr_get_lv
                0x000000000001bbe8                rf_txpwr_get_dbm
                0x000000000001bbf8                rf_agc_enable
 .com_text.isr.txrx
                0x000000000001bbfa       0x76 ..\..\..\Libraries\libs\libbtstack.a(rf.o)
                0x000000000001bbfa                bb_rf_ext_ctl_cb
                0x000000000001bbfc                bthw_txrx_isr
 *fill*         0x000000000001bc70        0x0 
 .com_text.bt21.isr
                0x000000000001bc70      0x5c8 ..\..\..\Libraries\libs\libbtstack.a(bt_hook.o)
                0x000000000001bc70                bt_page_init_func
                0x000000000001bc78                bt_acl_rx_header
                0x000000000001be70                bt_acl_test_rx_end
                0x000000000001be74                bt_acl_rx_end
                0x000000000001bedc                bt_acl_sniff_cacl_win_size
                0x000000000001bf34                bt_isr_hook
 .com_text.ble.isr
                0x000000000001c238       0x7c ..\..\..\Libraries\libs\libbtstack.a(ble_hook.o)
                0x000000000001c238                ble_isr_hook
 .com_text.bb.hct
                0x000000000001c2b4       0x18 ..\..\..\Libraries\libs\libbtstack.a(hct_fc.o)
                0x000000000001c2b4                hci_fc_acl_packet_sent
 .com_text.bt21.sco
                0x000000000001c2cc       0x1e ..\..\..\Libraries\libs\libbtstack.a(tws_sco.o)
                0x000000000001c2cc                bt_sco_get_index
 .com_text.bb.tws.sw.chk
                0x000000000001c2ea        0x4 ..\..\..\Libraries\libs\libbtstack.a(tws_acl.o)
                0x000000000001c2ea                tws_switch_acl_is_pause
 .com_text.bt21.isr
                0x000000000001c2ee       0x3c ..\..\..\Libraries\libs\libbtstack.a(bt_hal.o)
                0x000000000001c2ee                bt_channel_assess
 .com_text.bt21.isr
                0x000000000001c32a       0x52 ..\..\..\Libraries\libs\libbtstack.a(bt21.o)
                0x000000000001c32a                bt_buf_acl_rx_free
                0x000000000001c338                bt21_isr
 .com_text.ble.isr
                0x000000000001c37c      0x102 ..\..\..\Libraries\libs\libbtstack.a(ble_hal.o)
 .com_text.ble.isr.con
                0x000000000001c47e       0x3c ..\..\..\Libraries\libs\libbtstack.a(ble_hal.o)
                0x000000000001c47e                ble_channel_assess
 .com_text.ble.isr.adv
                0x000000000001c4ba       0x52 ..\..\..\Libraries\libs\libbtstack.a(ble_adv.o)
                0x000000000001c4ba                ble_adv_duration_update
 .com_text.bb.isr
                0x000000000001c50c       0x18 ..\..\..\Libraries\libs\libbtstack.a(ble.o)
                0x000000000001c50c                ble_isr
 .com_text.l2cap_test.con
                0x000000000001c524       0x4c ..\..\..\Libraries\libs\libbtstack.a(l2cap_test.o)
                0x000000000001c524                l2cap_vd_acl_check
 .com_text.stack.handler.l2cap
                0x000000000001c570       0x38 ..\..\..\Libraries\libs\libbtstack.a(l2cap.o)
                0x000000000001c570                l2cap_get_channel_for_local_cid
                0x000000000001c588                l2cap_get_channel_for_remote_cid
 .com_text.sco  0x000000000001c5a8        0x4 ..\..\..\Libraries\libs\libbtstack.a(hci_sco.o)
                0x000000000001c5a8                sco_init_var
                0x000000000001c5aa                sco_buffer_reset
 .com_text.stack.hci
                0x000000000001c5ac       0x5a ..\..\..\Libraries\libs\libbtstack.a(hci.o)
                0x000000000001c5ac                hci_connection_for_handle
                0x000000000001c5d4                hci_can_send_command_packet_now
 .com_text.stack.hci_recv
                0x000000000001c606        0xe ..\..\..\Libraries\libs\libbtstack.a(hci.o)
                0x000000000001c606                hci_host_recv_packet
 .com_text.bb.btisr
                0x000000000001c614        0x8 ..\..\..\Libraries\libs\libbtstack.a(avdtp.o)
                0x000000000001c614                a2dp_get_play_index
                0x000000000001c618                avdtp_rx_media_parse
 .com_text.stack.hcic
                0x000000000001c61c       0x10 ..\..\..\Libraries\libs\libbtstack.a(hci_transport_hcic.o)
                0x000000000001c61c                hcic_can_send_packet_now
 .com_text.ble.isr.test.clr
                0x000000000001c62c       0x22 ..\..\..\Libraries\libs\libbtstack.a(ble_test.o)
 .com_text.ble.init
                0x000000000001c64e      0xba2 ..\..\..\Libraries\libs\libbtstack.a(ble_init.o)
 .com_text.usbdev
                0x000000000001d1f0       0x20 ..\..\..\Libraries\libs\libdrivers.a(usb_device_hid.o)
                0x000000000001d1f0                ude_tmr_isr
 *fill*         0x000000000001d210        0x0 
 .com_text.epsize.table
                0x000000000001d210        0x4 ..\..\..\Libraries\libs\libdrivers.a(usb_comm.o)
                0x000000000001d210                epsize_tbl
 *(.com_text.stack.handler)
 *(.com_rodata*)
 .com_rodata.exception
                0x000000000001d214       0x29 ..\..\..\Libraries\libs\libplatform.a(main.o)
 *fill*         0x000000000001d23d        0x3 
 .com_rodata.irq
                0x000000000001d240       0x1b ..\..\..\Libraries\libs\libplatform.a(interrupt.o)
                0x000000000001d240                watch_point_str
 *fill*         0x000000000001d25b        0x1 
 .com_rodata.miss
                0x000000000001d25c       0x29 ..\..\..\Libraries\libs\libplatform.a(debug.o)
 *fill*         0x000000000001d285        0x3 
 .com_rodata.bb.sco
                0x000000000001d288       0x3c ..\..\..\Libraries\libs\libbtstack.a(bt_sco.o)
                0x000000000001d288                tbl_msbc_mute
 .com_rodata.bb.tbl
                0x000000000001d2c4       0x32 ..\..\..\Libraries\libs\libbtstack.a(bt_acl.o)
 *fill*         0x000000000001d2f6        0x2 
 .com_rodata.bb.tbl
                0x000000000001d2f8       0x10 ..\..\..\Libraries\libs\libbtstack.a(ble_con.o)
                0x000000000001d2f8                byte_tx_time
                0x000000000001d300                fixed_tx_time
 .com_rodata.bb.tbl
                0x000000000001d308       0x44 ..\..\..\Libraries\libs\libbtstack.a(bb_utils.o)
                0x000000000001d308                one_bits
                0x000000000001d318                bb_rate_to_byte_dur_us
                0x000000000001d320                bb_rate_to_phy_mask
                0x000000000001d324                bb_phy_value_to_mask
                0x000000000001d328                bb_phy_mask_to_value
                0x000000000001d330                bb_phy_to_rate
                0x000000000001d334                bb_rate_to_phy
                0x000000000001d33c                bb_sca2ppm
 .com_rodata.bb.tws
                0x000000000001d34c        0xd ..\..\..\Libraries\libs\libbtstack.a(bb_int.o)
                0x000000000001d34c                str_bb_err
 *fill*         0x000000000001d359        0x3 
 .com_rodata.bb.tbl
                0x000000000001d35c       0x3c ..\..\..\Libraries\libs\libbtstack.a(bb.o)
                0x000000000001d35c                bb_priority
 .com_rodata.bb.tbl
                0x000000000001d398        0xc ..\..\..\Libraries\libs\libbtstack.a(vs_proc.o)
                0x000000000001d398                vs_msg_env
 .com_rodata.bb.tbl
                0x000000000001d3a4        0x8 ..\..\..\Libraries\libs\libbtstack.a(rf.o)
 .com_rodata.bb.tbl
                0x000000000001d3ac        0xb ..\..\..\Libraries\libs\libbtstack.a(bt_hook.o)
 *fill*         0x000000000001d3b7        0x1 
 .com_rodata.bb.tbl
                0x000000000001d3b8       0x12 ..\..\..\Libraries\libs\libbtstack.a(bt21.o)
 *fill*         0x000000000001d3ca        0x2 
 .com_rodata.btstakc.hci
                0x000000000001d3cc        0x8 ..\..\..\Libraries\libs\libbtstack.a(hci_cmd.o)
                0x000000000001d3cc                hci_num_of_packet_complete
 .com_rodata.hci.trans
                0x000000000001d3d4       0x20 ..\..\..\Libraries\libs\libbtstack.a(hci_transport_hcic.o)
 .com_rodata.bb.tbl
                0x000000000001d3f4        0xc ..\..\..\Libraries\libs\libbtstack.a(lm_proc.o)
                0x000000000001d3f4                lm_msg_env
 .com_rodata.bb.tbl
                0x000000000001d400        0x8 ..\..\..\Libraries\libs\libbtstack.a(ble_init.o)
                0x000000000001d400                ble_init_max_aux_dur_tab
 .com_rodata.bb.tbl
                0x000000000001d408       0x18 ..\..\..\Libraries\libs\libbtstack.a(ble_buf.o)
 .com_rodata.bb.tbl
                0x000000000001d420        0xc ..\..\..\Libraries\libs\libbtstack.a(lc_proc.o)
                0x000000000001d420                lc_msg_env
 .com_rodata.bb.tbl
                0x000000000001d42c        0xc ..\..\..\Libraries\libs\libbtstack.a(mgr_proc.o)
                0x000000000001d42c                mgr_msg_env
 .com_rodata.bb.tbl
                0x000000000001d438        0xc ..\..\..\Libraries\libs\libbtstack.a(ll_proc.o)
                0x000000000001d438                ll_msg_env
 *debug.o(.rodata*)
 .rodata.str1.4
                0x000000000001d444       0xd0 ..\..\..\Libraries\libs\libplatform.a(debug.o)
                                         0xce (size before relaxing)
 *(.data*)
 .data          0x000000000001d514        0xc Output\obj\Libraries\BT\spp\profile.o
                0x000000000001d514                spp_sdp_record_item
 .data          0x000000000001d520       0x18 ..\..\..\Libraries\libs\libbtstack.a(btstack_link_key_db.o)
 .data          0x000000000001d538       0x31 ..\..\..\Libraries\libs\libbtstack.a(btstack_run_loop.o)
                0x000000000001d538                data_source_debug_info
 *(.sdata*)
 *fill*         0x000000000001d569        0x1 
 .sdata         0x000000000001d56a        0x2 Output\obj\Libraries\bsp\bsp_fot.o
                0x000000000001d56a                dev_version
 .sdata         0x000000000001d56c        0x1 Output\obj\Libraries\BT\ble\adv0.o
                0x000000000001d56c                cfg_ble_adv0_en
 .sdata         0x000000000001d56d        0x2 Output\obj\Libraries\BT\ble\ble.o
                0x000000000001d56d                cfg_ble_mtu_request_en
                0x000000000001d56e                cfg_ble_security_en
 *fill*         0x000000000001d56f        0x1 
 .sdata         0x000000000001d570       0x10 Output\obj\Libraries\BT\spp\bt.o
                0x000000000001d570                bt_local_addr
                0x000000000001d576                cfg_bt_link_info_items
                0x000000000001d578                cfg_bt_sup_to_connect_times
                0x000000000001d57a                cfg_bt_pwrup_connect_times
                0x000000000001d57b                cfg_bt_connect_times
                0x000000000001d57c                cfg_bt_support_profile
                0x000000000001d57e                cfg_bt_dual_mode
                0x000000000001d57f                cfg_bt_max_acl_link
 .sdata         0x000000000001d580        0x1 Output\obj\Libraries\libs\strong_symbol.o
                0x000000000001d580                cfg_bt_sniff_mode_dis
 *fill*         0x000000000001d581        0x3 
 .sdata         0x000000000001d584        0x4 Output\obj\Examples\Internal_Flash\Source\Internal_Flash.o
                0x000000000001d584                bt_Name
 .sdata         0x000000000001d588       0x11 ..\..\..\Libraries\libs\libbtstack.a(extern_bt.o)
                0x000000000001d588                cfg_bt_music_low_latency
                0x000000000001d58a                cfg_bt_music_normal_latency
                0x000000000001d58c                cfg_bt_ble_adv
                0x000000000001d598                cfg_bt_sniff_clk_sel
 *fill*         0x000000000001d599        0x3 
 .sdata         0x000000000001d59c        0x4 ..\..\..\Libraries\libs\libbtstack.a(sdp_server.o)
 .sdata         0x000000000001d5a0        0x3 ..\..\..\Libraries\libs\libbtstack.a(sm.o)
 *fill*         0x000000000001d5a3        0x1 
 .sdata         0x000000000001d5a4        0x4 ..\..\..\Libraries\libs\libbtstack.a(att_server.o)
 .sdata         0x000000000001d5a8        0xc ..\..\..\Libraries\libs\libbtstack.a(btstack_hal.o)
 .sdata         0x000000000001d5b4        0x1 ..\..\..\Libraries\libs\libbtstack.a(btstack_adv0.o)
 *fill*         0x000000000001d5b5        0x3 
 .sdata         0x000000000001d5b8        0x5 ..\..\..\Libraries\libs\libbtstack.a(ble_adv0.o)
 .sdata         0x000000000001d5bd        0x1 ..\..\..\Libraries\libs\libbtstack.a(extern_hfhs.o)
                0x000000000001d5bd                cfg_bt_hfp_feature
 .sdata         0x000000000001d5be        0x3 ..\..\..\Libraries\libs\libbtstack.a(l2cap_signaling.o)
 .sdata         0x000000000001d5c1        0x4 ..\..\..\Libraries\libs\libdrivers.a(usb_device_hid.o)
                0x000000000001d5c1                user_ep_type
                0x000000000001d5c2                user_ep_dir
                0x000000000001d5c3                user_ep_idx
                0x000000000001d5c4                hid_in_ep
 *(.load_text)
 *fill*         0x000000000001d5c5        0x1 
 .load_text     0x000000000001d5c6       0x10 ..\..\..\Libraries\libs\libplatform.a(main.o)
 *(.load_rodata)
                0x000000000001d600                . = ALIGN (0x200)
 *fill*         0x000000000001d5d6       0x2a 

.flash          0x0000000010006800    0x43000
                0x0000000010006800                __code_start_sniff = .
 *(.sniff*)
                0x0000000010006800                . = ALIGN (0x200)
                0x0000000010006800                __code_end_sniff = .
                0x0000000010006800                __code_start_usbdev = .
 *(.usbdev*)
 .usbdev.com    0x0000000010006800      0x1b2 ..\..\..\Libraries\libs\libdrivers.a(usb_device_hid.o)
                0x0000000010006800                usb_user_ep_tx_handler
                0x0000000010006802                usb_user_ep_rx_handler
                0x0000000010006804                ude_hid_setvalid
                0x0000000010006818                ude_hid_send
                0x0000000010006872                usb_user_ep_rx_ack
                0x0000000010006896                usb_user_ep_tx_process
                0x00000000100068b2                usb_user_ep_rx_process
                0x00000000100068e0                usb_int_ep_reset
                0x00000000100068f6                udh_init
                0x0000000010006952                udu_init
 .usbdev.com    0x00000000100069b2       0x7c ..\..\..\Libraries\libs\libdrivers.a(usb_device_printer.o)
                0x00000000100069b2                usb_bulk_reset
                0x00000000100069c8                ude_rx_ack
                0x00000000100069e0                bulk_tx_handler
                0x00000000100069e2                bulk_rx_handler
                0x00000000100069e4                ude_bulk_tx_process
                0x0000000010006a00                ude_bulk_rx_process
 .usbdev.com    0x0000000010006a2e      0x36c ..\..\..\Libraries\libs\libdrivers.a(usb_device_ep.o)
                0x0000000010006a2e                usb_set_cur_ep
                0x0000000010006a44                usb_ep_init
                0x0000000010006ad0                usb_ep_halt
                0x0000000010006b1c                usb_ep_clear
                0x0000000010006b5c                usb_ep_transfer
                0x0000000010006cea                usb_ep_reset
                0x0000000010006d5e                usb_ep_start_transfer
                0x0000000010006d78                usb_ep_do_transfer
                0x0000000010006e00                . = ALIGN (0x200)
 *fill*         0x0000000010006d9a       0x66 
                0x0000000010006e00                __code_end_usbdev = .
                0x0000000010006e00                __code_start_sleep = .
 *(.saradc_text*)
 *(.sleep_text*)
 .sleep_text.sleep.rc
                0x0000000010006e00       0xc2 ..\..\..\Libraries\libs\libplatform.a(rc.o)
                0x0000000010006e00                rc_sleep_trim_init
                0x0000000010006e02                rc_sleep_trim_clear
                0x0000000010006e04                rc_sleep_get_freqcnt
                0x0000000010006e72                rc_sleep_reset_sta
                0x0000000010006e74                rc_sleep_get_trim_freqcnt
 .sleep_text.rf
                0x0000000010006ec2      0x21a ..\..\..\Libraries\libs\libbtstack.a(rf_smart.o)
                0x0000000010006fa2                rfphy_deep_sleep
                0x000000001000704a                rfphy_idle
                0x0000000010007200                . = ALIGN (0x200)
 *fill*         0x00000000100070dc      0x124 
                0x0000000010007200                __code_end_sleep = .
                0x0000000010007200                __code_start_charge = .
 *(.charge_text*)
 *(.text.bsp.charge)
 *(.text.bsp.tkey)
 *(.text.vhouse)
                0x0000000010007200                . = ALIGN (0x200)
                0x0000000010007200                __code_end_charge = .
                0x0000000010007200                __code_start_pwrsave = .
 *(.text.pwroff*)
                0x0000000010007200                . = ALIGN (0x200)
                0x0000000010007200                __code_end_pwrsave = .
                0x0000000010007200                __code_start_bb_test = .
 *(.bb_test*)
 *(.bb_test_rodata*)
                0x0000000010007200                . = ALIGN (0x200)
                0x0000000010007200                __code_end_bb_test = .
                0x0000000010007200                __code_start_update = .
 *(.text.update*)
 .text.update_sd0baud
                0x0000000010007200       0x3c ..\..\..\Libraries\libs\libplatform.a(sys_clk.o)
                0x0000000010007200                update_sd0baud
 .text.update_complete
                0x000000001000723c        0x2 ..\..\..\Libraries\libs\libplatform.a(weak_symbol.o)
                0x000000001000723c                update_complete
                0x0000000010007400                . = ALIGN (0x200)
 *fill*         0x000000001000723e      0x1c2 
                0x0000000010007400                __code_end_update = .
                0x0000000010007400                __code_start_huart = .
 *(.com_huart*)
                0x0000000010007400                . = ALIGN (0x200)
                0x0000000010007400                __code_end_huart = .
                0x0000000010007400                __code_start_fota = .
 *(.text.fot.cache*)
 .text.fot.cache
                0x0000000010007400      0x744 Output\obj\Libraries\bsp\bsp_fot.o
                0x000000001000746a                fot_recv_proc
                0x000000001000795c                bsp_fot_process
                0x0000000010007a44                bsp_usb_fot_process
 *fill*         0x0000000010007b44        0x0 
 .text.fot.cache
                0x0000000010007b44      0x204 ..\..\..\Libraries\libs\libplatform.a(fot_update.o)
                0x0000000010007b44                fot_pkt_process_do
                0x0000000010007cae                fot_write
                0x0000000010007e00                . = ALIGN (0x200)
 *fill*         0x0000000010007d48       0xb8 
                0x0000000010007e00                __code_end_fota = .
                0x0000000010007e00                __code_start_bts = .
 *(.text.stk.tws.txreq*)
 *(.text.stk.l2cap.txreq*)
 .text.stk.l2cap.txreq
                0x0000000010007e00      0x110 ..\..\..\Libraries\libs\libbtstack.a(l2cap.o)
                0x0000000010007ed4                l2cap_request_can_send_now_event
                0x0000000010007eee                l2cap_request_can_send_fix_channel_now_event
 *fill*         0x0000000010007f10        0x0 
 .text.stk.l2cap.txreq.rodata
                0x0000000010007f10        0xa ..\..\..\Libraries\libs\libbtstack.a(l2cap.o)
                0x0000000010008000                . = ALIGN (0x200)
 *fill*         0x0000000010007f1a       0xe6 
 *(.text.stk.tws.send*)
                0x0000000010008000                . = ALIGN (0x200)
 *(.text.stk.tws.recv*)
                0x0000000010008000                . = ALIGN (0x200)
 *(.text.stk.hci.tx*)
                0x0000000010008000                . = ALIGN (0x200)
 *(.text.bts.hci.rx*)
                0x0000000010008000                . = ALIGN (0x200)
 *(.text.stk.bt.acl.tx*)
 .text.stk.bt.acl.tx.done
                0x0000000010008000       0x76 ..\..\..\Libraries\libs\libbtstack.a(lc_proc.o)
                0x0000000010008200                . = ALIGN (0x200)
 *fill*         0x0000000010008076      0x18a 
                0x0000000010008200                __code_end_bts = .
 *(.irq_init.aligned)
                0x0000000010008200                . = ALIGN (0x200)
 *(.text.ble.chmap*)
 .text.ble.chmap
                0x0000000010008200       0x50 ..\..\..\Libraries\libs\libbtstack.a(ble_con.o)
                0x0000000010008200                ble_con_ch_map_update
                0x0000000010008400                . = ALIGN (0x200)
 *fill*         0x0000000010008250      0x1b0 
 *(.text*)
 .text.btstack_ble_init_callback
                0x0000000010008400       0x6c Output\obj\Libraries\bsp\bsp_bt.o
                0x0000000010008400                btstack_ble_init_callback
 .text.ble_init_register
                0x000000001000846c        0xc Output\obj\Libraries\bsp\bsp_bt.o
                0x000000001000846c                ble_init_register
 .text.bsp_bt_init
                0x0000000010008478       0xaa Output\obj\Libraries\bsp\bsp_bt.o
                0x0000000010008478                bsp_bt_init
 .text.bt_emit_notice
                0x0000000010008522       0x40 Output\obj\Libraries\bsp\bsp_bt.o
                0x0000000010008522                bt_emit_notice
 .text.cm_loadparam
                0x0000000010008562       0x12 Output\obj\Libraries\bsp\bsp_cm.o
                0x0000000010008562                cm_loadparam
 .text.cm_factory
                0x0000000010008574       0x20 Output\obj\Libraries\bsp\bsp_cm.o
                0x0000000010008574                cm_factory
 .text.fot.update
                0x0000000010008594       0x6c Output\obj\Libraries\bsp\bsp_fot.o
                0x0000000010008594                is_fot_start
                0x00000000100085a0                fot_update_pause
                0x00000000100085ba                bsp_fot_init
                0x00000000100085e2                fot_update_continue
 .text.fot_ble_disconnect_callback
                0x0000000010008600       0x32 Output\obj\Libraries\bsp\bsp_fot.o
                0x0000000010008600                fot_ble_disconnect_callback
 .text.fot_ble_connect_callback
                0x0000000010008632        0xc Output\obj\Libraries\bsp\bsp_fot.o
                0x0000000010008632                fot_ble_connect_callback
 .text.fot_spp_connect_callback
                0x000000001000863e        0xc Output\obj\Libraries\bsp\bsp_fot.o
                0x000000001000863e                fot_spp_connect_callback
 .text.fot_spp_disconnect_callback
                0x000000001000864a       0x32 Output\obj\Libraries\bsp\bsp_fot.o
                0x000000001000864a                fot_spp_disconnect_callback
 .text.bsp.param
                0x000000001000867c       0xee Output\obj\Libraries\bsp\bsp_param.o
                0x000000001000867c                param_init
                0x000000001000869a                bsp_param_write
                0x000000001000869e                bsp_param_read
                0x00000000100086a2                bsp_param_sync
                0x00000000100086a6                param_sync
                0x00000000100086aa                param_get_xosc_addr
                0x00000000100086ae                param_fot_addr_write
                0x00000000100086c4                param_fot_addr_read
                0x00000000100086ce                param_fot_remote_ver_write
                0x00000000100086e4                param_fot_remote_ver_read
                0x00000000100086ee                param_fot_head_info_write
                0x0000000010008704                param_fot_head_info_read
                0x000000001000870e                param_fot_hash_write
                0x0000000010008724                param_fot_hash_read
                0x000000001000872e                param_qcheck_code_write
                0x0000000010008744                param_qcheck_code_read
                0x000000001000874e                param_sys_vol_write
                0x000000001000875c                param_sys_vol_read
 .text.bsp.sys.init
                0x000000001000876a      0x234 Output\obj\Libraries\bsp\bsp_sys.o
                0x00000000100087e2                rtc_init
                0x0000000010008854                bsp_update_init
                0x000000001000889a                bsp_sys_init
 .text.uart0_mapping_sel
                0x000000001000899e       0x90 Output\obj\Libraries\bsp\bsp_sys.o
                0x000000001000899e                uart0_mapping_sel
 .text.bsp_get_xosc_xcfg
                0x0000000010008a2e       0x20 Output\obj\Libraries\bsp\bsp_sys.o
                0x0000000010008a2e                bsp_get_xosc_xcfg
 .text.gatt_callback_fota
                0x0000000010008a4e       0x20 Output\obj\Libraries\BT\ble\ab_link\app.o
 .text.gatt_callback_app
                0x0000000010008a6e        0xe Output\obj\Libraries\BT\ble\ab_link\app.o
 .text.ble_get_scan_data
                0x0000000010008a7c       0x4e Output\obj\Libraries\BT\ble\ab_link\app.o
                0x0000000010008a7c                ble_get_scan_data
 .text.ble_get_adv_data
                0x0000000010008aca       0x50 Output\obj\Libraries\BT\ble\ab_link\app.o
                0x0000000010008aca                ble_get_adv_data
 .text.ble_txpkt_init
                0x0000000010008b1a       0x30 Output\obj\Libraries\BT\ble\ab_link\app.o
                0x0000000010008b1a                ble_txpkt_init
 .text.ble_fot_send_packet
                0x0000000010008b4a       0x1a Output\obj\Libraries\BT\ble\ab_link\app.o
                0x0000000010008b4a                ble_fot_send_packet
 .text.ble_app_gatts_service_init
                0x0000000010008b64      0x114 Output\obj\Libraries\BT\ble\ab_link\app.o
                0x0000000010008b64                ble_app_gatts_service_init
 .text.ble_app_init
                0x0000000010008c78        0x2 Output\obj\Libraries\BT\ble\ab_link\app.o
                0x0000000010008c78                ble_app_init
 .text.ble_get_local_bd_addr
                0x0000000010008c7a       0x28 Output\obj\Libraries\BT\ble\ble.o
                0x0000000010008c7a                ble_get_local_bd_addr
 .text.ble_disconnect_callback
                0x0000000010008ca2       0x18 Output\obj\Libraries\BT\ble\ble.o
                0x0000000010008ca2                ble_disconnect_callback
 .text.ble_connect_callback
                0x0000000010008cba       0x18 Output\obj\Libraries\BT\ble\ble.o
                0x0000000010008cba                ble_connect_callback
 .text.ble_init_att
                0x0000000010008cd2        0x2 Output\obj\Libraries\BT\ble\ble.o
                0x0000000010008cd2                ble_init_att
 .text.bt_get_class_of_device
                0x0000000010008cd4       0x18 Output\obj\Libraries\BT\spp\bt.o
                0x0000000010008cd4                bt_get_class_of_device
 .text.bt_get_pin_code
                0x0000000010008cec        0xa Output\obj\Libraries\BT\spp\bt.o
                0x0000000010008cec                bt_get_pin_code
 .text.bt_get_local_name
                0x0000000010008cf6        0x8 Output\obj\Libraries\BT\spp\bt.o
                0x0000000010008cf6                bt_get_local_name
 .text.bt_get_local_bd_addr
                0x0000000010008cfe       0x14 Output\obj\Libraries\BT\spp\bt.o
                0x0000000010008cfe                bt_get_local_bd_addr
 .text.bt_get_link_info
                0x0000000010008d12       0x24 Output\obj\Libraries\BT\spp\bt.o
                0x0000000010008d12                bt_get_link_info
 .text.bt_put_link_info
                0x0000000010008d36       0x24 Output\obj\Libraries\BT\spp\bt.o
                0x0000000010008d36                bt_put_link_info
 .text.bt_get_ext_link_info
                0x0000000010008d5a        0x8 Output\obj\Libraries\BT\spp\bt.o
                0x0000000010008d5a                bt_get_ext_link_info
 .text.bt_put_ext_link_info
                0x0000000010008d62        0x8 Output\obj\Libraries\BT\spp\bt.o
                0x0000000010008d62                bt_put_ext_link_info
 .text.bt_sync_link_info
                0x0000000010008d6a        0x4 Output\obj\Libraries\BT\spp\bt.o
                0x0000000010008d6a                bt_sync_link_info
 .text.bt_init_lib
                0x0000000010008d6e       0x24 Output\obj\Libraries\BT\spp\profile.o
                0x0000000010008d6e                bt_init_lib
 .text.spp_txpkt_init
                0x0000000010008d92       0x30 Output\obj\Libraries\BT\spp\spp.o
                0x0000000010008d92                spp_txpkt_init
 .text.spp_rxpkt_init
                0x0000000010008dc2        0x8 Output\obj\Libraries\BT\spp\spp.o
                0x0000000010008dc2                spp_rxpkt_init
 .text.get_spp_mtu_size
                0x0000000010008dca        0x6 Output\obj\Libraries\BT\spp\spp.o
                0x0000000010008dca                get_spp_mtu_size
 .text.spp_connect_callback
                0x0000000010008dd0       0x18 Output\obj\Libraries\BT\spp\spp.o
                0x0000000010008dd0                spp_connect_callback
 .text.spp_disconnect_callback
                0x0000000010008de8       0x18 Output\obj\Libraries\BT\spp\spp.o
                0x0000000010008de8                spp_disconnect_callback
 .text.spp_rx_callback
                0x0000000010008e00       0x86 Output\obj\Libraries\BT\spp\spp.o
                0x0000000010008e00                spp_rx_callback
 .text.vs_ble_test
                0x0000000010008e86        0x4 Output\obj\Libraries\libs\strong_symbol.o
                0x0000000010008e86                vs_ble_test
 .text.vs_fcc_test_cmd
                0x0000000010008e8a        0x4 Output\obj\Libraries\libs\strong_symbol.o
                0x0000000010008e8a                vs_fcc_test_cmd
 .text.is_fot_update_en
                0x0000000010008e8e        0x4 Output\obj\Libraries\libs\strong_symbol.o
                0x0000000010008e8e                is_fot_update_en
 .text.usb_init
                0x0000000010008e92        0x2 Output\obj\Libraries\libs\strong_symbol.o
                0x0000000010008e92                usb_init
 .text.usb_isr  0x0000000010008e94        0x2 Output\obj\Libraries\libs\strong_symbol.o
                0x0000000010008e94                usb_isr
 .text.ude_ep_reset
                0x0000000010008e96        0x2 Output\obj\Libraries\libs\strong_symbol.o
                0x0000000010008e96                ude_ep_reset
 .text.ude_control_flow
                0x0000000010008e98        0x2 Output\obj\Libraries\libs\strong_symbol.o
                0x0000000010008e98                ude_control_flow
 .text.internal_flash_write
                0x0000000010008e9a       0xa6 Output\obj\Examples\Internal_Flash\Source\Internal_Flash.o
                0x0000000010008e9a                internal_flash_write
 .text.internal_flash_erase_partial
                0x0000000010008f40       0x4c Output\obj\Examples\Internal_Flash\Source\Internal_Flash.o
                0x0000000010008f40                internal_flash_erase_partial
 .text.set_bluetooth_name
                0x0000000010008f8c       0xe0 Output\obj\Examples\Internal_Flash\Source\Internal_Flash.o
                0x0000000010008f8c                set_bluetooth_name
 .text.internal_flash_examples
                0x000000001000906c       0xf6 Output\obj\Examples\Internal_Flash\Source\Internal_Flash.o
                0x000000001000906c                internal_flash_examples
 .text.getcfg_vddbt_sel
                0x0000000010009162       0x18 Output\obj\Examples\Internal_Flash\Project\config.o
                0x0000000010009162                getcfg_vddbt_sel
 .text.getcfg_vddio_sel
                0x000000001000917a        0xc Output\obj\Examples\Internal_Flash\Project\config.o
                0x000000001000917a                getcfg_vddio_sel
 .text.getcfg_vddbt_capless_en
                0x0000000010009186        0xa Output\obj\Examples\Internal_Flash\Project\config.o
                0x0000000010009186                getcfg_vddbt_capless_en
 .text.startup.main
                0x0000000010009190       0x30 Output\obj\Examples\Internal_Flash\Project\main.o
                0x0000000010009190                main
 .text.pll_vco_band_trimming
                0x00000000100091c0       0x9a ..\..\..\Libraries\libs\libplatform.a(audio.o)
 *fill*         0x000000001000925a       0xa6 
 .text.adpll_divider_update_do
                0x0000000010009300       0xfa ..\..\..\Libraries\libs\libplatform.a(audio.o)
                0x0000000010009300                adpll_divider_update_do
 .text.adpll_divider_update
                0x00000000100093fa       0x68 ..\..\..\Libraries\libs\libplatform.a(audio.o)
                0x00000000100093fa                adpll_divider_update
 .text.adpll_init
                0x0000000010009462      0x106 ..\..\..\Libraries\libs\libplatform.a(audio.o)
                0x0000000010009462                adpll_init
 .text.cm_loadpage
                0x0000000010009568       0xb4 ..\..\..\Libraries\libs\libplatform.a(cm.o)
 .text.cm_next_freepage
                0x000000001000961c       0x54 ..\..\..\Libraries\libs\libplatform.a(cm.o)
 .text.cm_movepage
                0x0000000010009670       0x60 ..\..\..\Libraries\libs\libplatform.a(cm.o)
 .text.cm_release
                0x00000000100096d0      0x112 ..\..\..\Libraries\libs\libplatform.a(cm.o)
 .text.cm_savepage
                0x00000000100097e2       0xc8 ..\..\..\Libraries\libs\libplatform.a(cm.o)
 .text.cm_check_loadpage
                0x00000000100098aa       0xb0 ..\..\..\Libraries\libs\libplatform.a(cm.o)
 .text.cm_sync  0x000000001000995a       0x3e ..\..\..\Libraries\libs\libplatform.a(cm.o)
                0x000000001000995a                cm_sync
 .text.cm_read  0x0000000010009998       0x44 ..\..\..\Libraries\libs\libplatform.a(cm.o)
                0x0000000010009998                cm_read
 .text.cm_write
                0x00000000100099dc       0x5e ..\..\..\Libraries\libs\libplatform.a(cm.o)
                0x00000000100099dc                cm_write
 .text.cm_init  0x0000000010009a3a      0x1e8 ..\..\..\Libraries\libs\libplatform.a(cm.o)
                0x0000000010009a3a                cm_init
 .text.xcfg_init
                0x0000000010009c22       0x66 ..\..\..\Libraries\libs\libplatform.a(xcfg.o)
                0x0000000010009c22                xcfg_init
 .text.usb_disable
                0x0000000010009c88       0x22 ..\..\..\Libraries\libs\libplatform.a(device.o)
                0x0000000010009c88                usb_disable
 .text.device.init
                0x0000000010009caa       0xb2 ..\..\..\Libraries\libs\libplatform.a(device.o)
                0x0000000010009caa                dev_init
                0x0000000010009d04                dev_delay_times
                0x0000000010009d16                dev_delay_online_times
                0x0000000010009d24                dev_delay_offline_times
                0x0000000010009d32                dev_clr_sta
 .text.platform_main
                0x0000000010009d5c      0x212 ..\..\..\Libraries\libs\libplatform.a(main.o)
                0x0000000010009d5c                platform_main
 .text.main_startup
                0x0000000010009f6e       0x3e ..\..\..\Libraries\libs\libplatform.a(main.o)
                0x0000000010009f6e                main_startup
 .text.sys_irq_init.part.0
                0x0000000010009fac       0x50 ..\..\..\Libraries\libs\libplatform.a(interrupt.o)
 .text.timer0_init
                0x0000000010009ffc       0x64 ..\..\..\Libraries\libs\libplatform.a(interrupt.o)
                0x0000000010009ffc                timer0_init
 .text.soft_irq_init
                0x000000001000a060       0x3c ..\..\..\Libraries\libs\libplatform.a(interrupt.o)
                0x000000001000a060                soft_irq_init
 .text.bthw_irq_init
                0x000000001000a09c       0x38 ..\..\..\Libraries\libs\libplatform.a(interrupt.o)
                0x000000001000a09c                bthw_irq_init
 .text.sd0_irq_init
                0x000000001000a0d4       0x32 ..\..\..\Libraries\libs\libplatform.a(interrupt.o)
                0x000000001000a0d4                sd0_irq_init
 .text.usb_irq_init
                0x000000001000a106       0x26 ..\..\..\Libraries\libs\libplatform.a(interrupt.o)
                0x000000001000a106                usb_irq_init
 .text.aubuf_irq_init
                0x000000001000a12c       0x32 ..\..\..\Libraries\libs\libplatform.a(interrupt.o)
                0x000000001000a12c                aubuf_irq_init
 .text.thread_main_entry
                0x000000001000a15e      0x17a ..\..\..\Libraries\libs\libplatform.a(startup.o)
 .text.bt_set_timer_enable
                0x000000001000a2d8        0xa ..\..\..\Libraries\libs\libplatform.a(startup.o)
                0x000000001000a2d8                bt_set_timer_enable
 .text.sys_set_tmr_enable
                0x000000001000a2e2        0xe ..\..\..\Libraries\libs\libplatform.a(startup.o)
                0x000000001000a2e2                sys_set_tmr_enable
 .text.thread_idle_create
                0x000000001000a2f0       0x30 ..\..\..\Libraries\libs\libplatform.a(startup.o)
                0x000000001000a2f0                thread_idle_create
 .text.startup.init
                0x000000001000a320      0x116 ..\..\..\Libraries\libs\libplatform.a(startup.o)
                0x000000001000a320                platform_init
                0x000000001000a322                sys_startup
 .text.sys_hook_init
                0x000000001000a436        0x2 ..\..\..\Libraries\libs\libplatform.a(sys_hook.o)
                0x000000001000a436                sys_hook_init
 .text.debug_set
                0x000000001000a438       0x1a ..\..\..\Libraries\libs\libplatform.a(debug.o)
                0x000000001000a438                debug_set
 .text.fot.update
                0x000000001000a452      0x88e ..\..\..\Libraries\libs\libplatform.a(fot_update.o)
                0x000000001000a64e                get_keep_mac
                0x000000001000a692                calc_mac
                0x000000001000a6cc                mac_init
                0x000000001000a79a                set_macbuf
                0x000000001000a7ee                clear_macbuf
                0x000000001000a836                fot_head_info_analize
                0x000000001000a84a                fot_set_keep
                0x000000001000a8c2                fot_clear_keep
                0x000000001000a8f2                fot_down_first4k
                0x000000001000abbe                fot_tws_done_try
                0x000000001000abc0                fot_tws_done
                0x000000001000abfe                fot_tws_done_sync_err_deal
                0x000000001000ac24                fot_head_info_save
                0x000000001000ac30                fot_breakpoint_info_read
                0x000000001000acb2                fot_get_err
                0x000000001000acbc                is_fot_update_success
                0x000000001000accc                fot_get_curaddr
 .text.fot.init
                0x000000001000ace0       0xa2 ..\..\..\Libraries\libs\libplatform.a(fot_update.o)
 .text.is_fot_tws_support
                0x000000001000ad82        0x4 ..\..\..\Libraries\libs\libplatform.a(fot_update.o)
                0x000000001000ad82                is_fot_tws_support
 .text.get_spiloader_offset
                0x000000001000ad86        0xc ..\..\..\Libraries\libs\libplatform.a(fot_update.o)
                0x000000001000ad86                get_spiloader_offset
 .text.fot_checksum_cal
                0x000000001000ad92       0xde ..\..\..\Libraries\libs\libplatform.a(fot_update.o)
                0x000000001000ad92                fot_checksum_cal
 .text.fot_down_first4k_checksum_cal
                0x000000001000ae70       0x98 ..\..\..\Libraries\libs\libplatform.a(fot_update.o)
                0x000000001000ae70                fot_down_first4k_checksum_cal
 .text.fot_init
                0x000000001000af08       0x2e ..\..\..\Libraries\libs\libplatform.a(fot_update.o)
                0x000000001000af08                fot_init
 .text.fot_set_base_offset
                0x000000001000af36       0x28 ..\..\..\Libraries\libs\libplatform.a(fot_update.o)
                0x000000001000af36                fot_set_base_offset
 .text.lock_init
                0x000000001000af5e       0x10 ..\..\..\Libraries\libs\libplatform.a(lock.o)
                0x000000001000af5e                lock_init
 .text.lock_code_bt_comm
                0x000000001000af6e        0x2 ..\..\..\Libraries\libs\libplatform.a(lock.o)
                0x000000001000af6e                lock_code_bt_comm
 .text.unlock_code_bt_comm
                0x000000001000af70        0x2 ..\..\..\Libraries\libs\libplatform.a(lock.o)
                0x000000001000af70                unlock_code_bt_comm
 .text.load_code_fota
                0x000000001000af72       0x42 ..\..\..\Libraries\libs\libplatform.a(lock.o)
                0x000000001000af72                load_code_fota
 .text.patch_init
                0x000000001000afb4       0x1e ..\..\..\Libraries\libs\libplatform.a(patch.o)
                0x000000001000afb4                patch_init
 .text.set_buck_mode
                0x000000001000afd2       0x46 ..\..\..\Libraries\libs\libplatform.a(power.o)
                0x000000001000afd2                set_buck_mode
 .text.vddio_voltage_configure
                0x000000001000b018       0x54 ..\..\..\Libraries\libs\libplatform.a(power.o)
                0x000000001000b018                vddio_voltage_configure
 .text.vddbt_voltage_configure
                0x000000001000b06c       0x4e ..\..\..\Libraries\libs\libplatform.a(power.o)
                0x000000001000b06c                vddbt_voltage_configure
 .text.pmu_voltage_configure
                0x000000001000b0ba       0x64 ..\..\..\Libraries\libs\libplatform.a(power.o)
                0x000000001000b0ba                pmu_voltage_configure
 .text.pmu_init
                0x000000001000b11e      0x15e ..\..\..\Libraries\libs\libplatform.a(power.o)
                0x000000001000b11e                pmu_init
 .text.udivmoddi4
                0x000000001000b27c       0x96 ..\..\..\Libraries\libs\libplatform.a(sys.o)
 .text.sys_get_rc2m_clkhz
                0x000000001000b312      0x178 ..\..\..\Libraries\libs\libplatform.a(sys.o)
                0x000000001000b312                sys_get_rc2m_clkhz
 .text.sys_get_rand_key_init
                0x000000001000b48a       0x76 ..\..\..\Libraries\libs\libplatform.a(sys.o)
                0x000000001000b48a                sys_get_rand_key_init
 .text.sys_get_rand_key
                0x000000001000b500       0x5a ..\..\..\Libraries\libs\libplatform.a(sys.o)
                0x000000001000b500                sys_get_rand_key
 .text.bsp.param
                0x000000001000b55a       0x66 ..\..\..\Libraries\libs\libplatform.a(sys.o)
                0x000000001000b55a                param_bt_xosc_read
                0x000000001000b58e                bt_save_xosc_cap
 .text.xosc_init
                0x000000001000b5c0       0xa2 ..\..\..\Libraries\libs\libplatform.a(sys.o)
                0x000000001000b5c0                xosc_init
 .text.bt_restore_xosc_cap
                0x000000001000b662        0x4 ..\..\..\Libraries\libs\libplatform.a(sys.o)
                0x000000001000b662                bt_restore_xosc_cap
 .text.bt_get_xosc_cap
                0x000000001000b666       0x18 ..\..\..\Libraries\libs\libplatform.a(sys.o)
                0x000000001000b666                bt_get_xosc_cap
 .text.bt_set_xosc_cap
                0x000000001000b67e       0x26 ..\..\..\Libraries\libs\libplatform.a(sys.o)
                0x000000001000b67e                bt_set_xosc_cap
 .text.bt_adj_xosc_cap
                0x000000001000b6a4       0x8a ..\..\..\Libraries\libs\libplatform.a(sys.o)
                0x000000001000b6a4                bt_adj_xosc_cap
 .text.__udivdi3
                0x000000001000b72e        0x6 ..\..\..\Libraries\libs\libplatform.a(sys.o)
                0x000000001000b72e                __udivdi3
 .text.sys_clk_cacl_curr
                0x000000001000b734       0x24 ..\..\..\Libraries\libs\libplatform.a(sys_clk.o)
 *fill*         0x000000001000b758        0x0 
 .text.sys_clk  0x000000001000b758      0x1f4 ..\..\..\Libraries\libs\libplatform.a(sys_clk.o)
                0x000000001000b758                get_clksel_val
                0x000000001000b76a                get_cur_sysclk
                0x000000001000b772                set_audec_clkdiv
                0x000000001000b790                set_sbcec_clkdiv
                0x000000001000b792                sysclk_update_baud
                0x000000001000b7ca                update_uart1baud_in_sysclk_set
                0x000000001000b7ec                sys_clk_set_do
 *fill*         0x000000001000b94c       0xb4 
 .text.set_sys_clk_do
                0x000000001000ba00      0x1f0 ..\..\..\Libraries\libs\libplatform.a(sys_clk.o)
                0x000000001000ba00                set_sys_clk_do
 .text.set_peripherals_clkdiv
                0x000000001000bbf0      0x11c ..\..\..\Libraries\libs\libplatform.a(sys_clk.o)
                0x000000001000bbf0                set_peripherals_clkdiv
 .text.get_sysclk_nhz
                0x000000001000bd0c       0x7e ..\..\..\Libraries\libs\libplatform.a(sys_clk.o)
                0x000000001000bd0c                get_sysclk_nhz
 .text.set_sys_clk
                0x000000001000bd8a       0x34 ..\..\..\Libraries\libs\libplatform.a(sys_clk.o)
                0x000000001000bd8a                set_sys_clk
 *fill*         0x000000001000bdbe        0x2 
 .text.sys_clk.table
                0x000000001000bdc0        0xa ..\..\..\Libraries\libs\libplatform.a(sys_clk.o)
                0x000000001000bdc0                sysclk_sel_tbl
 .text.voltage.trim
                0x000000001000bdca      0x188 ..\..\..\Libraries\libs\libplatform.a(voltage_trim.o)
                0x000000001000bdca                bt_get_ft_trim_value
                0x000000001000be00                dac_get_ft_trim_value
                0x000000001000be1e                voltage_trim_value_init
 .text.stack.api
                0x000000001000bf52       0x2a ..\..\..\Libraries\libs\libplatform.a(bt.o)
                0x000000001000bf52                bt_send_msg_do
 .text          0x000000001000bf7c       0x70 ..\..\..\Libraries\libs\libbtstack.a(nanos.o)
                0x000000001000bf7c                nanos_init
                0x000000001000bfb0                nanos_var_init
 .text          0x000000001000bfec       0x68 ..\..\..\Libraries\libs\libbtstack.a(patch.o)
                0x000000001000bfec                bb_patch_init
 .text          0x000000001000c054        0x2 ..\..\..\Libraries\libs\libbtstack.a(platform.o)
                0x000000001000c054                timer_sync_init
 .text          0x000000001000c056       0x1c ..\..\..\Libraries\libs\libbtstack.a(bt_sco.o)
                0x000000001000c056                lc_sco_pkt_init
                0x000000001000c058                lc_sco_codec_init
                0x000000001000c05c                lc_sco_codec_exit
                0x000000001000c060                lc_sco_codec_setup
                0x000000001000c070                lc_sco_codec_kill
 *fill*         0x000000001000c072      0x18e 
 .text          0x000000001000c200     0x216e ..\..\..\Libraries\libs\libbtstack.a(bt_acl.o)
                0x000000001000c3d2                bt_acl_init
                0x000000001000c40e                bt_acl_reset
                0x000000001000c478                bt_acl_start
                0x000000001000c71e                bt_acl_init_param
                0x000000001000c800                bt_acl_stop
                0x000000001000c8c0                bt_acl_flow_off
                0x000000001000c900                bt_acl_flow_on
                0x000000001000c980                bt_acl_flush_to_get
                0x000000001000c9c0                bt_acl_flush_to_set
                0x000000001000ca00                bt_acl_poll_int_get
                0x000000001000ca40                bt_acl_poll_int_set
                0x000000001000cb00                bt_acl_sniff_trans
                0x000000001000cc00                bt_acl_sniff
                0x000000001000cd00                bt_acl_unsniff
                0x000000001000cdb2                bt_acl_tx_enc
                0x000000001000cdd4                bt_acl_rx_enc
                0x000000001000cdfa                bt_acl_bcst_rx_enc
                0x000000001000ce24                bt_acl_enc_key_set
                0x000000001000cf00                bt_acl_master_clock_get
                0x000000001000cf80                bt_acl_clock_offset_get
                0x000000001000d000                bt_acl_rsw_slot_offset_get
                0x000000001000d080                bt_acl_rsw_slot_offset_set
                0x000000001000d100                bt_acl_sup_to_get
                0x000000001000d140                bt_acl_sup_to_set
                0x000000001000d180                bt_acl_tim_acc_set
                0x000000001000d200                bt_acl_edr_set
                0x000000001000d300                bt_acl_tx_pkt_types_set
                0x000000001000d400                bt_acl_dm1_pkt_type_dis
                0x000000001000d480                bt_acl_curr_txpwr_get
                0x000000001000d600                bt_acl_afh_set
                0x000000001000d800                bt_acl_afh_new
                0x000000001000d900                bt_acl_afh_cfm
                0x000000001000d980                bt_acl_rx_max_slot_get
                0x000000001000d9c0                bt_acl_rx_max_slot_set
                0x000000001000da00                bt_acl_test_mode_set
                0x000000001000dac0                bt_acl_rssi_thr_get
                0x000000001000daf0                bt_sco_start
                0x000000001000df00                bt_sco_stop
                0x000000001000df80                bt_acl_sniff_clock_set
                0x000000001000e000                bt_acl_sniff_clock_diff
                0x000000001000e100                bt_acl_resche
 *fill*         0x000000001000e36e       0x92 
 .text          0x000000001000e400      0xca6 ..\..\..\Libraries\libs\libbtstack.a(ble_con.o)
                0x000000001000e400                ble_con_evt_time_update_fix
                0x000000001000e500                ble_con_start_do
                0x000000001000e528                ble_con_start
                0x000000001000ea00                ble_con_stop
                0x000000001000ea80                ble_con_param_update
                0x000000001000eb00                ble_con_phys_update
                0x000000001000eb80                ble_con_tx_len_update_for_intv
                0x000000001000ec00                ble_con_tx_len_update_for_rate
                0x000000001000ec80                ble_con_event_counter_get
                0x000000001000ecb0                ble_con_tx_enc
                0x000000001000ecfc                ble_con_rx_enc
                0x000000001000ed48                ble_con_enc_key_load
                0x000000001000ee00                ble_con_current_tx_power_get
                0x000000001000ee80                ble_con_rssi_get
                0x000000001000eeb0                ble_con_offset_get
                0x000000001000eeec                ble_con_pref_slave_latency_set
                0x000000001000ef2c                ble_con_pref_slave_evt_dur_set
                0x000000001000ef80                ble_con_peer_sca_set
                0x000000001000efaa                ble_con_duration_min_set
 *fill*         0x000000001000f0a6       0x5a 
 .text.bb.ble.con.flow
                0x000000001000f100       0xfa ..\..\..\Libraries\libs\libbtstack.a(ble_con.o)
                0x000000001000f100                ble_con_data_flow_set
 *fill*         0x000000001000f1fa        0x6 
 .text.bb.ble.con.data_len
                0x000000001000f200       0xfa ..\..\..\Libraries\libs\libbtstack.a(ble_con.o)
                0x000000001000f200                ble_con_data_len_update
 .text.le.con   0x000000001000f2fa       0x8c ..\..\..\Libraries\libs\libbtstack.a(ble_con.o)
                0x000000001000f2fa                ble_get_con_var
                0x000000001000f304                ble_con_init
 *fill*         0x000000001000f386        0x2 
 .text          0x000000001000f388      0x5d2 ..\..\..\Libraries\libs\libbtstack.a(bb_utils.o)
                0x000000001000f3d4                bb_bytes_to_string
                0x000000001000f412                bb_nb_good_channels
                0x000000001000f446                bb_util_pack
                0x000000001000f6c8                bb_util_unpack
 .text          0x000000001000f95a      0x1ba ..\..\..\Libraries\libs\libbtstack.a(bb_int.o)
                0x000000001000f95a                bb_time_set
                0x000000001000f978                bb_sleep_init
                0x000000001000f9d0                bb_driver_init
 *fill*         0x000000001000fb14       0xec 
 .text.bb.aes   0x000000001000fc00      0x1f6 ..\..\..\Libraries\libs\libbtstack.a(bb_int.o)
                0x000000001000fc00                bb_aes_encrypt
 .text          0x000000001000fdf6      0x2b6 ..\..\..\Libraries\libs\libbtstack.a(bb.o)
                0x000000001000fdf6                bb_rand_init
                0x000000001000fe00                bb_get_heap_info
                0x000000001000fe14                bb_var_init
                0x000000001000fe1c                bb_reset
                0x000000001000feac                bb_init
                0x000000001001002e                bb_off
                0x0000000010010080                bb_run_loop
 .text          0x00000000100100ac       0x1a ..\..\..\Libraries\libs\libbtstack.a(platform.o)
                0x00000000100100ac                lm_inq_start_do
                0x00000000100100b0                lm_inq_stop_do
                0x00000000100100b4                lm_inq_res_ind_do
                0x00000000100100b6                bt_pf_init
                0x00000000100100b8                bt_pf_exit
                0x00000000100100ba                bt_pf_post
                0x00000000100100bc                bt_pf_get_info
                0x00000000100100be                bt_is_ota_enable
 .text          0x00000000100100c6       0x50 ..\..\..\Libraries\libs\libbtstack.a(extern_tws.o)
                0x00000000100100c6                bt_tws_get_force_role
                0x00000000100100ca                tws_get_spp_eq_info
                0x00000000100100ce                tws_set_spp_eq_info
                0x00000000100100d0                bt_get_right_ear_sta
                0x00000000100100d4                bt_get_left_ear_sta
                0x00000000100100d8                bt_change_nr_sta
                0x00000000100100dc                bt_get_loc_nr_sta
                0x00000000100100e0                bt_get_auto_anwer_sta
                0x00000000100100e4                bt_set_menu_ctrl_sta
                0x00000000100100e6                tws_get_new_bt_name
                0x00000000100100ea                bt_get_serial_number
                0x00000000100100ee                bt_get_ch_serial_number
                0x00000000100100f2                bt_inear_test
                0x000000001001010e                bt_get_model_number
                0x0000000010010112                bt_get_fw_version
 .text          0x0000000010010116       0x9a ..\..\..\Libraries\libs\libbtstack.a(extern_bt.o)
                0x0000000010010116                bt_rf_get_inq_param
                0x000000001001011a                bt_rf_get_param
                0x000000001001011e                bt_rf_get_sco_param
                0x0000000010010122                bt_rf_get_fcc_param
                0x000000001001013a                bt_get_new_local_name
                0x000000001001013e                bt_set_new_local_name
                0x000000001001014e                bt_is_always_reconn
                0x0000000010010152                bt_get_conn_fail_delay
                0x0000000010010158                bt_get_connect_addr
                0x0000000010010180                tws_set_fot_data
                0x0000000010010184                tws_get_fot_data
                0x0000000010010188                tws_get_dueros_dma_data
                0x000000001001018c                tws_set_dueros_dma_data
                0x0000000010010190                tws_send_dueros_dma_data_cfm
                0x0000000010010192                tws_set_switch_fix_acl
                0x0000000010010196                is_bt_nor_linkkey_prohibit_del
                0x000000001001019a                bt_voice_callback
                0x000000001001019c                spp_custom1_rx_callback
                0x000000001001019e                spp_custom2_rx_callback
                0x00000000100101a2                spp_client_cfg_callback
                0x00000000100101a8                spp_custom1_connect_callback
                0x00000000100101aa                spp_custom1_disconnect_callback
                0x00000000100101ac                spp_custom2_connect_callback
                0x00000000100101ae                spp_custom2_disconnect_callback
 .text          0x00000000100101b0      0x398 ..\..\..\Libraries\libs\libbtstack.a(spp.o)
                0x0000000010010214                spp_disconnect
                0x00000000100102cc                spp_service_flush
                0x00000000100102d8                get_spp_connection_context_for_rfcomm_cid
                0x0000000010010308                get_spp_connection_context_for_bd_addr
                0x00000000100103e4                provide_spp_connection_context_for_bd_addr
                0x000000001001044c                spp_establish_service_level_connection
                0x00000000100104c6                spp_release_service_level_connection
                0x0000000010010510                spp_init
                0x0000000010010530                spp_init_var
                0x0000000010010540                spp_support_mul_server
 .text.stack.spp.handler
                0x0000000010010548      0x23c ..\..\..\Libraries\libs\libbtstack.a(spp.o)
                0x0000000010010548                spp_packet_handler
 .text.stack.sdp.util
                0x0000000010010784      0x60e ..\..\..\Libraries\libs\libbtstack.a(sdp_util.o)
                0x0000000010010836                de_get_size_type
                0x000000001001083e                de_get_element_type
                0x0000000010010846                de_get_header_size
                0x0000000010010864                de_get_data_size
                0x00000000100108a8                de_get_len
                0x0000000010010980                de_element_get_uint16
                0x00000000100109ac                de_get_normalized_uuid
                0x0000000010010a06                de_get_uuid32
                0x0000000010010a2e                de_store_descriptor_with_len
                0x0000000010010a6c                des_iterator_init
                0x0000000010010a9c                des_iterator_get_type
                0x0000000010010aac                des_iterator_get_size
                0x0000000010010ad4                des_iterator_has_more
                0x0000000010010ae2                des_iterator_get_element
                0x0000000010010af8                des_iterator_next
                0x0000000010010b16                sdp_attribute_list_constains_id
                0x0000000010010c42                sdp_filter_attributes_in_attributeIDList
                0x0000000010010c7a                spd_get_filtered_size
                0x0000000010010c9c                sdp_get_attribute_value_for_attribute_id
                0x0000000010010cbc                sdp_set_attribute_value_for_attribute_id
                0x0000000010010ce2                sdp_record_contains_UUID128
                0x0000000010010d40                sdp_traversal_match_pattern
                0x0000000010010d6c                sdp_record_matches_service_search_pattern
                0x0000000010010d90                de_dump_data_element
 .text          0x0000000010010d92       0x42 ..\..\..\Libraries\libs\libbtstack.a(sdp_server.o)
                0x0000000010010dca                remove_sdp_server_context
 .text.stack.sdp.server
                0x0000000010010dd4      0x750 ..\..\..\Libraries\libs\libbtstack.a(sdp_server.o)
                0x0000000010010e22                sdp_get_service_record_handle
                0x0000000010010e56                sdp_get_record_for_handle
                0x0000000010010e64                sdp_create_service_record_handle
                0x0000000010010e84                sdp_handle_service_search_request
                0x0000000010011024                sdp_handle_service_attribute_request
                0x00000000100111a0                sdp_handle_service_search_attribute_request
 .text.stack.setup
                0x0000000010011524       0x3a ..\..\..\Libraries\libs\libbtstack.a(sdp_server.o)
                0x0000000010011524                sdp_init
 .text.stack.sdp.server_add
                0x000000001001155e       0x46 ..\..\..\Libraries\libs\libbtstack.a(sdp_server.o)
                0x000000001001155e                sdp_add_service
 *fill*         0x00000000100115a4        0x0 
 .text          0x00000000100115a4      0x79c ..\..\..\Libraries\libs\libbtstack.a(sdp_client.o)
                0x00000000100115a4                remove_sdp_client_context
                0x00000000100115ae                de_state_init
                0x00000000100115be                de_state_size
                0x000000001001161c                sdp_parser_init
                0x0000000010011642                sdp_parser_handle_chunk
                0x0000000010011886                sdp_parser_handle_done
                0x00000000100118e2                sdp_client_packet_handler
                0x0000000010011c26                sdp_client_init
                0x0000000010011c42                sdp_client_free
                0x0000000010011c56                sdp_client_query
 .text          0x0000000010011d40     0x195a ..\..\..\Libraries\libs\libbtstack.a(rfcomm.o)
                0x0000000010012308                rfcomm_multiplexer_finalize
                0x00000000100123a2                rfcomm_set_required_security_level
                0x00000000100123aa                rfcomm_can_send_packet_now
                0x00000000100123bc                rfcomm_request_can_send_now_event
                0x00000000100123d8                rfcomm_reserve_packet_buffer
                0x00000000100123dc                rfcomm_release_packet_buffer
                0x00000000100123e0                rfcomm_get_outgoing_buffer
                0x00000000100123ee                rfcomm_get_max_frame_size
                0x0000000010012402                rfcomm_create_channel_with_initial_credits
                0x000000001001240a                rfcomm_create_channel
                0x0000000010012412                rfcomm_disconnect
                0x0000000010012442                rfcomm_register_service_with_initial_credits
                0x000000001001244a                rfcomm_unregister_service
                0x0000000010012480                rfcomm_accept_connection
                0x00000000100124d0                crc8_calc
                0x0000000010012506                rfcomm_send_prepared
                0x00000000100125c2                rfcomm_send
                0x00000000100135c6                provide_rfcomm_multiplexer
                0x00000000100135e2                provide_rfcomm_channel
                0x000000001001363a                rfcomm_set_packet_handler_for_channels
                0x000000001001364e                rfcomm_get_now_incoming_credit
                0x0000000010013664                rfcomm_set_to_send_new_incoming_credit
 .text.stack.rfcomm
                0x000000001001369a       0x90 ..\..\..\Libraries\libs\libbtstack.a(rfcomm.o)
                0x0000000010013724                rfcomm_register_service
 .text.stack.setup
                0x000000001001372a       0x22 ..\..\..\Libraries\libs\libbtstack.a(rfcomm.o)
                0x000000001001372a                rfcomm_init
 .text.stack.link_key
                0x000000001001374c      0x60c ..\..\..\Libraries\libs\libbtstack.a(btstack_link_key_db.o)
                0x00000000100138be                btstack_get_link_addr
                0x0000000010013972                btstack_get_link_key
                0x0000000010013a06                btstack_get_link_feature
                0x0000000010013a3a                btstack_delete_link_key
                0x0000000010013ad4                btstack_delete_all_link_key
                0x0000000010013b42                btstack_put_link_key
                0x0000000010013c40                btstack_put_link_offset
                0x0000000010013c8c                btstack_delete_all_link_offset
                0x0000000010013cf8                btstack_put_link_feature
 .text.stack.setup
                0x0000000010013d58      0x184 ..\..\..\Libraries\libs\libbtstack.a(btstack_link_key_db.o)
                0x0000000010013d58                btstack_open_link_info
 .text.stack.link_key.get.name
                0x0000000010013edc       0x62 ..\..\..\Libraries\libs\libbtstack.a(btstack_link_key_db.o)
                0x0000000010013edc                btstack_get_link_name
 .text.stack.link_key.put.name
                0x0000000010013f3e       0x94 ..\..\..\Libraries\libs\libbtstack.a(btstack_link_key_db.o)
                0x0000000010013f3e                btstack_put_link_name
 .text          0x0000000010013fd2       0xac ..\..\..\Libraries\libs\libbtstack.a(btstack_util.o)
                0x0000000010013fd2                log_info_hexdump
                0x0000000010013fd4                log_info_key
                0x0000000010013fd6                uuid_add_bluetooth_prefix
                0x0000000010013ff8                uuid_has_bluetooth_prefix
                0x0000000010014014                sscanf_bd_addr
 .text.stack.util
                0x000000001001407e      0x126 ..\..\..\Libraries\libs\libbtstack.a(btstack_util.o)
                0x000000001001407e                bd_addr_cmp
                0x0000000010014084                bd_addr_copy
                0x000000001001408a                big_endian_read_16
                0x000000001001409a                big_endian_read_32
                0x00000000100140ba                big_endian_store_16
                0x00000000100140ce                big_endian_store_32
                0x0000000010014102                reverse_bytes
                0x000000001001411e                reverse_24
                0x0000000010014122                reverse_48
                0x0000000010014126                reverse_56
                0x000000001001412a                reverse_64
                0x000000001001412e                reverse_128
                0x0000000010014132                reverse_256
                0x0000000010014138                reverse_bd_addr
                0x000000001001413a                btstack_min
                0x0000000010014140                btstack_max
                0x0000000010014146                char_for_nibble
                0x000000001001416c                nibble_for_char
 .text.stack.hci_dump
                0x00000000100141a4       0x52 ..\..\..\Libraries\libs\libbtstack.a(btstack_util.o)
                0x00000000100141a4                bd_addr_to_str
 .text          0x00000000100141f6       0x7c ..\..\..\Libraries\libs\libbtstack.a(btstack_txpkt.o)
                0x00000000100141f6                txpkt_init
 *fill*         0x0000000010014272        0xe 
 .text.stk.txpkt.flush
                0x0000000010014280       0x82 ..\..\..\Libraries\libs\libbtstack.a(btstack_txpkt.o)
                0x0000000010014280                txpkt_flush
 *fill*         0x0000000010014302       0x7e 
 .text.stack.run_loop
                0x0000000010014380      0x174 ..\..\..\Libraries\libs\libbtstack.a(btstack_run_loop.o)
                0x0000000010014380                btstack_run_loop_set_timer_handler
                0x0000000010014384                btstack_run_loop_set_data_source_handler
                0x0000000010014388                btstack_run_loop_set_data_source_fd
                0x000000001001438c                btstack_run_loop_get_data_source_fd
                0x0000000010014390                btstack_run_loop_enable_data_source_callbacks
                0x000000001001439c                btstack_run_loop_disable_data_source_callbacks
                0x00000000100143ac                btstack_run_loop_add_data_source
                0x00000000100143b8                btstack_run_loop_remove_data_source
                0x00000000100143c4                btstack_run_loop_set_timer
                0x00000000100143e0                btstack_run_loop_set_timer_context
                0x00000000100143e4                btstack_run_loop_get_timer_context
                0x0000000010014400                btstack_run_loop_set_trig_ticks
                0x000000001001443c                btstack_run_loop_add_timer
                0x000000001001446c                btstack_run_loop_remove_timer
                0x000000001001449a                btstack_run_loop_get_ticks
                0x00000000100144a6                btstack_run_loop_ticks_for_ms
                0x00000000100144ac                btstack_run_loop_get_time_ms
                0x00000000100144ba                btstack_run_loop_timer_dump
 .text.stack.setup
                0x00000000100144f4       0x34 ..\..\..\Libraries\libs\libbtstack.a(btstack_run_loop.o)
                0x00000000100144f4                btstack_run_loop_init
 .text.stack.memory
                0x0000000010014528       0x9a ..\..\..\Libraries\libs\libbtstack.a(btstack_memory.o)
                0x0000000010014528                btstack_memory_l2cap_service_get
                0x0000000010014532                btstack_memory_l2cap_service_free
                0x000000001001453e                btstack_memory_l2cap_channel_get
                0x0000000010014548                btstack_memory_l2cap_channel_free
                0x0000000010014554                btstack_memory_rfcomm_multiplexer_get
                0x000000001001455e                btstack_memory_rfcomm_multiplexer_free
                0x000000001001456a                btstack_memory_rfcomm_service_get
                0x0000000010014574                btstack_memory_rfcomm_service_free
                0x0000000010014580                btstack_memory_rfcomm_channel_get
                0x000000001001458a                btstack_memory_rfcomm_channel_free
                0x0000000010014596                btstack_memory_whitelist_entry_get
                0x00000000100145a0                btstack_memory_whitelist_entry_free
                0x00000000100145ac                btstack_memory_sm_lookup_entry_get
                0x00000000100145b6                btstack_memory_sm_lookup_entry_free
 .text.stack.setup
                0x00000000100145c2       0xa6 ..\..\..\Libraries\libs\libbtstack.a(btstack_memory.o)
                0x00000000100145c2                btstack_memory_init
 .text.stack.linked_list
                0x0000000010014668       0x6c ..\..\..\Libraries\libs\libbtstack.a(btstack_linked_list.o)
                0x0000000010014668                btstack_linked_list_get_last_item
                0x0000000010014676                btstack_linked_list_add
                0x000000001001468a                btstack_linked_list_add_tail
                0x000000001001469e                btstack_linked_list_remove
                0x00000000100146b6                btstack_linked_list_count
                0x00000000100146c4                btstack_linked_list_iterator_remove
 .text          0x00000000100146d4      0x270 ..\..\..\Libraries\libs\libbtstack.a(btstack_link_ctrl.o)
                0x00000000100146d4                alloc_link_ctrl_context_for_bd_addr
                0x0000000010014758                btstack_link_ctrl_stop_timer
                0x0000000010014774                btstack_link_ctrl_set_timer
                0x00000000100147aa                link_ctrl_timer_handler
                0x0000000010014836                btstack_link_ctrl_get_num
                0x0000000010014854                btstack_link_ctrl_get_recon_sta
                0x000000001001487e                btstack_link_ctrl_get_links
                0x0000000010014892                btstack_link_ctrl_is_exist
                0x00000000100148ca                btstack_link_ctrl_abort_reconnect
 .text.stack.linkctrl
                0x0000000010014944      0x17a ..\..\..\Libraries\libs\libbtstack.a(btstack_link_ctrl.o)
                0x0000000010014944                chk_link_ctrl_context_use_up
                0x000000001001495e                get_link_ctrl_context_for_bd_addr
                0x00000000100149a8                provide_link_ctrl_context_for_bd_addr
                0x00000000100149c0                remove_link_ctrl_context
                0x0000000010014a2a                remove_pending_link_ctrl_context
                0x0000000010014a6c                remove_waiting_link_ctrl_context_for_bd_addr
 .text.stack.setup
                0x0000000010014abe       0x16 ..\..\..\Libraries\libs\libbtstack.a(btstack_link_ctrl.o)
                0x0000000010014abe                btstack_link_ctrl_init
 *fill*         0x0000000010014ad4        0x0 
 .text          0x0000000010014ad4     0x245e ..\..\..\Libraries\libs\libbtstack.a(sm.o)
                0x000000001001691a                sm_address_resolution_lookup
                0x000000001001699c                sm_cmac_ready
                0x00000000100169aa                sm_cmac_general_start
                0x0000000010016a10                sm_cmac_signed_write_start
                0x0000000010016a42                get_rand_addr
                0x0000000010016a50                sm_register_oob_data_callback
                0x0000000010016a58                sm_add_event_handler
                0x0000000010016a66                sm_set_accepted_stk_generation_methods
                0x0000000010016a70                sm_set_encryption_key_size_range
                0x0000000010016a82                sm_set_authentication_requirements
                0x0000000010016a8a                sm_set_io_capabilities
                0x0000000010016a92                sm_set_request_security
                0x0000000010016a9c                sm_set_er
                0x0000000010016aac                sm_set_ir
                0x0000000010016abc                sm_test_set_irk
                0x0000000010016adc                sm_test_use_fixed_local_csrk
                0x0000000010016ae8                sm_init
                0x0000000010016bca                sm_use_fixed_ec_keypair
                0x0000000010016bcc                sm_test_use_fixed_ec_keypair
                0x0000000010016bce                sm_encryption_key_size
                0x0000000010016bee                sm_authenticated
                0x0000000010016c0e                sm_authorization_state
                0x0000000010016c32                sm_send_security_request
                0x0000000010016c56                sm_request_pairing
                0x0000000010016cda                sm_authorization_decline
                0x0000000010016d24                sm_authorization_grant
                0x0000000010016d70                sm_bonding_decline
                0x0000000010016dca                sm_just_works_confirm
                0x0000000010016e02                sm_numeric_comparison_confirm
                0x0000000010016e04                sm_passkey_input
                0x0000000010016e42                sm_keypress_notification
                0x0000000010016e64                sm_le_device_index
                0x0000000010016e78                gap_random_address_set_mode
                0x0000000010016eb4                gap_random_address_get_mode
                0x0000000010016ebc                gap_random_address_set_update_period
                0x0000000010016ee2                gap_random_address_set
                0x0000000010016f1e                gap_advertisements_set_params
 .text          0x0000000010016f32      0x3bc ..\..\..\Libraries\libs\libbtstack.a(le_device_db_memory.o)
                0x0000000010016f32                le_device_db_init
                0x0000000010016f4c                le_device_db_set_local_bd_addr
                0x0000000010016f4e                le_device_db_count
                0x0000000010016f7a                le_device_db_remove
                0x0000000010016f94                le_device_db_add
                0x000000001001700a                le_device_db_info
                0x000000001001706a                le_device_db_encryption_set
                0x00000000100170d4                le_device_db_encryption_get
                0x0000000010017198                le_device_db_remote_csrk_get
                0x00000000100171c2                le_device_db_remote_csrk_set
                0x00000000100171e8                le_device_db_local_csrk_get
                0x0000000010017212                le_device_db_local_csrk_set
                0x0000000010017238                le_device_db_remote_counter_get
                0x000000001001724e                le_device_db_remote_counter_set
                0x0000000010017264                le_device_db_local_counter_get
                0x000000001001727a                le_device_db_local_counter_set
                0x0000000010017290                le_device_db_dump
 .text          0x00000000100172ee      0x1cc ..\..\..\Libraries\libs\libbtstack.a(gatt_server.o)
                0x0000000010017312                ble_init_att_do
                0x0000000010017354                ble_init_att_for_handle
                0x0000000010017392                ble_register_att_buf_for_handle
                0x00000000100173dc                ble_tx_notify
                0x0000000010017436                ble_tx_indication
                0x0000000010017438                ble_update_conn_param
                0x000000001001745a                ble_set_adv_interval
                0x0000000010017486                btstack_ble_disconnect
                0x0000000010017492                btstack_ble_set_adv_data
                0x00000000100174a6                btstack_ble_set_scan_rsp_data
 .text.att.r_cb
                0x00000000100174ba       0xb6 ..\..\..\Libraries\libs\libbtstack.a(gatt_server.o)
                0x00000000100174ba                att_read_callback
 .text.att.w_cb
                0x0000000010017570      0x1c8 ..\..\..\Libraries\libs\libbtstack.a(gatt_server.o)
                0x0000000010017570                att_write_callback
 .text.ble.att  0x0000000010017738       0x76 ..\..\..\Libraries\libs\libbtstack.a(gatt_server.o)
                0x0000000010017738                btstack_gatt_init
                0x00000000100177a2                btstack_ble_send_req
 .text.ble.hci  0x00000000100177ae       0x6a ..\..\..\Libraries\libs\libbtstack.a(gatt_server.o)
                0x00000000100177ae                btstack_ble_update_conn_param
                0x00000000100177ec                btstack_ble_set_adv_interval
 .text          0x0000000010017818      0x5b4 ..\..\..\Libraries\libs\libbtstack.a(gatt_profile.o)
                0x0000000010017818                ble_gatts_service_add
                0x00000000100178d6                ble_gatts_characteristic_add
                0x0000000010017ac6                ble_gatts_add_server_characteristic_descriptor
                0x0000000010017d1a                ble_gatts_init
                0x0000000010017d46                ble_att_write_callback
                0x0000000010017d84                ble_att_read_callback
                0x0000000010017dc2                ble_get_profile_data
 .text          0x0000000010017dcc      0x726 ..\..\..\Libraries\libs\libbtstack.a(att_server.o)
                0x0000000010017ff8                ble_get_max_mtu
                0x0000000010017ffe                att_server_register_service_handler
                0x0000000010018026                att_server_init
                0x00000000100180a4                att_server_register_packet_handler
                0x00000000100180ac                att_server_can_send_packet_now
                0x00000000100180be                att_server_request_can_send_now_event
                0x0000000010018422                att_server_notify
                0x000000001001846e                att_server_indicate
 .text          0x00000000100184f2       0xe6 ..\..\..\Libraries\libs\libbtstack.a(att_dispatch.o)
                0x000000001001858c                att_dispatch_register_client
                0x00000000100185a0                att_dispatch_register_server
                0x00000000100185b4                att_dispatch_client_can_send_now
                0x00000000100185ba                att_dispatch_server_can_send_now
                0x00000000100185bc                att_dispatch_client_request_can_send_now_event
                0x00000000100185ca                att_dispatch_server_request_can_send_now_event
 .text          0x00000000100185d8      0xf8c ..\..\..\Libraries\libs\libbtstack.a(att_db.o)
                0x00000000100187d2                att_uuid_for_handle
                0x00000000100187fc                att_set_db
                0x0000000010018804                att_set_read_callback
                0x000000001001880c                att_set_write_callback
                0x0000000010018814                att_dump_attributes
                0x0000000010018858                att_clear_transaction_queue
                0x0000000010018874                att_prepare_handle_value_notification
                0x00000000100188b2                att_prepare_handle_value_indication
                0x00000000100188f0                att_handle_request
                0x000000001001932a                gatt_server_get_get_handle_range_for_service_with_uuid16
                0x00000000100193b0                gatt_server_get_value_handle_for_characteristic_with_uuid16
                0x00000000100193f2                gatt_server_get_client_configuration_handle_for_characteristic_with_uuid16
                0x000000001001947e                gatt_server_get_value_handle_for_characteristic_with_uuid128
                0x00000000100194cc                gatt_server_get_client_configuration_handle_for_characteristic_with_uuid128
 .text          0x0000000010019564       0x8c ..\..\..\Libraries\libs\libbtstack.a(btstack_main.o)
                0x00000000100195e6                btstack_test_func
                0x00000000100195e8                btstack_ble_set_init_callback
 .text.stack.handler
                0x00000000100195f0      0x1b6 ..\..\..\Libraries\libs\libbtstack.a(btstack_main.o)
 .text.stack.ble.sm
                0x00000000100197a6       0x20 ..\..\..\Libraries\libs\libbtstack.a(btstack_main.o)
                0x00000000100197a6                le_sm_init
 .text.stack.ble.setup
                0x00000000100197c6       0x1c ..\..\..\Libraries\libs\libbtstack.a(btstack_main.o)
                0x00000000100197c6                btstack_ble_init
 .text.stack.setup
                0x00000000100197e2       0x8c ..\..\..\Libraries\libs\libbtstack.a(btstack_main.o)
                0x00000000100197e2                btstack_main
 .text          0x000000001001986e       0x18 ..\..\..\Libraries\libs\libbtstack.a(btstack_hal.o)
                0x000000001001986e                hal_tick_init
                0x0000000010019874                hal_tick_set_handler
 .text          0x0000000010019886      0x760 ..\..\..\Libraries\libs\libbtstack.a(btstack_api.o)
                0x0000000010019886                dma_start_speech_to_ai
                0x0000000010019888                btstack_ctl0_api
                0x0000000010019898                btstack_comm_api
                0x00000000100198b2                btstack_hid_api
                0x00000000100198cc                btstack_fcc_test_func
                0x00000000100198d0                btstack_spp_api
                0x00000000100198dc                btstack_audio_bypass
                0x000000001001992e                btstack_audio_enable
                0x000000001001996c                btstack_ctl_api
                0x00000000100199f8                btstack_tws_api
                0x00000000100199fa                btstack_a2dp_msg
                0x00000000100199fc                dma_stop_speech_to_ai
                0x00000000100199fe                btstack_reset_bt_name
                0x0000000010019a00                btstack_tws_switch_role
                0x0000000010019a02                btstack_tws_connect
                0x0000000010019a04                btstack_low_latency_en
                0x0000000010019a06                btstack_low_latency_dis
                0x0000000010019a08                btstack_ble_conn_by_addr
                0x0000000010019a0a                btstack_ble_enable_scan
                0x0000000010019a0c                btstack_ble_set_scan_param
                0x0000000010019a0e                btstack_nor_connect
                0x0000000010019a10                btstack_ble_set_adv_param
                0x0000000010019a12                btstack_ble_disable_scan
                0x0000000010019a14                bt_decode_init
                0x0000000010019a16                btstack_var_init
                0x0000000010019a46                btstack_establish_service_connection_do
                0x0000000010019a66                btstack_establish_service_connection
                0x0000000010019a6e                btstack_continue_establish_service_connection
                0x0000000010019a96                btstack_tws_search_slave
                0x0000000010019a98                btstack_emit_notice_status
                0x0000000010019ad0                btstack_connect_address
                0x0000000010019b60                btstack_emit_notice
                0x0000000010019b74                btstack_tws_disc_continue
                0x0000000010019b76                bt_emit_player_notice
                0x0000000010019bc4                btstack_tws_set_status
                0x0000000010019bc6                btstack_clr_dis_flag
                0x0000000010019bde                btstack_get_ext_feature
                0x0000000010019c08                btstack_set_hfp_status_ptr
                0x0000000010019c3a                btstack_set_hsp_status_ptr
                0x0000000010019c50                btstack_clr_hfp_status_ptr
                0x0000000010019c96                btstack_clr_hsp_status_ptr
                0x0000000010019cb2                bt_get_siri_status
                0x0000000010019cb6                btstack_get_tws_key
                0x0000000010019ce2                btstack_get_tws_msg
                0x0000000010019d10                btstack_get_tws_hid_key
                0x0000000010019d36                btstack_get_tws_hid_msg
                0x0000000010019d74                bt_tws_is_playing
                0x0000000010019d8a                bt_tws_is_calling
                0x0000000010019d8e                btstack_clr_l2cap_status
                0x0000000010019e52                btstack_sco_setup
                0x0000000010019ea0                btstack_sco_kill
                0x0000000010019f08                btstack_msg_is_busy
                0x0000000010019f1c                btstack_msg_set_busy
                0x0000000010019f32                btstack_audio_is_busy
                0x0000000010019f46                btstack_audio_set_busy
                0x0000000010019f54                audio_bypass_get_cnt
                0x0000000010019f64                btstack_set_lmp_test
                0x0000000010019f7c                btstack_set_clk_offset
                0x0000000010019f94                tws_remote_is_busy
                0x0000000010019f98                btstack_tws_is_nego_ring
                0x0000000010019f9c                btstack_tws_is_connected_for_handle
                0x0000000010019fa0                btstack_tws_user_key
                0x0000000010019fa2                btstack_sync_info
                0x0000000010019fa4                btstack_tws_set_ring
                0x0000000010019fa6                btstack_tws_remote_switch_role
                0x0000000010019fa8                btstack_get_connect_delay
 .text.stack.api
                0x0000000010019fe6      0x5c8 ..\..\..\Libraries\libs\libbtstack.a(btstack_api.o)
                0x0000000010019fe6                btstack_tws_disconnect
                0x000000001001a006                btstack_nor_disconnect
                0x000000001001a008                btstack_dma_stat_change
                0x000000001001a00a                btstack_off
                0x000000001001a038                btstack_start_work
                0x000000001001a050                btstack_set_scan
                0x000000001001a078                btstack_set_scan_param
                0x000000001001a08e                btstack_hid_connect
                0x000000001001a0be                btstack_spp_disconnect
                0x000000001001a0fa                btstack_hid_disconnect
                0x000000001001a136                btstack_fot_resp
                0x000000001001a138                bt_init
                0x000000001001a150                btstack_tws_set_scan
                0x000000001001a152                btstack_connect_for_bd_addr_do
                0x000000001001a1e8                btstack_tws_disconnect_do
                0x000000001001a1ea                btstack_connect_for_bd_addr
                0x000000001001a20a                btstack_connect
                0x000000001001a262                btstack_disconnect_do
                0x000000001001a2dc                btstack_disconnect
                0x000000001001a304                bt_hid_is_ready_to_discon
                0x000000001001a344                btstack_set_l2cap_status
                0x000000001001a4a8                bt_get_call_indicate
                0x000000001001a524                bt_is_playing
                0x000000001001a542                bt_is_ios_device
                0x000000001001a546                bt_is_support_vol_ctrl
                0x000000001001a54a                bt_is_connected
                0x000000001001a562                dma_get_change_key
                0x000000001001a566                dma_get_change_value
                0x000000001001a56a                btstack_message
 .text.stack.sleep
                0x000000001001a5ae       0x32 ..\..\..\Libraries\libs\libbtstack.a(btstack_api.o)
                0x000000001001a5ae                btstack_enter_sleep
                0x000000001001a5c6                btstack_exit_sleep
 .text.stack.setup
                0x000000001001a5e0       0xc4 ..\..\..\Libraries\libs\libbtstack.a(btstack_api.o)
                0x000000001001a5e0                btstack_setup
 *fill*         0x000000001001a6a4      0x15c 
 .text.stack.status
                0x000000001001a800      0x1ec ..\..\..\Libraries\libs\libbtstack.a(btstack_api.o)
                0x000000001001a800                bt_get_status_do
 .text          0x000000001001a9ec      0x158 ..\..\..\Libraries\libs\libbtstack.a(bt_api.o)
                0x000000001001aa0c                bt_wait_disconnect
                0x000000001001aa50                bt_sync_info
                0x000000001001aa5e                bt_start_work
                0x000000001001aa6c                bt_updata_local_name
                0x000000001001aa76                bt_nor_connect
                0x000000001001aa78                bt_nor_disconnect
                0x000000001001aa7a                bt_tws_get_scan
                0x000000001001aa7e                bt_tws_set_scan
                0x000000001001aa80                bt_tws_get_link_info
                0x000000001001aa84                bt_tws_delete_link_info
                0x000000001001aa86                bt_tws_user_key
                0x000000001001aa8a                bt_tws_switch
                0x000000001001aa8c                bt_sync_init
                0x000000001001aa8e                bt_tws_get_first_role
                0x000000001001aa92                bt_tws_is_en
                0x000000001001aa96                bt_nor_delete_link_info
                0x000000001001aa9c                bt_nor_get_link_info_addr
                0x000000001001aacc                bt_nor_get_link_info
                0x000000001001aad0                bt_get_link_btname
                0x000000001001ab28                bt_is_low_latency
                0x000000001001ab36                bt_connect_address
                0x000000001001ab40                bt_map_start
                0x000000001001ab42                bt_map_abort
 .text.stack.api
                0x000000001001ab44      0x144 ..\..\..\Libraries\libs\libbtstack.a(bt_api.o)
                0x000000001001ab44                bt_off
                0x000000001001ab76                bt_setup
                0x000000001001aba8                bt_connect
                0x000000001001abd6                bt_disconnect
                0x000000001001ac08                bt_set_scan
                0x000000001001ac12                bt_audio_bypass
                0x000000001001ac3a                bt_audio_enable
                0x000000001001ac62                bt_get_stack_local_name
                0x000000001001ac78                bt_set_stack_local_name
 .text          0x000000001001ac88       0x9e ..\..\..\Libraries\libs\libbtstack.a(ble_api.o)
                0x000000001001ac88                ble_disconnect
                0x000000001001ac92                ble_set_adv_data
                0x000000001001acca                ble_set_scan_rsp_data
                0x000000001001ad02                ble_enable_adv
                0x000000001001ad08                ble_disable_adv
                0x000000001001ad0e                ble_set_scan_param
                0x000000001001ad12                ble_scan_en
                0x000000001001ad14                ble_scan_dis
                0x000000001001ad16                ble_adv0_set_ctrl
                0x000000001001ad1e                ble_connect_by_addr
                0x000000001001ad22                ble_init_callback_register
 .text.stack.le.api
                0x000000001001ad26       0x86 ..\..\..\Libraries\libs\libbtstack.a(ble_api.o)
                0x000000001001ad26                ble_set_adv_params
 .text          0x000000001001adac       0x44 ..\..\..\Libraries\libs\libbtstack.a(bb_sche.o)
                0x000000001001adac                bb_sche_frag_ble_dur_set
                0x000000001001adbe                bb_sche_init
 .text          0x000000001001adf0       0x68 ..\..\..\Libraries\libs\libbtstack.a(bb_dbg.o)
                0x000000001001adf0                my_spi_init
                0x000000001001ae56                bb_dbg_init
 .text          0x000000001001ae58       0xf6 ..\..\..\Libraries\libs\libbtstack.a(bb_clk.o)
                0x000000001001ae58                bb_clk_init
                0x000000001001af4c                bb_clk_off
 .text.bb.aes   0x000000001001af4e      0x2a6 ..\..\..\Libraries\libs\libbtstack.a(aes.o)
                0x000000001001af4e                aes_init
                0x000000001001af98                aes_alloc
                0x000000001001afba                aes_start
                0x000000001001aff8                aes_encrypt
                0x000000001001b044                aes_rand
                0x000000001001b080                aes_result_handler
                0x000000001001b0e8                aes_xor_128
                0x000000001001b10a                aes_shift_left_128
                0x000000001001b134                ble_ecpy
 .text          0x000000001001b1f4      0x102 ..\..\..\Libraries\libs\libbtstack.a(vs_proc.o)
                0x000000001001b2e6                bt_fcc_test_ctrl
 .text          0x000000001001b2f6       0xd4 ..\..\..\Libraries\libs\libbtstack.a(vs_fcc.o)
                0x000000001001b348                vs_con_start
                0x000000001001b374                vs_con_end
                0x000000001001b390                vs_fcc_3m_packet_filter
 .text.bb.vs.fcc
                0x000000001001b3ca      0x1b8 ..\..\..\Libraries\libs\libbtstack.a(vs_fcc.o)
                0x000000001001b3ce                vs_fcc_test_cmd_do
 .text          0x000000001001b582       0x9e ..\..\..\Libraries\libs\libbtstack.a(vs.o)
                0x000000001001b582                vs_init
                0x000000001001b5c0                vs_reset_complete_evt
 .text          0x000000001001b620      0xb48 ..\..\..\Libraries\libs\libbtstack.a(rf_smart.o)
                0x000000001001b7fa                rfphy_pll_afc
                0x000000001001b856                rfphy_pll_idle
                0x000000001001b86c                rfphy_rx_dcoc
                0x000000001001b880                rfphy_rx_rccal
                0x000000001001b90a                rfphy_t2r
                0x000000001001b99e                rfphy_tx_dcoc
                0x000000001001b9fa                rfphy_rx
                0x000000001001baa4                rfphy_tx
                0x000000001001bb3a                rfphy_tx_tone
                0x000000001001bb7e                rfphy_sw_ctrl
                0x000000001001bbac                rfphy_test
                0x000000001001bbae                rfphy_txrx_init
                0x000000001001bbf6                rfphy_init
 .text.bb.rf    0x000000001001c168       0x48 ..\..\..\Libraries\libs\libbtstack.a(rf_smart.o)
                0x000000001001c168                rfphy_tx_pwr
 .text          0x000000001001c1b0      0x3f6 ..\..\..\Libraries\libs\libbtstack.a(rf.o)
                0x000000001001c1b0                rf_txpwr_dec
                0x000000001001c1ec                rf_txpwr_inc
                0x000000001001c228                rf_txpwr_max
                0x000000001001c24e                rf_txpwr_epc_inc
                0x000000001001c28e                rf_txpwr_epc_dec
                0x000000001001c2d0                rf_off
                0x000000001001c2e0                rf_reset
                0x000000001001c2e2                rf_init
 *fill*         0x000000001001c5a6       0x5a 
 .text          0x000000001001c600       0x82 ..\..\..\Libraries\libs\libbtstack.a(bt_hook.o)
                0x000000001001c600                bt_scan_update_param
                0x000000001001c658                bt_inq_scan_hook
 .text          0x000000001001c682       0x1c ..\..\..\Libraries\libs\libbtstack.a(ble_hook.o)
                0x000000001001c682                ble_hal_init_hook
 *fill*         0x000000001001c69e      0x162 
 .text          0x000000001001c800      0xdcc ..\..\..\Libraries\libs\libbtstack.a(hct_tl.o)
                0x000000001001cc00                hct_flush_acl_rx_pend
                0x000000001001ce00                hci_tx_done_do
                0x000000001001cef4                hci_tx_done
                0x000000001001d000                hci_tl_send
                0x000000001001d154                hci_tl_init
                0x000000001001d192                hci_cmd_get_max_param_size
                0x000000001001d1aa                hci_cmd_received
                0x000000001001d3fe                hci_acl_tx_data_alloc
                0x000000001001d4f4                hci_acl_tx_data_received
 .text          0x000000001001d5cc      0x6da ..\..\..\Libraries\libs\libbtstack.a(hct_msg.o)
                0x000000001001db82                hci_check_desc_tabs_order
                0x000000001001db84                hci_look_for_cmd_desc
                0x000000001001dc06                hci_look_for_evt_desc
                0x000000001001dc4a                hci_look_for_dbg_evt_desc
                0x000000001001dc64                hci_look_for_le_evt_desc
 .text          0x000000001001dca6       0xb8 ..\..\..\Libraries\libs\libbtstack.a(hct_fc.o)
                0x000000001001dca6                hci_fc_init
                0x000000001001dcb6                hci_fc_acl_buf_size_set
                0x000000001001dccc                hci_fc_acl_en
                0x000000001001dd12                hci_fc_host_nb_acl_pkts_complete
                0x000000001001dd34                hci_fc_check_host_available_nb_acl_packets
 .text          0x000000001001dd5e      0x710 ..\..\..\Libraries\libs\libbtstack.a(hct.o)
                0x000000001001ddd0                hci_send_2_host
                0x000000001001e18e                hci_ble_conhdl_register
                0x000000001001e1a0                hci_ble_conhdl_unregister
                0x000000001001e1b0                hci_bt_acl_bdaddr_register
                0x000000001001e1da                hci_bt_acl_conhdl_register
                0x000000001001e1f2                hci_bt_acl_bdaddr_unregister
                0x000000001001e208                hci_evt_mask_set
                0x000000001001e246                hct_init
                0x000000001001e290                hci_evt_filter_add
                0x000000001001e458                hci_voice_settings_get
                0x000000001001e462                hci_voice_settings_set
 .text          0x000000001001e46e      0x81a ..\..\..\Libraries\libs\libbtstack.a(lm.o)
                0x000000001001e4c2                lm_init
                0x000000001001e654                lm_set_scan_int
                0x000000001001e668                lm_new_link_alloc
                0x000000001001e682                lm_stop_link_alloc
                0x000000001001e6a8                lm_lt_addr_alloc
                0x000000001001e6e0                lm_lt_addr_free
                0x000000001001e70c                lm_get_nb_acl
                0x000000001001e770                lm_role_switch_start
                0x000000001001e7ba                lm_role_switch_finished
                0x000000001001e842                lm_get_features
                0x000000001001e8c4                lm_pscan_start
                0x000000001001e914                lm_pscan_restart
                0x000000001001e924                lm_acl_disc
                0x000000001001e958                lm_get_auth_en
                0x000000001001e968                lm_get_sp_en
                0x000000001001e978                lm_get_sec_con_host_supp
                0x000000001001e986                lm_get_pin_type
                0x000000001001e990                lm_get_con_accept_timeout
                0x000000001001e99a                lm_set_loc_name
                0x000000001001ea04                lm_get_loc_name
                0x000000001001ea0e                lm_get_loc_name_seg
                0x000000001001ea68                lm_get_loopback_mode
                0x000000001001ea72                lm_get_pub_key_192
                0x000000001001ea94                lm_get_priv_key_192
                0x000000001001eab4                lm_get_oob_local_commit
                0x000000001001eade                lm_get_sp_debug_mode
                0x000000001001eae8                lm_debug_key_compare_192
                0x000000001001eb1a                lm_get_dut_mode_en
                0x000000001001eb24                lm_afh_get_ch_ass_en
                0x000000001001eb2e                lm_afh_get_host_ch_class
                0x000000001001eb38                lm_afh_set_peer_ch_class
                0x000000001001eb52                lm_afh_get_master_ch_map
                0x000000001001eb5c                lm_afh_init_timer
                0x000000001001eb88                lm_is_acl_con
                0x000000001001eba4                lm_is_acl_con_role
                0x000000001001ebce                lm_page_scan_rep_mode_get
                0x000000001001ebd8                lm_sco_move_en
                0x000000001001ebe2                lm_extract_max_enc_key_size
                0x000000001001ebfc                lm_create_master_key
                0x000000001001ec48                lm_create_master_key_rand
                0x000000001001ec54                lm_get_master_key
                0x000000001001ec62                lm_get_master_key_rand
                0x000000001001ec70                lm_get_master_enc_rand
                0x000000001001ec7e                lm_get_master_enc_key_size
 .text          0x000000001001ec88      0x382 ..\..\..\Libraries\libs\libbtstack.a(bt_hal.o)
                0x000000001001ec88                bt_hal_init
                0x000000001001ee0a                bt_hal_reset
                0x000000001001ef8e                bt_bd_addr_get
                0x000000001001ef9c                bt_bd_addr_set
                0x000000001001efc8                bt_class_of_dev_get
                0x000000001001efd6                bt_class_of_dev_set
                0x000000001001efe6                bt_tim_acc_get
                0x000000001001f000                bt_afh_ch_assess_get
 .text          0x000000001001f00a      0x14e ..\..\..\Libraries\libs\libbtstack.a(bt21.o)
                0x000000001001f00a                bt_buf_init
                0x000000001001f0f4                bt21_init
                0x000000001001f12e                bt21_reset
 .text          0x000000001001f158       0x62 ..\..\..\Libraries\libs\libbtstack.a(bc.o)
                0x000000001001f158                bc_init
                0x000000001001f17a                bc_reset
                0x000000001001f1aa                bc_get_nb_broadcast
                0x000000001001f1b2                bc_set_nb_broadcast
 *fill*         0x000000001001f1ba        0x6 
 .text          0x000000001001f1c0      0x430 ..\..\..\Libraries\libs\libbtstack.a(ble_hal.o)
                0x000000001001f1e6                ble_ral_search
                0x000000001001f238                ble_hal_init
                0x000000001001f4a4                ble_ch_assess_data_get
                0x000000001001f4ae                ble_rpa_renew
                0x000000001001f52c                ble_aa_gen
 *fill*         0x000000001001f5f0       0x10 
 .text          0x000000001001f600      0xb76 ..\..\..\Libraries\libs\libbtstack.a(ble_adv.o)
                0x000000001001f600                ble_get_adv_var
                0x000000001001f60a                ble_adv_init
                0x000000001001f700                ble_adv_stop
                0x000000001001f780                ble_adv_adv_data_update
                0x000000001001f800                ble_adv_scan_rsp_data_update
                0x000000001001f900                ble_adv_start_do
                0x000000001001f9ac                ble_adv_start
                0x0000000010020080                ble_adv_rand_addr_update
                0x0000000010020100                ble_adv_restart
 .text          0x0000000010020176       0x48 ..\..\..\Libraries\libs\libbtstack.a(ble.o)
                0x0000000010020176                ble_init
 .text.ble.var.init
                0x00000000100201be       0x38 ..\..\..\Libraries\libs\libbtstack.a(ble.o)
                0x00000000100201be                ble_var_init
 .text          0x00000000100201f6       0x4c ..\..\..\Libraries\libs\libbtstack.a(extern_ble.o)
                0x0000000010020210                ble_get_aap_addr
                0x000000001002021c                ble_client_cfg_callback
                0x000000001002021e                ble_adv0_get_adv_data_cb
                0x0000000010020222                ble_adv0_get_tws_role
                0x0000000010020236                ble_adv0_get_tws_loc_var
                0x000000001002023a                ble_adv0_set_tws_rem_var
                0x0000000010020240                ble_tx_test
 .text.bb.ble.adv0
                0x0000000010020242       0x28 ..\..\..\Libraries\libs\libbtstack.a(extern_ble.o)
                0x0000000010020242                ble_adv0_get_addr_cb
 .text          0x000000001002026a      0x30c ..\..\..\Libraries\libs\libbtstack.a(l2cap_test.o)
                0x0000000010020364                l2cap_end_of_test
                0x000000001002037a                l2cap_test_support_ext_feature
                0x0000000010020396                l2cap_test_cmd
                0x000000001002049e                l2cap_test_rsp
                0x00000000100204a0                l2cap_vd_acl_init
                0x00000000100204c2                l2cap_vd_enter_updateota
                0x00000000100204d0                l2cap_vd_exit_updateota
                0x00000000100204dc                l2cap_vd_acl_tx_request
 .text          0x0000000010020576      0x34e ..\..\..\Libraries\libs\libbtstack.a(l2cap.o)
                0x00000000100205c6                l2cap_register_packet_handler
                0x00000000100205ce                l2cap_send_test_cmd
                0x0000000010020620                l2cap_send_test_key
                0x000000001002064e                gap_request_connection_parameter_update
                0x0000000010020686                l2cap_get_outgoing_buffer
                0x0000000010020694                l2cap_reserve_packet_buffer
                0x0000000010020698                l2cap_release_packet_buffer
                0x000000001002069c                l2cap_send_prepared_connectionless
                0x00000000100206ee                l2cap_send_connectionless
                0x0000000010020724                l2cap_send_echo_request
                0x0000000010020730                l2cap_max_mtu
                0x0000000010020736                l2cap_max_le_mtu
                0x000000001002073c                l2cap_create_channel
                0x000000001002081c                l2cap_disconnect
                0x0000000010020838                provide_l2cap_channel
                0x000000001002089a                l2cap_unregister_service
 *fill*         0x00000000100208c4        0x0 
 .text.stack.handler.l2cap
                0x00000000100208c4      0x94c ..\..\..\Libraries\libs\libbtstack.a(l2cap.o)
                0x0000000010020b60                l2cap_emit_channel_closed
                0x00000000100211ae                l2cap_can_send_packet_now
                0x00000000100211cc                l2cap_can_send_prepared_packet_now
                0x00000000100211ea                l2cap_can_send_fixed_channel_packet_now
                0x00000000100211ee                l2cap_get_remote_mtu_for_local_cid
                0x0000000010021208                l2cap_stop_rtx
 .text.stack.l2cap
                0x0000000010021210      0x860 ..\..\..\Libraries\libs\libbtstack.a(l2cap.o)
                0x0000000010021228                l2cap_clear_pending_tx
                0x0000000010021938                l2cap_send_prepared
                0x00000000100219a0                l2cap_send
                0x00000000100219f2                l2cap_accept_connection
                0x0000000010021a0c                l2cap_decline_connection
                0x0000000010021a2c                l2cap_register_service
 .text.stack.setup
                0x0000000010021a70       0x72 ..\..\..\Libraries\libs\libbtstack.a(l2cap.o)
                0x0000000010021a70                l2cap_init
                0x0000000010021ac0                l2cap_register_fixed_channel
 .text.stack.setup
                0x0000000010021ae2        0x2 ..\..\..\Libraries\libs\libbtstack.a(hci_dump.o)
                0x0000000010021ae2                hci_dump_open
 .text.stack.hci_send
                0x0000000010021ae4      0x26c ..\..\..\Libraries\libs\libbtstack.a(hci_cmd.o)
                0x0000000010021ae4                hci_cmd_create_from_template
 .text          0x0000000010021d50      0x562 ..\..\..\Libraries\libs\libbtstack.a(hci.o)
                0x0000000010021efc                hci_alloc_num_packets_sent
                0x0000000010021f3c                hci_shutdown_connection
                0x0000000010021f78                gap_advertisements_get_address
                0x0000000010021fa4                hci_free_connect_waiting
                0x0000000010022002                gap_local_bd_addr
                0x0000000010022012                hci_emit_start_action
                0x0000000010022048                hci_emit_service_establish
                0x0000000010022076                gap_get_connection_type
                0x00000000100220ac                hci_set_sco_voice_setting_for_addr
                0x00000000100220c4                hci_get_sco_voice_setting_for_addr
                0x000000001002212e                gap_advertisements_set_data
                0x000000001002214a                gap_scan_response_set_data
                0x0000000010022166                hci_le_advertisements_set_params
                0x00000000100221aa                gap_advertisements_enable
                0x00000000100221e0                gap_inquiry
                0x00000000100221f6                gap_inquiry_cancel
                0x000000001002220c                gap_disconnect
                0x000000001002225e                hci_set_sco_voice_setting
                0x000000001002226a                hci_setup_sync
                0x00000000100222ae                hci_rx_flush
 .text.stack.hci
                0x00000000100222b2      0x934 ..\..\..\Libraries\libs\libbtstack.a(hci.o)
                0x00000000100223a2                hci_authentication_active_for_handle
                0x00000000100223c2                gap_drop_link_key_for_bd_addr
                0x00000000100223e4                gap_store_link_key_for_bd_addr
                0x0000000010022408                gap_get_link_feature_for_bd_addr
                0x0000000010022426                gap_store_link_feature_for_bd_addr
                0x0000000010022444                gap_get_link_addr_by_order
                0x0000000010022448                hci_number_free_acl_slots_for_handle
                0x0000000010022462                hci_can_send_acl_classic_packet_now
                0x0000000010022478                hci_can_send_acl_le_packet_now
                0x000000001002248a                hci_can_send_prepared_acl_packet_now
                0x00000000100224aa                hci_can_send_acl_packet_now
                0x00000000100224bc                hci_is_packet_buffer_reserved
                0x00000000100224c8                hci_reserve_packet_buffer
                0x00000000100224e0                hci_release_packet_buffer
                0x00000000100225b0                hci_send_acl_packet_buffer
                0x0000000010022600                hci_usable_acl_packet_types
                0x000000001002260c                hci_get_outgoing_packet_buffer
                0x0000000010022616                hci_max_acl_data_packet_length
                0x0000000010022622                hci_non_flushable_packet_boundary_flag_supported
                0x0000000010022632                hci_disconnect_security_block
                0x000000001002264c                gap_ssp_set_enable
                0x0000000010022658                update_extend_inquiry_response
                0x0000000010022680                hci_run_le_connection
                0x0000000010022764                hci_remote_esco_supported
                0x000000001002277e                gap_ssp_supported_on_both_sides
                0x00000000100227b0                hci_local_had_auth_request
                0x00000000100227da                gap_security_level_for_link_key_type
                0x000000001002280c                hci_run_pend_connection
                0x0000000010022aa4                gap_mitm_protection_required_for_security_level
                0x0000000010022aae                gap_security_level
                0x0000000010022ac6                hci_run_w2_connection
                0x0000000010022b86                gap_w_scan_control
                0x0000000010022ba0                gap_request_security_level
 *fill*         0x0000000010022be6        0x2 
 .text.stack.hci_init
                0x0000000010022be8      0x3c6 ..\..\..\Libraries\libs\libbtstack.a(hci.o)
                0x0000000010022c20                gap_set_local_name
                0x0000000010022f7c                hci_power_control
 .text.stack.handler.acl
                0x0000000010022fae       0x16 ..\..\..\Libraries\libs\libbtstack.a(hci.o)
 .text.stack.setup
                0x0000000010022fc4      0x166 ..\..\..\Libraries\libs\libbtstack.a(hci.o)
                0x0000000010023014                hci_add_event_handler
                0x0000000010023022                hci_register_acl_packet_handler
                0x000000001002302c                hci_init
                0x00000000100230c8                hci_set_chipset
                0x00000000100230dc                gap_set_class_of_device
                0x00000000100230e6                hci_set_bd_addr
                0x0000000010023106                gap_ssp_set_io_capability
                0x0000000010023112                gap_ssp_set_authentication_requirement
                0x000000001002311e                gap_ssp_set_auto_accept
 .text.stack.hci_emit
                0x000000001002312a      0x148 ..\..\..\Libraries\libs\libbtstack.a(hci.o)
                0x00000000100231d8                hci_emit_state
                0x0000000010023206                hci_emit_scan_ctrl
                0x000000001002322c                hci_emit_inquiry_ctrl
                0x0000000010023252                hci_emit_test_active
 .text.stack.hci.conn
                0x0000000010023272      0x1e2 ..\..\..\Libraries\libs\libbtstack.a(hci.o)
                0x0000000010023272                create_connection_for_bd_addr_and_type
                0x000000001002337c                gap_get_connection_parameter_range
                0x000000001002338c                gap_set_connection_parameter_range
                0x000000001002339e                hci_get_connections
                0x00000000100233a8                hci_connection_for_bd_addr_and_type
                0x00000000100233e6                hci_connection_get_other_for_bd_addr_and_type
                0x0000000010023424                hci_connection_for_index
 .text.ble.hci  0x0000000010023454      0x132 ..\..\..\Libraries\libs\libbtstack.a(hci.o)
                0x0000000010023454                ble_event_cmd_complete
                0x00000000100234f2                ble_event_meta
 .text.stack.hci_send
                0x0000000010023586      0x2bc ..\..\..\Libraries\libs\libbtstack.a(hci.o)
                0x0000000010023586                hci_send_cmd_packet
                0x0000000010023746                hci_send_cmd
                0x000000001002379c                hci_send_create_connection_cmd
 *fill*         0x0000000010023842      0x1be 
 .text.stack.hci.run
                0x0000000010023a00      0x1c8 ..\..\..\Libraries\libs\libbtstack.a(hci.o)
 .text.stack.hci_rx
                0x0000000010023bc8      0x106 ..\..\..\Libraries\libs\libbtstack.a(hci.o)
                0x0000000010023bc8                acl_handler
 *fill*         0x0000000010023cce        0x2 
 .text.stack.handler.event
                0x0000000010023cd0      0xd3c ..\..\..\Libraries\libs\libbtstack.a(hci.o)
 .text          0x0000000010024a0c      0x1d4 ..\..\..\Libraries\libs\libbtstack.a(hid_usage.o)
                0x0000000010024a0c                hid_report_init
                0x0000000010024a1e                hid_report_set
                0x0000000010024a3e                hid_send_report_callback
                0x0000000010024a8c                btstack_hid_send
                0x0000000010024ab2                btstack_hid_key
                0x0000000010024b0c                btstack_hid_consumer
                0x0000000010024b40                btstack_hid_touch_screen
                0x0000000010024bce                bt_hid_is_send_complete
 .text          0x0000000010024be0      0x55e ..\..\..\Libraries\libs\libbtstack.a(hid_device.o)
                0x0000000010024ffe                bt_hid_is_connected
                0x0000000010025026                hid_device_init
                0x0000000010025066                hid_device_request_can_send_now_event
                0x000000001002506a                hid_device_send_interrupt_message
                0x000000001002506e                hid_device_send_contro_message
                0x0000000010025072                hid_establish_service_level_connection
                0x00000000100250e8                hid_release_service_level_connection
                0x000000001002510e                bt_hid_index_set
                0x0000000010025110                hid_get_interrupt_cid
 *fill*         0x000000001002513e        0x2 
 .text          0x0000000010025140      0xbd8 ..\..\..\Libraries\libs\libbtstack.a(hfp_hf.o)
                0x0000000010025b68                hfp_hf_packet_handler
                0x0000000010025bda                hfp_hf_init_codecs
                0x0000000010025c04                hfp_hf_init_supported_features
                0x0000000010025c0c                hfp_hf_init_hf_indicators
                0x0000000010025c0e                hfp_hf_establish_service_level_connection
                0x0000000010025c18                hfp_hf_release_service_level_connection
                0x0000000010025c32                hfp_hf_get_siri_status
                0x0000000010025c66                hfp_hf_set_call_switch_flag
                0x0000000010025c7a                hfp_hf_call_switch_for_index
                0x0000000010025cd8                hfp_hf_call_for_index
                0x0000000010025d16                hfp_hf_init
 .text.stack.api
                0x0000000010025d18      0x316 ..\..\..\Libraries\libs\libbtstack.a(hfp_hf.o)
                0x0000000010025d18                hfp_hf_switch_siri
                0x0000000010025d50                hfp_hf_is_calling
                0x0000000010025d6c                hfp_hf_answer_incoming_call
                0x0000000010025de2                hfp_hf_terminate_call
                0x0000000010025e36                hfp_hf_reject_incoming_call
                0x0000000010025e38                hfp_hf_swap_calls
                0x0000000010025e68                hfp_hf_dial_number
                0x0000000010025ea6                hfp_hf_at_cmd
                0x0000000010025edc                hfp_hf_custom_at_cmd
                0x0000000010025f0a                hfp_hf_redial_last_number_do
                0x0000000010025f4a                hfp_hf_redial_last_number
                0x0000000010025f5e                hfp_hf_set_speaker_gain
                0x0000000010025f98                hfp_hf_set_microphone_gain
                0x0000000010025fd2                hfp_hf_report_bat_state
                0x0000000010026010                hfp_hf_start_codec
 .text.stack.hfp.api1
                0x000000001002602e       0x28 ..\..\..\Libraries\libs\libbtstack.a(hfp_hf.o)
                0x000000001002602e                hfp_is_connect
 *fill*         0x0000000010026056        0x2 
 .text          0x0000000010026058      0xbcc ..\..\..\Libraries\libs\libbtstack.a(hfp.o)
                0x0000000010026058                hfp_init
                0x000000001002606a                hfp_var_init
                0x000000001002606c                send_str_over_rfcomm
                0x0000000010026094                join
                0x0000000010026108                join_bitmap
                0x0000000010026186                hfp_emit_call_indicate
                0x0000000010026188                hfp_get_connections
                0x0000000010026192                hfp_get_connection_for_index
                0x0000000010026196                get_hfp_connection_context_for_rfcomm_cid
                0x000000001002619a                get_hfp_connection_context_for_bd_addr
                0x000000001002619e                get_hfp_connection_context_for_sco_handle
                0x00000000100261a2                hfp_reset_context_flags
                0x00000000100261ca                hfp_reset_voice_recognition_flags
                0x00000000100261e4                provide_hfp_connection_context_for_bd_addr
                0x00000000100261fc                hfp_handle_hci_event
                0x00000000100262b0                hfp_parse
                0x0000000010026b14                hfp_establish_service_level_connection
                0x0000000010026b56                hfp_rfcomm_service_supported
                0x0000000010026b5a                hfp_release_audio_connection
                0x0000000010026b72                hfp_release_service_level_connection
                0x0000000010026bcc                hfp_setup_synchronous_connection
                0x0000000010026c22                hfp_set_packet_handler_for_rfcomm_connections
 .text          0x0000000010026c24        0x8 ..\..\..\Libraries\libs\libbtstack.a(a2dp.o)
                0x0000000010026c24                a2dp_is_playing
                0x0000000010026c28                a2dp_is_playing_fast
 .text.stack.memory
                0x0000000010026c2c       0x46 ..\..\..\Libraries\libs\libbtstack.a(btstack_memory_pool.o)
                0x0000000010026c2c                btstack_memory_pool_get
                0x0000000010026c38                btstack_memory_pool_free
                0x0000000010026c4c                btstack_memory_pool_create
 .text          0x0000000010026c72       0x92 ..\..\..\Libraries\libs\libbtstack.a(btstack_adv0.o)
                0x0000000010026c72                btstack_adv0_ctrl
                0x0000000010026cd6                ble_adv0_set_intv
                0x0000000010026cf2                ble_adv0_get_adv_en
                0x0000000010026d02                ble_adv0_idx_update
 .text          0x0000000010026d04       0x7c ..\..\..\Libraries\libs\libbtstack.a(hci_transport_hcic.o)
                0x0000000010026d04                hcic_recv_packet
                0x0000000010026d20                hcic_send_acl_segment
                0x0000000010026d54                hcic_rx_flush
                0x0000000010026d72                hci_init_var
 .text.stack.hcic
                0x0000000010026d80      0x128 ..\..\..\Libraries\libs\libbtstack.a(hci_transport_hcic.o)
                0x0000000010026d82                hcic_register_packet_handler
                0x0000000010026dea                hcic_close
                0x0000000010026e00                hcic_open
                0x0000000010026e42                hcic_send_packet
 .text          0x0000000010026ea8       0x24 ..\..\..\Libraries\libs\libbtstack.a(btstack_chipset_inner.o)
                0x0000000010026ec2                btstack_chipset_inner_instance
 .text          0x0000000010026ecc       0x1e ..\..\..\Libraries\libs\libbtstack.a(lm_hook.o)
                0x0000000010026ecc                lm_init_hook
                0x0000000010026ee6                lm_set_iac_en
                0x0000000010026ee8                lm_page_scan_end_hook
 .text          0x0000000010026eea     0x1d9a ..\..\..\Libraries\libs\libbtstack.a(lm_sp.o)
                0x0000000010027602                lm_n_is_zero
                0x0000000010027a2c                lm_sp_sha256_calculate
                0x0000000010027ab4                lm_sp_n_one
                0x0000000010027c70                lm_sp_n192_convert_wnaf
                0x0000000010027d14                lm_sp_p192_point_to_inf
                0x0000000010027d28                lm_sp_p192_point_jacobian_to_affine
                0x0000000010027d9e                lm_sp_p192_points_jacobian_to_affine
                0x0000000010027eae                lm_sp_p192_dbl
                0x0000000010028026                lm_sp_p192_add
                0x00000000100282be                lm_sp_pre_compute_points
                0x0000000010028306                lm_sp_p192_invert
                0x000000001002834c                lm_f1
                0x00000000100284be                lm_f2
                0x000000001002863c                lm_oob_f1
                0x00000000100287ae                lm_g
                0x0000000010028870                lm_f3
                0x0000000010028a1a                lm_generate_rand_16bytes
                0x0000000010028a78                lm_dhkey_calc_init
                0x0000000010028bb0                lm_dhkey_compare
 .text          0x0000000010028c84     0x1cca ..\..\..\Libraries\libs\libbtstack.a(lm_proc.o)
                0x000000001002a90a                lm_inq_start
                0x000000001002a924                lm_inq_stop
 .text          0x000000001002a94e      0xd3c ..\..\..\Libraries\libs\libbtstack.a(lm_key.o)
                0x000000001002ada0                lm_e1
                0x000000001002adfc                lm_e21
                0x000000001002ae38                lm_e22
                0x000000001002aeb8                lm_e3
                0x000000001002af16                lm_kc_key
                0x000000001002b666                lm_xor_key
                0x000000001002b66a                lm_get_rand_vec
 *fill*         0x000000001002b68a        0x2 
 .text          0x000000001002b68c     0x2e60 ..\..\..\Libraries\libs\libbtstack.a(lc.o)
                0x000000001002b6fe                lc_util_set_loc_trans_coll
                0x000000001002b71a                lc_cmd_stat_send
                0x000000001002b742                lc_mode_chg_evt_send
                0x000000001002b77e                lc_init
                0x000000001002b7c4                lc_reset
                0x000000001002b814                lc_afh_set
                0x000000001002b8e2                lc_chg_pkt_type_cmp
                0x000000001002b948                lc_chg_pkt_type_cont
                0x000000001002b9b6                lc_afh_start
                0x000000001002ba20                lc_con_cmp_evt_send
                0x000000001002ba88                lc_max_slot_mgt
                0x000000001002bb3a                lc_mst_qos_done
                0x000000001002bbae                lc_ptt
                0x000000001002bc54                lc_ptt_cmp
                0x000000001002bcba                lc_resp_auth
                0x000000001002bd74                lc_release
                0x000000001002bd94                lc_restore_to
                0x000000001002bde0                lc_start_lmp_to
                0x000000001002be4a                lc_start
                0x000000001002c06e                lc_comb_key_svr
                0x000000001002c170                lc_locepr_rsw
                0x000000001002c1c4                lc_locepr_lkref
                0x000000001002c21c                lc_enc_key_refresh
                0x000000001002c2fe                lc_initiator_epr
                0x000000001002c348                lc_init_calc_f3
                0x000000001002c3ca                lc_dhkey
                0x000000001002c410                lc_init_start_mutual_auth
                0x000000001002c45e                lc_mst_send_mst_key
                0x000000001002c54e                lc_init_passkey_loop
                0x000000001002c5bc                lc_pairing_cont
                0x000000001002c6ee                lc_legacy_pair
                0x000000001002c752                lc_passkey_comm
                0x000000001002c7ea                lc_qos_setup
                0x000000001002c862                lc_rd_rem_name
                0x000000001002c8b2                lc_resp_oob_wait_nonce
                0x000000001002c8d0                lc_start_enc
                0x000000001002c9d2                lc_epr_rsw_cmp
                0x000000001002ca3a                lc_start_enc_key_size
                0x000000001002caa6                lc_start_key_exch
                0x000000001002cb16                lc_resp_num_comp
                0x000000001002cb7a                lc_stop_enc
                0x000000001002cbe2                lc_epr_resp
                0x000000001002cc5c                lc_rem_enc
                0x000000001002ccd6                lc_stop_afh_reporting
                0x000000001002cd04                lc_local_switch
                0x000000001002cdde                lc_restore_afh_reporting
                0x000000001002ce32                lc_skip_hl_oob_req
                0x000000001002ce8c                lc_start_oob
                0x000000001002ceb8                lc_send_enc_mode
                0x000000001002cf22                lc_restart_enc
                0x000000001002cf68                lc_restart_enc_cont
                0x000000001002d020                lc_detach
                0x000000001002d0d0                lc_chg_pkt_type_retry
                0x000000001002d1b2                lc_rem_name_cont
                0x000000001002d228                lc_semi_key_cmp
                0x000000001002d2f2                lc_mst_key
                0x000000001002d3d8                lc_feat
                0x000000001002d430                lc_hl_connect
                0x000000001002d47c                lc_version
                0x000000001002d4b8                lc_ext_feat
                0x000000001002d4f6                lc_loc_auth
                0x000000001002d5a4                lc_packet_type
                0x000000001002d62e                lc_conn_seq_done
                0x000000001002d650                lc_rsw_done
                0x000000001002d776                lc_switch_cmp
                0x000000001002d792                lc_rem_switch
                0x000000001002d87e                lc_send_enc_chg_evt
                0x000000001002d8d4                lc_auth_cmp
                0x000000001002d9b2                lc_con_cmp
                0x000000001002da8a                lc_end_chk_colli
                0x000000001002dade                lc_enc_cmp
                0x000000001002db94                lc_mutual_auth_end2
                0x000000001002dcd4                lc_epr_change_lk
                0x000000001002dd2a                lc_epr_cmp
                0x000000001002ddb6                lc_mutual_auth_end
                0x000000001002dee8                lc_key_exch_end
                0x000000001002df5a                lc_sp_end
                0x000000001002dfb0                lc_calc_link_key
                0x000000001002e04c                lc_sp_fail
                0x000000001002e084                lc_resp_oob_nonce
                0x000000001002e10a                lc_resp_calc_f3
                0x000000001002e1d6                lc_start_passkey_loop
                0x000000001002e242                lc_start_passkey
                0x000000001002e310                lc_resp_pair
                0x000000001002e3cc                lc_pair
                0x000000001002e482                lc_check_all_slaves_support_sec_con
                0x000000001002e4b8                lc_get_curr_mode
 .text          0x000000001002e4ec      0x52c ..\..\..\Libraries\libs\libbtstack.a(mgr.o)
                0x000000001002e4ec                mgr_cmd_cmp_send
                0x000000001002e514                mgr_cmd_stat_send
                0x000000001002e53c                mgr_is_dev_connected
                0x000000001002e590                mgr_is_dev_synced
                0x000000001002e5fc                mgr_ral_search
                0x000000001002e642                mgr_ral_is_empty
                0x000000001002e654                mgr_ch_map_update
                0x000000001002e7c2                mgr_init
                0x000000001002e8c4                mgr_clk_acc_set
                0x000000001002e904                mgr_link_disc
                0x000000001002e93c                mgr_master_ch_map_get
                0x000000001002e946                mgr_le_evt_mask_check
                0x000000001002e962                mgr_le_get_features
                0x000000001002e986                mgr_ral_get
                0x000000001002e990                mgr_plan_elt_get
                0x000000001002e9a2                mgr_act_get_free
                0x000000001002e9f2                mgr_act_set_free
 .text.le.ll_cntl
                0x000000001002ea18      0x2f4 ..\..\..\Libraries\libs\libbtstack.a(ll.o)
                0x000000001002ea80                ll_cleanup
                0x000000001002eb0c                ll_init
                0x000000001002eb78                ll_role_get
                0x000000001002ebae                ll_proc_reg
                0x000000001002ebfa                ll_proc_id_get
                0x000000001002ec1a                ll_proc_state_get
                0x000000001002ec20                ll_proc_state_set
                0x000000001002ec26                ll_proc_get
                0x000000001002ec3e                ll_proc_err_ind
                0x000000001002ec66                ll_proc_unreg
                0x000000001002ecd6                ll_proc_collision_check
 .text.le.ll_cntl.start
                0x000000001002ed0c      0x20e ..\..\..\Libraries\libs\libbtstack.a(ll.o)
                0x000000001002ed0c                ll_start
 .text.le.ll_cntl.state
                0x000000001002ef1a       0x60 ..\..\..\Libraries\libs\libbtstack.a(ll.o)
                0x000000001002ef1a                ll_cntl_state_set
 .text.le.ll_cntl.stop
                0x000000001002ef7a       0x48 ..\..\..\Libraries\libs\libbtstack.a(ll.o)
                0x000000001002ef7a                ll_stop
 .text.le.ll_cntl.timer
                0x000000001002efc2       0xd8 ..\..\..\Libraries\libs\libbtstack.a(ll.o)
                0x000000001002efc2                ll_proc_timer_set
                0x000000001002f032                ll_proc_timer_set_state
 .text          0x000000001002f09a       0x20 ..\..\..\Libraries\libs\libbtstack.a(ble_test.o)
                0x000000001002f09a                ble_test_init
 *fill*         0x000000001002f0ba       0x46 
 .text          0x000000001002f100      0x702 ..\..\..\Libraries\libs\libbtstack.a(ble_scan.o)
                0x000000001002f166                ble_get_scan_var
                0x000000001002f170                ble_get_sync_var
                0x000000001002f17a                ble_scan_init
                0x000000001002f1f2                ble_scan_start
                0x000000001002f700                ble_scan_stop
                0x000000001002f738                ble_scan_params_update
 .text          0x000000001002f802        0x4 ..\..\..\Libraries\libs\libbtstack.a(ble_per_adv.o)
                0x000000001002f802                ble_get_per_adv_var
 *fill*         0x000000001002f806       0x3a 
 .text          0x000000001002f840      0x86e ..\..\..\Libraries\libs\libbtstack.a(ble_init.o)
                0x000000001002f840                ble_init_connect_req_pack
                0x000000001002f8ea                ble_init_init
                0x000000001002f958                ble_init_start
                0x0000000010030040                ble_init_stop
 .text          0x00000000100300ae      0x158 ..\..\..\Libraries\libs\libbtstack.a(ble_buf.o)
                0x00000000100300ae                ble_buf_init_do
                0x00000000100301bc                ble_buf_init
 .text.bb.ble.adv0
                0x0000000010030206      0x20a ..\..\..\Libraries\libs\libbtstack.a(ble_adv0.o)
                0x00000000100302be                ble_adv0_init
                0x0000000010030310                ble_adv0_end_ind
                0x000000001003034a                ble_adv0_set_en
                0x00000000100303a2                ble_adv0_update_adv_data
                0x0000000010030406                ble_adv0_set_interval
                0x000000001003040e                ble_adv0_copy
 .text          0x0000000010030410       0x2a ..\..\..\Libraries\libs\libbtstack.a(extern_hfhs.o)
                0x0000000010030410                hfp_notice_network_time
                0x0000000010030412                hfp_notice_ring_number
                0x0000000010030418                hfp_get_last_call_number
                0x000000001003041c                msbc_exit
                0x000000001003041e                bt_pbap_data_callback
                0x0000000010030420                hfp_get_mic_gain
                0x0000000010030424                hfp_get_spk_gain
                0x0000000010030428                hfp_get_bat_level
                0x000000001003042c                hfp_hf_established_hook
                0x0000000010030430                hfp_hf_send_custom_at_cmd_hook
                0x0000000010030434                hfp_hf_recv_custom_at_cmd_hook
                0x0000000010030438                hfp_hf_release_hook
 .text.func.outgoing
                0x000000001003043a       0x14 ..\..\..\Libraries\libs\libbtstack.a(extern_hfhs.o)
                0x000000001003043a                hfp_get_outgoing_number
                0x0000000010030444                hfp_get_at_cmd
 .text.func.btring
                0x000000001003044e        0x6 ..\..\..\Libraries\libs\libbtstack.a(extern_hfhs.o)
                0x000000001003044e                hfp_is_list_curr_calls
                0x0000000010030452                hfp_hf_emit_curr_calls
 .text.stack.l2cap_sig
                0x0000000010030454      0x134 ..\..\..\Libraries\libs\libbtstack.a(l2cap_signaling.o)
                0x0000000010030534                l2cap_next_sig_id
                0x0000000010030550                l2cap_next_local_cid
                0x0000000010030574                l2cap_create_signaling_classic
                0x000000001003057e                l2cap_create_signaling_le
 .text          0x0000000010030588       0xdc ..\..\..\Libraries\libs\libbtstack.a(lc_hook.o)
                0x0000000010030588                lc_lmp_ver_req_hook
                0x00000000100305ae                lc_lmp_ver_res_hook
                0x00000000100305b0                lc_loc_sniff_req_hook
                0x00000000100305ec                lmp_sniff_req_hook
                0x000000001003060e                lc_auto_sniff_step_set
 *fill*         0x0000000010030664        0x0 
 .text          0x0000000010030664     0x17ca ..\..\..\Libraries\libs\libbtstack.a(lm_sco.o)
                0x00000000100310e8                lm_get_sync_param
                0x0000000010031a62                lm_init_sync
                0x0000000010031a84                lm_reset_sync
                0x0000000010031ab4                lm_check_active_sync
                0x0000000010031ac2                lm_add_sync
                0x0000000010031c4c                lm_check_sync_hl_rsp
                0x0000000010031d20                lm_get_synchdl
                0x0000000010031d3e                lm_look_for_sync
                0x0000000010031d88                lm_get_nb_sync_link
                0x0000000010031d92                lm_get_min_sync_intv
                0x0000000010031db6                lm_remove_sync
                0x0000000010031e24                lm_sco_nego_end
 .text          0x0000000010031e2e      0x498 ..\..\..\Libraries\libs\libbtstack.a(lc_util.o)
                0x0000000010031e2e                lc_get_max_pkt_size
                0x0000000010031e9a                lc_compute_pkt_types
                0x0000000010031ec0                lc_update_acl_pkt_types
                0x0000000010031f12                lc_update_acl_edr_pkt_types
                0x0000000010031f8a                lc_reduce_acl_pkt_types
                0x0000000010031fc0                lc_pkt_types_to_max_slot
                0x0000000010032006                lc_get_qos_param
                0x0000000010032134                lc_gen_cof_for_addr
                0x000000001003215a                lc_check_edr_feature_for_pkt_types
                0x000000001003216a                lc_check_feature
                0x0000000010032198                lc_pref_rate_to_pkt_types
                0x0000000010032228                lc_max_slot_to_pkt_types
                0x0000000010032248                lc_get_common_pkt_types
 .text          0x00000000100322c6      0x9b2 ..\..\..\Libraries\libs\libbtstack.a(lc_sniff.o)
                0x0000000010032502                lc_sniff_init
                0x0000000010032514                lc_sniff_clear
                0x000000001003254a                lc_sniff_interval_get
                0x000000001003256a                lc_sniff_offset_update
                0x000000001003259a                lc_sniff_host_request
                0x0000000010032730                lc_sniff_peer_request
                0x0000000010032a00                lc_sniff_peer_accept
                0x0000000010032ad0                lc_sniff_peer_reject
                0x0000000010032afa                lc_sniff_acc_tx_cfm
                0x0000000010032afc                lc_sniff_timeout
                0x0000000010032b02                lc_sniff_unsniff
                0x0000000010032b66                lc_sniff_unsniff_peer_request
                0x0000000010032c12                lc_sniff_unsniff_peer_accept
                0x0000000010032c32                lc_sniff_unsniff_peer_reject
 .text          0x0000000010032c78     0x164c ..\..\..\Libraries\libs\libbtstack.a(lc_sco.o)
                0x0000000010033446                lc_sco_alloc_link
                0x000000001003348e                lc_sco_free_link
                0x00000000100334c6                lc_sco_get_conhdl
                0x0000000010033502                lc_sco_get_snoop_service
                0x0000000010033546                lc_sco_set_snoop_service
                0x0000000010033576                lc_sco_start_snoop
                0x0000000010033668                lc_sco_init
                0x0000000010033696                lc_sco_reset
                0x00000000100336e2                lc_sco_detach
                0x000000001003377a                lc_sco_release
                0x00000000100337f4                lc_sco_host_request
                0x00000000100338f2                lc_sco_host_accept
                0x0000000010033a80                lc_sco_host_reject
                0x0000000010033b1a                lc_sco_host_request_disc
                0x0000000010033ba4                lc_sco_peer_request
                0x0000000010033e0c                lc_sco_peer_accept
                0x0000000010033e7c                lc_sco_peer_reject
                0x0000000010033efe                lc_sco_peer_request_disc
                0x0000000010033fee                lc_sco_peer_accept_disc
                0x0000000010034094                lc_sco_peer_reject_disc
                0x0000000010034114                lc_sco_baseband_ack
                0x00000000100341e4                lc_sco_timeout
                0x0000000010034290                lc_sco_offset_update
 *fill*         0x00000000100342c4        0x0 
 .text          0x00000000100342c4     0x9234 ..\..\..\Libraries\libs\libbtstack.a(lc_proc.o)
                0x000000001003449e                hci_acl_data_lc_func
                0x0000000010034a50                lmp_detach_func
                0x0000000010034b46                lc_acl_rx_ind_func
                0x000000001003d4ae                lc_flush_acl_tx_pend
 .text          0x000000001003d4f8      0x6dc ..\..\..\Libraries\libs\libbtstack.a(lc_lmppdu.o)
                0x000000001003d4f8                lmp_find_desc
                0x000000001003d546                lmp_estab_allowed
                0x000000001003d57e                lmp_msg_pk
                0x000000001003d5e2                lmp_msg_unpk
                0x000000001003d654                lc_send_lmp
                0x000000001003d6be                lc_send_pdu_acc
                0x000000001003d6dc                lc_send_pdu_acc_ext4
                0x000000001003d706                lc_send_pdu_not_acc
                0x000000001003d728                lc_send_pdu_not_acc_ext4
                0x000000001003d756                lc_send_pdu_set_afh
                0x000000001003d798                lc_send_pdu_au_rand
                0x000000001003d7c2                lc_send_pdu_in_rand
                0x000000001003d7ec                lc_send_pdu_comb_key
                0x000000001003d816                lc_send_pdu_max_slot
                0x000000001003d834                lc_send_pdu_max_slot_req
                0x000000001003d852                lc_send_pdu_encaps_payl
                0x000000001003d87c                lc_send_pdu_encaps_head
                0x000000001003d8a2                lc_send_pdu_ptt_req
                0x000000001003d8c4                lc_send_pdu_sp_nb
                0x000000001003d8ee                lc_send_pdu_sp_cfm
                0x000000001003d918                lc_send_pdu_sres
                0x000000001003d942                lc_send_pdu_sco_lk_rem_req
                0x000000001003d964                lc_send_pdu_esco_lk_rem_req
                0x000000001003d98a                lc_send_pdu_auto_rate
                0x000000001003d9a4                lc_send_pdu_sup_to
                0x000000001003d9c2                lc_send_pdu_enc_key_sz_req
                0x000000001003d9e0                lc_send_pdu_feats_res
                0x000000001003da0c                lc_send_pdu_tim_acc
                0x000000001003da26                lc_send_pdu_feats_ext_req
                0x000000001003da5c                lc_send_pdu_io_cap_res
                0x000000001003daa6                lc_send_pdu_num_comp_fail
                0x000000001003dac4                lc_send_pdu_paus_enc_req
                0x000000001003dae2                lc_send_pdu_resu_enc_req
                0x000000001003db00                lc_send_pdu_setup_cmp
                0x000000001003db1a                lc_send_pdu_qos_req
                0x000000001003db3c                lc_send_pdu_slot_off
                0x000000001003db7e                lc_send_pdu_vers_req
                0x000000001003dbac                lc_send_pdu_dhkey_chk
 .text          0x000000001003dbd4      0x11a ..\..\..\Libraries\libs\libbtstack.a(mgr_proc.o)
 .text          0x000000001003dcee      0xa60 ..\..\..\Libraries\libs\libbtstack.a(mgr_init.o)
                0x000000001003dcee                hci_le_create_con_cmd_func
                0x000000001003e006                hci_le_ext_create_con_cmd_func
                0x000000001003e364                hci_le_create_con_cancel_cmd_func
                0x000000001003e3da                ble_init_end_ind_func
 .text          0x000000001003e74e      0x6da ..\..\..\Libraries\libs\libbtstack.a(mgr_hci.o)
 .text.le.mgr   0x000000001003ee28       0x38 ..\..\..\Libraries\libs\libbtstack.a(mgr_hci.o)
                0x000000001003ee28                hci_command_mgr_func
 .text          0x000000001003ee60      0x40a ..\..\..\Libraries\libs\libbtstack.a(ll_scan.o)
                0x000000001003ee60                hci_le_set_scan_param_cmd_func
                0x000000001003efae                hci_le_set_scan_en_cmd_func
 .text.le.ll_scan
                0x000000001003f26a      0x628 ..\..\..\Libraries\libs\libbtstack.a(ll_scan.o)
                0x000000001003f26a                ble_adv_rep_ind_func
                0x000000001003f800                ble_scan_end_ind_func
 .text          0x000000001003f892      0x826 ..\..\..\Libraries\libs\libbtstack.a(ll_adv.o)
                0x000000001003f94a                ll_adv_hdl_to_idx
                0x000000001003f98e                hci_le_rd_adv_ch_tx_pw_cmd_func
                0x000000001003f9ee                hci_le_set_adv_param_cmd_func
                0x000000001003fb98                hci_le_set_adv_data_cmd_func
                0x000000001003fc6c                hci_le_set_scan_rsp_data_cmd_func
                0x000000001003fd40                hci_le_set_adv_en_cmd_func
                0x000000001003ffc2                ll_adv_get_act_idx
                0x000000001004002c                ll_adv_get_set_id
 .text.le.ll_adv
                0x00000000100400b8      0x30a ..\..\..\Libraries\libs\libbtstack.a(ll_adv.o)
                0x00000000100400b8                ble_scan_req_ind_func
                0x0000000010040120                ble_adv_end_ind_func
 .text.le.ll_adv.con
                0x00000000100403c2      0x250 ..\..\..\Libraries\libs\libbtstack.a(ll_adv.o)
                0x00000000100403c2                ble_adv_end_con_ind
 .text          0x0000000010040612      0x3ae ..\..\..\Libraries\libs\libbtstack.a(ll_proc.o)
                0x0000000010040612                hci_command_ll_func
                0x0000000010040662                ble_acl_rx_ind_func
                0x00000000100407f8                ble_acl_tx_cfm_func
                0x0000000010040808                hci_acl_data_func
                0x00000000100408da                ll_cmd_cmp_send
                0x0000000010040908                hci_vs_set_pref_slave_latency_cmd_func
                0x000000001004094c                hci_vs_set_pref_slave_evt_dur_cmd_func
                0x0000000010040998                ll_cmd_stat_send
 .text          0x00000000100409c0      0x32e ..\..\..\Libraries\libs\libbtstack.a(ll_ping.o)
                0x0000000010040a40                hci_rd_auth_payl_to_cmd_func
                0x0000000010040aa4                ll_op_ping_ind_func
                0x0000000010040afa                ll_auth_payl_nearly_to_func
                0x0000000010040b68                ll_ping_restart
                0x0000000010040bc0                ll_auth_payl_real_to_func
                0x0000000010040c1e                ll_ping_set
                0x0000000010040c86                hci_wr_auth_payl_to_cmd_func
 .text.le.ll_cntl.pdu
                0x0000000010040cee       0x3c ..\..\..\Libraries\libs\libbtstack.a(ll_ping.o)
                0x0000000010040cee                ll_ping_req_func
                0x0000000010040d0a                ll_ping_rsp_func
 *fill*         0x0000000010040d2a        0x2 
 .text          0x0000000010040d2c      0xad0 ..\..\..\Libraries\libs\libbtstack.a(ll_phy_upd.o)
                0x0000000010041520                hci_le_rd_phy_cmd_func
                0x0000000010041588                hci_le_set_phy_cmd_func
                0x00000000100416ca                ll_op_phy_upd_ind_func
                0x0000000010041754                ble_phy_upd_cfm_func
                0x0000000010041790                ll_phy_upd_proc_start
 .text.le.ll_cntl.pdu
                0x00000000100417fc      0x212 ..\..\..\Libraries\libs\libbtstack.a(ll_phy_upd.o)
                0x00000000100417fc                ll_phy_req_func
                0x00000000100418c0                ll_phy_rsp_func
                0x0000000010041954                ll_phy_update_ind_func
 .text          0x0000000010041a0e      0x136 ..\..\..\Libraries\libs\libbtstack.a(ll_past.o)
                0x0000000010041a0e                hci_le_per_adv_set_info_transf_cmd_func
                0x0000000010041ac2                hci_le_set_per_adv_sync_transf_param_cmd_func
 .text          0x0000000010041b44      0x57c ..\..\..\Libraries\libs\libbtstack.a(ll_length.o)
                0x0000000010041dac                hci_le_set_data_len_cmd_func
                0x0000000010041eba                hci_vs_set_max_rx_size_and_time_cmd_func
                0x0000000010041fce                ll_op_length_upd_ind_func
                0x0000000010042034                ll_length_proc_start
 .text.le.ll_cntl.pdu
                0x00000000100420c0      0x204 ..\..\..\Libraries\libs\libbtstack.a(ll_length.o)
                0x00000000100420c0                ll_length_req_func
                0x000000001004222a                ll_length_rsp_func
 .text          0x00000000100422c4      0x2d6 ..\..\..\Libraries\libs\libbtstack.a(ll_feature.o)
                0x0000000010042474                hci_le_rd_rem_feats_cmd_func
                0x0000000010042524                ll_op_feats_exch_ind_func
 .text.le.ll_cntl.pdu
                0x000000001004259a      0x168 ..\..\..\Libraries\libs\libbtstack.a(ll_feature.o)
                0x000000001004259a                ll_feature_req_func
                0x0000000010042610                ll_slave_feature_req_func
                0x0000000010042686                ll_feature_rsp_func
 *fill*         0x0000000010042702        0x2 
 .text          0x0000000010042704      0xaa0 ..\..\..\Libraries\libs\libbtstack.a(ll_encrypt.o)
                0x0000000010042e5c                hci_le_en_enc_cmd_func
                0x0000000010042f32                hci_le_ltk_req_reply_cmd_func
                0x0000000010042fa6                hci_le_ltk_req_neg_reply_cmd_func
                0x0000000010043032                ll_encrypt_ind_func
                0x000000001004313c                ll_op_encrypt_ind_func
 .text.le.ll_cntl.pdu
                0x00000000100431a4      0x2fa ..\..\..\Libraries\libs\libbtstack.a(ll_encrypt.o)
                0x00000000100431a4                ll_pause_enc_req_func
                0x0000000010043222                ll_pause_enc_rsp_func
                0x0000000010043284                ll_enc_req_func
                0x000000001004336a                ll_enc_rsp_func
                0x00000000100433ec                ll_start_enc_req_func
                0x0000000010043446                ll_start_enc_rsp_func
 .text          0x000000001004349e      0x30a ..\..\..\Libraries\libs\libbtstack.a(ll_disconnect.o)
                0x000000001004349e                ble_disc_ind_func
                0x00000000100434f6                ll_stopped_ind_func
                0x000000001004354e                hci_disconnect_cmd_func
                0x00000000100435fc                ll_disconnect
                0x00000000100436de                ll_op_disconnect_ind_func
                0x0000000010043758                ll_init_term_proc
 .text.le.ll_cntl.pdu
                0x00000000100437a8       0x44 ..\..\..\Libraries\libs\libbtstack.a(ll_disconnect.o)
                0x00000000100437a8                ll_terminate_ind_func
 .text          0x00000000100437ec      0xce4 ..\..\..\Libraries\libs\libbtstack.a(ll_con_upd.o)
                0x0000000010044062                hci_le_con_upd_cmd_func
                0x000000001004418e                hci_le_rem_con_param_req_reply_cmd_func
                0x0000000010044228                hci_le_rem_con_param_req_neg_reply_cmd_func
                0x000000001004428a                ll_op_con_upd_ind_func
                0x000000001004431c                ble_con_param_upd_cfm_func
                0x0000000010044388                ble_con_offset_upd_ind_func
                0x00000000100443da                ll_con_move_cb
 .text.le.ll_cntl.pdu
                0x00000000100444d0      0x30c ..\..\..\Libraries\libs\libbtstack.a(ll_con_upd.o)
                0x00000000100444d0                ll_con_update_ind_func
                0x0000000010044630                ll_con_param_req_func
                0x0000000010044746                ll_con_param_rsp_func
 .text          0x00000000100447dc      0x2cc ..\..\..\Libraries\libs\libbtstack.a(ll_cntl.o)
                0x00000000100447dc                ll_pdu_send_reject_ind
                0x0000000010044830                ble_cntl_rx_ind_func
                0x0000000010044998                ble_cntl_tx_cfm_func
                0x00000000100449f0                hci_vs_send_cntl_cmd_func
                0x0000000010044a54                hci_vs_cntl_discard_cmd_func
 .text.le.ll_cntl.pdu
                0x0000000010044aa8       0x64 ..\..\..\Libraries\libs\libbtstack.a(ll_cntl.o)
 .text.le.ll_cntl.send
                0x0000000010044b0c      0x18a ..\..\..\Libraries\libs\libbtstack.a(ll_cntl.o)
                0x0000000010044b0c                ll_cntl_tx_check
                0x0000000010044bfc                ll_cntl_send
 .text          0x0000000010044c96      0x2d6 ..\..\..\Libraries\libs\libbtstack.a(ll_clk_acc.o)
                0x0000000010044df6                ll_op_clk_acc_ind_func
                0x0000000010044e4c                ll_clk_acc_modify
                0x0000000010044eca                hci_le_req_peer_sca_cmd_func
 .text.le.ll_cntl.pdu
                0x0000000010044f6c       0xb4 ..\..\..\Libraries\libs\libbtstack.a(ll_clk_acc.o)
                0x0000000010044f6c                ll_clk_acc_req_func
                0x0000000010044fca                ll_clk_acc_rsp_func
 .text          0x0000000010045020      0x37a ..\..\..\Libraries\libs\libbtstack.a(ll_chmap_upd.o)
                0x0000000010045222                hci_le_rd_chnl_map_cmd_func
                0x000000001004528c                ll_op_ch_map_upd_ind_func
                0x00000000100452ec                mgr_ch_map_update_ind_func
                0x0000000010045366                ble_ch_map_upd_cfm_func
 .text.le.ll_cntl.pdu
                0x000000001004539a      0x172 ..\..\..\Libraries\libs\libbtstack.a(ll_chmap_upd.o)
                0x000000001004539a                ll_channel_map_ind_func
                0x0000000010045462                ll_min_used_channels_ind_func
 .text          0x000000001004550c      0x176 ..\..\..\Libraries\libs\libbtstack.a(aes_rpa.o)
                0x00000000100455ce                aes_rpa_gen
                0x0000000010045620                aes_rpa_resolve
 .text          0x0000000010045682        0x4 ..\..\..\Libraries\libs\libbtstack.a(scan_hook.o)
                0x0000000010045682                ble_scan_end_ind_hook
 .text          0x0000000010045686        0x8 ..\..\..\Libraries\libs\libbtstack.a(adv_hook.o)
                0x0000000010045686                ble_adv_end_ind_hook
 .text          0x000000001004568e      0x21e ..\..\..\Libraries\libs\libbtstack.a(ll_version.o)
                0x000000001004579c                ll_op_ver_exch_ind_func
                0x0000000010045812                hci_rd_rem_ver_info_cmd_func
 .text.le.ll_cntl.pdu
                0x00000000100458ac       0x6e ..\..\..\Libraries\libs\libbtstack.a(ll_version.o)
                0x00000000100458ac                ll_version_ind_func
 .text          0x000000001004591a      0x11a ..\..\..\Libraries\libs\libbtstack.a(ll_pwr.o)
                0x000000001004591a                hci_rd_tx_pwr_lvl_cmd_func
                0x00000000100459b0                hci_rd_rssi_cmd_func
 *(.rodata*)
 *fill*         0x0000000010045a34        0x0 
 .rodata.str1.4
                0x0000000010045a34       0x3e Output\obj\Libraries\bsp\bsp_bt.o
 *fill*         0x0000000010045a72        0x2 
 .rodata.str1.4
                0x0000000010045a74      0x11d Output\obj\Libraries\bsp\bsp_fot.o
 *fill*         0x0000000010045b91        0x3 
 .rodata.str1.4
                0x0000000010045b94       0x76 Output\obj\Libraries\bsp\bsp_sys.o
 *fill*         0x0000000010045c0a        0x2 
 .rodata        0x0000000010045c0c       0xbc Output\obj\Libraries\BT\ble\ab_link\app.o
                0x0000000010045c0c                scan_data_const
                0x0000000010045c18                adv_data_const
                0x0000000010045c28                printer_primay_uuid16
                0x0000000010045c38                printer_write_uuid16
                0x0000000010045c48                printer_notify_uuid16
                0x0000000010045c58                printer2_primay_uuid16
                0x0000000010045c68                printer2_write_uuid16
                0x0000000010045c78                printer2_notify_uuid16
                0x0000000010045c88                app_primay_uuid16
                0x0000000010045c98                app_write_uuid16
                0x0000000010045ca8                app_notify_uuid16
                0x0000000010045cb8                fota_uuid16
 .rodata.str1.4
                0x0000000010045cc8        0xe Output\obj\Libraries\BT\ble\ab_link\app.o
 *fill*         0x0000000010045cd6        0x2 
 .rodata.str1.4
                0x0000000010045cd8       0x3a Output\obj\Libraries\BT\ble\ble.o
 *fill*         0x0000000010045d12        0x2 
 .rodata.str1.4
                0x0000000010045d14        0x5 Output\obj\Libraries\BT\spp\bt.o
 *fill*         0x0000000010045d19        0x3 
 .rodata.str1.4
                0x0000000010045d1c       0x58 Output\obj\Libraries\BT\spp\spp.o
 .rodata.str1.4
                0x0000000010045d74       0x7c Output\obj\Examples\Internal_Flash\Source\Internal_Flash.o
                                         0x80 (size before relaxing)
 .rodata.str1.4
                0x0000000010045df0       0x1e Output\obj\Examples\Internal_Flash\Project\main.o
 *fill*         0x0000000010045e0e        0x2 
 .rodata.str1.4
                0x0000000010045e10       0xfc ..\..\..\Libraries\libs\libplatform.a(cm.o)
 .rodata.str1.4
                0x0000000010045f0c       0x10 ..\..\..\Libraries\libs\libplatform.a(main.o)
 .rodata.str1.4
                0x0000000010045f1c       0x57 ..\..\..\Libraries\libs\libplatform.a(startup.o)
 *fill*         0x0000000010045f73        0x1 
 .rodata.str1.4
                0x0000000010045f74      0x104 ..\..\..\Libraries\libs\libplatform.a(lock.o)
 .rodata.str1.4
                0x0000000010046078       0x1d ..\..\..\Libraries\libs\libplatform.a(sys.o)
 *fill*         0x0000000010046095        0x3 
 .rodata.volt_trim
                0x0000000010046098       0xbc ..\..\..\Libraries\libs\libplatform.a(voltage_trim.o)
                0x0000000010046098                charge_trim_step
                0x00000000100460ac                vddcore_trim_step
                0x00000000100460cc                vddio_trim_step
                0x00000000100460ec                vddbko_trim_step
 .rodata.bb.tbl
                0x0000000010046154        0x8 ..\..\..\Libraries\libs\libbtstack.a(ble_con.o)
                0x0000000010046154                connect_req_dur_tab
 .rodata.bb.tbl
                0x000000001004615c       0x16 ..\..\..\Libraries\libs\libbtstack.a(bb_utils.o)
                0x000000001004615c                null_array
                0x000000001004616c                dft_addr
 *fill*         0x0000000010046172        0x2 
 .rodata        0x0000000010046174       0x20 ..\..\..\Libraries\libs\libbtstack.a(bb.o)
                0x0000000010046174                bb_hook
 .rodata.str1.4
                0x0000000010046194        0x5 ..\..\..\Libraries\libs\libbtstack.a(extern_bt.o)
                                          0xd (size before relaxing)
 *fill*         0x0000000010046199        0x3 
 .rodata        0x000000001004619c       0x18 ..\..\..\Libraries\libs\libbtstack.a(spp.o)
 .rodata.stack.spp
                0x00000000100461b4        0x2 ..\..\..\Libraries\libs\libbtstack.a(spp.o)
 *fill*         0x00000000100461b6        0x2 
 .rodata        0x00000000100461b8       0x10 ..\..\..\Libraries\libs\libbtstack.a(sdp_util.o)
                0x00000000100461b8                mfi_search_uuid128
 .rodata.sdp.tbl.spp
                0x00000000100461c8      0x11f ..\..\..\Libraries\libs\libbtstack.a(sdp_tbl.o)
                0x00000000100461c8                sdp_spp_dueros_ota_service_record
                0x000000001004622c                sdp_spp_proc_test_service_record
                0x0000000010046290                sdp_spp_service_record
 *fill*         0x00000000100462e7        0x1 
 .rodata.str1.4
                0x00000000100462e8        0x8 ..\..\..\Libraries\libs\libbtstack.a(sdp_client.o)
 .rodata        0x00000000100462f0       0x17 ..\..\..\Libraries\libs\libbtstack.a(sdp_client.o)
 *fill*         0x0000000010046307        0x1 
 .rodata        0x0000000010046308      0x100 ..\..\..\Libraries\libs\libbtstack.a(rfcomm.o)
 .rodata        0x0000000010046408       0x20 ..\..\..\Libraries\libs\libbtstack.a(btstack_util.o)
                0x0000000010046418                bluetooth_base_uuid
 .rodata.str1.4
                0x0000000010046428       0x1a ..\..\..\Libraries\libs\libbtstack.a(btstack_link_ctrl.o)
 *fill*         0x0000000010046442        0x2 
 .rodata.str1.4
                0x0000000010046444       0x51 ..\..\..\Libraries\libs\libbtstack.a(sm.o)
                                         0x55 (size before relaxing)
 *fill*         0x0000000010046495        0x3 
 .rodata        0x0000000010046498       0x64 ..\..\..\Libraries\libs\libbtstack.a(sm.o)
 .rodata.str1.4
                0x00000000100464fc       0x18 ..\..\..\Libraries\libs\libbtstack.a(le_device_db_memory.o)
                                         0x1c (size before relaxing)
 .rodata        0x0000000010046514       0x11 ..\..\..\Libraries\libs\libbtstack.a(gatt_server.o)
 *fill*         0x0000000010046525        0x3 
 .rodata        0x0000000010046528       0x38 ..\..\..\Libraries\libs\libbtstack.a(gatt_profile.o)
 .rodata        0x0000000010046560       0x10 ..\..\..\Libraries\libs\libbtstack.a(att_db.o)
 .rodata.str1.4
                0x0000000010046570       0x2e ..\..\..\Libraries\libs\libbtstack.a(btstack_api.o)
 *fill*         0x000000001004659e        0x2 
 .rodata        0x00000000100465a0       0xe0 ..\..\..\Libraries\libs\libbtstack.a(btstack_api.o)
                0x00000000100465a0                tws_key_tbl
                0x0000000010046668                tws_hid_key_tbl
 .rodata.stack.api
                0x0000000010046680      0x184 ..\..\..\Libraries\libs\libbtstack.a(btstack_api.o)
                0x0000000010046680                btstack_ctl0_tbl
                0x00000000100466d8                btstack_comm_tbl
                0x00000000100466f8                btstack_hid_tbl
                0x0000000010046704                btstack_ctl_tbl
                0x00000000100467d0                btstack_api_tbl
                0x0000000010046800                btstack_spp_tbl
 .rodata.stack.setup
                0x0000000010046804       0x14 ..\..\..\Libraries\libs\libbtstack.a(btstack_api.o)
 .rodata        0x0000000010046818       0x2c ..\..\..\Libraries\libs\libbtstack.a(bb_sche.o)
 .rodata        0x0000000010046844       0x18 ..\..\..\Libraries\libs\libbtstack.a(vs_proc.o)
 .rodata.bb.tbl
                0x000000001004685c        0x6 ..\..\..\Libraries\libs\libbtstack.a(rf_smart.o)
 *fill*         0x0000000010046862        0x2 
 .rodata.str1.4
                0x0000000010046864       0x20 ..\..\..\Libraries\libs\libbtstack.a(hct_tl.o)
 .rodata.str1.4
                0x0000000010046884      0x312 ..\..\..\Libraries\libs\libbtstack.a(hct_msg.o)
                                        0x362 (size before relaxing)
 *fill*         0x0000000010046b96        0x2 
 .rodata        0x0000000010046b98      0xc20 ..\..\..\Libraries\libs\libbtstack.a(hct_msg.o)
                0x0000000010046b98                hci_cmd_desc_root_tab
                0x0000000010046bd8                hci_evt_desc_tab
                0x0000000010046d58                hci_evt_le_desc_tab
                0x0000000010046dc8                hci_cmd_desc_tab_vs
                0x0000000010046e94                hci_cmd_desc_tab_le
                0x00000000100470f8                hci_cmd_desc_tab_testing
                0x0000000010047134                hci_cmd_desc_tab_stat_par
                0x0000000010047188                hci_cmd_desc_tab_info_par
                0x000000001004720c                hci_cmd_desc_tab_ctrl_bb
                0x0000000010047584                hci_cmd_desc_tab_lk_pol
                0x0000000010047608                hci_cmd_desc_tab_lk_ctrl
 .rodata        0x00000000100477b8       0x9c ..\..\..\Libraries\libs\libbtstack.a(lm.o)
 .rodata.bb.tbl
                0x0000000010047854       0x14 ..\..\..\Libraries\libs\libbtstack.a(bt21.o)
                0x0000000010047854                bt_ctl
 .rodata.bb.tbl
                0x0000000010047868        0x7 ..\..\..\Libraries\libs\libbtstack.a(ble_hal.o)
 *fill*         0x000000001004786f        0x1 
 .rodata.bb.tbl
                0x0000000010047870       0x14 ..\..\..\Libraries\libs\libbtstack.a(ble.o)
                0x0000000010047870                ble_ctl
 .rodata.l2cap  0x0000000010047884        0x9 ..\..\..\Libraries\libs\libbtstack.a(l2cap_test.o)
                0x0000000010047884                vs_test_actived_cmd
 *fill*         0x000000001004788d        0x3 
 .rodata.stack.l2cap
                0x0000000010047890        0x5 ..\..\..\Libraries\libs\libbtstack.a(l2cap.o)
 *fill*         0x0000000010047895        0x3 
 .rodata.str1.4
                0x0000000010047898       0xb8 ..\..\..\Libraries\libs\libbtstack.a(hci_cmd.o)
                                         0xd0 (size before relaxing)
 .rodata.stack.hci_send
                0x0000000010047950      0x2a0 ..\..\..\Libraries\libs\libbtstack.a(hci_cmd.o)
                0x0000000010047950                hci_le_set_default_phy
                0x0000000010047958                hci_le_write_suggested_default_data_len
                0x0000000010047960                hci_le_test_end
                0x0000000010047968                hci_le_transmitter_test
                0x0000000010047970                hci_le_receiver_test
                0x0000000010047978                hci_le_read_supported_states
                0x0000000010047980                hci_le_long_term_key_negative_reply
                0x0000000010047988                hci_le_long_term_key_request_reply
                0x0000000010047990                hci_le_start_encryption
                0x0000000010047998                hci_le_rand
                0x00000000100479a0                hci_le_encrypt
                0x00000000100479a8                hci_le_read_remote_used_features
                0x00000000100479b0                hci_le_read_channel_map
                0x00000000100479b8                hci_le_set_host_channel_classification
                0x00000000100479c0                hci_le_connection_update
                0x00000000100479c8                hci_le_remove_device_from_white_list
                0x00000000100479d0                hci_le_add_device_to_white_list
                0x00000000100479d8                hci_le_clear_white_list
                0x00000000100479e0                hci_le_read_white_list_size
                0x00000000100479e8                hci_le_create_connection_cancel
                0x00000000100479f0                hci_le_create_connection
                0x00000000100479f8                hci_le_set_scan_enable
                0x0000000010047a00                hci_le_set_scan_parameters
                0x0000000010047a08                hci_le_set_advertise_enable
                0x0000000010047a10                hci_le_set_scan_response_data
                0x0000000010047a18                hci_le_set_advertising_data
                0x0000000010047a20                hci_le_read_advertising_channel_tx_power
                0x0000000010047a28                hci_le_set_advertising_parameters
                0x0000000010047a30                hci_le_set_random_address
                0x0000000010047a38                hci_le_read_supported_features
                0x0000000010047a40                hci_le_read_buffer_size
                0x0000000010047a48                hci_le_set_event_mask
                0x0000000010047a50                hci_test_mode_emul
                0x0000000010047a58                hci_read_rssi
                0x0000000010047a60                hci_read_bd_addr
                0x0000000010047a68                hci_read_buffer_size
                0x0000000010047a70                hci_read_local_supported_features
                0x0000000010047a78                hci_read_local_supported_commands
                0x0000000010047a80                hci_write_loopback_mode
                0x0000000010047a88                hci_read_loopback_mode
                0x0000000010047a90                hci_write_le_host_supported
                0x0000000010047a98                hci_read_le_host_supported
                0x0000000010047aa0                hci_write_simple_pairing_mode
                0x0000000010047aa8                hci_write_extended_inquiry_response
                0x0000000010047ab0                hci_write_inquiry_scan_type
                0x0000000010047ab8                hci_write_inquiry_mode
                0x0000000010047ac0                hci_write_link_supervision_timeout
                0x0000000010047ac8                hci_host_buffer_size
                0x0000000010047ad0                hci_write_class_of_device
                0x0000000010047ad8                hci_write_scan_enable
                0x0000000010047ae0                hci_write_page_timeout
                0x0000000010047ae8                hci_write_local_name
                0x0000000010047af0                hci_reset
                0x0000000010047af8                hci_set_event_mask
                0x0000000010047b00                hci_switch_role_command
                0x0000000010047b08                hci_role_discovery
                0x0000000010047b10                hci_io_capability_request_negative_reply
                0x0000000010047b18                hci_remote_oob_data_request_negative_reply
                0x0000000010047b20                hci_user_passkey_request_negative_reply
                0x0000000010047b28                hci_user_passkey_request_reply
                0x0000000010047b30                hci_user_confirmation_request_negative_reply
                0x0000000010047b38                hci_user_confirmation_request_reply
                0x0000000010047b40                hci_io_capability_request_reply
                0x0000000010047b48                hci_accept_synchronous_connection
                0x0000000010047b50                hci_setup_synchronous_connection
                0x0000000010047b58                hci_read_clock_offset_command
                0x0000000010047b60                hci_read_remote_version_info_command
                0x0000000010047b68                hci_read_remote_supported_features_command
                0x0000000010047b70                hci_remote_name_request_cancel
                0x0000000010047b78                hci_remote_name_request
                0x0000000010047b80                hci_change_connection_link_key
                0x0000000010047b88                hci_set_connection_encryption
                0x0000000010047b90                hci_authentication_requested
                0x0000000010047b98                hci_pin_code_request_negative_reply
                0x0000000010047ba0                hci_pin_code_request_reply
                0x0000000010047ba8                hci_link_key_request_negative_reply
                0x0000000010047bb0                hci_link_key_request_reply
                0x0000000010047bb8                hci_reject_connection_request
                0x0000000010047bc0                hci_accept_connection_request
                0x0000000010047bc8                hci_create_connection_cancel
                0x0000000010047bd0                hci_disconnect
                0x0000000010047bd8                hci_create_connection
                0x0000000010047be0                hci_inquiry_cancel
                0x0000000010047be8                hci_inquiry
 .rodata        0x0000000010047bf0        0xc ..\..\..\Libraries\libs\libbtstack.a(hci.o)
 .rodata        0x0000000010047bfc       0x2d ..\..\..\Libraries\libs\libbtstack.a(hid_usage.o)
                0x0000000010047c14                ts_release
                0x0000000010047c20                ts_press
 *fill*         0x0000000010047c29        0x3 
 .rodata.str1.4
                0x0000000010047c2c      0x116 ..\..\..\Libraries\libs\libbtstack.a(hfp_hf.o)
                                        0x11a (size before relaxing)
 *fill*         0x0000000010047d42        0x2 
 .rodata.str1.4
                0x0000000010047d44       0x6d ..\..\..\Libraries\libs\libbtstack.a(hfp.o)
                                         0xd5 (size before relaxing)
 *fill*         0x0000000010047db1        0x3 
 .rodata        0x0000000010047db4       0x12 ..\..\..\Libraries\libs\libbtstack.a(hfp.o)
 *fill*         0x0000000010047dc6        0x2 
 .rodata.str1.4
                0x0000000010047dc8        0x6 ..\..\..\Libraries\libs\libbtstack.a(btstack_chipset_inner.o)
 *fill*         0x0000000010047dce        0x2 
 .rodata        0x0000000010047dd0       0x14 ..\..\..\Libraries\libs\libbtstack.a(btstack_chipset_inner.o)
 .rodata        0x0000000010047de4      0x1c8 ..\..\..\Libraries\libs\libbtstack.a(lm_sp.o)
 .rodata        0x0000000010047fac      0x2f4 ..\..\..\Libraries\libs\libbtstack.a(lm_proc.o)
 .rodata.bb.tbl
                0x00000000100482a0       0x1e ..\..\..\Libraries\libs\libbtstack.a(lm_proc.o)
                0x00000000100482a0                lm_local_supp_feats
 *fill*         0x00000000100482be        0x2 
 .rodata        0x00000000100482c0      0x420 ..\..\..\Libraries\libs\libbtstack.a(lm_key.o)
 .rodata        0x00000000100486e0       0x10 ..\..\..\Libraries\libs\libbtstack.a(lc.o)
 .rodata.str1.4
                0x00000000100486f0        0x2 ..\..\..\Libraries\libs\libbtstack.a(extern_hfhs.o)
                                          0x6 (size before relaxing)
 *fill*         0x00000000100486f2        0x2 
 .rodata.str1.4
                0x00000000100486f4       0x16 ..\..\..\Libraries\libs\libbtstack.a(l2cap_signaling.o)
                                         0x2a (size before relaxing)
 *fill*         0x000000001004870a        0x2 
 .rodata        0x000000001004870c       0x58 ..\..\..\Libraries\libs\libbtstack.a(l2cap_signaling.o)
 .rodata        0x0000000010048764       0x7c ..\..\..\Libraries\libs\libbtstack.a(lm_sco.o)
 .rodata        0x00000000100487e0       0x40 ..\..\..\Libraries\libs\libbtstack.a(lc_util.o)
 .rodata        0x0000000010048820      0x5dc ..\..\..\Libraries\libs\libbtstack.a(lc_proc.o)
 .rodata.str1.4
                0x0000000010048dfc       0x6b ..\..\..\Libraries\libs\libbtstack.a(lc_lmppdu.o)
                                         0x9b (size before relaxing)
 *fill*         0x0000000010048e67        0x1 
 .rodata        0x0000000010048e68      0x280 ..\..\..\Libraries\libs\libbtstack.a(lc_lmppdu.o)
 .rodata        0x00000000100490e8       0x60 ..\..\..\Libraries\libs\libbtstack.a(mgr_proc.o)
 .rodata.le.mgr_cntl.tbl
                0x0000000010049148       0xf0 ..\..\..\Libraries\libs\libbtstack.a(mgr_hci.o)
                0x0000000010049148                mgr_hci_cmd_tbl
 .rodata        0x0000000010049238       0x1c ..\..\..\Libraries\libs\libbtstack.a(ll_scan.o)
 .rodata.le.ll_cntl.tbl
                0x0000000010049254      0x1a8 ..\..\..\Libraries\libs\libbtstack.a(ll_proc.o)
                0x0000000010049254                ll_msg_tbl
                0x0000000010049334                ll_hci_cmd_tbl
 .rodata.str1.4
                0x00000000100493fc       0x3c ..\..\..\Libraries\libs\libbtstack.a(ll_cntl.o)
                                         0x59 (size before relaxing)
 .rodata.le.ll_cntl.tbl
                0x0000000010049438      0x1c8 ..\..\..\Libraries\libs\libbtstack.a(ll_cntl.o)
                0x0000000010049438                ll_cntl_pdu_tbl
 *(.srodata*)
 .srodata       0x0000000010049600        0x4 ..\..\..\Libraries\libs\libbtstack.a(bt_acl.o)
 .srodata       0x0000000010049604        0x3 ..\..\..\Libraries\libs\libbtstack.a(extern_bt.o)
                0x0000000010049605                cfg_bb_rf_ctl
 *fill*         0x0000000010049607        0x1 
 .srodata       0x0000000010049608        0x2 ..\..\..\Libraries\libs\libbtstack.a(btstack_link_key_db.o)
                0x0000000010049608                link_info_page_size
 *fill*         0x000000001004960a        0x2 
 .srodata       0x000000001004960c        0x8 ..\..\..\Libraries\libs\libbtstack.a(vs_proc.o)
 .srodata       0x0000000010049614        0x8 ..\..\..\Libraries\libs\libbtstack.a(hct_msg.o)
                0x0000000010049614                hci_evt_dbg_desc_tab
 .srodata       0x000000001004961c       0x1c ..\..\..\Libraries\libs\libbtstack.a(hct.o)
 .srodata       0x0000000010049638        0x6 ..\..\..\Libraries\libs\libbtstack.a(hci.o)
 *fill*         0x000000001004963e        0x2 
 .srodata       0x0000000010049640       0x10 ..\..\..\Libraries\libs\libbtstack.a(mgr.o)
 .srodata       0x0000000010049650        0x3 ..\..\..\Libraries\libs\libbtstack.a(lc_proc.o)
 *fill*         0x0000000010049653        0x1 
 .srodata       0x0000000010049654        0x8 ..\..\..\Libraries\libs\libbtstack.a(mgr_hci.o)
 .srodata       0x000000001004965c        0x5 ..\..\..\Libraries\libs\libbtstack.a(ll_adv.o)
 *(.rela*)
 .rela.text.btstack_ble_init_callback
                0x0000000010049661        0x0 Output\obj\Libraries\bsp\bsp_bt.o
 .rela.text.ble_init_register
                0x0000000010049661        0x0 Output\obj\Libraries\bsp\bsp_bt.o
 .rela.text.bsp_bt_init
                0x0000000010049661        0x0 Output\obj\Libraries\bsp\bsp_bt.o
 .rela.text.bsp_spp_disinit
                0x0000000010049661        0x0 Output\obj\Libraries\bsp\bsp_bt.o
 .rela.text.bt_emit_notice
                0x0000000010049661        0x0 Output\obj\Libraries\bsp\bsp_bt.o
 .rela.text.cm_factory
                0x0000000010049661        0x0 Output\obj\Libraries\bsp\bsp_bt.o
 .rela.text.fot.cache
                0x0000000010049661        0x0 Output\obj\Libraries\bsp\bsp_bt.o
 .rela.text.fot.update
                0x0000000010049661        0x0 Output\obj\Libraries\bsp\bsp_bt.o
 .rela.text.fot_ble_disconnect_callback
                0x0000000010049661        0x0 Output\obj\Libraries\bsp\bsp_bt.o
 .rela.text.fot_ble_connect_callback
                0x0000000010049661        0x0 Output\obj\Libraries\bsp\bsp_bt.o
 .rela.text.fot_spp_connect_callback
                0x0000000010049661        0x0 Output\obj\Libraries\bsp\bsp_bt.o
 .rela.text.fot_spp_disconnect_callback
                0x0000000010049661        0x0 Output\obj\Libraries\bsp\bsp_bt.o
 .rela.com_text.fot
                0x0000000010049661        0x0 Output\obj\Libraries\bsp\bsp_bt.o
 .rela.text.bsp.param
                0x0000000010049661        0x0 Output\obj\Libraries\bsp\bsp_bt.o
 .rela.text.bsp.sys.init
                0x0000000010049661        0x0 Output\obj\Libraries\bsp\bsp_bt.o
 .rela.com_text.timer
                0x0000000010049661        0x0 Output\obj\Libraries\bsp\bsp_bt.o
 .rela.text.bsp_get_xosc_xcfg
                0x0000000010049661        0x0 Output\obj\Libraries\bsp\bsp_bt.o
 .rela.text.gatt_callback_fota
                0x0000000010049661        0x0 Output\obj\Libraries\bsp\bsp_bt.o
 .rela.text.gatt_callback_app
                0x0000000010049661        0x0 Output\obj\Libraries\bsp\bsp_bt.o
 .rela.text.ble_get_scan_data
                0x0000000010049661        0x0 Output\obj\Libraries\bsp\bsp_bt.o
 .rela.text.ble_get_adv_data
                0x0000000010049661        0x0 Output\obj\Libraries\bsp\bsp_bt.o
 .rela.text.ble_txpkt_init
                0x0000000010049661        0x0 Output\obj\Libraries\bsp\bsp_bt.o
 .rela.text.ble_send_packet1
                0x0000000010049661        0x0 Output\obj\Libraries\bsp\bsp_bt.o
 .rela.text.ble_send_packet2
                0x0000000010049661        0x0 Output\obj\Libraries\bsp\bsp_bt.o
 .rela.text.ble_read_value
                0x0000000010049661        0x0 Output\obj\Libraries\bsp\bsp_bt.o
 .rela.text.ble_fot_send_packet
                0x0000000010049661        0x0 Output\obj\Libraries\bsp\bsp_bt.o
 .rela.text.ble_app_gatts_service_init
                0x0000000010049661        0x0 Output\obj\Libraries\bsp\bsp_bt.o
 .rela.text.ble_get_local_bd_addr
                0x0000000010049661        0x0 Output\obj\Libraries\bsp\bsp_bt.o
 .rela.text.ble_enter_transmit
                0x0000000010049661        0x0 Output\obj\Libraries\bsp\bsp_bt.o
 .rela.text.ble_exit_transmit
                0x0000000010049661        0x0 Output\obj\Libraries\bsp\bsp_bt.o
 .rela.text.ble_disconnect_callback
                0x0000000010049661        0x0 Output\obj\Libraries\bsp\bsp_bt.o
 .rela.text.ble_connect_callback
                0x0000000010049661        0x0 Output\obj\Libraries\bsp\bsp_bt.o
 .rela.text.bt_get_local_name
                0x0000000010049661        0x0 Output\obj\Libraries\bsp\bsp_bt.o
 .rela.text.bt_clr_all_link_info
                0x0000000010049661        0x0 Output\obj\Libraries\bsp\bsp_bt.o
 .rela.text.bt_get_local_bd_addr
                0x0000000010049661        0x0 Output\obj\Libraries\bsp\bsp_bt.o
 .rela.text.bt_get_link_info
                0x0000000010049661        0x0 Output\obj\Libraries\bsp\bsp_bt.o
 .rela.text.bt_put_link_info
                0x0000000010049661        0x0 Output\obj\Libraries\bsp\bsp_bt.o
 .rela.text.bt_get_ext_link_info
                0x0000000010049661        0x0 Output\obj\Libraries\bsp\bsp_bt.o
 .rela.text.bt_put_ext_link_info
                0x0000000010049661        0x0 Output\obj\Libraries\bsp\bsp_bt.o
 .rela.text.bt_sync_link_info
                0x0000000010049661        0x0 Output\obj\Libraries\bsp\bsp_bt.o
 .rela.text.bsp_bt_hid_screen_left
                0x0000000010049661        0x0 Output\obj\Libraries\bsp\bsp_bt.o
 .rela.text.bsp_bt_hid_screen_right
                0x0000000010049661        0x0 Output\obj\Libraries\bsp\bsp_bt.o
 .rela.data     0x0000000010049661        0x0 Output\obj\Libraries\bsp\bsp_bt.o
 .rela.text.bt_init_lib
                0x0000000010049661        0x0 Output\obj\Libraries\bsp\bsp_bt.o
 .rela.text.spp_txpkt_init
                0x0000000010049661        0x0 Output\obj\Libraries\bsp\bsp_bt.o
 .rela.text.spp_connect_callback
                0x0000000010049661        0x0 Output\obj\Libraries\bsp\bsp_bt.o
 .rela.text.spp_disconnect_callback
                0x0000000010049661        0x0 Output\obj\Libraries\bsp\bsp_bt.o
 .rela.text.spp_rx_callback
                0x0000000010049661        0x0 Output\obj\Libraries\bsp\bsp_bt.o
 .rela.text.gpio_pic_config
                0x0000000010049661        0x0 Output\obj\Libraries\bsp\bsp_bt.o
 .rela.text.internal_flash_write
                0x0000000010049661        0x0 Output\obj\Libraries\bsp\bsp_bt.o
 .rela.text.internal_flash_erase_partial
                0x0000000010049661        0x0 Output\obj\Libraries\bsp\bsp_bt.o
 .rela.text.set_bluetooth_name
                0x0000000010049661        0x0 Output\obj\Libraries\bsp\bsp_bt.o
 .rela.text.read_bluetooth_name
                0x0000000010049661        0x0 Output\obj\Libraries\bsp\bsp_bt.o
 .rela.text.internal_flash_examples
                0x0000000010049661        0x0 Output\obj\Libraries\bsp\bsp_bt.o
 .rela.text.getcfg_vddbt_sel
                0x0000000010049661        0x0 Output\obj\Libraries\bsp\bsp_bt.o
 .rela.text.getcfg_vddio_sel
                0x0000000010049661        0x0 Output\obj\Libraries\bsp\bsp_bt.o
 .rela.text.getcfg_vddbt_capless_en
                0x0000000010049661        0x0 Output\obj\Libraries\bsp\bsp_bt.o
 .rela.text.startup.main
                0x0000000010049661        0x0 Output\obj\Libraries\bsp\bsp_bt.o
 .rela.text.pll_vco_band_trimming
                0x0000000010049661        0x0 Output\obj\Libraries\bsp\bsp_bt.o
 .rela.com_text.dac
                0x0000000010049661        0x0 Output\obj\Libraries\bsp\bsp_bt.o
 .rela.text.adpll_divider_update_do
                0x0000000010049661        0x0 Output\obj\Libraries\bsp\bsp_bt.o
 .rela.text.adpll_divider_update
                0x0000000010049661        0x0 Output\obj\Libraries\bsp\bsp_bt.o
 .rela.text.adpll_init
                0x0000000010049661        0x0 Output\obj\Libraries\bsp\bsp_bt.o
 .rela.text.spires
                0x0000000010049661        0x0 Output\obj\Libraries\bsp\bsp_bt.o
 .rela.text.cm_loadpage
                0x0000000010049661        0x0 Output\obj\Libraries\bsp\bsp_bt.o
 .rela.text.cm_next_freepage
                0x0000000010049661        0x0 Output\obj\Libraries\bsp\bsp_bt.o
 .rela.text.cm_movepage
                0x0000000010049661        0x0 Output\obj\Libraries\bsp\bsp_bt.o
 .rela.text.cm_move_allpages
                0x0000000010049661        0x0 Output\obj\Libraries\bsp\bsp_bt.o
 .rela.text.cm_release
                0x0000000010049661        0x0 Output\obj\Libraries\bsp\bsp_bt.o
 .rela.text.cm_savepage
                0x0000000010049661        0x0 Output\obj\Libraries\bsp\bsp_bt.o
 .rela.text.cm_check_loadpage
                0x0000000010049661        0x0 Output\obj\Libraries\bsp\bsp_bt.o
 .rela.text.cm_sync
                0x0000000010049661        0x0 Output\obj\Libraries\bsp\bsp_bt.o
 .rela.text.cm_release_all
                0x0000000010049661        0x0 Output\obj\Libraries\bsp\bsp_bt.o
 .rela.text.cm_read
                0x0000000010049661        0x0 Output\obj\Libraries\bsp\bsp_bt.o
 .rela.text.cm_read8
                0x0000000010049661        0x0 Output\obj\Libraries\bsp\bsp_bt.o
 .rela.text.cm_read16
                0x0000000010049661        0x0 Output\obj\Libraries\bsp\bsp_bt.o
 .rela.text.cm_read32
                0x0000000010049661        0x0 Output\obj\Libraries\bsp\bsp_bt.o
 .rela.text.cm_write
                0x0000000010049661        0x0 Output\obj\Libraries\bsp\bsp_bt.o
 .rela.text.cm_write8
                0x0000000010049661        0x0 Output\obj\Libraries\bsp\bsp_bt.o
 .rela.text.cm_write16
                0x0000000010049661        0x0 Output\obj\Libraries\bsp\bsp_bt.o
 .rela.text.cm_write32
                0x0000000010049661        0x0 Output\obj\Libraries\bsp\bsp_bt.o
 .rela.text.cm_clear
                0x0000000010049661        0x0 Output\obj\Libraries\bsp\bsp_bt.o
 .rela.text.cm_init
                0x0000000010049661        0x0 Output\obj\Libraries\bsp\bsp_bt.o
 .rela.com_text.spiflash
                0x0000000010049661        0x0 Output\obj\Libraries\bsp\bsp_bt.o
 .rela.text.xcfg_init
                0x0000000010049661        0x0 Output\obj\Libraries\bsp\bsp_bt.o
 .rela.text.sd_disable_user
                0x0000000010049661        0x0 Output\obj\Libraries\bsp\bsp_bt.o
 .rela.text.device.init
                0x0000000010049661        0x0 Output\obj\Libraries\bsp\bsp_bt.o
 .rela.text.device
                0x0000000010049661        0x0 Output\obj\Libraries\bsp\bsp_bt.o
 .rela.com_text.sd.isr
                0x0000000010049661        0x0 Output\obj\Libraries\bsp\bsp_bt.o
 .rela.com_text.sd.api
                0x0000000010049661        0x0 Output\obj\Libraries\bsp\bsp_bt.o
 .rela.text.fs_lock
                0x0000000010049661        0x0 Output\obj\Libraries\bsp\bsp_bt.o
 .rela.text.fs_unlock
                0x0000000010049661        0x0 Output\obj\Libraries\bsp\bsp_bt.o
 .rela.com_text.exception.hook
                0x0000000010049661        0x0 Output\obj\Libraries\bsp\bsp_bt.o
 .rela.com_text.exception
                0x0000000010049661        0x0 Output\obj\Libraries\bsp\bsp_bt.o
 .rela.com_text.delay
                0x0000000010049661        0x0 Output\obj\Libraries\bsp\bsp_bt.o
 .rela.com_text.exception.do
                0x0000000010049661        0x0 Output\obj\Libraries\bsp\bsp_bt.o
 .rela.com_text.ledseg
                0x0000000010049661        0x0 Output\obj\Libraries\bsp\bsp_bt.o
 .rela.text.platform_main
                0x0000000010049661        0x0 Output\obj\Libraries\bsp\bsp_bt.o
 .rela.text.main_startup
                0x0000000010049661        0x0 Output\obj\Libraries\bsp\bsp_bt.o
 .rela.text.compiler
                0x0000000010049661        0x0 Output\obj\Libraries\bsp\bsp_bt.o
 .rela.com_text.irq
                0x0000000010049661        0x0 Output\obj\Libraries\bsp\bsp_bt.o
 .rela.text.sys_irq_init
                0x0000000010049661        0x0 Output\obj\Libraries\bsp\bsp_bt.o
 .rela.text.timer0_init
                0x0000000010049661        0x0 Output\obj\Libraries\bsp\bsp_bt.o
 .rela.text.soft_irq_init
                0x0000000010049661        0x0 Output\obj\Libraries\bsp\bsp_bt.o
 .rela.text.bthw_irq_init
                0x0000000010049661        0x0 Output\obj\Libraries\bsp\bsp_bt.o
 .rela.text.sd0_irq_init
                0x0000000010049661        0x0 Output\obj\Libraries\bsp\bsp_bt.o
 .rela.text.usb_irq_init
                0x0000000010049661        0x0 Output\obj\Libraries\bsp\bsp_bt.o
 .rela.text.timer1_irq_init
                0x0000000010049661        0x0 Output\obj\Libraries\bsp\bsp_bt.o
 .rela.com_text.tws.isr
                0x0000000010049661        0x0 Output\obj\Libraries\bsp\bsp_bt.o
 .rela.text.aubuf_irq_init
                0x0000000010049661        0x0 Output\obj\Libraries\bsp\bsp_bt.o
 .rela.text.huart_irq_init
                0x0000000010049661        0x0 Output\obj\Libraries\bsp\bsp_bt.o
 .rela.text.watch_point_set
                0x0000000010049661        0x0 Output\obj\Libraries\bsp\bsp_bt.o
 .rela.text.thread_main_entry
                0x0000000010049661        0x0 Output\obj\Libraries\bsp\bsp_bt.o
 .rela.text.thread_idle_create
                0x0000000010049661        0x0 Output\obj\Libraries\bsp\bsp_bt.o
 .rela.text.startup.init
                0x0000000010049661        0x0 Output\obj\Libraries\bsp\bsp_bt.o
 .rela.reset    0x0000000010049661        0x0 Output\obj\Libraries\bsp\bsp_bt.o
 .rela.vector   0x0000000010049661        0x0 Output\obj\Libraries\bsp\bsp_bt.o
 .rela.com_text.debug
                0x0000000010049661        0x0 Output\obj\Libraries\bsp\bsp_bt.o
 .rela.text.fot_init
                0x0000000010049661        0x0 Output\obj\Libraries\bsp\bsp_bt.o
 .rela.text.lock_code_bt_sleep
                0x0000000010049661        0x0 Output\obj\Libraries\bsp\bsp_bt.o
 .rela.text.lock_code_pwrsave
                0x0000000010049661        0x0 Output\obj\Libraries\bsp\bsp_bt.o
 .rela.text.lock_code_charge
                0x0000000010049661        0x0 Output\obj\Libraries\bsp\bsp_bt.o
 .rela.text.lock_code_usbdev
                0x0000000010049661        0x0 Output\obj\Libraries\bsp\bsp_bt.o
 .rela.text.load_code_btdec
                0x0000000010049661        0x0 Output\obj\Libraries\bsp\bsp_bt.o
 .rela.text.load_code_bt_voice
                0x0000000010049661        0x0 Output\obj\Libraries\bsp\bsp_bt.o
 .rela.text.lock_code_sniff
                0x0000000010049661        0x0 Output\obj\Libraries\bsp\bsp_bt.o
 .rela.text.lock_code_huart
                0x0000000010049661        0x0 Output\obj\Libraries\bsp\bsp_bt.o
 .rela.text.lock_code_bb_test
                0x0000000010049661        0x0 Output\obj\Libraries\bsp\bsp_bt.o
 .rela.text.load_code_fota
                0x0000000010049661        0x0 Output\obj\Libraries\bsp\bsp_bt.o
 .rela.text.patch_init
                0x0000000010049661        0x0 Output\obj\Libraries\bsp\bsp_bt.o
 .rela.text.vddio_voltage_configure
                0x0000000010049661        0x0 Output\obj\Libraries\bsp\bsp_bt.o
 .rela.text.vddbt_voltage_configure
                0x0000000010049661        0x0 Output\obj\Libraries\bsp\bsp_bt.o
 .rela.text.pmu_voltage_configure
                0x0000000010049661        0x0 Output\obj\Libraries\bsp\bsp_bt.o
 .rela.text.pmu_init
                0x0000000010049661        0x0 Output\obj\Libraries\bsp\bsp_bt.o
 .rela.com_text.voltage.trim
                0x0000000010049661        0x0 Output\obj\Libraries\bsp\bsp_bt.o
 .rela.text.sys_clk
                0x0000000010049661        0x0 Output\obj\Libraries\bsp\bsp_bt.o
 .rela.text.set_peripherals_clkdiv
                0x0000000010049661        0x0 Output\obj\Libraries\bsp\bsp_bt.o
 .rela.com_huart.text
                0x0000000010049661        0x0 Output\obj\Libraries\bsp\bsp_bt.o
 .rela.com_text.thread.usb
                0x0000000010049661        0x0 Output\obj\Libraries\bsp\bsp_bt.o
 .rela.bt_voice.plc
                0x0000000010049661        0x0 Output\obj\Libraries\bsp\bsp_bt.o
 .rela.text.stack.api
                0x0000000010049661        0x0 Output\obj\Libraries\bsp\bsp_bt.o
 .rela.com_text.stack.run_loop
                0x0000000010049661        0x0 Output\obj\Libraries\bsp\bsp_bt.o
 .rela.com_text.bb.bthw
                0x0000000010049661        0x0 Output\obj\Libraries\bsp\bsp_bt.o
 .rela.text     0x0000000010049661        0x0 Output\obj\Libraries\bsp\bsp_bt.o
 .rela.com_text.bb.nanos
                0x0000000010049661        0x0 Output\obj\Libraries\bsp\bsp_bt.o
 .rela.com_text.bb.patch
                0x0000000010049661        0x0 Output\obj\Libraries\bsp\bsp_bt.o
 .rela.com_text.ble.isr.con
                0x0000000010049661        0x0 Output\obj\Libraries\bsp\bsp_bt.o
 .rela.com_text.bb.isr.timer
                0x0000000010049661        0x0 Output\obj\Libraries\bsp\bsp_bt.o
 .rela.com_text.bb.isr
                0x0000000010049661        0x0 Output\obj\Libraries\bsp\bsp_bt.o
 .rela.sleep_text.bb
                0x0000000010049661        0x0 Output\obj\Libraries\bsp\bsp_bt.o
 .rela.com_text.bb.sleep
                0x0000000010049661        0x0 Output\obj\Libraries\bsp\bsp_bt.o
 .rela.com_text.bb.btisr
                0x0000000010049661        0x0 Output\obj\Libraries\bsp\bsp_bt.o
 .rela.rodata   0x0000000010049661        0x0 Output\obj\Libraries\bsp\bsp_bt.o
 .rela.com_text.pp.send_pkt
                0x0000000010049661        0x0 Output\obj\Libraries\bsp\bsp_bt.o
 .rela.com_text.spp.tx
                0x0000000010049661        0x0 Output\obj\Libraries\bsp\bsp_bt.o
 .rela.com_text.spp.send_req
                0x0000000010049661        0x0 Output\obj\Libraries\bsp\bsp_bt.o
 .rela.com_text.spp.event_send
                0x0000000010049661        0x0 Output\obj\Libraries\bsp\bsp_bt.o
 .rela.com_text.spp.rx_set_new_credit
                0x0000000010049661        0x0 Output\obj\Libraries\bsp\bsp_bt.o
 .rela.text.stack.spp.handler
                0x0000000010049661        0x0 Output\obj\Libraries\bsp\bsp_bt.o
 .rela.text.stack.sdp.util
                0x0000000010049661        0x0 Output\obj\Libraries\bsp\bsp_bt.o
 .rela.text.stack.sdp.server
                0x0000000010049661        0x0 Output\obj\Libraries\bsp\bsp_bt.o
 .rela.text.stack.setup
                0x0000000010049661        0x0 Output\obj\Libraries\bsp\bsp_bt.o
 .rela.text.stack.sdp.server_add
                0x0000000010049661        0x0 Output\obj\Libraries\bsp\bsp_bt.o
 .rela.text.stack.sdp.server_rmv
                0x0000000010049661        0x0 Output\obj\Libraries\bsp\bsp_bt.o
 .rela.text.stack.rfcomm
                0x0000000010049661        0x0 Output\obj\Libraries\bsp\bsp_bt.o
 .rela.text.stack.link_key
                0x0000000010049661        0x0 Output\obj\Libraries\bsp\bsp_bt.o
 .rela.text.stack.run_loop
                0x0000000010049661        0x0 Output\obj\Libraries\bsp\bsp_bt.o
 .rela.com_text.stack.ticks
                0x0000000010049661        0x0 Output\obj\Libraries\bsp\bsp_bt.o
 .rela.text.stack.memory
                0x0000000010049661        0x0 Output\obj\Libraries\bsp\bsp_bt.o
 .rela.text.stack.linkctrl
                0x0000000010049661        0x0 Output\obj\Libraries\bsp\bsp_bt.o
 .rela.com_text.ble.send_pkt
                0x0000000010049661        0x0 Output\obj\Libraries\bsp\bsp_bt.o
 .rela.text.att.r_cb
                0x0000000010049661        0x0 Output\obj\Libraries\bsp\bsp_bt.o
 .rela.text.att.w_cb
                0x0000000010049661        0x0 Output\obj\Libraries\bsp\bsp_bt.o
 .rela.com_text.stack.ble.mtu
                0x0000000010049661        0x0 Output\obj\Libraries\bsp\bsp_bt.o
 .rela.text.ble.notify_handle
                0x0000000010049661        0x0 Output\obj\Libraries\bsp\bsp_bt.o
 .rela.text.ble.att
                0x0000000010049661        0x0 Output\obj\Libraries\bsp\bsp_bt.o
 .rela.text.ble.hci
                0x0000000010049661        0x0 Output\obj\Libraries\bsp\bsp_bt.o
 .rela.text.stack.handler
                0x0000000010049661        0x0 Output\obj\Libraries\bsp\bsp_bt.o
 .rela.text.stack.ble.setup
                0x0000000010049661        0x0 Output\obj\Libraries\bsp\bsp_bt.o
 .rela.text.stack.status
                0x0000000010049661        0x0 Output\obj\Libraries\bsp\bsp_bt.o
 .rela.rodata.stack.api
                0x0000000010049661        0x0 Output\obj\Libraries\bsp\bsp_bt.o
 .rela.text.stack.api.hid_con
                0x0000000010049661        0x0 Output\obj\Libraries\bsp\bsp_bt.o
 .rela.text.stack.api.hid_disc
                0x0000000010049661        0x0 Output\obj\Libraries\bsp\bsp_bt.o
 .rela.text.stack.api.hid_send
                0x0000000010049661        0x0 Output\obj\Libraries\bsp\bsp_bt.o
 .rela.text.stack.le.api
                0x0000000010049661        0x0 Output\obj\Libraries\bsp\bsp_bt.o
 .rela.text.bb.vs.fcc
                0x0000000010049661        0x0 Output\obj\Libraries\bsp\bsp_bt.o
 .rela.com_text.isr.txrx
                0x0000000010049661        0x0 Output\obj\Libraries\bsp\bsp_bt.o
 .rela.com_text.bt21.isr
                0x0000000010049661        0x0 Output\obj\Libraries\bsp\bsp_bt.o
 .rela.text.ble.var.init
                0x0000000010049661        0x0 Output\obj\Libraries\bsp\bsp_bt.o
 .rela.text.bb.ble.adv0
                0x0000000010049661        0x0 Output\obj\Libraries\bsp\bsp_bt.o
 .rela.text.stk.l2cap.txreq
                0x0000000010049661        0x0 Output\obj\Libraries\bsp\bsp_bt.o
 .rela.text.stack.handler.l2cap
                0x0000000010049661        0x0 Output\obj\Libraries\bsp\bsp_bt.o
 .rela.text.stack.l2cap
                0x0000000010049661        0x0 Output\obj\Libraries\bsp\bsp_bt.o
 .rela.text.stack.hci
                0x0000000010049661        0x0 Output\obj\Libraries\bsp\bsp_bt.o
 .rela.text.stack.hci_init
                0x0000000010049661        0x0 Output\obj\Libraries\bsp\bsp_bt.o
 .rela.com_text.stack.hci
                0x0000000010049661        0x0 Output\obj\Libraries\bsp\bsp_bt.o
 .rela.text.stack.hci_send
                0x0000000010049661        0x0 Output\obj\Libraries\bsp\bsp_bt.o
 .rela.text.stack.hci.run
                0x0000000010049661        0x0 Output\obj\Libraries\bsp\bsp_bt.o
 .rela.text.stack.handler.event
                0x0000000010049661        0x0 Output\obj\Libraries\bsp\bsp_bt.o
 .rela.com_text.stack.hci_recv
                0x0000000010049661        0x0 Output\obj\Libraries\bsp\bsp_bt.o
 .rela.text.stack.hfp.api1
                0x0000000010049661        0x0 Output\obj\Libraries\bsp\bsp_bt.o
 .rela.text.bb.lm.inq.start
                0x0000000010049661        0x0 Output\obj\Libraries\bsp\bsp_bt.o
 .rela.text.le.ll_cntl
                0x0000000010049661        0x0 Output\obj\Libraries\bsp\bsp_bt.o
 .rela.text.le.ll_cntl.start
                0x0000000010049661        0x0 Output\obj\Libraries\bsp\bsp_bt.o
 .rela.text.le.ll_cntl.state
                0x0000000010049661        0x0 Output\obj\Libraries\bsp\bsp_bt.o
 .rela.text.le.ll_cntl.stop
                0x0000000010049661        0x0 Output\obj\Libraries\bsp\bsp_bt.o
 .rela.text.le.mgr
                0x0000000010049661        0x0 Output\obj\Libraries\bsp\bsp_bt.o
 .rela.rodata.le.mgr_cntl.tbl
                0x0000000010049661        0x0 Output\obj\Libraries\bsp\bsp_bt.o
 .rela.text.le.ll_scan
                0x0000000010049661        0x0 Output\obj\Libraries\bsp\bsp_bt.o
 .rela.text.le.ll_adv
                0x0000000010049661        0x0 Output\obj\Libraries\bsp\bsp_bt.o
 .rela.text.le.ll_adv.con
                0x0000000010049661        0x0 Output\obj\Libraries\bsp\bsp_bt.o
 .rela.com_rodata.bb.tbl
                0x0000000010049661        0x0 Output\obj\Libraries\bsp\bsp_bt.o
 .rela.rodata.le.ll_cntl.tbl
                0x0000000010049661        0x0 Output\obj\Libraries\bsp\bsp_bt.o
 .rela.text.le.ll_cntl.pdu
                0x0000000010049661        0x0 Output\obj\Libraries\bsp\bsp_bt.o
 .rela.text.le.ll_cntl.send
                0x0000000010049661        0x0 Output\obj\Libraries\bsp\bsp_bt.o
 .rela.com_text.usbdev
                0x0000000010049661        0x0 Output\obj\Libraries\bsp\bsp_bt.o
 .rela.usbdev.com
                0x0000000010049661        0x0 Output\obj\Libraries\bsp\bsp_bt.o
 .rela.com_text.bulkep
                0x0000000010049661        0x0 Output\obj\Libraries\bsp\bsp_bt.o
 .rela.text.udp_init
                0x0000000010049661        0x0 Output\obj\Libraries\bsp\bsp_bt.o
 .rela.text.usb_device_init
                0x0000000010049661        0x0 Output\obj\Libraries\bsp\bsp_bt.o
 .rela.text.usb_device_enter
                0x0000000010049661        0x0 Output\obj\Libraries\bsp\bsp_bt.o
 .rela.com_text.usb.device
                0x0000000010049661        0x0 Output\obj\Libraries\bsp\bsp_bt.o
 .rela.text.usb.host.init
                0x0000000010049661        0x0 Output\obj\Libraries\bsp\bsp_bt.o
 .rela.com_text.usb.host
                0x0000000010049661        0x0 Output\obj\Libraries\bsp\bsp_bt.o
 .rela.text.udisk_read
                0x0000000010049661        0x0 Output\obj\Libraries\bsp\bsp_bt.o
 .rela.text.udisk_write
                0x0000000010049661        0x0 Output\obj\Libraries\bsp\bsp_bt.o
 .rela.text.do_transfer
                0x0000000010049661        0x0 Output\obj\Libraries\bsp\bsp_bt.o
 .rela.text.do_receive
                0x0000000010049661        0x0 Output\obj\Libraries\bsp\bsp_bt.o
 .rela.text.uhs_start
                0x0000000010049661        0x0 Output\obj\Libraries\bsp\bsp_bt.o
 .rela.text.uhs_init
                0x0000000010049661        0x0 Output\obj\Libraries\bsp\bsp_bt.o
 .rela.text.usb_init
                0x0000000010049661        0x0 Output\obj\Libraries\bsp\bsp_bt.o
 .rela.text.usb_host_enter
                0x0000000010049661        0x0 Output\obj\Libraries\bsp\bsp_bt.o
 .rela.text.uhe_start
                0x0000000010049661        0x0 Output\obj\Libraries\bsp\bsp_bt.o
                0x0000000010049661        0x4 LONG 0x0
                0x0000000010049800                . = ALIGN (0x200)
 *fill*         0x0000000010049665      0x19b 

.stack          0x0000000000010800      0x400
                0x0000000000010800                __irq_stack_start = .
                0x0000000000000400                . = 0x400
 *fill*         0x0000000000010800      0x400 
                0x0000000000010c00                __irq_stack = .
                0x0000000000000400                __irq_stack_size = (__irq_stack - __irq_stack_start)

.bss            0x0000000000013c00     0x17f8
                0x0000000000013c00                __bss_start = .
 *(COMMON)
 COMMON         0x0000000000013c00        0x7 Output\obj\Libraries\bsp\bsp_bt.o
                0x0000000000013c00                f_bt
 *fill*         0x0000000000013c07        0x1 
 COMMON         0x0000000000013c08       0x22 Output\obj\Libraries\bsp\bsp_fot.o
                0x0000000000013c08                fot_var
 *fill*         0x0000000000013c2a        0x2 
 COMMON         0x0000000000013c2c       0xb2 Output\obj\Libraries\bsp\bsp_sys.o
                0x0000000000013c2c                ticks_50ms
                0x0000000000013c30                xcfg_cb
 *fill*         0x0000000000013cde        0x2 
 COMMON         0x0000000000013ce0       0x60 Output\obj\Examples\Internal_Flash\Source\Internal_Flash.o
                0x0000000000013ce0                mySavePara
                0x0000000000013d20                g_ucMcuId
 *(.bss*)
 .bss           0x0000000000013d40      0x22c ..\..\..\Libraries\libs\libplatform.a(cm.o)
 .bss           0x0000000000013f6c       0xa0 ..\..\..\Libraries\libs\libplatform.a(main.o)
                0x0000000000013f6c                cpu_gprs
                0x0000000000013fec                sys
 .bss.irq_tbl   0x000000000001400c       0x84 ..\..\..\Libraries\libs\libplatform.a(interrupt.o)
                0x000000000001400c                tbl_irq_vector
                0x000000000001408c                irq_mask
 .bss           0x0000000000014090       0x28 ..\..\..\Libraries\libs\libplatform.a(startup.o)
 .bss           0x00000000000140b8       0x20 ..\..\..\Libraries\libs\libplatform.a(fot_update.o)
 .bss           0x00000000000140d8       0x78 ..\..\..\Libraries\libs\libplatform.a(lock.o)
 .bss           0x0000000000014150        0xc ..\..\..\Libraries\libs\libplatform.a(voltage_trim.o)
                0x0000000000014150                sys_trim
 .bss           0x000000000001415c        0x9 ..\..\..\Libraries\libs\libbtstack.a(bb.o)
                0x000000000001415c                rf_api
 *fill*         0x0000000000014165        0x3 
 .bss           0x0000000000014168       0x3e ..\..\..\Libraries\libs\libbtstack.a(btstack_link_key_db.o)
 *fill*         0x00000000000141a6        0x2 
 .bss           0x00000000000141a8      0x4fc ..\..\..\Libraries\libs\libbtstack.a(btstack_memory.o)
 .bss           0x00000000000146a4       0x10 ..\..\..\Libraries\libs\libbtstack.a(sm.o)
 .bss           0x00000000000146b4       0x48 ..\..\..\Libraries\libs\libbtstack.a(btstack_api.o)
                0x00000000000146b4                btstack_cb
                0x00000000000146c0                btstack_st
 .bss           0x00000000000146fc      0x184 ..\..\..\Libraries\libs\libbtstack.a(bb_sche.o)
                0x00000000000146fc                ss_params
 .bss           0x0000000000014880        0xc ..\..\..\Libraries\libs\libbtstack.a(aes.o)
                0x0000000000014880                aes_env
 .bss           0x000000000001488c       0x24 ..\..\..\Libraries\libs\libbtstack.a(hct_tl.o)
 .bss           0x00000000000148b0       0x26 ..\..\..\Libraries\libs\libbtstack.a(bc.o)
                0x00000000000148b0                bc_env
 *fill*         0x00000000000148d6        0x2 
 .bss           0x00000000000148d8       0x40 ..\..\..\Libraries\libs\libbtstack.a(l2cap_test.o)
                0x00000000000148d8                vd_tx
 .bss           0x0000000000014918       0xc0 ..\..\..\Libraries\libs\libbtstack.a(lm_sp.o)
 .bss           0x00000000000149d8      0x100 ..\..\..\Libraries\libs\libbtstack.a(ble_buf.o)
 .bss           0x0000000000014ad8      0x21c ..\..\..\Libraries\libs\libbtstack.a(ll_proc.o)
 .bss           0x0000000000014cf4       0x24 ..\..\..\Libraries\libs\libdrivers.a(usb_device_ep.o)
                0x0000000000014cf4                eps
 *(.sbss*)
 .sbss          0x0000000000014d18        0x4 Output\obj\Libraries\bsp\bsp_fot.o
 .sbss          0x0000000000014d1c       0x1e Output\obj\Libraries\BT\ble\ab_link\app.o
                0x0000000000014d20                str
 .sbss          0x0000000000014d3a        0xc Output\obj\Libraries\BT\spp\bt.o
                0x0000000000014d3a                cfg_bt_hid_type
                0x0000000000014d3c                cfg_bt_support_codec
                0x0000000000014d3e                cfg_bt_simple_pair_mode
                0x0000000000014d3f                cfg_bt_scan_ctrl_mode
                0x0000000000014d40                cfg_bt_work_mode
                0x0000000000014d41                cfg_ble_page_rssi_thr
                0x0000000000014d42                cfg_ble_page_txpwr
                0x0000000000014d43                cfg_bt_inq_txpwr
                0x0000000000014d44                cfg_bt_page_txpwr
                0x0000000000014d45                cfg_bt_rf_def_txpwr
 .sbss          0x0000000000014d46        0x2 Output\obj\Libraries\BT\spp\spp.o
                0x0000000000014d46                SPP_CreditCount
                0x0000000000014d47                BtFlowControl_start
 .sbss          0x0000000000014d48        0x8 ..\..\..\Libraries\libs\libplatform.a(audio.o)
                0x0000000000014d4c                aux_cur_gain
 .sbss          0x0000000000014d50        0x8 ..\..\..\Libraries\libs\libplatform.a(os_flash.o)
                0x0000000000014d50                spi_baud_w
                0x0000000000014d54                spi_baud_r
 .sbss          0x0000000000014d58        0xc ..\..\..\Libraries\libs\libplatform.a(interrupt.o)
                0x0000000000014d58                tmr5ms_cnt
                0x0000000000014d5c                ms_tick
                0x0000000000014d60                tmr0_counter
 .sbss          0x0000000000014d64       0x3c ..\..\..\Libraries\libs\libplatform.a(startup.o)
                0x0000000000014d64                user_timer_isr_en
                0x0000000000014d68                bt_timer_isr_en
                0x0000000000014d6c                pmutex_pff
                0x0000000000014d70                pmutex_bt_sta
                0x0000000000014d74                pmutex_math
                0x0000000000014d78                pmutex_dac
                0x0000000000014d7c                pmutex_uart
                0x0000000000014d80                pmutex_clk
                0x0000000000014d84                pmutex_cm
                0x0000000000014d88                pmq_usb
                0x0000000000014d8c                pmq_btstack
                0x0000000000014d90                psem_sd
                0x0000000000014d94                psem_aubuf
                0x0000000000014d98                psem_btstack
                0x0000000000014d9c                psem_bthw
 .sbss          0x0000000000014da0        0xc ..\..\..\Libraries\libs\libplatform.a(fot_update.o)
 .sbss          0x0000000000014dac        0x4 ..\..\..\Libraries\libs\libplatform.a(bt.o)
                0x0000000000014dac                bt_thread_res
 .sbss          0x0000000000014db0        0x1 ..\..\..\Libraries\libs\libbtstack.a(bb.o)
 .sbss          0x0000000000014db1        0x1 ..\..\..\Libraries\libs\libbtstack.a(platform.o)
                0x0000000000014db1                cfg_bt_spp_rx_flow_ctrl_en
 .sbss          0x0000000000014db2        0x6 ..\..\..\Libraries\libs\libbtstack.a(extern_tws.o)
                0x0000000000014db2                cfg_bt_tws_limit_pair_time
                0x0000000000014db4                cfg_bt_tws_feat
                0x0000000000014db6                cfg_bt_tws_pair_mode
 .sbss          0x0000000000014db8        0x9 ..\..\..\Libraries\libs\libbtstack.a(extern_bt.o)
                0x0000000000014dba                cfg_bt_tws_mode
 *fill*         0x0000000000014dc1        0x3 
 .sbss          0x0000000000014dc4        0x4 ..\..\..\Libraries\libs\libbtstack.a(sdp_server.o)
 .sbss          0x0000000000014dc8       0x13 ..\..\..\Libraries\libs\libbtstack.a(rfcomm.o)
                0x0000000000014dd0                rfcomm_channels
                0x0000000000014dd4                rfcomm_multiplexers
 *fill*         0x0000000000014ddb        0x1 
 .sbss          0x0000000000014ddc        0x5 ..\..\..\Libraries\libs\libbtstack.a(btstack_run_loop.o)
 *fill*         0x0000000000014de1        0x3 
 .sbss          0x0000000000014de4       0x20 ..\..\..\Libraries\libs\libbtstack.a(btstack_memory.o)
 .sbss          0x0000000000014e04        0xf ..\..\..\Libraries\libs\libbtstack.a(sm.o)
 *fill*         0x0000000000014e13        0x1 
 .sbss          0x0000000000014e14       0x1f ..\..\..\Libraries\libs\libbtstack.a(att_server.o)
 *fill*         0x0000000000014e33        0x1 
 .sbss          0x0000000000014e34        0xc ..\..\..\Libraries\libs\libbtstack.a(att_dispatch.o)
 .sbss          0x0000000000014e40       0x10 ..\..\..\Libraries\libs\libbtstack.a(att_db.o)
 .sbss          0x0000000000014e50        0xd ..\..\..\Libraries\libs\libbtstack.a(btstack_main.o)
 *fill*         0x0000000000014e5d        0x3 
 .sbss          0x0000000000014e60        0x8 ..\..\..\Libraries\libs\libbtstack.a(hct_fc.o)
 .sbss          0x0000000000014e68        0xd ..\..\..\Libraries\libs\libbtstack.a(l2cap_test.o)
                0x0000000000014e68                vd_tx_cnt
                0x0000000000014e6c                vd_tx_w
                0x0000000000014e70                vd_tx_r
 *fill*         0x0000000000014e75        0x3 
 .sbss          0x0000000000014e78        0x5 ..\..\..\Libraries\libs\libbtstack.a(hci.o)
 *fill*         0x0000000000014e7d        0x3 
 .sbss          0x0000000000014e80        0x5 ..\..\..\Libraries\libs\libbtstack.a(hid_usage.o)
                0x0000000000014e80                ts_ctl
 *fill*         0x0000000000014e85        0x3 
 .sbss          0x0000000000014e88        0x9 ..\..\..\Libraries\libs\libbtstack.a(hfp_hf.o)
 *fill*         0x0000000000014e91        0x3 
 .sbss          0x0000000000014e94        0x9 ..\..\..\Libraries\libs\libbtstack.a(hci_transport_hcic.o)
                0x0000000000014e98                p_hci_transport
 *fill*         0x0000000000014e9d        0x3 
 .sbss          0x0000000000014ea0        0x2 ..\..\..\Libraries\libs\libbtstack.a(lc_proc.o)
                0x0000000000014ea0                lc_state
 *fill*         0x0000000000014ea2        0x2 
 .sbss          0x0000000000014ea4        0x1 ..\..\..\Libraries\libs\libbtstack.a(mgr_proc.o)
 *fill*         0x0000000000014ea5        0x3 
 .sbss          0x0000000000014ea8        0x4 ..\..\..\Libraries\libs\libbtstack.a(ll_proc.o)
 *(.buf*)
 .buf.bsp.sys_cb
                0x0000000000014eac       0x40 Output\obj\Libraries\bsp\bsp_sys.o
                0x0000000000014eac                sys_cb
 .buf.device.cb
                0x0000000000014eec       0x1b ..\..\..\Libraries\libs\libplatform.a(device.o)
                0x0000000000014eec                dev_cb
 *fill*         0x0000000000014f07        0x1 
 .buf.usb       0x0000000000014f08      0x15c ..\..\..\Libraries\libs\libdrivers.a(usb_device_run_loop.o)
                0x0000000000014f08                ude_0
                0x0000000000014f30                udp_0
                0x0000000000014f3c                epcb_printer_tx
                0x0000000000014f54                epcb_printer_rx
                0x0000000000014f6c                udh_0
                0x0000000000014f74                epcb3_tx
                0x0000000000014f8c                udu_0
                0x0000000000014f90                epcb_user
                0x0000000000014fa8                uds_0
                0x0000000000014fdc                epcb2_rx
                0x0000000000014ff4                epcb2_tx
                0x000000000001500c                uda_0
                0x000000000001501c                epcb1_rx
                0x0000000000015034                epcb1_tx
                0x000000000001504c                lun_0
 *(.dac_obuf)
 *(.btmem.stack.sdp)
 .btmem.stack.sdp
                0x0000000000015064      0x18c ..\..\..\Libraries\libs\libbtstack.a(sdp_server.o)
 .btmem.stack.sdp
                0x00000000000151f0       0xba ..\..\..\Libraries\libs\libbtstack.a(sdp_client.o)
 *(.btmem.stack.spp)
 *fill*         0x00000000000152aa        0x2 
 .btmem.stack.spp
                0x00000000000152ac       0x58 ..\..\..\Libraries\libs\libbtstack.a(spp.o)
                0x00000000000152ac                spp_connections
 *(.btmem.stack.l2cap)
 .btmem.stack.l2cap
                0x0000000000015304       0xbc ..\..\..\Libraries\libs\libbtstack.a(l2cap.o)
                0x000000000001532c                l2cap_channels
 *(.btmem.stack.hid)
 .btmem.stack.hid
                0x00000000000153c0       0x38 ..\..\..\Libraries\libs\libbtstack.a(hid_device.o)
 *(.qtest_buf)
                0x00000000000153f8                __bss_end = .
                0x00000000000017f8                __bss_size = (__bss_end - __bss_start)

.heap           0x0000000000010c00     0x3000
 *(.mem_heap)
 .mem_heap      0x0000000000010c00     0x3000 ..\..\..\Libraries\libs\libplatform.a(startup.o)
                0x0000000000010c00                mem_heap

.bram           0x0000000000020000     0xbbe0
 *(.btmem.bthw)
 .btmem.bthw    0x0000000000020000     0x45f8 ..\..\..\Libraries\libs\libbtstack.a(bb.o)
                0x0000000000020000                bthw_mem
 *(.btmem*)
 .btmem.bb.buf  0x00000000000245f8       0x4c ..\..\..\Libraries\libs\libbtstack.a(nanos.o)
 .btmem.bt.sco  0x0000000000024644        0xa ..\..\..\Libraries\libs\libbtstack.a(bt_sco.o)
 *fill*         0x000000000002464e        0x2 
 .btmem.bt.acl  0x0000000000024650        0x8 ..\..\..\Libraries\libs\libbtstack.a(bt_acl.o)
                0x0000000000024650                bt_acl_env
 .btmem.bt.sco  0x0000000000024658        0x8 ..\..\..\Libraries\libs\libbtstack.a(bt_acl.o)
                0x0000000000024658                bt_sco_env
 .btmem.ble.con
                0x0000000000024660       0x14 ..\..\..\Libraries\libs\libbtstack.a(ble_con.o)
 .btmem.bb.env  0x0000000000024674       0x4c ..\..\..\Libraries\libs\libbtstack.a(bb_int.o)
                0x0000000000024674                bb_env
 .btmem.bb.buf  0x00000000000246c0     0x3278 ..\..\..\Libraries\libs\libbtstack.a(bb.o)
 .btmem.stack.util
                0x0000000000027938       0x12 ..\..\..\Libraries\libs\libbtstack.a(btstack_util.o)
 *fill*         0x000000000002794a        0x2 
 .btmem.stack   0x000000000002794c       0x14 ..\..\..\Libraries\libs\libbtstack.a(btstack_run_loop.o)
 .btmem.stack.linkctrl
                0x0000000000027960       0x58 ..\..\..\Libraries\libs\libbtstack.a(btstack_link_ctrl.o)
                0x0000000000027964                hci_link_max
 .btmem.ble.adv
                0x00000000000279b8       0x40 ..\..\..\Libraries\libs\libbtstack.a(btstack_main.o)
                0x00000000000279b8                scan_data
                0x00000000000279d7                scan_data_len
                0x00000000000279d8                adv_data
                0x00000000000279f7                adv_data_len
 .btmem.bb.vs   0x00000000000279f8        0xd ..\..\..\Libraries\libs\libbtstack.a(vs_proc.o)
                0x00000000000279f8                vs_env
                0x0000000000027a04                vs_state
 *fill*         0x0000000000027a05        0x3 
 .btmem.bb.rf   0x0000000000027a08        0x4 ..\..\..\Libraries\libs\libbtstack.a(rf_smart.o)
 .btmem.bb.hci  0x0000000000027a0c       0x62 ..\..\..\Libraries\libs\libbtstack.a(hct.o)
                0x0000000000027a0c                hci_env
 *fill*         0x0000000000027a6e        0x2 
 .btmem.bt.lm   0x0000000000027a70      0x1ac ..\..\..\Libraries\libs\libbtstack.a(lm.o)
                0x0000000000027a74                lm_env
 .btmem.bt.env  0x0000000000027c1c      0x1cc ..\..\..\Libraries\libs\libbtstack.a(bt_hal.o)
                0x0000000000027c1c                bt_env
 .btmem.bt.buf  0x0000000000027de8       0xdc ..\..\..\Libraries\libs\libbtstack.a(bt21.o)
 .btmem.ble.hal
                0x0000000000027ec4      0x130 ..\..\..\Libraries\libs\libbtstack.a(ble_hal.o)
                0x0000000000027ec8                ble_env
                0x0000000000027fec                ble_exp_sync_pos_tab
 .btmem.ble.adv
                0x0000000000027ff4       0x10 ..\..\..\Libraries\libs\libbtstack.a(ble_adv.o)
 .btmem.stack.hci
                0x0000000000028004      0xad1 ..\..\..\Libraries\libs\libbtstack.a(hci.o)
 *fill*         0x0000000000028ad5        0x3 
 .btmem.stack.hci_buf
                0x0000000000028ad8      0x3c4 ..\..\..\Libraries\libs\libbtstack.a(hci.o)
 .btmem.stack.hid.usage
                0x0000000000028e9c       0x12 ..\..\..\Libraries\libs\libbtstack.a(hid_usage.o)
                0x0000000000028e9c                hrpt_cb
                0x0000000000028ea4                hid_report_buf
 *fill*         0x0000000000028eae        0x2 
 .btmem.stack.hfp
                0x0000000000028eb0        0x5 ..\..\..\Libraries\libs\libbtstack.a(hfp.o)
                0x0000000000028eb0                hfp_connections
                0x0000000000028eb4                hfp_index
 *fill*         0x0000000000028eb5        0x3 
 .btmem.ble.adv
                0x0000000000028eb8       0x1f ..\..\..\Libraries\libs\libbtstack.a(btstack_adv0.o)
 *fill*         0x0000000000028ed7        0x1 
 .btmem.hci.transport
                0x0000000000028ed8       0x20 ..\..\..\Libraries\libs\libbtstack.a(hci_transport_hcic.o)
 .btmem.bt.lm   0x0000000000028ef8        0x1 ..\..\..\Libraries\libs\libbtstack.a(lm_proc.o)
                0x0000000000028ef8                lm_state
 *fill*         0x0000000000028ef9        0x3 
 .btmem.bt.lc   0x0000000000028efc        0x8 ..\..\..\Libraries\libs\libbtstack.a(lc.o)
                0x0000000000028efc                lc_env
 .btmem.ble.lm  0x0000000000028f04      0x24c ..\..\..\Libraries\libs\libbtstack.a(mgr.o)
                0x0000000000028f04                mgr_env
 .btmem.ble.lc  0x0000000000029150       0x10 ..\..\..\Libraries\libs\libbtstack.a(ll.o)
                0x0000000000029150                ll_env
 .btmem.ble.test
                0x0000000000029160        0x4 ..\..\..\Libraries\libs\libbtstack.a(ble_test.o)
 .btmem.ble.scan
                0x0000000000029164        0x8 ..\..\..\Libraries\libs\libbtstack.a(ble_scan.o)
 .btmem.ble.init
                0x000000000002916c        0x4 ..\..\..\Libraries\libs\libbtstack.a(ble_init.o)
 .btmem.ble.buf
                0x0000000000029170       0x30 ..\..\..\Libraries\libs\libbtstack.a(ble_buf.o)
 .btmem.bt.lm.sco
                0x00000000000291a0        0xf ..\..\..\Libraries\libs\libbtstack.a(lm_sco.o)
 *fill*         0x00000000000291af        0x1 
 .btmem.bt.lc.sniff
                0x00000000000291b0       0x68 ..\..\..\Libraries\libs\libbtstack.a(lc_sniff.o)
                0x00000000000291b0                lc_sniff_env
 .btmem.bt.lc.sco
                0x0000000000029218       0x12 ..\..\..\Libraries\libs\libbtstack.a(lc_sco.o)
 *(.ble_cache*)
 *fill*         0x000000000002922a        0x2 
 .ble_cache.sm  0x000000000002922c      0x214 ..\..\..\Libraries\libs\libbtstack.a(sm.o)
 .ble_cache.att
                0x0000000000029440       0x10 ..\..\..\Libraries\libs\libbtstack.a(gatt_server.o)
                0x0000000000029440                notify_tx
 .ble_cache.att
                0x0000000000029450      0x458 ..\..\..\Libraries\libs\libbtstack.a(gatt_profile.o)
 .ble_cache.att
                0x00000000000298a8       0x50 ..\..\..\Libraries\libs\libbtstack.a(ad_parser.o)
                0x00000000000298a8                ad_param
 *(.ble_buf*)
 .ble_buf.stack.spp
                0x00000000000298f8       0x10 ..\..\..\Libraries\libs\libbtstack.a(spp.o)
                0x00000000000298f8                spp_tx
 .ble_buf.att   0x0000000000029908      0x180 ..\..\..\Libraries\libs\libbtstack.a(le_device_db_memory.o)
 .ble_buf.att   0x0000000000029a88      0x138 ..\..\..\Libraries\libs\libbtstack.a(gatt_server.o)
                0x0000000000029a88                att_attributes
 .ble_buf.att.buf
                0x0000000000029bc0      0x400 ..\..\..\Libraries\libs\libbtstack.a(gatt_server.o)
                0x0000000000029bc0                attribute_buf
 .ble_buf.queue.buf
                0x0000000000029fc0       0xc0 ..\..\..\Libraries\libs\libbtstack.a(gatt_server.o)
                0x0000000000029fc0                att_queue_buf
 .ble_buf.att   0x000000000002a080      0x2e0 ..\..\..\Libraries\libs\libbtstack.a(att_server.o)
                0x000000000002a080                att_connection
 *(.spp_tx_buff.*)
 .spp_tx_buff.spp_tx_pool
                0x000000000002a360     0x1040 Output\obj\Libraries\BT\spp\spp.o
                0x000000000002a360                spp_tx_pool
 *(.ble_tx_buff.*)
 .ble_tx_buff.att
                0x000000000002b3a0      0x840 Output\obj\Libraries\BT\ble\ab_link\app.o
                0x000000000002b3a0                notify_tx_pool

.aram           0x0000000000050000     0x1000
 *(.usb_buf*)
 .usb_buf.hid   0x0000000000050000        0x8 ..\..\..\Libraries\libs\libdrivers.a(usb_device_run_loop.o)
                0x0000000000050000                ep3_buf
 .usb_buf.user  0x0000000000050008      0x400 ..\..\..\Libraries\libs\libdrivers.a(usb_device_run_loop.o)
                0x0000000000050008                ep_user_buf
                0x0000000000001000                . = 0x1000
 *fill*         0x0000000000050408      0xbf8 

.fcc_buf        0x0000000000050000     0x1000
                0x0000000000001000                . = 0x1000
 *fill*         0x0000000000050000     0x1000 
 *(.fcc_buf.huart)

.aram_msc_stm   0x0000000000050000     0x1000
 *(.stm_buf)
                0x0000000000001000                . = 0x1000
 *fill*         0x0000000000050000     0x1000 

.cram_user
 *(.user.*)

.dram_upd       0x0000000000058000     0x4500
                0x0000000000003800                . = 0x3800
 *fill*         0x0000000000058000     0x3800 
 *(.upd_ota*)
 *(.upd_buf*)
                0x0000000000004500                . = 0x4500
 *fill*         0x000000000005b800      0xd00 

.eram_fot       0x0000000000054000      0xa00
 *(.fot_data.*)
 .fot_data.buf  0x0000000000054000      0x200 Output\obj\Libraries\bsp\bsp_fot.o
                0x0000000000054000                fot_data
 .fot_data.buf  0x0000000000054200      0x4e4 ..\..\..\Libraries\libs\libplatform.a(fot_update.o)
                0x0000000000054478                mac_ctl
                0x0000000000000a00                . = 0xa00
 *fill*         0x00000000000546e4      0x31c 
                0x0000000000043000                __bank_size = SIZEOF (.flash)
                0x0000000010000200                __comm_lma = LOADADDR (.comm)
                0x0000000000006600                __comm_size = SIZEOF (.comm)
LOAD ..\..\..\Libraries\libs\libplatform.a
LOAD ..\..\..\Libraries\libs\libbtstack.a
LOAD ..\..\..\Libraries\libs\libdrivers.a
LOAD ..\..\..\Libraries\libs\libbtstack_master.a
LOAD ..\..\..\Libraries\libs\libc.a
LOAD ..\..\..\Libraries\libs\libgcc.a
LOAD ..\..\..\Libraries\libs\libm.a
LOAD D:\×ÀÃæ\¼ÖÌìº½\×ªÕý¹¤×÷ÎÄ¼þ-2024\ÉÏ´«¹ÙÍøGW3323-¾«¼ò°æ\GW3323_SDK_V2.5_GW3323HGU6_À¶ÑÀ3+1_ÐÂ±±Ñó\Libraries\libs\libbtstack.a
LOAD D:\×ÀÃæ\¼ÖÌìº½\×ªÕý¹¤×÷ÎÄ¼þ-2024\ÉÏ´«¹ÙÍøGW3323-¾«¼ò°æ\GW3323_SDK_V2.5_GW3323HGU6_À¶ÑÀ3+1_ÐÂ±±Ñó\Libraries\libs\libc.a
LOAD D:\×ÀÃæ\¼ÖÌìº½\×ªÕý¹¤×÷ÎÄ¼þ-2024\ÉÏ´«¹ÙÍøGW3323-¾«¼ò°æ\GW3323_SDK_V2.5_GW3323HGU6_À¶ÑÀ3+1_ÐÂ±±Ñó\Libraries\libs\libdrivers.a
LOAD D:\×ÀÃæ\¼ÖÌìº½\×ªÕý¹¤×÷ÎÄ¼þ-2024\ÉÏ´«¹ÙÍøGW3323-¾«¼ò°æ\GW3323_SDK_V2.5_GW3323HGU6_À¶ÑÀ3+1_ÐÂ±±Ñó\Libraries\libs\libgcc.a
LOAD D:\×ÀÃæ\¼ÖÌìº½\×ªÕý¹¤×÷ÎÄ¼þ-2024\ÉÏ´«¹ÙÍøGW3323-¾«¼ò°æ\GW3323_SDK_V2.5_GW3323HGU6_À¶ÑÀ3+1_ÐÂ±±Ñó\Libraries\libs\libm.a
LOAD D:\×ÀÃæ\¼ÖÌìº½\×ªÕý¹¤×÷ÎÄ¼þ-2024\ÉÏ´«¹ÙÍøGW3323-¾«¼ò°æ\GW3323_SDK_V2.5_GW3323HGU6_À¶ÑÀ3+1_ÐÂ±±Ñó\Libraries\libs\libplatform.a
OUTPUT(Output\bin\app.rv32 elf32-littleriscv)

.comment        0x0000000000000000       0x23
 .comment       0x0000000000000000       0x11 Output\obj\Libraries\bsp\bsp_bt.o
                                         0x12 (size before relaxing)
 .comment       0x0000000000000011       0x12 Output\obj\Libraries\bsp\bsp_cm.o
 .comment       0x0000000000000011       0x12 Output\obj\Libraries\bsp\bsp_fot.o
 .comment       0x0000000000000011       0x12 Output\obj\Libraries\bsp\bsp_param.o
 .comment       0x0000000000000011       0x12 Output\obj\Libraries\bsp\bsp_sys.o
 .comment       0x0000000000000011       0x12 Output\obj\Libraries\BT\ble\ab_link\app.o
 .comment       0x0000000000000011       0x12 Output\obj\Libraries\BT\ble\adv0.o
 .comment       0x0000000000000011       0x12 Output\obj\Libraries\BT\ble\ble.o
 .comment       0x0000000000000011       0x12 Output\obj\Libraries\BT\spp\bt.o
 .comment       0x0000000000000011       0x12 Output\obj\Libraries\BT\spp\profile.o
 .comment       0x0000000000000011       0x12 Output\obj\Libraries\BT\spp\spp.o
 .comment       0x0000000000000011       0x12 Output\obj\Libraries\Device\Source\gw3323_gpio.o
 .comment       0x0000000000000011       0x12 Output\obj\Libraries\libs\strong_symbol.o
 .comment       0x0000000000000011       0x12 Output\obj\Examples\Internal_Flash\Source\Internal_Flash.o
 .comment       0x0000000000000011       0x12 Output\obj\Examples\Internal_Flash\Project\config.o
 .comment       0x0000000000000011       0x12 Output\obj\Examples\Internal_Flash\Project\main.o
 .comment       0x0000000000000011       0x12 ..\..\..\Libraries\libs\libplatform.a(audio.o)
                                         0x13 (size before relaxing)
 .comment       0x0000000000000023       0x13 ..\..\..\Libraries\libs\libplatform.a(cm.o)
 .comment       0x0000000000000023       0x13 ..\..\..\Libraries\libs\libplatform.a(os_flash.o)
 .comment       0x0000000000000023       0x13 ..\..\..\Libraries\libs\libplatform.a(xcfg.o)
 .comment       0x0000000000000023       0x13 ..\..\..\Libraries\libs\libplatform.a(device.o)
 .comment       0x0000000000000023       0x13 ..\..\..\Libraries\libs\libplatform.a(main.o)
 .comment       0x0000000000000023       0x13 ..\..\..\Libraries\libs\libplatform.a(interrupt.o)
 .comment       0x0000000000000023       0x13 ..\..\..\Libraries\libs\libplatform.a(startup.o)
 .comment       0x0000000000000023       0x13 ..\..\..\Libraries\libs\libplatform.a(sys_hook.o)
 .comment       0x0000000000000023       0x13 ..\..\..\Libraries\libs\libplatform.a(spiflash.o)
 .comment       0x0000000000000023       0x13 ..\..\..\Libraries\libs\libplatform.a(debug.o)
 .comment       0x0000000000000023       0x13 ..\..\..\Libraries\libs\libplatform.a(fot_update.o)
 .comment       0x0000000000000023       0x13 ..\..\..\Libraries\libs\libplatform.a(lock.o)
 .comment       0x0000000000000023       0x13 ..\..\..\Libraries\libs\libplatform.a(patch.o)
 .comment       0x0000000000000023       0x13 ..\..\..\Libraries\libs\libplatform.a(power.o)
 .comment       0x0000000000000023       0x13 ..\..\..\Libraries\libs\libplatform.a(rc.o)
 .comment       0x0000000000000023       0x13 ..\..\..\Libraries\libs\libplatform.a(sys.o)
 .comment       0x0000000000000023       0x13 ..\..\..\Libraries\libs\libplatform.a(sys_clk.o)
 .comment       0x0000000000000023       0x13 ..\..\..\Libraries\libs\libplatform.a(voltage_trim.o)
 .comment       0x0000000000000023       0x13 ..\..\..\Libraries\libs\libplatform.a(weak_symbol.o)
 .comment       0x0000000000000023       0x13 ..\..\..\Libraries\libs\libplatform.a(usb.o)
 .comment       0x0000000000000023       0x13 ..\..\..\Libraries\libs\libplatform.a(bt.o)
 .comment       0x0000000000000023       0x13 ..\..\..\Libraries\libs\libbtstack.a(nanos.o)
 .comment       0x0000000000000023       0x13 ..\..\..\Libraries\libs\libbtstack.a(patch.o)
 .comment       0x0000000000000023       0x13 ..\..\..\Libraries\libs\libbtstack.a(platform.o)
 .comment       0x0000000000000023       0x13 ..\..\..\Libraries\libs\libbtstack.a(bt_sco.o)
 .comment       0x0000000000000023       0x13 ..\..\..\Libraries\libs\libbtstack.a(bt_acl.o)
 .comment       0x0000000000000023       0x13 ..\..\..\Libraries\libs\libbtstack.a(ble_con.o)
 .comment       0x0000000000000023       0x13 ..\..\..\Libraries\libs\libbtstack.a(bb_utils.o)
 .comment       0x0000000000000023       0x13 ..\..\..\Libraries\libs\libbtstack.a(bb_int.o)
 .comment       0x0000000000000023       0x13 ..\..\..\Libraries\libs\libbtstack.a(bb.o)
 .comment       0x0000000000000023       0x13 ..\..\..\Libraries\libs\libbtstack.a(platform.o)
 .comment       0x0000000000000023       0x13 ..\..\..\Libraries\libs\libbtstack.a(extern_tws.o)
 .comment       0x0000000000000023       0x13 ..\..\..\Libraries\libs\libbtstack.a(extern_bt.o)
 .comment       0x0000000000000023       0x13 ..\..\..\Libraries\libs\libbtstack.a(extern.o)
 .comment       0x0000000000000023       0x13 ..\..\..\Libraries\libs\libbtstack.a(spp.o)
 .comment       0x0000000000000023       0x13 ..\..\..\Libraries\libs\libbtstack.a(sdp_util.o)
 .comment       0x0000000000000023       0x13 ..\..\..\Libraries\libs\libbtstack.a(sdp_tbl.o)
 .comment       0x0000000000000023       0x13 ..\..\..\Libraries\libs\libbtstack.a(sdp_server.o)
 .comment       0x0000000000000023       0x13 ..\..\..\Libraries\libs\libbtstack.a(sdp_client.o)
 .comment       0x0000000000000023       0x13 ..\..\..\Libraries\libs\libbtstack.a(rfcomm.o)
 .comment       0x0000000000000023       0x13 ..\..\..\Libraries\libs\libbtstack.a(btstack_link_key_db.o)
 .comment       0x0000000000000023       0x13 ..\..\..\Libraries\libs\libbtstack.a(btstack_util.o)
 .comment       0x0000000000000023       0x13 ..\..\..\Libraries\libs\libbtstack.a(btstack_txpkt.o)
 .comment       0x0000000000000023       0x13 ..\..\..\Libraries\libs\libbtstack.a(btstack_run_loop.o)
 .comment       0x0000000000000023       0x13 ..\..\..\Libraries\libs\libbtstack.a(btstack_memory.o)
 .comment       0x0000000000000023       0x13 ..\..\..\Libraries\libs\libbtstack.a(btstack_linked_list.o)
 .comment       0x0000000000000023       0x13 ..\..\..\Libraries\libs\libbtstack.a(btstack_link_ctrl.o)
 .comment       0x0000000000000023       0x13 ..\..\..\Libraries\libs\libbtstack.a(sm.o)
 .comment       0x0000000000000023       0x13 ..\..\..\Libraries\libs\libbtstack.a(le_device_db_memory.o)
 .comment       0x0000000000000023       0x13 ..\..\..\Libraries\libs\libbtstack.a(gatt_server.o)
 .comment       0x0000000000000023       0x13 ..\..\..\Libraries\libs\libbtstack.a(gatt_profile.o)
 .comment       0x0000000000000023       0x13 ..\..\..\Libraries\libs\libbtstack.a(att_server.o)
 .comment       0x0000000000000023       0x13 ..\..\..\Libraries\libs\libbtstack.a(att_dispatch.o)
 .comment       0x0000000000000023       0x13 ..\..\..\Libraries\libs\libbtstack.a(att_db.o)
 .comment       0x0000000000000023       0x13 ..\..\..\Libraries\libs\libbtstack.a(ad_parser.o)
 .comment       0x0000000000000023       0x13 ..\..\..\Libraries\libs\libbtstack.a(btstack_main.o)
 .comment       0x0000000000000023       0x13 ..\..\..\Libraries\libs\libbtstack.a(btstack_hal.o)
 .comment       0x0000000000000023       0x13 ..\..\..\Libraries\libs\libbtstack.a(btstack_api.o)
 .comment       0x0000000000000023       0x13 ..\..\..\Libraries\libs\libbtstack.a(bt_api.o)
 .comment       0x0000000000000023       0x13 ..\..\..\Libraries\libs\libbtstack.a(ble_api.o)
 .comment       0x0000000000000023       0x13 ..\..\..\Libraries\libs\libbtstack.a(bb_sche.o)
 .comment       0x0000000000000023       0x13 ..\..\..\Libraries\libs\libbtstack.a(bb_dbg.o)
 .comment       0x0000000000000023       0x13 ..\..\..\Libraries\libs\libbtstack.a(bb_clk.o)
 .comment       0x0000000000000023       0x13 ..\..\..\Libraries\libs\libbtstack.a(aes.o)
 .comment       0x0000000000000023       0x13 ..\..\..\Libraries\libs\libbtstack.a(vs_proc.o)
 .comment       0x0000000000000023       0x13 ..\..\..\Libraries\libs\libbtstack.a(vs_fcc.o)
 .comment       0x0000000000000023       0x13 ..\..\..\Libraries\libs\libbtstack.a(vs.o)
 .comment       0x0000000000000023       0x13 ..\..\..\Libraries\libs\libbtstack.a(rf_smart.o)
 .comment       0x0000000000000023       0x13 ..\..\..\Libraries\libs\libbtstack.a(rf.o)
 .comment       0x0000000000000023       0x13 ..\..\..\Libraries\libs\libbtstack.a(bt_hook.o)
 .comment       0x0000000000000023       0x13 ..\..\..\Libraries\libs\libbtstack.a(ble_hook.o)
 .comment       0x0000000000000023       0x13 ..\..\..\Libraries\libs\libbtstack.a(hct_tl.o)
 .comment       0x0000000000000023       0x13 ..\..\..\Libraries\libs\libbtstack.a(hct_msg.o)
 .comment       0x0000000000000023       0x13 ..\..\..\Libraries\libs\libbtstack.a(hct_fc.o)
 .comment       0x0000000000000023       0x13 ..\..\..\Libraries\libs\libbtstack.a(hct.o)
 .comment       0x0000000000000023       0x13 ..\..\..\Libraries\libs\libbtstack.a(tws_sco.o)
 .comment       0x0000000000000023       0x13 ..\..\..\Libraries\libs\libbtstack.a(tws_acl.o)
 .comment       0x0000000000000023       0x13 ..\..\..\Libraries\libs\libbtstack.a(lm.o)
 .comment       0x0000000000000023       0x13 ..\..\..\Libraries\libs\libbtstack.a(bt_hal.o)
 .comment       0x0000000000000023       0x13 ..\..\..\Libraries\libs\libbtstack.a(bt21.o)
 .comment       0x0000000000000023       0x13 ..\..\..\Libraries\libs\libbtstack.a(bc.o)
 .comment       0x0000000000000023       0x13 ..\..\..\Libraries\libs\libbtstack.a(ble_hal.o)
 .comment       0x0000000000000023       0x13 ..\..\..\Libraries\libs\libbtstack.a(ble_adv.o)
 .comment       0x0000000000000023       0x13 ..\..\..\Libraries\libs\libbtstack.a(ble.o)
 .comment       0x0000000000000023       0x13 ..\..\..\Libraries\libs\libbtstack.a(extern_ble.o)
 .comment       0x0000000000000023       0x13 ..\..\..\Libraries\libs\libbtstack.a(l2cap_test.o)
 .comment       0x0000000000000023       0x13 ..\..\..\Libraries\libs\libbtstack.a(l2cap.o)
 .comment       0x0000000000000023       0x13 ..\..\..\Libraries\libs\libbtstack.a(hci_sco.o)
 .comment       0x0000000000000023       0x13 ..\..\..\Libraries\libs\libbtstack.a(hci_dump.o)
 .comment       0x0000000000000023       0x13 ..\..\..\Libraries\libs\libbtstack.a(hci_cmd.o)
 .comment       0x0000000000000023       0x13 ..\..\..\Libraries\libs\libbtstack.a(hci.o)
 .comment       0x0000000000000023       0x13 ..\..\..\Libraries\libs\libbtstack.a(hid_usage.o)
 .comment       0x0000000000000023       0x13 ..\..\..\Libraries\libs\libbtstack.a(hid_device.o)
 .comment       0x0000000000000023       0x13 ..\..\..\Libraries\libs\libbtstack.a(hfp_hf.o)
 .comment       0x0000000000000023       0x13 ..\..\..\Libraries\libs\libbtstack.a(hfp.o)
 .comment       0x0000000000000023       0x13 ..\..\..\Libraries\libs\libbtstack.a(avdtp.o)
 .comment       0x0000000000000023       0x13 ..\..\..\Libraries\libs\libbtstack.a(a2dp.o)
 .comment       0x0000000000000023       0x13 ..\..\..\Libraries\libs\libbtstack.a(btstack_memory_pool.o)
 .comment       0x0000000000000023       0x13 ..\..\..\Libraries\libs\libbtstack.a(btstack_adv0.o)
 .comment       0x0000000000000023       0x13 ..\..\..\Libraries\libs\libbtstack.a(hci_transport_hcic.o)
 .comment       0x0000000000000023       0x13 ..\..\..\Libraries\libs\libbtstack.a(btstack_chipset_inner.o)
 .comment       0x0000000000000023       0x13 ..\..\..\Libraries\libs\libbtstack.a(lm_hook.o)
 .comment       0x0000000000000023       0x13 ..\..\..\Libraries\libs\libbtstack.a(lm_sp.o)
 .comment       0x0000000000000023       0x13 ..\..\..\Libraries\libs\libbtstack.a(lm_proc.o)
 .comment       0x0000000000000023       0x13 ..\..\..\Libraries\libs\libbtstack.a(lm_key.o)
 .comment       0x0000000000000023       0x13 ..\..\..\Libraries\libs\libbtstack.a(lc.o)
 .comment       0x0000000000000023       0x13 ..\..\..\Libraries\libs\libbtstack.a(mgr.o)
 .comment       0x0000000000000023       0x13 ..\..\..\Libraries\libs\libbtstack.a(ll.o)
 .comment       0x0000000000000023       0x13 ..\..\..\Libraries\libs\libbtstack.a(ble_test.o)
 .comment       0x0000000000000023       0x13 ..\..\..\Libraries\libs\libbtstack.a(ble_scan.o)
 .comment       0x0000000000000023       0x13 ..\..\..\Libraries\libs\libbtstack.a(ble_per_adv.o)
 .comment       0x0000000000000023       0x13 ..\..\..\Libraries\libs\libbtstack.a(ble_init.o)
 .comment       0x0000000000000023       0x13 ..\..\..\Libraries\libs\libbtstack.a(ble_buf.o)
 .comment       0x0000000000000023       0x13 ..\..\..\Libraries\libs\libbtstack.a(ble_adv0.o)
 .comment       0x0000000000000023       0x13 ..\..\..\Libraries\libs\libbtstack.a(extern_hfhs.o)
 .comment       0x0000000000000023       0x13 ..\..\..\Libraries\libs\libbtstack.a(l2cap_signaling.o)
 .comment       0x0000000000000023       0x13 ..\..\..\Libraries\libs\libbtstack.a(lc_hook.o)
 .comment       0x0000000000000023       0x13 ..\..\..\Libraries\libs\libbtstack.a(lm_sco.o)
 .comment       0x0000000000000023       0x13 ..\..\..\Libraries\libs\libbtstack.a(lc_util.o)
 .comment       0x0000000000000023       0x13 ..\..\..\Libraries\libs\libbtstack.a(lc_sniff.o)
 .comment       0x0000000000000023       0x13 ..\..\..\Libraries\libs\libbtstack.a(lc_sco.o)
 .comment       0x0000000000000023       0x13 ..\..\..\Libraries\libs\libbtstack.a(lc_proc.o)
 .comment       0x0000000000000023       0x13 ..\..\..\Libraries\libs\libbtstack.a(lc_lmppdu.o)
 .comment       0x0000000000000023       0x13 ..\..\..\Libraries\libs\libbtstack.a(mgr_proc.o)
 .comment       0x0000000000000023       0x13 ..\..\..\Libraries\libs\libbtstack.a(mgr_init.o)
 .comment       0x0000000000000023       0x13 ..\..\..\Libraries\libs\libbtstack.a(mgr_hci.o)
 .comment       0x0000000000000023       0x13 ..\..\..\Libraries\libs\libbtstack.a(ll_scan.o)
 .comment       0x0000000000000023       0x13 ..\..\..\Libraries\libs\libbtstack.a(ll_adv.o)
 .comment       0x0000000000000023       0x13 ..\..\..\Libraries\libs\libbtstack.a(ll_proc.o)
 .comment       0x0000000000000023       0x13 ..\..\..\Libraries\libs\libbtstack.a(ll_ping.o)
 .comment       0x0000000000000023       0x13 ..\..\..\Libraries\libs\libbtstack.a(ll_phy_upd.o)
 .comment       0x0000000000000023       0x13 ..\..\..\Libraries\libs\libbtstack.a(ll_past.o)
 .comment       0x0000000000000023       0x13 ..\..\..\Libraries\libs\libbtstack.a(ll_length.o)
 .comment       0x0000000000000023       0x13 ..\..\..\Libraries\libs\libbtstack.a(ll_feature.o)
 .comment       0x0000000000000023       0x13 ..\..\..\Libraries\libs\libbtstack.a(ll_encrypt.o)
 .comment       0x0000000000000023       0x13 ..\..\..\Libraries\libs\libbtstack.a(ll_disconnect.o)
 .comment       0x0000000000000023       0x13 ..\..\..\Libraries\libs\libbtstack.a(ll_con_upd.o)
 .comment       0x0000000000000023       0x13 ..\..\..\Libraries\libs\libbtstack.a(ll_cntl.o)
 .comment       0x0000000000000023       0x13 ..\..\..\Libraries\libs\libbtstack.a(ll_clk_acc.o)
 .comment       0x0000000000000023       0x13 ..\..\..\Libraries\libs\libbtstack.a(ll_chmap_upd.o)
 .comment       0x0000000000000023       0x13 ..\..\..\Libraries\libs\libbtstack.a(aes_rpa.o)
 .comment       0x0000000000000023       0x13 ..\..\..\Libraries\libs\libbtstack.a(scan_hook.o)
 .comment       0x0000000000000023       0x13 ..\..\..\Libraries\libs\libbtstack.a(adv_hook.o)
 .comment       0x0000000000000023       0x13 ..\..\..\Libraries\libs\libbtstack.a(ll_version.o)
 .comment       0x0000000000000023       0x13 ..\..\..\Libraries\libs\libbtstack.a(ll_pwr.o)
 .comment       0x0000000000000023       0x13 ..\..\..\Libraries\libs\libdrivers.a(usb_device_hid.o)
 .comment       0x0000000000000023       0x13 ..\..\..\Libraries\libs\libdrivers.a(usb_device_printer.o)
 .comment       0x0000000000000023       0x13 ..\..\..\Libraries\libs\libdrivers.a(usb_device_run_loop.o)
 .comment       0x0000000000000023       0x13 ..\..\..\Libraries\libs\libdrivers.a(usb_comm.o)
 .comment       0x0000000000000023       0x13 ..\..\..\Libraries\libs\libdrivers.a(usb_device_ep.o)

.riscv.attributes
                0x0000000000000000     0x1e12
 .riscv.attributes
                0x0000000000000000       0x32 ..\..\..\Libraries\libs\libplatform.a(audio.o)
 .riscv.attributes
                0x0000000000000032       0x32 ..\..\..\Libraries\libs\libplatform.a(cm.o)
 .riscv.attributes
                0x0000000000000064       0x32 ..\..\..\Libraries\libs\libplatform.a(os_flash.o)
 .riscv.attributes
                0x0000000000000096       0x32 ..\..\..\Libraries\libs\libplatform.a(xcfg.o)
 .riscv.attributes
                0x00000000000000c8       0x32 ..\..\..\Libraries\libs\libplatform.a(device.o)
 .riscv.attributes
                0x00000000000000fa       0x32 ..\..\..\Libraries\libs\libplatform.a(main.o)
 .riscv.attributes
                0x000000000000012c       0x32 ..\..\..\Libraries\libs\libplatform.a(interrupt.o)
 .riscv.attributes
                0x000000000000015e       0x32 ..\..\..\Libraries\libs\libplatform.a(startup.o)
 .riscv.attributes
                0x0000000000000190       0x32 ..\..\..\Libraries\libs\libplatform.a(sys_hook.o)
 .riscv.attributes
                0x00000000000001c2       0x34 ..\..\..\Libraries\libs\libplatform.a(reset.o)
 .riscv.attributes
                0x00000000000001f6       0x32 ..\..\..\Libraries\libs\libplatform.a(spiflash.o)
 .riscv.attributes
                0x0000000000000228       0x32 ..\..\..\Libraries\libs\libplatform.a(debug.o)
 .riscv.attributes
                0x000000000000025a       0x32 ..\..\..\Libraries\libs\libplatform.a(fot_update.o)
 .riscv.attributes
                0x000000000000028c       0x32 ..\..\..\Libraries\libs\libplatform.a(lock.o)
 .riscv.attributes
                0x00000000000002be       0x32 ..\..\..\Libraries\libs\libplatform.a(patch.o)
 .riscv.attributes
                0x00000000000002f0       0x32 ..\..\..\Libraries\libs\libplatform.a(power.o)
 .riscv.attributes
                0x0000000000000322       0x32 ..\..\..\Libraries\libs\libplatform.a(rc.o)
 .riscv.attributes
                0x0000000000000354       0x30 ..\..\..\Libraries\libs\libplatform.a(s_sys.o)
 .riscv.attributes
                0x0000000000000384       0x32 ..\..\..\Libraries\libs\libplatform.a(sys.o)
 .riscv.attributes
                0x00000000000003b6       0x32 ..\..\..\Libraries\libs\libplatform.a(sys_clk.o)
 .riscv.attributes
                0x00000000000003e8       0x32 ..\..\..\Libraries\libs\libplatform.a(voltage_trim.o)
 .riscv.attributes
                0x000000000000041a       0x32 ..\..\..\Libraries\libs\libplatform.a(weak_symbol.o)
 .riscv.attributes
                0x000000000000044c       0x32 ..\..\..\Libraries\libs\libplatform.a(usb.o)
 .riscv.attributes
                0x000000000000047e       0x32 ..\..\..\Libraries\libs\libplatform.a(bt.o)
 .riscv.attributes
                0x00000000000004b0       0x32 ..\..\..\Libraries\libs\libbtstack.a(nanos.o)
 .riscv.attributes
                0x00000000000004e2       0x32 ..\..\..\Libraries\libs\libbtstack.a(patch.o)
 .riscv.attributes
                0x0000000000000514       0x32 ..\..\..\Libraries\libs\libbtstack.a(platform.o)
 .riscv.attributes
                0x0000000000000546       0x32 ..\..\..\Libraries\libs\libbtstack.a(bt_sco.o)
 .riscv.attributes
                0x0000000000000578       0x32 ..\..\..\Libraries\libs\libbtstack.a(bt_acl.o)
 .riscv.attributes
                0x00000000000005aa       0x32 ..\..\..\Libraries\libs\libbtstack.a(ble_con.o)
 .riscv.attributes
                0x00000000000005dc       0x32 ..\..\..\Libraries\libs\libbtstack.a(bb_utils.o)
 .riscv.attributes
                0x000000000000060e       0x32 ..\..\..\Libraries\libs\libbtstack.a(bb_int.o)
 .riscv.attributes
                0x0000000000000640       0x32 ..\..\..\Libraries\libs\libbtstack.a(bb.o)
 .riscv.attributes
                0x0000000000000672       0x32 ..\..\..\Libraries\libs\libbtstack.a(platform.o)
 .riscv.attributes
                0x00000000000006a4       0x32 ..\..\..\Libraries\libs\libbtstack.a(extern_tws.o)
 .riscv.attributes
                0x00000000000006d6       0x32 ..\..\..\Libraries\libs\libbtstack.a(extern_bt.o)
 .riscv.attributes
                0x0000000000000708       0x32 ..\..\..\Libraries\libs\libbtstack.a(extern.o)
 .riscv.attributes
                0x000000000000073a       0x32 ..\..\..\Libraries\libs\libbtstack.a(spp.o)
 .riscv.attributes
                0x000000000000076c       0x32 ..\..\..\Libraries\libs\libbtstack.a(sdp_util.o)
 .riscv.attributes
                0x000000000000079e       0x32 ..\..\..\Libraries\libs\libbtstack.a(sdp_tbl.o)
 .riscv.attributes
                0x00000000000007d0       0x32 ..\..\..\Libraries\libs\libbtstack.a(sdp_server.o)
 .riscv.attributes
                0x0000000000000802       0x32 ..\..\..\Libraries\libs\libbtstack.a(sdp_client.o)
 .riscv.attributes
                0x0000000000000834       0x32 ..\..\..\Libraries\libs\libbtstack.a(rfcomm.o)
 .riscv.attributes
                0x0000000000000866       0x32 ..\..\..\Libraries\libs\libbtstack.a(btstack_link_key_db.o)
 .riscv.attributes
                0x0000000000000898       0x32 ..\..\..\Libraries\libs\libbtstack.a(btstack_util.o)
 .riscv.attributes
                0x00000000000008ca       0x32 ..\..\..\Libraries\libs\libbtstack.a(btstack_txpkt.o)
 .riscv.attributes
                0x00000000000008fc       0x32 ..\..\..\Libraries\libs\libbtstack.a(btstack_run_loop.o)
 .riscv.attributes
                0x000000000000092e       0x32 ..\..\..\Libraries\libs\libbtstack.a(btstack_memory.o)
 .riscv.attributes
                0x0000000000000960       0x32 ..\..\..\Libraries\libs\libbtstack.a(btstack_linked_list.o)
 .riscv.attributes
                0x0000000000000992       0x32 ..\..\..\Libraries\libs\libbtstack.a(btstack_link_ctrl.o)
 .riscv.attributes
                0x00000000000009c4       0x32 ..\..\..\Libraries\libs\libbtstack.a(sm.o)
 .riscv.attributes
                0x00000000000009f6       0x32 ..\..\..\Libraries\libs\libbtstack.a(le_device_db_memory.o)
 .riscv.attributes
                0x0000000000000a28       0x32 ..\..\..\Libraries\libs\libbtstack.a(gatt_server.o)
 .riscv.attributes
                0x0000000000000a5a       0x32 ..\..\..\Libraries\libs\libbtstack.a(gatt_profile.o)
 .riscv.attributes
                0x0000000000000a8c       0x32 ..\..\..\Libraries\libs\libbtstack.a(att_server.o)
 .riscv.attributes
                0x0000000000000abe       0x32 ..\..\..\Libraries\libs\libbtstack.a(att_dispatch.o)
 .riscv.attributes
                0x0000000000000af0       0x32 ..\..\..\Libraries\libs\libbtstack.a(att_db.o)
 .riscv.attributes
                0x0000000000000b22       0x32 ..\..\..\Libraries\libs\libbtstack.a(ad_parser.o)
 .riscv.attributes
                0x0000000000000b54       0x32 ..\..\..\Libraries\libs\libbtstack.a(btstack_main.o)
 .riscv.attributes
                0x0000000000000b86       0x32 ..\..\..\Libraries\libs\libbtstack.a(btstack_hal.o)
 .riscv.attributes
                0x0000000000000bb8       0x32 ..\..\..\Libraries\libs\libbtstack.a(btstack_api.o)
 .riscv.attributes
                0x0000000000000bea       0x32 ..\..\..\Libraries\libs\libbtstack.a(bt_api.o)
 .riscv.attributes
                0x0000000000000c1c       0x32 ..\..\..\Libraries\libs\libbtstack.a(ble_api.o)
 .riscv.attributes
                0x0000000000000c4e       0x32 ..\..\..\Libraries\libs\libbtstack.a(bb_sche.o)
 .riscv.attributes
                0x0000000000000c80       0x30 ..\..\..\Libraries\libs\libbtstack.a(patch_asm.o)
 .riscv.attributes
                0x0000000000000cb0       0x32 ..\..\..\Libraries\libs\libbtstack.a(bb_dbg.o)
 .riscv.attributes
                0x0000000000000ce2       0x32 ..\..\..\Libraries\libs\libbtstack.a(bb_clk.o)
 .riscv.attributes
                0x0000000000000d14       0x32 ..\..\..\Libraries\libs\libbtstack.a(aes.o)
 .riscv.attributes
                0x0000000000000d46       0x32 ..\..\..\Libraries\libs\libbtstack.a(vs_proc.o)
 .riscv.attributes
                0x0000000000000d78       0x32 ..\..\..\Libraries\libs\libbtstack.a(vs_fcc.o)
 .riscv.attributes
                0x0000000000000daa       0x32 ..\..\..\Libraries\libs\libbtstack.a(vs.o)
 .riscv.attributes
                0x0000000000000ddc       0x32 ..\..\..\Libraries\libs\libbtstack.a(rf_smart.o)
 .riscv.attributes
                0x0000000000000e0e       0x32 ..\..\..\Libraries\libs\libbtstack.a(rf.o)
 .riscv.attributes
                0x0000000000000e40       0x32 ..\..\..\Libraries\libs\libbtstack.a(bt_hook.o)
 .riscv.attributes
                0x0000000000000e72       0x32 ..\..\..\Libraries\libs\libbtstack.a(ble_hook.o)
 .riscv.attributes
                0x0000000000000ea4       0x32 ..\..\..\Libraries\libs\libbtstack.a(hct_tl.o)
 .riscv.attributes
                0x0000000000000ed6       0x32 ..\..\..\Libraries\libs\libbtstack.a(hct_msg.o)
 .riscv.attributes
                0x0000000000000f08       0x32 ..\..\..\Libraries\libs\libbtstack.a(hct_fc.o)
 .riscv.attributes
                0x0000000000000f3a       0x32 ..\..\..\Libraries\libs\libbtstack.a(hct.o)
 .riscv.attributes
                0x0000000000000f6c       0x32 ..\..\..\Libraries\libs\libbtstack.a(tws_sco.o)
 .riscv.attributes
                0x0000000000000f9e       0x32 ..\..\..\Libraries\libs\libbtstack.a(tws_acl.o)
 .riscv.attributes
                0x0000000000000fd0       0x32 ..\..\..\Libraries\libs\libbtstack.a(lm.o)
 .riscv.attributes
                0x0000000000001002       0x32 ..\..\..\Libraries\libs\libbtstack.a(bt_hal.o)
 .riscv.attributes
                0x0000000000001034       0x32 ..\..\..\Libraries\libs\libbtstack.a(bt21.o)
 .riscv.attributes
                0x0000000000001066       0x32 ..\..\..\Libraries\libs\libbtstack.a(bc.o)
 .riscv.attributes
                0x0000000000001098       0x32 ..\..\..\Libraries\libs\libbtstack.a(ble_hal.o)
 .riscv.attributes
                0x00000000000010ca       0x32 ..\..\..\Libraries\libs\libbtstack.a(ble_adv.o)
 .riscv.attributes
                0x00000000000010fc       0x32 ..\..\..\Libraries\libs\libbtstack.a(ble.o)
 .riscv.attributes
                0x000000000000112e       0x32 ..\..\..\Libraries\libs\libbtstack.a(extern_ble.o)
 .riscv.attributes
                0x0000000000001160       0x32 ..\..\..\Libraries\libs\libbtstack.a(l2cap_test.o)
 .riscv.attributes
                0x0000000000001192       0x32 ..\..\..\Libraries\libs\libbtstack.a(l2cap.o)
 .riscv.attributes
                0x00000000000011c4       0x32 ..\..\..\Libraries\libs\libbtstack.a(hci_sco.o)
 .riscv.attributes
                0x00000000000011f6       0x32 ..\..\..\Libraries\libs\libbtstack.a(hci_dump.o)
 .riscv.attributes
                0x0000000000001228       0x32 ..\..\..\Libraries\libs\libbtstack.a(hci_cmd.o)
 .riscv.attributes
                0x000000000000125a       0x32 ..\..\..\Libraries\libs\libbtstack.a(hci.o)
 .riscv.attributes
                0x000000000000128c       0x32 ..\..\..\Libraries\libs\libbtstack.a(hid_usage.o)
 .riscv.attributes
                0x00000000000012be       0x32 ..\..\..\Libraries\libs\libbtstack.a(hid_device.o)
 .riscv.attributes
                0x00000000000012f0       0x32 ..\..\..\Libraries\libs\libbtstack.a(hfp_hf.o)
 .riscv.attributes
                0x0000000000001322       0x32 ..\..\..\Libraries\libs\libbtstack.a(hfp.o)
 .riscv.attributes
                0x0000000000001354       0x32 ..\..\..\Libraries\libs\libbtstack.a(avdtp.o)
 .riscv.attributes
                0x0000000000001386       0x32 ..\..\..\Libraries\libs\libbtstack.a(a2dp.o)
 .riscv.attributes
                0x00000000000013b8       0x32 ..\..\..\Libraries\libs\libbtstack.a(btstack_memory_pool.o)
 .riscv.attributes
                0x00000000000013ea       0x32 ..\..\..\Libraries\libs\libbtstack.a(btstack_adv0.o)
 .riscv.attributes
                0x000000000000141c       0x32 ..\..\..\Libraries\libs\libbtstack.a(hci_transport_hcic.o)
 .riscv.attributes
                0x000000000000144e       0x32 ..\..\..\Libraries\libs\libbtstack.a(btstack_chipset_inner.o)
 .riscv.attributes
                0x0000000000001480       0x32 ..\..\..\Libraries\libs\libbtstack.a(lm_hook.o)
 .riscv.attributes
                0x00000000000014b2       0x32 ..\..\..\Libraries\libs\libbtstack.a(lm_sp.o)
 .riscv.attributes
                0x00000000000014e4       0x32 ..\..\..\Libraries\libs\libbtstack.a(lm_proc.o)
 .riscv.attributes
                0x0000000000001516       0x32 ..\..\..\Libraries\libs\libbtstack.a(lm_key.o)
 .riscv.attributes
                0x0000000000001548       0x32 ..\..\..\Libraries\libs\libbtstack.a(lc.o)
 .riscv.attributes
                0x000000000000157a       0x32 ..\..\..\Libraries\libs\libbtstack.a(mgr.o)
 .riscv.attributes
                0x00000000000015ac       0x32 ..\..\..\Libraries\libs\libbtstack.a(ll.o)
 .riscv.attributes
                0x00000000000015de       0x32 ..\..\..\Libraries\libs\libbtstack.a(ble_test.o)
 .riscv.attributes
                0x0000000000001610       0x32 ..\..\..\Libraries\libs\libbtstack.a(ble_scan.o)
 .riscv.attributes
                0x0000000000001642       0x32 ..\..\..\Libraries\libs\libbtstack.a(ble_per_adv.o)
 .riscv.attributes
                0x0000000000001674       0x32 ..\..\..\Libraries\libs\libbtstack.a(ble_init.o)
 .riscv.attributes
                0x00000000000016a6       0x32 ..\..\..\Libraries\libs\libbtstack.a(ble_buf.o)
 .riscv.attributes
                0x00000000000016d8       0x32 ..\..\..\Libraries\libs\libbtstack.a(ble_adv0.o)
 .riscv.attributes
                0x000000000000170a       0x32 ..\..\..\Libraries\libs\libbtstack.a(extern_hfhs.o)
 .riscv.attributes
                0x000000000000173c       0x32 ..\..\..\Libraries\libs\libbtstack.a(l2cap_signaling.o)
 .riscv.attributes
                0x000000000000176e       0x32 ..\..\..\Libraries\libs\libbtstack.a(lc_hook.o)
 .riscv.attributes
                0x00000000000017a0       0x32 ..\..\..\Libraries\libs\libbtstack.a(lm_sco.o)
 .riscv.attributes
                0x00000000000017d2       0x32 ..\..\..\Libraries\libs\libbtstack.a(lc_util.o)
 .riscv.attributes
                0x0000000000001804       0x32 ..\..\..\Libraries\libs\libbtstack.a(lc_sniff.o)
 .riscv.attributes
                0x0000000000001836       0x32 ..\..\..\Libraries\libs\libbtstack.a(lc_sco.o)
 .riscv.attributes
                0x0000000000001868       0x32 ..\..\..\Libraries\libs\libbtstack.a(lc_proc.o)
 .riscv.attributes
                0x000000000000189a       0x32 ..\..\..\Libraries\libs\libbtstack.a(lc_lmppdu.o)
 .riscv.attributes
                0x00000000000018cc       0x32 ..\..\..\Libraries\libs\libbtstack.a(mgr_proc.o)
 .riscv.attributes
                0x00000000000018fe       0x32 ..\..\..\Libraries\libs\libbtstack.a(mgr_init.o)
 .riscv.attributes
                0x0000000000001930       0x32 ..\..\..\Libraries\libs\libbtstack.a(mgr_hci.o)
 .riscv.attributes
                0x0000000000001962       0x32 ..\..\..\Libraries\libs\libbtstack.a(ll_scan.o)
 .riscv.attributes
                0x0000000000001994       0x32 ..\..\..\Libraries\libs\libbtstack.a(ll_adv.o)
 .riscv.attributes
                0x00000000000019c6       0x32 ..\..\..\Libraries\libs\libbtstack.a(ll_proc.o)
 .riscv.attributes
                0x00000000000019f8       0x32 ..\..\..\Libraries\libs\libbtstack.a(ll_ping.o)
 .riscv.attributes
                0x0000000000001a2a       0x32 ..\..\..\Libraries\libs\libbtstack.a(ll_phy_upd.o)
 .riscv.attributes
                0x0000000000001a5c       0x32 ..\..\..\Libraries\libs\libbtstack.a(ll_past.o)
 .riscv.attributes
                0x0000000000001a8e       0x32 ..\..\..\Libraries\libs\libbtstack.a(ll_length.o)
 .riscv.attributes
                0x0000000000001ac0       0x32 ..\..\..\Libraries\libs\libbtstack.a(ll_feature.o)
 .riscv.attributes
                0x0000000000001af2       0x32 ..\..\..\Libraries\libs\libbtstack.a(ll_encrypt.o)
 .riscv.attributes
                0x0000000000001b24       0x32 ..\..\..\Libraries\libs\libbtstack.a(ll_disconnect.o)
 .riscv.attributes
                0x0000000000001b56       0x32 ..\..\..\Libraries\libs\libbtstack.a(ll_con_upd.o)
 .riscv.attributes
                0x0000000000001b88       0x32 ..\..\..\Libraries\libs\libbtstack.a(ll_cntl.o)
 .riscv.attributes
                0x0000000000001bba       0x32 ..\..\..\Libraries\libs\libbtstack.a(ll_clk_acc.o)
 .riscv.attributes
                0x0000000000001bec       0x32 ..\..\..\Libraries\libs\libbtstack.a(ll_chmap_upd.o)
 .riscv.attributes
                0x0000000000001c1e       0x32 ..\..\..\Libraries\libs\libbtstack.a(aes_rpa.o)
 .riscv.attributes
                0x0000000000001c50       0x32 ..\..\..\Libraries\libs\libbtstack.a(scan_hook.o)
 .riscv.attributes
                0x0000000000001c82       0x32 ..\..\..\Libraries\libs\libbtstack.a(adv_hook.o)
 .riscv.attributes
                0x0000000000001cb4       0x32 ..\..\..\Libraries\libs\libbtstack.a(ll_version.o)
 .riscv.attributes
                0x0000000000001ce6       0x32 ..\..\..\Libraries\libs\libbtstack.a(ll_pwr.o)
 .riscv.attributes
                0x0000000000001d18       0x32 ..\..\..\Libraries\libs\libdrivers.a(usb_device_hid.o)
 .riscv.attributes
                0x0000000000001d4a       0x32 ..\..\..\Libraries\libs\libdrivers.a(usb_device_printer.o)
 .riscv.attributes
                0x0000000000001d7c       0x32 ..\..\..\Libraries\libs\libdrivers.a(usb_device_run_loop.o)
 .riscv.attributes
                0x0000000000001dae       0x32 ..\..\..\Libraries\libs\libdrivers.a(usb_comm.o)
 .riscv.attributes
                0x0000000000001de0       0x32 ..\..\..\Libraries\libs\libdrivers.a(usb_device_ep.o)
